 CryPhysics

 Timestamp is 5036e413 (Fri Aug 24 04:16:51 2012)

 Preferred load address is 0000000035000000

 Start         Length     Name                   Class
 0001:00000000 0020119aH .text                   CODE
 0001:002011a0 00000092H .text$x                 CODE
 0001:00201240 000004a0H .text$yc                CODE
 0001:002016e0 00000295H .text$yd                CODE
 0002:00000000 00000238H .idata$5                DATA
 0002:00000238 00000008H .CRT$XCA                DATA
 0002:00000240 00000080H .CRT$XCU                DATA
 0002:000002c0 00000008H .CRT$XCZ                DATA
 0002:000002c8 00000008H .CRT$XIA                DATA
 0002:000002d0 00000008H .CRT$XIAA               DATA
 0002:000002d8 00000008H .CRT$XIZ                DATA
 0002:000002e0 00005cc8H .rdata                  DATA
 0002:00005fa8 00000055H .rdata$debug            DATA
 0002:00006000 00000008H .rtc$IAA                DATA
 0002:00006008 00000008H .rtc$IZZ                DATA
 0002:00006010 00000008H .rtc$TAA                DATA
 0002:00006018 00000008H .rtc$TZZ                DATA
 0002:00006020 0000da8cH .xdata                  DATA
 0002:00013aac 0000003cH .idata$2                DATA
 0002:00013ae8 00000014H .idata$3                DATA
 0002:00013b00 00000238H .idata$4                DATA
 0002:00013d38 0000043aH .idata$6                DATA
 0002:00014180 00000092H .edata                  DATA
 0003:00000000 000010c8H .data                   DATA
 0003:000010d0 00145cb0H .bss                    DATA
 0004:00000000 00007860H .pdata                  DATA
 0005:00000000 00000008H .tls$                   DATA
 0006:00000000 00000058H .rsrc$01                DATA
 0006:00000060 00000248H .rsrc$02                DATA

  Address         Publics by Value              Rva+Base               Lib:Object

 0000:00000000       ___safe_se_handler_count   0000000000000000     <absolute>
 0000:00000000       ___safe_se_handler_table   0000000000000000     <absolute>
 0000:00000000       __ImageBase                0000000035000000     <linker-defined>
 0001:00000000       ?AlertNeighbourhoodND@CArticulatedEntity@@UEAAXH@Z 0000000035001000 f   articulatedentity.obj
 0001:00000040       ??_H@YAXPEAX_KHP6APEAX0@Z@Z 0000000035001040 f i articulatedentity.obj
 0001:00000090       ?GetPotentialColliders@CArticulatedEntity@@UEAAHAEAPEAPEAVCPhysicalEntity@@M@Z 0000000035001090 f   articulatedentity.obj
 0001:000000b0       ?CheckSelfCollision@CArticulatedEntity@@UEAAHHH@Z 00000000350010b0 f   articulatedentity.obj
 0001:000000f0       ?GetRigidBody@CArticulatedEntity@@UEAAPEAVRigidBody@@HH@Z 00000000350010f0 f   articulatedentity.obj
 0001:00000130       ?GetDamping@CArticulatedEntity@@UEAAMM@Z 0000000035001130 f   articulatedentity.obj
 0001:000001a0       ?IsAwake@CArticulatedEntity@@UEBAHH@Z 00000000350011a0 f   articulatedentity.obj
 0001:000001e0       ?GetMaxTimeStep@CArticulatedEntity@@UEAAMM@Z 00000000350011e0 f   articulatedentity.obj
 0001:000001f0       ?JointListUpdated@CArticulatedEntity@@QEAAXXZ 00000000350011f0 f   articulatedentity.obj
 0001:000002c0       ?BreakableConstraintsUpdated@CArticulatedEntity@@UEAAXXZ 00000000350012c0 f   articulatedentity.obj
 0001:00000310       ?OnContactResolved@CArticulatedEntity@@UEAAXPEAUentity_contact@@HH@Z 0000000035001310 f   articulatedentity.obj
 0001:000003a0       ?GetMemoryStatistics@CArticulatedEntity@@UEBAXPEAVICrySizer@@@Z 00000000350013a0 f   articulatedentity.obj
 0001:00000430       ??4?$matrix_tpl@M@@QEAAAEAV0@AEBV0@@Z 0000000035001430 f i articulatedentity.obj
 0001:00000540       ?zero@?$matrix_tpl@M@@QEAAAEAV1@XZ 0000000035001540 f i articulatedentity.obj
 0001:000005b0       ?identity@?$matrix_tpl@M@@QEAAAEAV1@XZ 00000000350015b0 f i articulatedentity.obj
 0001:00000690       ?get_iCaller@@YAHXZ        0000000035001690 f i articulatedentity.obj
 0001:000006d0       ?assign_to@?$matrix_product_tpl@M@@QEBAXPEAM@Z 00000000350016d0 f i articulatedentity.obj
 0001:000008d0       ??$ReallocateList@PEAUentity_contact@@@@YAPEAPEAUentity_contact@@AEAPEAPEAU0@HH_N1@Z 00000000350018d0 f i rigidentity.obj
 0001:000008d0       ??$ReallocateList@PEAD@@YAPEAPEADAEAPEAPEADHH_N1@Z 00000000350018d0 f i articulatedentity.obj
 0001:000008d0       ??$ReallocateList@_K@@YAPEA_KAEAPEA_KHH_N1@Z 00000000350018d0 f i rigidentity.obj
 0001:000009b0       ??$?XM@@YAAEAV?$matrix_tpl@M@@AEAV0@M@Z 00000000350019b0 f i articulatedentity.obj
 0001:00000a50       ??$?0M@?$Ang3_tpl@M@@QEAA@AEBU?$Matrix33_tpl@M@@@Z 0000000035001a50 f i articulatedentity.obj
 0001:00000b70       ?AddLabelFmt@CDummyMemReplay@@UEAAXPEBDZZ 0000000035001b70 f i articulatedentity.obj
 0001:00000b80       ?StepBack@CLivingEntity@@UEAAXM@Z 0000000035001b80 f i livingentity.obj
 0001:00000b80       ?UnbindFromContainer@CDummyMemReplay@@UEAAXPEBX0@Z 0000000035001b80 f i articulatedentity.obj
 0001:00000b80       ?AddContextV@CDummyMemReplay@@UEAAXHIPEBDPEAD@Z 0000000035001b80 f i articulatedentity.obj
 0001:00000b80       ?UnMarkBucket@CDummyMemReplay@@UEAAXHPEAX@Z 0000000035001b80 f i articulatedentity.obj
 0001:00000b80       ?Start@CDummyMemReplay@@UEAAX_NPEBD@Z 0000000035001b80 f i articulatedentity.obj
 0001:00000b80       ?ExitScope_Realloc@CDummyMemReplay@@UEAAX_K000@Z 0000000035001b80 f i articulatedentity.obj
 0001:00000b80       ?GetNodeChildrenBVs@CBVTree@@UEAAXPEBUBV@@AEAPEAU2@1H@Z 0000000035001b80 f i livingentity.obj
 0001:00000b80       ?GetBBox@CBVTree@@UEAAXPEAUbox@primitives@@@Z 0000000035001b80 f i livingentity.obj
 0001:00000b80       ?RemapForeignIdx@CGeometry@@UEAAXPEAH0H@Z 0000000035001b80 f i livingentity.obj
 0001:00000b80       ?BucketEnableCleanups@CDummyMemReplay@@UEAAXPEAX_N@Z 0000000035001b80 f i articulatedentity.obj
 0001:00000b80       ?SpuUnfriendly@CGeometry@@UEAAXPEADAEA_K@Z 0000000035001b80 f i livingentity.obj
 0001:00000b80       ?BindToContainer@CDummyMemReplay@@UEAAXPEBX0@Z 0000000035001b80 f i articulatedentity.obj
 0001:00000b80       ?AddScreenshot@CDummyMemReplay@@UEAAXXZ 0000000035001b80 f i articulatedentity.obj
 0001:00000b80       ?CalcVolumetricPressure@CGeometry@@UEAAXPEAUgeom_world_data@@AEBU?$Vec3_tpl@M@@MM1AEAU3@2@Z 0000000035001b80 f i livingentity.obj
 0001:00000b80       ?MarkUsedTriangle@CBVTree@@UEAAXHPEAUgeometry_under_test@@@Z 0000000035001b80 f i livingentity.obj
 0001:00000b80       ?SetDynPoolSize@CPhysicalWorld@@UEAAXH@Z 0000000035001b80 f i physicalworld.obj
 0001:00000b80       ?CleanupAfterIntersectionTest@CGeometry@@UEAAXPEAUgeometry_under_test@@@Z 0000000035001b80 f i livingentity.obj
 0001:00000b80       ?PrepareForRayTest@CHeightfield@@UEAAXM@Z 0000000035001b80 f i waterman.obj
 0001:00000b80       ?RemoveContext@CDummyMemReplay@@UEAAXXZ 0000000035001b80 f i articulatedentity.obj
 0001:00000b80       ?Load@CBVTree@@UEAAXAEAVCMemStream@@PEAVCGeometry@@@Z 0000000035001b80 f i livingentity.obj
 0001:00000b80       ?SwapContainers@CDummyMemReplay@@UEAAXPEBX0@Z 0000000035001b80 f i articulatedentity.obj
 0001:00000b80       ?ReleaseLastBVs@CBVTree@@UEAAXH@Z 0000000035001b80 f i livingentity.obj
 0001:00000b80       ?AppendVertices@CGeometry@@UEAAXPEAU?$Vec3_tpl@M@@PEAHH@Z 0000000035001b80 f i livingentity.obj
 0001:00000b80       ?ReleaseLastSweptBVs@CBVTree@@UEAAXH@Z 0000000035001b80 f i livingentity.obj
 0001:00000b80       ?AddContext@CDummyMemReplay@@UEAAXHIPEBD@Z 0000000035001b80 f i articulatedentity.obj
 0001:00000b80       ?AllocUsage@CDummyMemReplay@@UEAAXW4Class@EMemReplayAllocClass@@_K1@Z 0000000035001b80 f i articulatedentity.obj
 0001:00000b80       ?GetMemoryStatistics@CGeometry@@UEAAXPEAVICrySizer@@@Z 0000000035001b80 f i livingentity.obj
 0001:00000b80       ?ExitScope@CDummyMemReplay@@UEAAXXZ 0000000035001b80 f i articulatedentity.obj
 0001:00000b80       ?StartOnCommandLine@CDummyMemReplay@@UEAAXPEBD@Z 0000000035001b80 f i articulatedentity.obj
 0001:00000b80       ?Load@CGeometry@@UEAAXAEAVCMemStream@@@Z 0000000035001b80 f i livingentity.obj
 0001:00000b80       ?GetNodeChildrenBVs@CBVTree@@UEAAXAEBU?$Matrix33_tpl@M@@AEBU?$Vec3_tpl@M@@MPEBUBV@@AEAPEAU4@3H@Z 0000000035001b80 f i livingentity.obj
 0001:00000b80       ?GetMemoryStatistics@CBVTree@@UEAAXPEAVICrySizer@@@Z 0000000035001b80 f i livingentity.obj
 0001:00000b80       ?RecomputeMassDistribution@CPhysicalEntity@@UEAAXHH@Z 0000000035001b80 f i livingentity.obj
 0001:00000b80       ?CalcVolumetricPressure@CVoxelGeom@@UEAAXPEAUgeom_world_data@@AEBU?$Vec3_tpl@M@@MM1AEAU3@2@Z 0000000035001b80 f i geoman.obj
 0001:00000b80       ?GetMemoryStatistics@CPhysicalPlaceholder@@UEBAXPEAVICrySizer@@@Z 0000000035001b80 f i physarea.obj
 0001:00000b80       ?GetInfo@CDummyMemReplay@@UEAAXAEAUCryReplayInfo@@@Z 0000000035001b80 f i articulatedentity.obj
 0001:00000b80       ?CompactMemory@CGeometry@@UEAAXXZ 0000000035001b80 f i livingentity.obj
 0001:00000b80       ?GetNodeBV@CRayBV@@UEAAXAEBU?$Matrix33_tpl@M@@AEBU?$Vec3_tpl@M@@MAEAPEAUBV@@1MHH@Z 0000000035001b80 f i livingentity.obj
 0001:00000b80       ?CleanupAfterIntersectionTest@CBVTree@@UEAAXPEAUgeometry_under_test@@@Z 0000000035001b80 f i livingentity.obj
 0001:00000b80       ?GetSpatialContactMatrix@CPhysicalEntity@@UEAAXAEBU?$Vec3_tpl@M@@HQEAY05M@Z 0000000035001b80 f i articulatedentity.obj
 0001:00000b80       ?AddAllocReference@CDummyMemReplay@@UEAAXPEAX0@Z 0000000035001b80 f i articulatedentity.obj
 0001:00000b80       ?MarkPool@CDummyMemReplay@@UEAAXH_KPEAX0PEBD@Z 0000000035001b80 f i articulatedentity.obj
 0001:00000b80       ?CreateJobThreads@@YAXHH@Z 0000000035001b80 f i jobq.obj
 0001:00000b80       ?Flush@CDummyMemReplay@@UEAAXXZ 0000000035001b80 f i articulatedentity.obj
 0001:00000b80       ?DumpStats@CDummyMemReplay@@UEAAXXZ 0000000035001b80 f i articulatedentity.obj
 0001:00000b80       ?GetNodeBV@CRayBV@@UEAAXAEAPEAUBV@@AEBU?$Vec3_tpl@M@@MHH@Z 0000000035001b80 f i livingentity.obj
 0001:00000b80       ?GetMemoryStatistics@CPhysicalStub@@UEBAXPEAVICrySizer@@@Z 0000000035001b80 f i physarea.obj
 0001:00000b80       ?Save@CGeometry@@UEAAXAEAVCMemStream@@@Z 0000000035001b80 f i livingentity.obj
 0001:00000b80       ?ExitScope_Alloc@CDummyMemReplay@@UEAAX_K00@Z 0000000035001b80 f i articulatedentity.obj
 0001:00000b80       ?RegisterFixedAddressRange@CDummyMemReplay@@UEAAXPEAX_KPEBD@Z 0000000035001b80 f i articulatedentity.obj
 0001:00000b80       ?DumpSymbols@CDummyMemReplay@@UEAAXXZ 0000000035001b80 f i articulatedentity.obj
 0001:00000b80       ?GetNodeChildrenBVs@CBVTree@@UEAAXPEBUBV@@AEBU?$Vec3_tpl@M@@MAEAPEAU2@2H@Z 0000000035001b80 f i livingentity.obj
 0001:00000b80       ?RemoveGeometry@CPhysicalStub@@UEAAXHH@Z 0000000035001b80 f i physarea.obj
 0001:00000b80       ?RegisterContainer@CDummyMemReplay@@UEAAXPEBXH@Z 0000000035001b80 f i articulatedentity.obj
 0001:00000b80       ?CalcVolumetricPressure@CHeightfield@@UEAAXPEAUgeom_world_data@@AEBU?$Vec3_tpl@M@@MM1AEAU3@2@Z 0000000035001b80 f i heightfieldgeom.obj
 0001:00000b80       ?SetNetworkAuthority@CPhysicalEntity@@UEAAXHH@Z 0000000035001b80 f i livingentity.obj
 0001:00000b80       ?Stop@CDummyMemReplay@@UEAAXXZ 0000000035001b80 f i articulatedentity.obj
 0001:00000b80       ?MarkBucket@CDummyMemReplay@@UEAAXH_KPEAX0@Z 0000000035001b80 f i articulatedentity.obj
 0001:00000b80       ?OnDelayedStep@CPhysicalEntity@@UEAAXAEAVCMemStreamA@@@Z 0000000035001b80 f i livingentity.obj
 0001:00000b80       ?UnMarkPool@CDummyMemReplay@@UEAAXHPEAX@Z 0000000035001b80 f i articulatedentity.obj
 0001:00000b80       ?AddLabel@CDummyMemReplay@@UEAAXPEBD@Z 0000000035001b80 f i articulatedentity.obj
 0001:00000b80       ?WriteCompressedPos@@YAXAEAVCStream@@AEBU?$Vec3_tpl@M@@_N@Z 0000000035001b80 f i utils.obj
 0001:00000b80       ?PrepareForRayTest@CGeometry@@UEAAXM@Z 0000000035001b80 f i livingentity.obj
 0001:00000b80       ?OnStructureUpdate@CPhysicalEntity@@UEAAXXZ 0000000035001b80 f i articulatedentity.obj
 0001:00000b80       ?PrepareForRayTest@CVoxelGeom@@UEAAXM@Z 0000000035001b80 f i geoman.obj
 0001:00000b80       ?AddAdditionalImpulses@CRigidEntity@@UEAAXM@Z 0000000035001b80 f i articulatedentity.obj
 0001:00000b80       ?WriteCompressedQuat@@YAXAEAVCStream@@AEBU?$Quat_tpl@M@@@Z 0000000035001b80 f i utils.obj
 0001:00000b80       ?UnMapPage@CDummyMemReplay@@UEAAXPEAX_K@Z 0000000035001b80 f i articulatedentity.obj
 0001:00000b80       ?AddFrameStart@CDummyMemReplay@@UEAAXXZ 0000000035001b80 f i articulatedentity.obj
 0001:00000b80       ?GetContactMatrix@CPhysicalEntity@@UEAAXAEBU?$Vec3_tpl@M@@HAEAU?$Matrix33_tpl@M@@@Z 0000000035001b80 f i particleentity.obj
 0001:00000b80       ?DestroyAuxilaryMeshData@CGeometry@@UEAAXH@Z 0000000035001b80 f i livingentity.obj
 0001:00000b80       ?RemoveAllocReference@CDummyMemReplay@@UEAAXPEAX@Z 0000000035001b80 f i articulatedentity.obj
 0001:00000b80       ?SetStateFromSnapshotTxt@CPhysicalStub@@UEAAXPEBDH@Z 0000000035001b80 f i physarea.obj
 0001:00000b80       ?StepBack@CPhysicalEntity@@UEAAXM@Z 0000000035001b80 f i particleentity.obj
 0001:00000b80       ?StepBack@CPhysicalStub@@UEAAXM@Z 0000000035001b80 f i physarea.obj
 0001:00000b80       ?GetNodeBV@CHeightfieldBV@@UEAAXAEBU?$Matrix33_tpl@M@@AEBU?$Vec3_tpl@M@@MAEAPEAUBV@@1MHH@Z 0000000035001b80 f i waterman.obj
 0001:00000b80       ?GetNodeBV@COBBTree@@UEAAXAEBU?$Matrix33_tpl@M@@AEBU?$Vec3_tpl@M@@MAEAPEAUBV@@1MHH@Z 0000000035001b80 f i trimesh.obj
 0001:00000b80       ?AddSizerTree@CDummyMemReplay@@UEAAXPEBD@Z 0000000035001b80 f i articulatedentity.obj
 0001:00000b80       ?OnNeighbourSplit@CPhysicalEntity@@UEAAXPEAV1@0@Z 0000000035001b80 f i livingentity.obj
 0001:00000b80       ?StartStep@CPhysicalEntity@@UEAAXM@Z 0000000035001b80 f i physicalentity.obj
 0001:00000b80       ?UnregisterContainer@CDummyMemReplay@@UEAAXPEBX@Z 0000000035001b80 f i articulatedentity.obj
 0001:00000b80       ?SetNetworkAuthority@CPhysicalStub@@UEAAXHH@Z 0000000035001b80 f i physarea.obj
 0001:00000b80       ?CheckAdditionalGeometry@CRigidEntity@@UEAAXM@Z 0000000035001b80 f i articulatedentity.obj
 0001:00000b80       ?SetData@CGeometry@@UEAAXPEBUprimitive@primitives@@@Z 0000000035001b80 f i livingentity.obj
 0001:00000b80       ?ExitScope_Free@CDummyMemReplay@@UEAAX_K@Z 0000000035001b80 f i articulatedentity.obj
 0001:00000b80       ?ApplyVolumetricPressure@CPhysicalEntity@@UEAAXAEBU?$Vec3_tpl@M@@MM@Z 0000000035001b80 f i articulatedentity.obj
 0001:00000b80       ?GetNodeBV@CAABBTree@@UEAAXAEBU?$Matrix33_tpl@M@@AEBU?$Vec3_tpl@M@@MAEAPEAUBV@@1MHH@Z 0000000035001b80 f i trimesh.obj
 0001:00000b80       ?Save@CBVTree@@UEAAXAEAVCMemStream@@@Z 0000000035001b80 f i livingentity.obj
 0001:00000b80       ?MapPage@CDummyMemReplay@@UEAAXPEAX_K@Z 0000000035001b80 f i articulatedentity.obj
 0001:00000b80       ?DelayedIntersect@CPhysicalEntity@@UEAAXPEAUgeom_contact@@HPEAPEAV1@PEAY01H@Z 0000000035001b80 f i livingentity.obj
 0001:00000b80       ?StartStep@CPhysicalStub@@UEAAXM@Z 0000000035001b80 f i physarea.obj
 0001:00000b80       ?AddTexturePoolContext@CDummyMemReplay@@UEAAXPEAXHHHPEBDI@Z 0000000035001b80 f i articulatedentity.obj
 0001:00000b80       ?SetGeomConvex@CBVTree@@UEAAXXZ 0000000035001b80 f i livingentity.obj
 0001:00000b80       ?DetachPartContacts@CPhysicalEntity@@UEAAXHHPEAV1@HH@Z 0000000035001b80 f i livingentity.obj
 0001:00000b80       ?GetNodeBV@CHeightfieldBV@@UEAAXAEAPEAUBV@@AEBU?$Vec3_tpl@M@@MHH@Z 0000000035001b80 f i waterman.obj
 0001:00000b80       ?ResetCollisionArea@CBVTree@@UEAAXXZ 0000000035001b80 f i livingentity.obj
 0001:00000b90       ??_GIMemReplay@@UEAAPEAXI@Z 0000000035001b90 f i articulatedentity.obj
 0001:00000b90       ??_ECDummyMemReplay@@UEAAPEAXI@Z 0000000035001b90 f i articulatedentity.obj
 0001:00000b90       ??_EIMemReplay@@UEAAPEAXI@Z 0000000035001b90 f i articulatedentity.obj
 0001:00000b90       ??_GCDummyMemReplay@@UEAAPEAXI@Z 0000000035001b90 f i articulatedentity.obj
 0001:00000bc0       ?AllocRequestsQueue@CPhysicalWorld@@QEAAXH@Z 0000000035001bc0 f i articulatedentity.obj
 0001:00000c70       ?FreeEntityPart@CPhysicalWorld@@QEAAXPEAUgeom@@@Z 0000000035001c70 f i articulatedentity.obj
 0001:00000cd0       ?FreeEntityParts@CPhysicalWorld@@QEAAXPEAUgeom@@H@Z 0000000035001cd0 f i articulatedentity.obj
 0001:00000d00       ?IsPODThread@@YAHPEAVCPhysicalWorld@@@Z 0000000035001d00 f i articulatedentity.obj
 0001:00000d30       ?Loc2Glob@@YA?AU?$Vec3_tpl@M@@AEBUentity_contact@@AEBU1@H@Z 0000000035001d30 f i articulatedentity.obj
 0001:00001010       ??0ae_joint@@QEAA@XZ       0000000035002010 f i articulatedentity.obj
 0001:000012d0       ??0CArticulatedEntity@@QEAA@PEAVCPhysicalWorld@@@Z 00000000350022d0 f   articulatedentity.obj
 0001:000014a0       ?GetForeignData@CPhysicalPlaceholder@@UEBAPEAXH@Z 00000000350024a0 f i articulatedentity.obj
 0001:000014b0       ?GetiForeignData@CPhysicalPlaceholder@@UEBAHXZ 00000000350024b0 f i articulatedentity.obj
 0001:000014c0       ?GetWorld@CPhysicalEntity@@UEBAPEAUIPhysicalWorld@@XZ 00000000350024c0 f i articulatedentity.obj
 0001:000014c0       ?GetWorld@CPhysArea@@UEBAPEAUIPhysicalWorld@@XZ 00000000350024c0 f i physarea.obj
 0001:000014d0       ?GetMass@CPhysicalEntity@@UEAAMH@Z 00000000350024d0 f i articulatedentity.obj
 0001:000014f0       ?GetMassInv@CRigidEntity@@UEAAMXZ 00000000350024f0 f i articulatedentity.obj
 0001:00001510       ?GetSnapshotVersion@CRigidEntity@@UEAAHXZ 0000000035002510 f i articulatedentity.obj
 0001:00001510       ?GetType@CPhysArea@@UEBA?AW4pe_type@@XZ 0000000035002510 f i physarea.obj
 0001:00001520       ?GetLastTimeStep@CRigidEntity@@UEAAMM@Z 0000000035002520 f i articulatedentity.obj
 0001:00001530       ?GetMaxFriction@CRigidEntity@@UEAAMXZ 0000000035002530 f i articulatedentity.obj
 0001:00001540       ?GetType@CCapsuleGeom@@UEAAHXZ 0000000035002540 f i livingentity.obj
 0001:00001540       ?GetType@CArticulatedEntity@@UEBA?AW4pe_type@@XZ 0000000035002540 f i articulatedentity.obj
 0001:00001550       ?GetSleepSpeedChange@CArticulatedEntity@@UEAAXHAEAU?$Vec3_tpl@M@@0@Z 0000000035002550 f i articulatedentity.obj
 0001:000015c0       ??4geom@@QEAAAEAU0@AEBU0@@Z 00000000350025c0 f i articulatedentity.obj
 0001:000016d0       ??0CFrameProfiler@@QEAA@PEAUISystem@@PEBDW4EProfiledSubsystem@@@Z 00000000350026d0 f i articulatedentity.obj
 0001:00001760       ?GetStatus@CArticulatedEntity@@UEBAHPEAUpe_status@@@Z 0000000035002760 f   articulatedentity.obj
 0001:000021e0       ??4RigidBody@@QEAAAEAV0@AEBV0@@Z 00000000350031e0 f i articulatedentity.obj
 0001:000023c0       ?UpdatePosition@CArticulatedEntity@@QEAAXH@Z 00000000350033c0 f   articulatedentity.obj
 0001:00002560       ?UpdateJointDyn@CArticulatedEntity@@QEAAXXZ 0000000035003560 f   articulatedentity.obj
 0001:00002710       ?CalcEnergy@CArticulatedEntity@@UEAAMM@Z 0000000035003710 f   articulatedentity.obj
 0001:00003190       ?validate@pe_params_joint@@QEAA_NPEBDPEAUILog@@AEBU?$Vec3_tpl@M@@PEAUIPhysRenderer@@PEAXHH@Z 0000000035004190 f i articulatedentity.obj
 0001:00003650       ??0pe_params_articulated_body@@QEAA@XZ 0000000035004650 f i articulatedentity.obj
 0001:000037b0       ?GetContactMatrix@CArticulatedEntity@@UEAAXAEBU?$Vec3_tpl@M@@HAEAU?$Matrix33_tpl@M@@@Z 00000000350047b0 f   articulatedentity.obj
 0001:00003840       ?CreateConstraintContact@CArticulatedEntity@@QEAAPEAUentity_contact@@H@Z 0000000035004840 f   articulatedentity.obj
 0001:00003b00       ?validate@pe_action_impulse@@QEAA_NPEBDPEAUILog@@AEBU?$Vec3_tpl@M@@PEAUIPhysRenderer@@PEAXHH@Z 0000000035004b00 f i articulatedentity.obj
 0001:000040f0       ??0pe_articgeomparams@@QEAA@AEAUpe_geomparams@@@Z 00000000350050f0 f i articulatedentity.obj
 0001:00004220       ??0geom_world_data@@QEAA@XZ 0000000035005220 f i articulatedentity.obj
 0001:00004270       ??0?$ChangeRequest@Upe_geomparams@@@@QEAA@PEAVCPhysicalPlaceholder@@PEAVCPhysicalWorld@@PEAUpe_geomparams@@HPEAXH@Z 0000000035005270 f i articulatedentity.obj
 0001:00004770       ??0?$ChangeRequest@X@@QEAA@PEAVCPhysicalPlaceholder@@PEAVCPhysicalWorld@@PEAXH2H@Z 0000000035005770 f i articulatedentity.obj
 0001:00004ad0       ??0?$ChangeRequest@Upe_params@@@@QEAA@PEAVCPhysicalPlaceholder@@PEAVCPhysicalWorld@@PEAUpe_params@@HPEAXH@Z 0000000035005ad0 f i articulatedentity.obj
 0001:00004f90       ??0?$ChangeRequest@Upe_action@@@@QEAA@PEAVCPhysicalPlaceholder@@PEAVCPhysicalWorld@@PEAUpe_action@@HPEAXH@Z 0000000035005f90 f i articulatedentity.obj
 0001:000053d0       ??$AllocPooledObj@Ugeom@@@CPhysicalWorld@@QEAAPEAUgeom@@AEAPEAU1@AEAH1AECH@Z 00000000350063d0 f i articulatedentity.obj
 0001:00005540       ??$ReallocateList@Uae_joint@@@@YAPEAUae_joint@@AEAPEAU0@HH_N1@Z 0000000035006540 f i articulatedentity.obj
 0001:000056b0       ??$ReallocateList@Uae_part_info@@@@YAPEAUae_part_info@@AEAPEAU0@HH_N1@Z 00000000350066b0 f i articulatedentity.obj
 0001:00005790       ?CryGetIMemReplay@@YAPEAUIMemReplay@@XZ 0000000035006790 f i articulatedentity.obj
 0001:00005810       ?GetLocTransform@CPhysicalEntity@@UEAAXHAEAU?$Vec3_tpl@M@@AEAU?$Quat_tpl@M@@AEAM@Z 0000000035006810 f i articulatedentity.obj
 0001:00005af0       ?AllocEntityParts@CPhysicalWorld@@QEAAPEAUgeom@@H@Z 0000000035006af0 f i articulatedentity.obj
 0001:00005b50       ??1CArticulatedEntity@@UEAA@XZ 0000000035006b50 f   articulatedentity.obj
 0001:00005bf0       ??0geom@@QEAA@AEBU0@@Z     0000000035006bf0 f i articulatedentity.obj
 0001:00005d00       ?RemoveGeometry@CArticulatedEntity@@UEAAXHH@Z 0000000035006d00 f   articulatedentity.obj
 0001:00006400       ?GetParams@CArticulatedEntity@@UEBAHPEAUpe_params@@@Z 0000000035007400 f   articulatedentity.obj
 0001:00006c80       ?GetRigidBodyData@CArticulatedEntity@@UEAAPEAVRigidBody@@PEAV2@H@Z 0000000035007c80 f   articulatedentity.obj
 0001:00006d10       ?OnDelayedStep@CArticulatedEntity@@UEAAXAEAVCMemStreamA@@@Z 0000000035007d10 f   articulatedentity.obj
 0001:00006ff0       ?UpdateJointRotationAxes@CArticulatedEntity@@QEAAXH@Z 0000000035007ff0 f   articulatedentity.obj
 0001:00007740       ?CheckForGimbalLock@CArticulatedEntity@@QEAAXH@Z 0000000035008740 f   articulatedentity.obj
 0001:00007b80       ?SyncJointWithBody@CArticulatedEntity@@QEAAXHH@Z 0000000035008b80 f   articulatedentity.obj
 0001:000087a0       ?CalcBodyZa@CArticulatedEntity@@QEAAHHMAEAV?$vectorn_tpl@M@@@Z 00000000350097a0 f   articulatedentity.obj
 0001:0000a050       ?CalcBodyIa@CArticulatedEntity@@QEAAHHAEAV?$matrix_tpl@M@@@Z 000000003500b050 f   articulatedentity.obj
 0001:0000c9f0       ?CollectPendingImpulses@CArticulatedEntity@@QEAAHHAEAH@Z 000000003500d9f0 f   articulatedentity.obj
 0001:0000dca0       ?PropagateImpulses@CArticulatedEntity@@QEAAXAEBU?$Vec3_tpl@M@@H@Z 000000003500eca0 f   articulatedentity.obj
 0001:0000e6b0       ?CalcVelocityChanges@CArticulatedEntity@@QEAAXMAEBU?$Vec3_tpl@M@@0@Z 000000003500f6b0 f   articulatedentity.obj
 0001:0000f050       ?CalcBodiesIinv@CArticulatedEntity@@QEAAXH@Z 0000000035010050 f   articulatedentity.obj
 0001:00011cd0       ?GetStateSnapshot@CArticulatedEntity@@UEAAHAEAVCStream@@MH@Z 0000000035012cd0 f   articulatedentity.obj
 0001:00012290       ??0pe_params_buoyancy@@QEAA@XZ 0000000035013290 f i articulatedentity.obj
 0001:00012360       ?GetStateSnapshot@CArticulatedEntity@@UEAAHV?$CSerializeWrapper@UISerialize@@@@MH@Z 0000000035013360 f   articulatedentity.obj
 0001:000127b0       ?RegisterContacts@CArticulatedEntity@@UEAAHMH@Z 00000000350137b0 f   articulatedentity.obj
 0001:00013f20       ??_GCArticulatedEntity@@UEAAPEAXI@Z 0000000035014f20 f i articulatedentity.obj
 0001:00013f20       ??_ECArticulatedEntity@@UEAAPEAXI@Z 0000000035014f20 f i articulatedentity.obj
 0001:00013f50       ?AddGeometry@CArticulatedEntity@@UEAAHPEAUphys_geometry@@PEAUpe_geomparams@@HH@Z 0000000035014f50 f   articulatedentity.obj
 0001:000160b0       ?RecomputeMassDistribution@CArticulatedEntity@@UEAAXHH@Z 00000000350170b0 f   articulatedentity.obj
 0001:00017860       ?Action@CArticulatedEntity@@UEAAHPEAUpe_action@@H@Z 0000000035018860 f   articulatedentity.obj
 0001:0001a6b0       ?SyncBodyWithJoint@CArticulatedEntity@@QEAAXHH@Z 000000003501b6b0 f   articulatedentity.obj
 0001:0001bdc0       ?StepJoint@CArticulatedEntity@@QEAAHHMAEAHHH@Z 000000003501cdc0 f   articulatedentity.obj
 0001:0001eec0       ?StepFeatherstone@CArticulatedEntity@@QEAA?AU?$Vec3_tpl@M@@MHAEAU?$Matrix33_tpl@M@@@Z 000000003501fec0 f   articulatedentity.obj
 0001:00020a30       ?StepBack@CArticulatedEntity@@UEAAXM@Z 0000000035021a30 f   articulatedentity.obj
 0001:000217d0       ?SetStateFromSnapshot@CArticulatedEntity@@UEAAHV?$CSerializeWrapper@UISerialize@@@@H@Z 00000000350227d0 f   articulatedentity.obj
 0001:00022020       ?Update@CArticulatedEntity@@UEAAHMM@Z 0000000035023020 f   articulatedentity.obj
 0001:00022eb0       ?SyncWithHost@CArticulatedEntity@@QEAAHHM@Z 0000000035023eb0 f   articulatedentity.obj
 0001:00023b10       ?Step@CArticulatedEntity@@UEAAHM@Z 0000000035024b10 f   articulatedentity.obj
 0001:00025d00       ?SetParams@CArticulatedEntity@@UEAAHPEAUpe_params@@H@Z 0000000035026d00 f   articulatedentity.obj
 0001:0002a410       ?PrepareForIntersectionTest@CBVTree@@UEAAHPEAUgeometry_under_test@@PEAVCGeometry@@0@Z 000000003502b410 f i livingentity.obj
 0001:0002a430       ?GetVolume@CGeometry@@UEAAMXZ 000000003502b430 f i livingentity.obj
 0001:0002a430       ?ComputeExtent@CPhysicalStub@@UEAAMAEAUGeomQuery@@W4EGeomForm@@@Z 000000003502b430 f i physarea.obj
 0001:0002a430       ?GetMassInv@CPhysicalEntity@@UEAAMXZ 000000003502b430 f i particleentity.obj
 0001:0002a430       ?CalcEnergy@CPhysicalEntity@@UEAAMM@Z 000000003502b430 f i particleentity.obj
 0001:0002a430       ?GetMaxSkipDim@CBVTree@@UEAAMXZ 000000003502b430 f i livingentity.obj
 0001:0002a430       ?SplitPriority@CBVTree@@UEAAMPEBUBV@@@Z 000000003502b430 f i livingentity.obj
 0001:0002a440       ?GetNodeContentsIdx@CBVTree@@UEAAHHAEAH@Z 000000003502b440 f i livingentity.obj
 0001:0002a450       ?GetType@CRayBV@@UEAAHXZ   000000003502b450 f i livingentity.obj
 0001:0002a450       ?GetType@CRayGeom@@UEAAHXZ 000000003502b450 f i livingentity.obj
 0001:0002a450       ?GetType@CWheeledVehicleEntity@@UEBA?AW4pe_type@@XZ 000000003502b450 f i wheeledvehicleentity.obj
 0001:0002a460       ??1CLivingEntity@@UEAA@XZ  000000003502b460 f   livingentity.obj
 0001:0002a540       ?GetDamping@CPhysicalEntity@@UEAAMM@Z 000000003502b540 f i livingentity.obj
 0001:0002a550       ?GetMaxFriction@CPhysicalEntity@@UEAAMXZ 000000003502b550 f i livingentity.obj
 0001:0002a560       ?EnterScope@CDummyMemReplay@@UEAA_NW4Class@EMemReplayAllocClass@@GH@Z 000000003502b560 f i articulatedentity.obj
 0001:0002a560       ?IgnoreCollisionsWith@CPhysicalEntity@@UEBA_NPEBV1@H@Z 000000003502b560 f i livingentity.obj
 0001:0002a570       ?GetRigidBodyData@CLivingEntity@@UEAAPEAVRigidBody@@PEAV2@H@Z 000000003502b570 f i livingentity.obj
 0001:0002a5e0       ?GetMassInv@CLivingEntity@@UEAAMXZ 000000003502b5e0 f i livingentity.obj
 0001:0002a5f0       ?GetSpatialContactMatrix@CLivingEntity@@UEAAXAEBU?$Vec3_tpl@M@@HQEAY05M@Z 000000003502b5f0 f i livingentity.obj
 0001:0002a640       ?ReleaseGroundCollider@CLivingEntity@@QEAAXXZ 000000003502b640 f   livingentity.obj
 0001:0002a670       ?GetParams@CLivingEntity@@UEBAHPEAUpe_params@@@Z 000000003502b670 f   livingentity.obj
 0001:0002a9c0       ?AddGeometry@CLivingEntity@@UEAAHPEAUphys_geometry@@PEAUpe_geomparams@@HH@Z 000000003502b9c0 f   livingentity.obj
 0001:0002aa10       ?RemoveGeometry@CLivingEntity@@UEAAXHH@Z 000000003502ba10 f   livingentity.obj
 0001:0002aa50       ?UpdatePosition@CLivingEntity@@QEAAXAEBU?$Vec3_tpl@M@@PEBU2@H@Z 000000003502ba50 f   livingentity.obj
 0001:0002aba0       ?StartStep@CLivingEntity@@UEAAXM@Z 000000003502bba0 f   livingentity.obj
 0001:0002abe0       ?GetMemoryStatistics@CLivingEntity@@UEBAXPEAVICrySizer@@@Z 000000003502bbe0 f   livingentity.obj
 0001:0002ac30       ??$SignalEvent@UEventPhysBBoxOverlap@@@CPhysicalWorld@@QEAAHPEAUEventPhysBBoxOverlap@@H@Z 000000003502bc30 f i livingentity.obj
 0001:0002acc0       ??$SignalEvent@UEventPhysCollision@@@CPhysicalWorld@@QEAAHPEAUEventPhysCollision@@H@Z 000000003502bcc0 f i livingentity.obj
 0001:0002ad50       ??$SignalEvent@UEventPhysPostStep@@@CPhysicalWorld@@QEAAHPEAUEventPhysPostStep@@H@Z 000000003502bd50 f i livingentity.obj
 0001:0002ade0       ??_GIGeometry@@UEAAPEAXI@Z 000000003502bde0 f i livingentity.obj
 0001:0002ade0       ??_EIGeometry@@UEAAPEAXI@Z 000000003502bde0 f i livingentity.obj
 0001:0002ae10       ?AddRef@CGeometry@@UEAAHXZ 000000003502be10 f i livingentity.obj
 0001:0002ae20       ?GetForeignIdx@CGeometry@@UEAAHH@Z 000000003502be20 f i livingentity.obj
 0001:0002ae20       ?PreparePrimitive@CGeometry@@UEAAHPEAUgeom_world_data@@AEAPEAUprimitive@primitives@@H@Z 000000003502be20 f i livingentity.obj
 0001:0002ae20       ?RemoveContactPoint@CPhysicalEntity@@UEAAHPEAV1@AEBU?$Vec3_tpl@M@@M@Z 000000003502be20 f i livingentity.obj
 0001:0002ae20       ?WaitForJobFinish@@YAHAEAHH@Z 000000003502be20 f i jobq.obj
 0001:0002ae20       ?PointInsideStatus@CVoxelGeom@@UEAAHAEBU?$Vec3_tpl@M@@@Z 000000003502be20 f i geoman.obj
 0001:0002ae20       ?AddGeometry@CPhysicalStub@@UEAAHPEAUphys_geometry@@PEAUpe_geomparams@@HH@Z 000000003502be20 f i physarea.obj
 0001:0002ae20       ?GetPrimitiveId@CGeometry@@UEAAHHH@Z 000000003502be20 f i livingentity.obj
 0001:0002ae20       ?PointInsideStatus@CGeometry@@UEAAHAEBU?$Vec3_tpl@M@@@Z 000000003502be20 f i livingentity.obj
 0001:0002ae30       ?GetForeignData@CGeometry@@UEAAPEAXH@Z 000000003502be30 f i livingentity.obj
 0001:0002ae40       ?SetForeignData@CGeometry@@UEAAXPEAXH@Z 000000003502be40 f i livingentity.obj
 0001:0002ae50       ?Load@CGeometry@@UEAAXAEAVCMemStream@@V?$strided_pointer@$$CBU?$Vec3_tpl@M@@@@V?$strided_pointer@G@@PEAD@Z 000000003502be50 f i livingentity.obj
 0001:0002ae50       ?GetEntityFast@CPhysArea@@UEAAPEAVCPhysicalEntity@@XZ 000000003502be50 f i physarea.obj
 0001:0002ae60       ?GetUnprojectionCandidates@CGeometry@@UEAAHHPEBUcontact@@AEAPEAUprimitive@primitives@@AEAPEAHPEAUgeometry_under_test@@@Z 000000003502be60 f i livingentity.obj
 0001:0002ae80       ?DrawWireframe@CGeometry@@UEAAXPEAUIPhysRenderer@@PEAUgeom_world_data@@HH@Z 000000003502be80 f i livingentity.obj
 0001:0002aed0       ?CalculateBuoyancy@CGeometry@@UEAAMPEBUplane@primitives@@PEBUgeom_world_data@@AEAU?$Vec3_tpl@M@@@Z 000000003502bed0 f i livingentity.obj
 0001:0002aee0       ?CalculateMediumResistance@CGeometry@@UEAAXPEBUplane@primitives@@PEBUgeom_world_data@@AEAU?$Vec3_tpl@M@@2@Z 000000003502bee0 f i livingentity.obj
 0001:0002af00       ?GetNormal@CGeometry@@UEAA?AU?$Vec3_tpl@M@@HAEBU2@@Z 000000003502bf00 f i livingentity.obj
 0001:0002af10       ?GetCenter@CGeometry@@UEAA?AU?$Vec3_tpl@M@@XZ 000000003502bf10 f i livingentity.obj
 0001:0002af20       ?Lock@CGeometry@@UEAAXH@Z  000000003502bf20 f i livingentity.obj
 0001:0002af80       ?Unlock@CGeometry@@UEAAXH@Z 000000003502bf80 f i livingentity.obj
 0001:0002afa0       ??_GCGeometry@@UEAAPEAXI@Z 000000003502bfa0 f i livingentity.obj
 0001:0002afa0       ??_ECGeometry@@UEAAPEAXI@Z 000000003502bfa0 f i livingentity.obj
 0001:0002b000       ??_GCSingleBoxTree@@UEAAPEAXI@Z 000000003502c000 f i livingentity.obj
 0001:0002b000       ??_ECVoxelBV@@UEAAPEAXI@Z  000000003502c000 f i geoman.obj
 0001:0002b000       ??_ECBVTree@@UEAAPEAXI@Z   000000003502c000 f i livingentity.obj
 0001:0002b000       ??_GCRayBV@@UEAAPEAXI@Z    000000003502c000 f i livingentity.obj
 0001:0002b000       ??_GCBVTree@@UEAAPEAXI@Z   000000003502c000 f i livingentity.obj
 0001:0002b000       ??_GCVoxelBV@@UEAAPEAXI@Z  000000003502c000 f i geoman.obj
 0001:0002b000       ??_ECRayBV@@UEAAPEAXI@Z    000000003502c000 f i livingentity.obj
 0001:0002b000       ??_ECSingleBoxTree@@UEAAPEAXI@Z 000000003502c000 f i livingentity.obj
 0001:0002b030       ?GetSleepSpeedChange@CPhysicalEntity@@UEAAXHAEAU?$Vec3_tpl@M@@0@Z 000000003502c030 f i livingentity.obj
 0001:0002b050       ?GetMatId@CPhysicalEntity@@QEAAHHH@Z 000000003502c050 f i livingentity.obj
 0001:0002b100       ?CheckAreas@CPhysicalWorld@@QEAAHPEAVCPhysicalEntity@@AEAU?$Vec3_tpl@M@@PEAUpe_params_buoyancy@@HAEBU3@H@Z 000000003502c100 f i livingentity.obj
 0001:0002b1b0       ?AlertNeighbourhoodND@CLivingEntity@@UEAAXH@Z 000000003502c1b0 f i livingentity.obj
 0001:0002b1f0       ?GetContactMatrix@CLivingEntity@@UEAAXAEBU?$Vec3_tpl@M@@HAEAU?$Matrix33_tpl@M@@@Z 000000003502c1f0 f i livingentity.obj
 0001:0002b230       ?EncodeVec6b@@YA?AU?$Vec3_tpl@F@@AEBU?$Vec3_tpl@M@@@Z 000000003502c230 f i livingentity.obj
 0001:0002b310       ?EncodeVec4b@@YA?AUvec4b@@AEBU?$Vec3_tpl@M@@@Z 000000003502c310 f i livingentity.obj
 0001:0002b460       ??_ECLivingEntity@@UEAAPEAXI@Z 000000003502c460 f i livingentity.obj
 0001:0002b460       ??_GCLivingEntity@@UEAAPEAXI@Z 000000003502c460 f i livingentity.obj
 0001:0002b490       ?Awake@CLivingEntity@@UEAAHHH@Z 000000003502c490 f   livingentity.obj
 0001:0002b530       ?GetStateSnapshot@CLivingEntity@@UEAAHV?$CSerializeWrapper@UISerialize@@@@MH@Z 000000003502c530 f   livingentity.obj
 0001:0002b640       ?GetMaxTimeStep@CLivingEntity@@UEAAMM@Z 000000003502c640 f   livingentity.obj
 0001:0002b680       ?CalcEnergy@CLivingEntity@@UEAAMM@Z 000000003502c680 f   livingentity.obj
 0001:0002b860       ?Step_HandleWasFlying@CLivingEntity@@QEAAXAEAU?$Vec3_tpl@M@@AEAHAEBU2@H@Z 000000003502c860 f   livingentity.obj
 0001:0002bda0       ??$OnEvent@UEventPhysBBoxOverlap@@@CPhysicalWorld@@QEAAHIPEAUEventPhysBBoxOverlap@@PEAPEAU1@@Z 000000003502cda0 f i livingentity.obj
 0001:0002be80       ??$OnEvent@UEventPhysCollision@@@CPhysicalWorld@@QEAAHIPEAUEventPhysCollision@@PEAPEAU1@@Z 000000003502ce80 f i livingentity.obj
 0001:0002bf60       ??$OnEvent@UEventPhysPostStep@@@CPhysicalWorld@@QEAAHIPEAUEventPhysPostStep@@PEAPEAU1@@Z 000000003502cf60 f i livingentity.obj
 0001:0002c050       ?validate@pe_player_dimensions@@QEAA_NPEBDPEAUILog@@AEBU?$Vec3_tpl@M@@PEAUIPhysRenderer@@PEAXHH@Z 000000003502d050 f i livingentity.obj
 0001:0002c430       ?validate@pe_action_move@@QEAA_NPEBDPEAUILog@@AEBU?$Vec3_tpl@M@@PEAUIPhysRenderer@@PEAXHH@Z 000000003502d430 f i livingentity.obj
 0001:0002c730       ?SetGeomConvex@CSingleBoxTree@@UEAAXXZ 000000003502d730 f i livingentity.obj
 0001:0002c740       ?MaxPrimsInNode@CSingleBoxTree@@UEAAHXZ 000000003502d740 f i livingentity.obj
 0001:0002c750       ?GetNodeContentsIdx@CSingleBoxTree@@UEAAHHAEAH@Z 000000003502d750 f i livingentity.obj
 0001:0002c760       ?GetType@CVoxelBV@@UEAAHXZ 000000003502d760 f i geoman.obj
 0001:0002c760       ?GetType@CCylinderGeom@@UEAAHXZ 000000003502d760 f i livingentity.obj
 0001:0002c760       ?GetType@CParticleEntity@@UEBA?AW4pe_type@@XZ 000000003502d760 f i particleentity.obj
 0001:0002c770       ?GetBBox@CCylinderGeom@@UEAAXPEAUbox@primitives@@@Z 000000003502d770 f i livingentity.obj
 0001:0002c780       ?GetBVTree@CCylinderGeom@@UEAAPEAVCBVTree@@XZ 000000003502d780 f i livingentity.obj
 0001:0002c780       ?GetBVTree@CRayGeom@@UEAAPEAVCBVTree@@XZ 000000003502d780 f i livingentity.obj
 0001:0002c790       ?GetPrimitive@CCylinderGeom@@UEAAHHPEAUprimitive@primitives@@@Z 000000003502d790 f i livingentity.obj
 0001:0002c7d0       ?SetData@CCylinderGeom@@UEAAXPEBUprimitive@primitives@@@Z 000000003502d7d0 f i livingentity.obj
 0001:0002c7e0       ?GetCenter@CSphereGeom@@UEAA?AU?$Vec3_tpl@M@@XZ 000000003502d7e0 f i physicalentity.obj
 0001:0002c7e0       ?GetCenter@CCylinderGeom@@UEAA?AU?$Vec3_tpl@M@@XZ 000000003502d7e0 f i livingentity.obj
 0001:0002c800       ?GetSizeFast@CCylinderGeom@@UEAAHXZ 000000003502d800 f i livingentity.obj
 0001:0002c810       ?GetVolume@CCylinderGeom@@UEAAMXZ 000000003502d810 f i livingentity.obj
 0001:0002c840       ??_GCCylinderGeom@@UEAAPEAXI@Z 000000003502d840 f i livingentity.obj
 0001:0002c840       ??_GCRayGeom@@UEAAPEAXI@Z  000000003502d840 f i livingentity.obj
 0001:0002c840       ??_ECCapsuleGeom@@UEAAPEAXI@Z 000000003502d840 f i livingentity.obj
 0001:0002c840       ??_ECRayGeom@@UEAAPEAXI@Z  000000003502d840 f i livingentity.obj
 0001:0002c840       ??_GCCapsuleGeom@@UEAAPEAXI@Z 000000003502d840 f i livingentity.obj
 0001:0002c840       ??_ECCylinderGeom@@UEAAPEAXI@Z 000000003502d840 f i livingentity.obj
 0001:0002c8a0       ?SetData@CCapsuleGeom@@UEAAXPEBUprimitive@primitives@@@Z 000000003502d8a0 f i livingentity.obj
 0001:0002c8b0       ?PreparePrimitive@CCapsuleGeom@@UEAAHPEAUgeom_world_data@@AEAPEAUprimitive@primitives@@H@Z 000000003502d8b0 f i livingentity.obj
 0001:0002c8d0       ?GetVolume@CCapsuleGeom@@UEAAMXZ 000000003502d8d0 f i livingentity.obj
 0001:0002c910       ??0CRayGeom@@QEAA@XZ       000000003502d910 f i livingentity.obj
 0001:0002c980       ?GetPrimitive@CRayGeom@@UEAAHHPEAUprimitive@primitives@@@Z 000000003502d980 f i livingentity.obj
 0001:0002c9b0       ?GetData@CSphereGeom@@UEAAPEBUprimitive@primitives@@XZ 000000003502d9b0 f i physicalentity.obj
 0001:0002c9b0       ?GetData@CCylinderGeom@@UEAAPEBUprimitive@primitives@@XZ 000000003502d9b0 f i livingentity.obj
 0001:0002c9b0       ?GetData@CRayGeom@@UEAAPEBUprimitive@primitives@@XZ 000000003502d9b0 f i livingentity.obj
 0001:0002c9b0       ?GetData@CBoxGeom@@UEAAPEBUprimitive@primitives@@XZ 000000003502d9b0 f i physicalentity.obj
 0001:0002c9c0       ?GetSizeFast@CRayGeom@@UEAAHXZ 000000003502d9c0 f i livingentity.obj
 0001:0002c9d0       ?GetCenter@CRayGeom@@UEAA?AU?$Vec3_tpl@M@@XZ 000000003502d9d0 f i livingentity.obj
 0001:0002ca40       ?SetData@CRayGeom@@UEAAXPEBUprimitive@primitives@@@Z 000000003502da40 f i livingentity.obj
 0001:0002cb00       ?PrepareForRayTest@CRayGeom@@UEAAXM@Z 000000003502db00 f i livingentity.obj
 0001:0002cba0       ??0CLivingEntity@@QEAA@PEAVCPhysicalWorld@@@Z 000000003502dba0 f   livingentity.obj
 0001:0002d1a0       ?UnprojectionNeeded@CLivingEntity@@QEBAMAEBU?$Vec3_tpl@M@@AEBU?$Quat_tpl@M@@MM0HAEAU2@H@Z 000000003502e1a0 f   livingentity.obj
 0001:0002e1c0       ?SetParams@CLivingEntity@@UEAAHPEAUpe_params@@H@Z 000000003502f1c0 f   livingentity.obj
 0001:0002f310       ?GetStatus@CLivingEntity@@UEBAHPEAUpe_status@@@Z 0000000035030310 f   livingentity.obj
 0001:0002fcf0       ?Action@CLivingEntity@@UEAAHPEAUpe_action@@H@Z 0000000035030cf0 f   livingentity.obj
 0001:00030440       ?GetStateSnapshot@CLivingEntity@@UEAAHAEAVCStream@@MH@Z 0000000035031440 f   livingentity.obj
 0001:000307e0       ?SetStateFromSnapshot@CLivingEntity@@UEAAHV?$CSerializeWrapper@UISerialize@@@@H@Z 00000000350317e0 f   livingentity.obj
 0001:00030a10       ?AddLegsImpulse@CLivingEntity@@QEAAXAEBU?$Vec3_tpl@M@@0_N@Z 0000000035031a10 f   livingentity.obj
 0001:00030fc0       ?RegisterContact@CLivingEntity@@QEAAXAEBU?$Vec3_tpl@M@@00PEAVCPhysicalEntity@@HHMHH@Z 0000000035031fc0 f   livingentity.obj
 0001:000317b0       ?RegisterUnprojContact@CLivingEntity@@QEAAXAEBUle_contact@@@Z 00000000350327b0 f   livingentity.obj
 0001:000318b0       ?ComputeBBox@CLivingEntity@@UEAAXPEAU?$Vec3_tpl@M@@H@Z 00000000350328b0 f   livingentity.obj
 0001:00031b00       ?ComputeBBoxLE@CLivingEntity@@QEAAXAEBU?$Vec3_tpl@M@@PEAU2@PEAUcoord_block_BBox@@@Z 0000000035032b00 f   livingentity.obj
 0001:00031bf0       ?RegisterContacts@CLivingEntity@@UEAAHMH@Z 0000000035032bf0 f   livingentity.obj
 0001:000322a0       ?GetRigidBody@CLivingEntity@@UEAAPEAVRigidBody@@HH@Z 00000000350332a0 f   livingentity.obj
 0001:00032620       ?OnContactResolved@CLivingEntity@@UEAAXPEAUentity_contact@@HH@Z 0000000035033620 f   livingentity.obj
 0001:000328f0       ?DrawHelperInformation@CLivingEntity@@UEAAXPEAUIPhysRenderer@@H@Z 00000000350338f0 f   livingentity.obj
 0001:00032930       ?Step_HandleFlying@CLivingEntity@@QEAAXAEAU?$Vec3_tpl@M@@AEBU2@H1MM@Z 0000000035033930 f   livingentity.obj
 0001:00032cb0       ?ShootRayDown@CLivingEntity@@QEAAMPEAUle_precomp_entity@@HPEAUle_precomp_part@@AEBU?$Vec3_tpl@M@@AEAU4@M_N44@Z 0000000035033cb0 f   livingentity.obj
 0001:000344f0       ?SyncWithGroundCollider@CLivingEntity@@QEAA?AU?$Vec3_tpl@M@@M@Z 00000000350354f0 f   livingentity.obj
 0001:00035250       ?Step@CLivingEntity@@UEAAHM@Z 0000000035036250 f   livingentity.obj
 0001:0003e4a0       ?Update@CLivingEntity@@UEAAHMM@Z 000000003503f4a0 f   livingentity.obj
 0001:0003ea60       ??1CParticleEntity@@UEAA@XZ 000000003503fa60 f   particleentity.obj
 0001:0003eae0       ?GetRigidBodyData@CPhysicalEntity@@UEAAPEAVRigidBody@@PEAV2@H@Z 000000003503fae0 f i particleentity.obj
 0001:0003eaf0       ?GetMass@CParticleEntity@@UEAAMH@Z 000000003503faf0 f i particleentity.obj
 0001:0003eb00       ?AlertNeighbourhoodND@CParticleEntity@@UEAAXH@Z 000000003503fb00 f i particleentity.obj
 0001:0003eb30       ?StartStep@CParticleEntity@@UEAAXM@Z 000000003503fb30 f   particleentity.obj
 0001:0003eb50       ?GetMemoryStatistics@CParticleEntity@@UEBAXPEAVICrySizer@@@Z 000000003503fb50 f   particleentity.obj
 0001:0003eba0       ?ComputeBBox@CParticleEntity@@UEAAXPEAU?$Vec3_tpl@M@@H@Z 000000003503fba0 f i particleentity.obj
 0001:0003ec40       ?Step@CParticleEntity@@UEAAHM@Z 000000003503fc40 f i particleentity.obj
 0001:0003eca0       ??0CParticleEntity@@QEAA@PEAVCPhysicalWorld@@@Z 000000003503fca0 f   particleentity.obj
 0001:0003ef70       ??_ECParticleEntity@@UEAAPEAXI@Z 000000003503ff70 f i particleentity.obj
 0001:0003ef70       ??_GCParticleEntity@@UEAAPEAXI@Z 000000003503ff70 f i particleentity.obj
 0001:0003efa0       ?GetParams@CParticleEntity@@UEBAHPEAUpe_params@@@Z 000000003503ffa0 f   particleentity.obj
 0001:0003f1a0       ?GetStateSnapshot@CParticleEntity@@UEAAHAEAVCStream@@MH@Z 00000000350401a0 f   particleentity.obj
 0001:0003f220       ?Awake@CParticleEntity@@UEAAHHH@Z 0000000035040220 f   particleentity.obj
 0001:0003f260       ?IsAwake@CParticleEntity@@UEBAHH@Z 0000000035040260 f   particleentity.obj
 0001:0003f380       ?GetMaxTimeStep@CParticleEntity@@UEAAMM@Z 0000000035040380 f   particleentity.obj
 0001:0003f3c0       ??0box@primitives@@QEAA@XZ 00000000350403c0 f i articulatedentity.obj
 0001:0003f3c0       ??0geom_contact@@QEAA@XZ   00000000350403c0 f i particleentity.obj
 0001:0003f3c0       ?PrepGeomExt@@YAPEAUIGeometry@@PEAU1@@Z 00000000350403c0 f i rwi.obj
 0001:0003f3c0       ??0?$Vec3_tpl@M@@QEAA@XZ   00000000350403c0 f i articulatedentity.obj
 0001:0003f3c0       ??0BBoxExt@@QEAA@XZ        00000000350403c0 f i geometry.obj
 0001:0003f3c0       ??0ray@primitives@@QEAA@XZ 00000000350403c0 f i livingentity.obj
 0001:0003f3c0       ?GetEntity@CPhysicalEntity@@UEAAPEAV1@XZ 00000000350403c0 f i rwi.obj
 0001:0003f3c0       ??0sphere@primitives@@QEAA@XZ 00000000350403c0 f i livingentity.obj
 0001:0003f3c0       ??0indexed_triangle@primitives@@QEAA@XZ 00000000350403c0 f i physarea.obj
 0001:0003f3c0       ??0geom_contact_area@@QEAA@XZ 00000000350403c0 f i geometry.obj
 0001:0003f3c0       ??0edge_desc@@QEAA@XZ      00000000350403c0 f i geometry.obj
 0001:0003f3c0       ??0surface_desc@@QEAA@XZ   00000000350403c0 f i geometry.obj
 0001:0003f3c0       ??0cylinder@primitives@@QEAA@XZ 00000000350403c0 f i livingentity.obj
 0001:0003f3c0       ??0?$Vec2_tpl@M@@QEAA@XZ   00000000350403c0 f i livingentity.obj
 0001:0003f3c0       ??0BBox@@QEAA@XZ           00000000350403c0 f i geometry.obj
 0001:0003f3c0       ?GetEntityFast@CPhysicalEntity@@UEAAPEAV1@XZ 00000000350403c0 f i articulatedentity.obj
 0001:0003f3d0       ??0pe_params_particle@@QEAA@XZ 00000000350403d0 f i particleentity.obj
 0001:0003f560       ?validate@pe_params_particle@@QEAA_NPEBDPEAUILog@@AEBU?$Vec3_tpl@M@@PEAUIPhysRenderer@@PEAXHH@Z 0000000035040560 f i particleentity.obj
 0001:0003fc70       ?GetStateSnapshot@CParticleEntity@@UEAAHV?$CSerializeWrapper@UISerialize@@@@MH@Z 0000000035040c70 f   particleentity.obj
 0001:0003fd80       ?SetStateFromSnapshot@CParticleEntity@@UEAAHV?$CSerializeWrapper@UISerialize@@@@H@Z 0000000035040d80 f   particleentity.obj
 0001:0003ff50       ?GetStatus@CParticleEntity@@UEBAHPEAUpe_status@@@Z 0000000035040f50 f   particleentity.obj
 0001:00040350       ?RayTrace@CParticleEntity@@UEAAHAEAUSRayTraceRes@@@Z 0000000035041350 f   particleentity.obj
 0001:00040920       ?DrawHelperInformation@CParticleEntity@@UEAAXPEAUIPhysRenderer@@H@Z 0000000035041920 f   particleentity.obj
 0001:00041470       ?SetParams@CParticleEntity@@UEAAHPEAUpe_params@@H@Z 0000000035042470 f   particleentity.obj
 0001:00042260       ?Action@CParticleEntity@@UEAAHPEAUpe_action@@H@Z 0000000035043260 f   particleentity.obj
 0001:00042700       ?DoStep@CParticleEntity@@UEAAHMH@Z 0000000035043700 f   particleentity.obj
 0001:00047c90       ?GetEntity@CPhysArea@@UEAAPEAVCPhysicalEntity@@XZ 0000000035048c90 f   physarea.obj
 0001:00047ca0       ?GetParams@CPhysArea@@UEBAHPEAUpe_params@@@Z 0000000035048ca0 f   physarea.obj
 0001:00047d80       ?GetMemoryStatistics@CPhysArea@@UEBAXPEAVICrySizer@@@Z 0000000035048d80 f   physarea.obj
 0001:000480f0       ?GetNextArea@CPhysicalWorld@@UEAAPEAUIPhysicalEntity@@PEAU2@@Z 00000000350490f0 f   physarea.obj
 0001:00048160       ??$SignalEvent@UEventPhysAreaChange@@@CPhysicalWorld@@QEAAHPEAUEventPhysAreaChange@@H@Z 0000000035049160 f i physarea.obj
 0001:000481f0       ??$SignalEvent@UEventPhysArea@@@CPhysicalWorld@@QEAAHPEAUEventPhysArea@@H@Z 00000000350491f0 f i physarea.obj
 0001:00048280       ??_GCPhysicalStub@@UEAAPEAXI@Z 0000000035049280 f i physarea.obj
 0001:00048280       ??_ECPhysicalStub@@UEAAPEAXI@Z 0000000035049280 f i physarea.obj
 0001:00048280       ??_EIPhysicalEntity@@UEAAPEAXI@Z 0000000035049280 f i physarea.obj
 0001:00048280       ??_GIPhysicalEntity@@UEAAPEAXI@Z 0000000035049280 f i physarea.obj
 0001:000482b0       ?GetEntityFast@CPhysicalPlaceholder@@UEAAPEAVCPhysicalEntity@@XZ 00000000350492b0 f i physarea.obj
 0001:000482c0       ?CircleRandomPoint@@YA?AU?$Vec2_tpl@M@@W4EGeomForm@@M@Z 00000000350492c0 f i physarea.obj
 0001:000483a0       ?GetRandomPos@CPhysicalStub@@UEAAXAEAURandomPos@@AEAUGeomQuery@@W4EGeomForm@@@Z 00000000350493a0 f i physarea.obj
 0001:000483b0       ??1CPhysArea@@UEAA@XZ      00000000350493b0 f   physarea.obj
 0001:00048440       ?AddRef@CPhysArea@@UEAAHXZ 0000000035049440 f i physarea.obj
 0001:00048460       ?Release@CPhysArea@@UEAAHXZ 0000000035049460 f i physarea.obj
 0001:00048480       ?IsAreaNonWater@@YAHPEAVCPhysArea@@@Z 0000000035049480 f   physarea.obj
 0001:00048500       ?IsAreaGravity@@YAHPEAVCPhysArea@@@Z 0000000035049500 f   physarea.obj
 0001:00048540       ?SetWaterMat@CPhysicalWorld@@UEAAXH@Z 0000000035049540 f   physarea.obj
 0001:00048590       ?alloc@?$AllocPrefix@UStandardAlloc@NAlloc@@@NAlloc@@SAPEAXAEA_K_NHH@Z 0000000035049590 f i physarea.obj
 0001:00048640       ??$move_init@M@NArray@@YAXPEAM0_K@Z 0000000035049640 f i physarea.obj
 0001:000486e0       ??0CRayGeom@@QEAA@AEBU?$Vec3_tpl@M@@0@Z 00000000350496e0 f i physarea.obj
 0001:00048820       ?GetRandomPart@GeomQuery@@QEBAHXZ 0000000035049820 f i physarea.obj
 0001:000489d0       ??_ECPhysArea@@UEAAPEAXI@Z 00000000350499d0 f i physarea.obj
 0001:000489d0       ??_GCPhysArea@@UEAAPEAXI@Z 00000000350499d0 f i physarea.obj
 0001:00048a00       ?DrawHelperInformation@CPhysArea@@UEAAXPEAUIPhysRenderer@@H@Z 0000000035049a00 f   physarea.obj
 0001:00049a00       ?RepositionArea@CPhysicalWorld@@QEAAXPEAVCPhysArea@@@Z 000000003504aa00 f   physarea.obj
 0001:00049b40       ?RemoveArea@CPhysicalWorld@@UEAAXPEAUIPhysicalEntity@@@Z 000000003504ab40 f   physarea.obj
 0001:00049dd0       ?resize_raw@?$SmallDynStorage@MHUStandardAlloc@NAlloc@@@NArray@@QEAAXHH_N@Z 000000003504add0 f i physarea.obj
 0001:00049f40       ?set_size@?$SmallDynStorage@MHUStandardAlloc@NAlloc@@@NArray@@QEAAXH@Z 000000003504af40 f i physarea.obj
 0001:00049fe0       ?destroy@?$DynArray@UGeomQuery@@HU?$SmallDynStorage@UGeomQuery@@HUStandardAlloc@NAlloc@@@NArray@@@@KAXU?$Array@UGeomQuery@@HU?$ArrayStorage@UGeomQuery@@H@NArray@@@@@Z 000000003504afe0 f i physarea.obj
 0001:0004a020       ?set_size@?$SmallDynStorage@UGeomQuery@@HUStandardAlloc@NAlloc@@@NArray@@QEAAXH@Z 000000003504b020 f i physarea.obj
 0001:0004a0d0       ?findroots@?$polynomial_tpl@N$02@@QEBAHNNPEANHH_N@Z 000000003504b0d0 f i physarea.obj
 0001:0004b280       ??0EventPhysArea@@QEAA@XZ  000000003504c280 f i physarea.obj
 0001:0004b360       ??0CPhysArea@@QEAA@PEAVCPhysicalWorld@@@Z 000000003504c360 f   physarea.obj
 0001:0004b600       ?FindSplineClosestPt@CPhysArea@@QEBAMAEBU?$Vec3_tpl@M@@AEAHAEAM@Z 000000003504c600 f   physarea.obj
 0001:0004c1a0       ?FindSplineClosestPt@CPhysArea@@QEBAHAEBU?$Vec3_tpl@M@@0AEAU2@1@Z 000000003504d1a0 f   physarea.obj
 0001:0004e150       ?SetParams@CPhysArea@@UEAAHPEAUpe_params@@H@Z 000000003504f150 f   physarea.obj
 0001:0004f960       ?AddArea@CPhysicalWorld@@UEAAPEAUIPhysicalEntity@@PEAU?$Vec3_tpl@M@@HMMAEBU3@AEBU?$Quat_tpl@M@@M1PEAHH0@Z 0000000035050960 f   physarea.obj
 0001:000518a0       ?AddArea@CPhysicalWorld@@UEAAPEAUIPhysicalEntity@@PEAUIGeometry@@AEBU?$Vec3_tpl@M@@AEBU?$Quat_tpl@M@@M@Z 00000000350528a0 f   physarea.obj
 0001:00052010       ?AddArea@CPhysicalWorld@@UEAAPEAUIPhysicalEntity@@PEAU?$Vec3_tpl@M@@HMAEBU3@AEBU?$Quat_tpl@M@@M@Z 0000000035053010 f   physarea.obj
 0001:000527f0       ?AddGlobalArea@CPhysicalWorld@@UEAAPEAUIPhysicalEntity@@XZ 00000000350537f0 f   physarea.obj
 0001:00052900       ?destroy@?$DynArray@UGeomQuery@@HU?$SmallDynStorage@UGeomQuery@@HUStandardAlloc@NAlloc@@@NArray@@@@IEAAXXZ 0000000035053900 f i physarea.obj
 0001:00052950       ?append_raw@?$DynArray@MHU?$SmallDynStorage@MHUStandardAlloc@NAlloc@@@NArray@@@@QEAA?AU?$Array@MHU?$ArrayStorage@MH@NArray@@@@H@Z 0000000035053950 f i physarea.obj
 0001:00052a10       ?ApplyParams@CPhysArea@@QEBAHAEBU?$Vec3_tpl@M@@AEAU2@0PEAUpe_params_buoyancy@@HHAEAHPEAUIPhysicalEntity@@@Z 0000000035053a10 f   physarea.obj
 0001:00054c20       ?CheckPoint@CPhysArea@@QEBAHAEBU?$Vec3_tpl@M@@M@Z 0000000035055c20 f   physarea.obj
 0001:00055310       ?RayTraceInternal@CPhysArea@@QEAAHAEBU?$Vec3_tpl@M@@0PEAUray_hit@@PEAUpe_params_pos@@@Z 0000000035056310 f   physarea.obj
 0001:000564a0       ?CheckAreas@CPhysicalWorld@@UEAAHAEBU?$Vec3_tpl@M@@AEAU2@PEAUpe_params_buoyancy@@HH0PEAUIPhysicalEntity@@H@Z 00000000350574a0 f   physarea.obj
 0001:00056bf0       ?clear@?$DynArray@MHU?$SmallDynStorage@MHUStandardAlloc@NAlloc@@@NArray@@@@QEAAXXZ 0000000035057bf0 f i physarea.obj
 0001:00056cc0       ??1?$DynArray@UGeomQuery@@HU?$SmallDynStorage@UGeomQuery@@HUStandardAlloc@NAlloc@@@NArray@@@@QEAA@XZ 0000000035057cc0 f i physarea.obj
 0001:00056d40       ??0?$DynArray@MHU?$SmallDynStorage@MHUStandardAlloc@NAlloc@@@NArray@@@@QEAA@AEBU0@@Z 0000000035057d40 f i physarea.obj
 0001:00056e00       ??_GGeomQuery@@QEAAPEAXI@Z 0000000035057e00 f i physarea.obj
 0001:00056e70       ??0GeomQuery@@QEAA@XZ      0000000035057e70 f i physarea.obj
 0001:00056f30       ??$move_init@UGeomQuery@@@NArray@@YAXPEAUGeomQuery@@0_K@Z 0000000035057f30 f i physarea.obj
 0001:00057110       ?resize_raw@?$SmallDynStorage@UGeomQuery@@HUStandardAlloc@NAlloc@@@NArray@@QEAAXHH_N@Z 0000000035058110 f i physarea.obj
 0001:00057290       ?expand_raw@?$DynArray@UGeomQuery@@HU?$SmallDynStorage@UGeomQuery@@HUStandardAlloc@NAlloc@@@NArray@@@@IEAAPEAUGeomQuery@@PEAU2@H@Z 0000000035058290 f i physarea.obj
 0001:00057350       ?clear@?$DynArray@UGeomQuery@@HU?$SmallDynStorage@UGeomQuery@@HUStandardAlloc@NAlloc@@@NArray@@@@QEAAXXZ 0000000035058350 f i physarea.obj
 0001:00057550       ?grow@?$DynArray@UGeomQuery@@HU?$SmallDynStorage@UGeomQuery@@HUStandardAlloc@NAlloc@@@NArray@@@@QEAAPEAUGeomQuery@@H@Z 0000000035058550 f i physarea.obj
 0001:000575c0       ??$GetExtent@UIGeometry@@@GeomQuery@@QEAAMPEAUIGeometry@@W4EGeomForm@@@Z 00000000350585c0 f i physarea.obj
 0001:00057640       ??$GetExtent@VCPhysArea@@@GeomQuery@@QEAAMPEAVCPhysArea@@W4EGeomForm@@@Z 0000000035058640 f i physarea.obj
 0001:000576c0       ??0?$DynArray@UGeomQuery@@HU?$SmallDynStorage@UGeomQuery@@HUStandardAlloc@NAlloc@@@NArray@@@@QEAA@AEBU0@@Z 00000000350586c0 f i physarea.obj
 0001:00057780       ?GetRandomPos@CPhysArea@@UEBAXAEAURandomPos@@AEAUGeomQuery@@W4EGeomForm@@@Z 0000000035058780 f   physarea.obj
 0001:00057f40       ?GetStatus@CPhysArea@@UEBAHPEAUpe_status@@@Z 0000000035058f40 f   physarea.obj
 0001:00058b80       ?resize@?$DynArray@UGeomQuery@@HU?$SmallDynStorage@UGeomQuery@@HUStandardAlloc@NAlloc@@@NArray@@@@QEAAXH@Z 0000000035059b80 f i physarea.obj
 0001:00058d70       ??0GeomQuery@@QEAA@AEBU0@@Z 0000000035059d70 f i physarea.obj
 0001:00058dc0       ?init@?$DynArray@UGeomQuery@@HU?$SmallDynStorage@UGeomQuery@@HUStandardAlloc@NAlloc@@@NArray@@@@KAPEAUGeomQuery@@U?$Array@UGeomQuery@@HU?$ArrayStorage@UGeomQuery@@H@NArray@@@@PEBU2@@Z 0000000035059dc0 f i physarea.obj
 0001:00058e70       ?ComputeExtent@CPhysArea@@UEBAMAEAUGeomQuery@@W4EGeomForm@@@Z 0000000035059e70 f   physarea.obj
 0001:00059020       ?CleanupGlobalState@CPhysicalEntity@@SAXXZ 000000003505a020 f   physicalentity.obj
 0001:00059090       ?UpdatePartIdmatBreakable@CPhysicalEntity@@QEAAXHH@Z 000000003505a090 f   physicalentity.obj
 0001:00059400       ?RemoveCollider@CPhysicalEntity@@UEAAHPEAV1@_N@Z 000000003505a400 f   physicalentity.obj
 0001:000594c0       ?GetMemoryStatistics@CPhysicalEntity@@UEBAXPEAVICrySizer@@@Z 000000003505a4c0 f   physicalentity.obj
 0001:000597e0       ?GetStateSnapshotTxt@CPhysicalEntity@@UEAAHPEADHM@Z 000000003505a7e0 f   physicalentity.obj
 0001:00059810       ?SetStateFromSnapshotTxt@CPhysicalEntity@@UEAAXPEBDH@Z 000000003505a810 f   physicalentity.obj
 0001:00059850       ?ReleasePartPlaceholder@CPhysicalEntity@@QEAAPEAVCPhysicalPlaceholder@@H@Z 000000003505a850 f   physicalentity.obj
 0001:00059970       ??$ReallocateList@USPartInfo@@@@YAPEAUSPartInfo@@AEAPEAU0@HH_N1@Z 000000003505a970 f i physicalentity.obj
 0001:00059a50       ??$SignalEvent@UEventPhysUpdateMesh@@@CPhysicalWorld@@QEAAHPEAUEventPhysUpdateMesh@@H@Z 000000003505aa50 f i physicalentity.obj
 0001:00059ae0       ??$SignalEvent@UEventPhysCreateEntityPart@@@CPhysicalWorld@@QEAAHPEAUEventPhysCreateEntityPart@@H@Z 000000003505aae0 f i physicalentity.obj
 0001:00059b70       ??$SignalEvent@UEventPhysRemoveEntityParts@@@CPhysicalWorld@@QEAAHPEAUEventPhysRemoveEntityParts@@H@Z 000000003505ab70 f i physicalentity.obj
 0001:00059c00       ??$SignalEvent@UEventPhysRevealEntityPart@@@CPhysicalWorld@@QEAAHPEAUEventPhysRevealEntityPart@@H@Z 000000003505ac00 f i physicalentity.obj
 0001:00059c90       ??$SignalEvent@UEventPhysJointBroken@@@CPhysicalWorld@@QEAAHPEAUEventPhysJointBroken@@H@Z 000000003505ac90 f i physicalentity.obj
 0001:00059d20       ??0CPhysicalEntity@@QEAA@PEAVCPhysicalWorld@@@Z 000000003505ad20 f   physicalentity.obj
 0001:00059ec0       ?GetMaxTimeStep@CPhysicalEntity@@UEAAMM@Z 000000003505aec0 f i physicalentity.obj
 0001:00059ec0       ?GetLastTimeStep@CPhysicalEntity@@UEAAMM@Z 000000003505aec0 f i livingentity.obj
 0001:00059ed0       ??1CPhysicalEntity@@UEAA@XZ 000000003505aed0 f   physicalentity.obj
 0001:0005a1f0       ?AddRef@CPhysicalEntity@@UEAAHXZ 000000003505b1f0 f   physicalentity.obj
 0001:0005a260       ?Release@CPhysicalEntity@@UEAAHXZ 000000003505b260 f   physicalentity.obj
 0001:0005a2e0       ?GetRigidBody@CPhysicalEntity@@UEAAPEAVRigidBody@@HH@Z 000000003505b2e0 f   physicalentity.obj
 0001:0005a350       ?IsPointInside@CPhysicalEntity@@UEBAHU?$Vec3_tpl@M@@@Z 000000003505b350 f   physicalentity.obj
 0001:0005a6e0       ?AlertNeighbourhoodND@CPhysicalEntity@@UEAAXH@Z 000000003505b6e0 f   physicalentity.obj
 0001:0005aa20       ?AddCollider@CPhysicalEntity@@UEAAHPEAV1@@Z 000000003505ba20 f   physicalentity.obj
 0001:0005ac10       ?FillGeomParams@@YAXAEAUpe_geomparams@@AEAUgeom@@@Z 000000003505bc10 f i physicalentity.obj
 0001:0005aca0       ?AABB_OBB@Overlap@@YA_NAEBUAABB@@AEBU?$Vec3_tpl@M@@AEBU?$OBB_tpl@M@@@Z 000000003505bca0 f i physicalentity.obj
 0001:0005b470       ?validate@pe_params_pos@@QEAA_NPEBDPEAUILog@@AEBU?$Vec3_tpl@M@@PEAUIPhysRenderer@@PEAXHH@Z 000000003505c470 f i physicalentity.obj
 0001:0005b8b0       ?validate@pe_params_bbox@@QEAA_NPEBDPEAUILog@@AEBU?$Vec3_tpl@M@@PEAUIPhysRenderer@@PEAXHH@Z 000000003505c8b0 f i physicalentity.obj
 0001:0005bb20       ??0pe_params_part@@QEAA@XZ 000000003505cb20 f i physicalentity.obj
 0001:0005bc30       ?validate@pe_params_part@@QEAA_NPEBDPEAUILog@@AEBU?$Vec3_tpl@M@@PEAUIPhysRenderer@@PEAXHH@Z 000000003505cc30 f i physicalentity.obj
 0001:0005c070       ??0pe_simulation_params@@QEAA@XZ 000000003505d070 f i physicalentity.obj
 0001:0005c150       ??0pe_params_structural_joint@@QEAA@XZ 000000003505d150 f i physicalentity.obj
 0001:0005c290       ??0pe_params_softbody@@QEAA@XZ 000000003505d290 f i physicalentity.obj
 0001:0005c430       ??0pe_action_add_constraint@@QEAA@XZ 000000003505d430 f i physicalentity.obj
 0001:0005c530       ??4pe_geomparams@@QEAAAEAU0@AEBU0@@Z 000000003505d530 f i physicalentity.obj
 0001:0005c5c0       ?validate@pe_geomparams@@QEAA_NPEBDPEAUILog@@AEBU?$Vec3_tpl@M@@PEAUIPhysRenderer@@PEAXHH@Z 000000003505d5c0 f i physicalentity.obj
 0001:0005caf0       ?RepositionParts@CPhysicalEntity@@QEAAXXZ 000000003505daf0 f   physicalentity.obj
 0001:0005ccc0       ?AllocStructureInfo@CPhysicalEntity@@QEAAXXZ 000000003505dcc0 f   physicalentity.obj
 0001:0005cda0       ??0?$Matrix34_tpl@M@@QEAA@AEBU?$Vec3_tpl@M@@AEBU?$Quat_tpl@M@@0@Z 000000003505dda0 f i physicalentity.obj
 0001:0005cf50       ?invert@?$Diag33_tpl@M@@QEAAAEAU1@XZ 000000003505df50 f i physicalentity.obj
 0001:0005cfb0       ??$OnEvent@UEventPhysUpdateMesh@@@CPhysicalWorld@@QEAAHIPEAUEventPhysUpdateMesh@@PEAPEAU1@@Z 000000003505dfb0 f i physicalentity.obj
 0001:0005d080       ??$OnEvent@UEventPhysCreateEntityPart@@@CPhysicalWorld@@QEAAHIPEAUEventPhysCreateEntityPart@@PEAPEAU1@@Z 000000003505e080 f i physicalentity.obj
 0001:0005d150       ??$OnEvent@UEventPhysRemoveEntityParts@@@CPhysicalWorld@@QEAAHIPEAUEventPhysRemoveEntityParts@@PEAPEAU1@@Z 000000003505e150 f i physicalentity.obj
 0001:0005d260       ??$OnEvent@UEventPhysRevealEntityPart@@@CPhysicalWorld@@QEAAHIPEAUEventPhysRevealEntityPart@@PEAPEAU1@@Z 000000003505e260 f i physicalentity.obj
 0001:0005d360       ??$OnEvent@UEventPhysJointBroken@@@CPhysicalWorld@@QEAAHIPEAUEventPhysJointBroken@@PEAPEAU1@@Z 000000003505e360 f i physicalentity.obj
 0001:0005d430       ??$ReallocateList@Uplane@primitives@@@@YAPEAUplane@primitives@@AEAPEAU01@HH_N1@Z 000000003505e430 f i physicalentity.obj
 0001:0005d520       ??$ReallocateList@USSkelInfo@@@@YAPEAUSSkelInfo@@AEAPEAU0@HH_N1@Z 000000003505e520 f i physicalentity.obj
 0001:0005d610       ??$ReallocateList@Ubox@primitives@@@@YAPEAUbox@primitives@@AEAPEAU01@HH_N1@Z 000000003505e610 f i physicalentity.obj
 0001:0005d610       ??$ReallocateList@Ubop_newtri@@@@YAPEAUbop_newtri@@AEAPEAU0@HH_N1@Z 000000003505e610 f i boolean3d.obj
 0001:0005d6f0       ?GetBBox@CBoxGeom@@UEAAXPEAUbox@primitives@@@Z 000000003505e6f0 f i physicalentity.obj
 0001:0005d700       ?GetBVTree@CBoxGeom@@UEAAPEAVCBVTree@@XZ 000000003505e700 f i physicalentity.obj
 0001:0005d710       ?SetData@CBoxGeom@@UEAAXPEBUprimitive@primitives@@@Z 000000003505e710 f i physicalentity.obj
 0001:0005d720       ?GetCenter@CBoxGeom@@UEAA?AU?$Vec3_tpl@M@@XZ 000000003505e720 f i physicalentity.obj
 0001:0005d740       ?GetSizeFast@CBoxGeom@@UEAAHXZ 000000003505e740 f i physicalentity.obj
 0001:0005d750       ?GetVolume@CBoxGeom@@UEAAMXZ 000000003505e750 f i physicalentity.obj
 0001:0005d770       ?GetPrimitive@CBoxGeom@@UEAAHHPEAUprimitive@primitives@@@Z 000000003505e770 f i physicalentity.obj
 0001:0005d7f0       ??_GCBoxGeom@@UEAAPEAXI@Z  000000003505e7f0 f i physicalentity.obj
 0001:0005d7f0       ??_ECBoxGeom@@UEAAPEAXI@Z  000000003505e7f0 f i physicalentity.obj
 0001:0005d850       ?GetType@CHeightfieldBV@@UEAAHXZ 000000003505e850 f i waterman.obj
 0001:0005d850       ?GetType@CSphereGeom@@UEAAHXZ 000000003505e850 f i physicalentity.obj
 0001:0005d850       ?GetType@CLivingEntity@@UEBA?AW4pe_type@@XZ 000000003505e850 f i livingentity.obj
 0001:0005d860       ?GetBBox@CSphereGeom@@UEAAXPEAUbox@primitives@@@Z 000000003505e860 f i physicalentity.obj
 0001:0005d870       ?GetBVTree@CSphereGeom@@UEAAPEAVCBVTree@@XZ 000000003505e870 f i physicalentity.obj
 0001:0005d880       ?GetPrimitive@CSphereGeom@@UEAAHHPEAUprimitive@primitives@@@Z 000000003505e880 f i physicalentity.obj
 0001:0005d8b0       ?SetData@CSphereGeom@@UEAAXPEBUprimitive@primitives@@@Z 000000003505e8b0 f i physicalentity.obj
 0001:0005d8c0       ?GetSizeFast@CSphereGeom@@UEAAHXZ 000000003505e8c0 f i physicalentity.obj
 0001:0005d8d0       ?GetVolume@CSphereGeom@@UEAAMXZ 000000003505e8d0 f i physicalentity.obj
 0001:0005d900       ??_GCSphereGeom@@UEAAPEAXI@Z 000000003505e900 f i physicalentity.obj
 0001:0005d900       ??_ECSphereGeom@@UEAAPEAXI@Z 000000003505e900 f i physicalentity.obj
 0001:0005d960       ??_GCPhysicalEntity@@UEAAPEAXI@Z 000000003505e960 f i physicalentity.obj
 0001:0005d960       ??_ECPhysicalEntity@@UEAAPEAXI@Z 000000003505e960 f i physicalentity.obj
 0001:0005d990       ?GetParams@CPhysicalEntity@@UEBAHPEAUpe_params@@@Z 000000003505e990 f   physicalentity.obj
 0001:0005e420       ?AddGeometry@CPhysicalEntity@@UEAAHPEAUphys_geometry@@PEAUpe_geomparams@@HH@Z 000000003505f420 f   physicalentity.obj
 0001:0005f1b0       ?RemoveGeometry@CPhysicalEntity@@UEAAXHH@Z 00000000350601b0 f   physicalentity.obj
 0001:0005f9a0       ?RemoveBrokenParent@CPhysicalEntity@@QEAAXHH@Z 00000000350609a0 f   physicalentity.obj
 0001:0005fbe0       ?MapHitPointFromParent@CPhysicalEntity@@QEAAHHAEBU?$Vec3_tpl@M@@@Z 0000000035060be0 f   physicalentity.obj
 0001:000602b0       ?OnContactResolved@CPhysicalEntity@@UEAAXPEAUentity_contact@@HH@Z 00000000350612b0 f   physicalentity.obj
 0001:000615d0       ?TouchesSphere@CPhysicalEntity@@QEAAHAEBU?$Vec3_tpl@M@@M@Z 00000000350625d0 f   physicalentity.obj
 0001:00061cb0       ?MakeDeformable@CPhysicalEntity@@QEAA_NHHM@Z 0000000035062cb0 f   physicalentity.obj
 0001:000636c0       ?UpdateDeformablePart@CPhysicalEntity@@QEAAXH@Z 00000000350646c0 f   physicalentity.obj
 0001:00064640       ?_Assign@?$CryStringT@D@@IEAAXPEBD_K@Z 0000000035065640 f i physicalentity.obj
 0001:00064720       ?ComputeBBox@CPhysicalEntity@@UEAAXPEAU?$Vec3_tpl@M@@H@Z 0000000035065720 f   physicalentity.obj
 0001:00065700       ?Action@CPhysicalEntity@@UEAAHPEAUpe_action@@H@Z 0000000035066700 f   physicalentity.obj
 0001:000680f0       ?OccupiesEntityGridSquare@CPhysicalEntity@@QEAA_NAEBUAABB@@@Z 00000000350690f0 f   physicalentity.obj
 0001:00068990       ?DrawHelperInformation@CPhysicalEntity@@UEAAXPEAUIPhysRenderer@@H@Z 0000000035069990 f   physicalentity.obj
 0001:0006aa10       ?CapsulizePart@CPhysicalEntity@@QEAAHH@Z 000000003506ba10 f   physicalentity.obj
 0001:0006cea0       ?UpdateStructure@CPhysicalEntity@@QEAAHMPEAUpe_explosion@@HU?$Vec3_tpl@M@@@Z 000000003506dea0 f   physicalentity.obj
 0001:0007b8c0       ?GenerateJoints@CPhysicalEntity@@QEAAHXZ 000000003507c8c0 f   physicalentity.obj
 0001:0007d400       ?SetParams@CPhysicalEntity@@UEAAHPEAUpe_params@@H@Z 000000003507e400 f   physicalentity.obj
 0001:00080460       ?GetStateSnapshot@CPhysicalEntity@@UEAAHV?$CSerializeWrapper@UISerialize@@@@MH@Z 0000000035081460 f   physicalentity.obj
 0001:00080ad0       ?SetStateFromSnapshot@CPhysicalEntity@@UEAAHV?$CSerializeWrapper@UISerialize@@@@H@Z 0000000035081ad0 f   physicalentity.obj
 0001:000811e0       ??$GetExtent@VCPhysicalEntity@@@GeomQuery@@QEAAMPEAVCPhysicalEntity@@W4EGeomForm@@@Z 00000000350821e0 f i physicalentity.obj
 0001:00081260       ?GetStatus@CPhysicalEntity@@UEBAHPEAUpe_status@@@Z 0000000035082260 f   physicalentity.obj
 0001:00081dd0       ?GetRandomPos@CPhysicalEntity@@UEBAXAEAURandomPos@@AEAUGeomQuery@@W4EGeomForm@@@Z 0000000035082dd0 f   physicalentity.obj
 0001:00082210       ?ComputeExtent@CPhysicalEntity@@UEBAMAEAUGeomQuery@@W4EGeomForm@@@Z 0000000035083210 f   physicalentity.obj
 0001:000822d0       ?IsPlaceholder@CPhysicalWorld@@QEAAHPEBVCPhysicalPlaceholder@@@Z 00000000350832d0 f i physicalplaceholder.obj
 0001:00082390       ?GetWorld@CPhysicalPlaceholder@@UEBAPEAUIPhysicalWorld@@XZ 0000000035083390 f   physicalplaceholder.obj
 0001:000824d0       ?GetEntity@CPhysicalPlaceholder@@UEAAPEAVCPhysicalEntity@@XZ 00000000350834d0 f   physicalplaceholder.obj
 0001:00082630       ?GetType@CPhysicalPlaceholder@@UEBA?AW4pe_type@@XZ 0000000035083630 f   physicalplaceholder.obj
 0001:00082670       ?GetParams@CPhysicalPlaceholder@@UEBAHPEAUpe_params@@@Z 0000000035083670 f   physicalplaceholder.obj
 0001:000826f0       ?GetStatus@CPhysicalPlaceholder@@UEBAHPEAUpe_status@@@Z 00000000350836f0 f   physicalplaceholder.obj
 0001:00082740       ?Action@CPhysicalPlaceholder@@UEAAHPEAUpe_action@@H@Z 0000000035083740 f   physicalplaceholder.obj
 0001:000827f0       ?AddGeometry@CPhysicalPlaceholder@@UEAAHPEAUphys_geometry@@PEAUpe_geomparams@@HH@Z 00000000350837f0 f   physicalplaceholder.obj
 0001:00082840       ?RemoveGeometry@CPhysicalPlaceholder@@UEAAXHH@Z 0000000035083840 f   physicalplaceholder.obj
 0001:00082880       ?GetStateSnapshot@CPhysicalPlaceholder@@UEAAHAEAVCStream@@MH@Z 0000000035083880 f   physicalplaceholder.obj
 0001:000828d0       ?GetStateSnapshot@CPhysicalPlaceholder@@UEAAHV?$CSerializeWrapper@UISerialize@@@@MH@Z 00000000350838d0 f   physicalplaceholder.obj
 0001:00082910       ?SetStateFromSnapshot@CPhysicalPlaceholder@@UEAAHAEAVCStream@@H@Z 0000000035083910 f   physicalplaceholder.obj
 0001:00082950       ?SetStateFromSnapshot@CPhysicalPlaceholder@@UEAAHV?$CSerializeWrapper@UISerialize@@@@H@Z 0000000035083950 f   physicalplaceholder.obj
 0001:00082980       ?SetStateFromTypedSnapshot@CPhysicalPlaceholder@@UEAAHV?$CSerializeWrapper@UISerialize@@@@HH@Z 0000000035083980 f   physicalplaceholder.obj
 0001:000829d0       ?PostSetStateFromSnapshot@CPhysicalPlaceholder@@UEAAHXZ 00000000350839d0 f   physicalplaceholder.obj
 0001:000829f0       ?GetStateSnapshotTxt@CPhysicalPlaceholder@@UEAAHPEADHM@Z 00000000350839f0 f   physicalplaceholder.obj
 0001:00082a40       ?SetStateFromSnapshotTxt@CPhysicalPlaceholder@@UEAAXPEBDH@Z 0000000035083a40 f   physicalplaceholder.obj
 0001:00082a80       ?GetStateChecksum@CPhysicalPlaceholder@@UEAAIXZ 0000000035083a80 f   physicalplaceholder.obj
 0001:00082aa0       ?SetNetworkAuthority@CPhysicalPlaceholder@@UEAAXHH@Z 0000000035083aa0 f   physicalplaceholder.obj
 0001:00082ae0       ?Step@CPhysicalPlaceholder@@UEAAHM@Z 0000000035083ae0 f   physicalplaceholder.obj
 0001:00082b10       ?StartStep@CPhysicalPlaceholder@@UEAAXM@Z 0000000035083b10 f   physicalplaceholder.obj
 0001:00082b40       ?StepBack@CPhysicalPlaceholder@@UEAAXM@Z 0000000035083b40 f   physicalplaceholder.obj
 0001:00082b70       ??$SignalEvent@UEventPhysStateChange@@@CPhysicalWorld@@QEAAHPEAUEventPhysStateChange@@H@Z 0000000035083b70 f i physicalplaceholder.obj
 0001:00082c00       ??$OnEvent@UEventPhysStateChange@@@CPhysicalWorld@@QEAAHIPEAUEventPhysStateChange@@PEAPEAU1@@Z 0000000035083c00 f i physicalplaceholder.obj
 0001:00082ce0       ?SetParams@CPhysicalPlaceholder@@UEAAHPEAUpe_params@@H@Z 0000000035083ce0 f   physicalplaceholder.obj
 0001:00082fe0       ??_EIThreadTask@@UEAAPEAXI@Z 0000000035083fe0 f i physicalworld.obj
 0001:00082fe0       ??_GIThreadTask@@UEAAPEAXI@Z 0000000035083fe0 f i physicalworld.obj
 0001:00083010       ??Ape_entgrid@@QEAAAEAHI@Z 0000000035084010 f i physicalworld.obj
 0001:000830b0       ?GetGridSize@@YAHAEAUpe_entgrid@@AEBU?$Vec2_tpl@H@@@Z 00000000350840b0 f i physicalworld.obj
 0001:00083190       ?GetTmpEntList@CPhysicalWorld@@QEAAHAEAPEAPEAVCPhysicalEntity@@H@Z 0000000035084190 f i physicalworld.obj
 0001:00083230       ?CryLog@@YAXPEBDZZ         0000000035084230 f i physicalworld.obj
 0001:00083290       ?CryLogAlways@@YAXPEBDZZ   0000000035084290 f i physicalworld.obj
 0001:000832f0       ?IsEnd@CPhysicalEntityIt@CPhysicalWorld@@UEAA_NXZ 00000000350842f0 f   physicalworld.obj
 0001:00083300       ?Next@CPhysicalEntityIt@CPhysicalWorld@@UEAAPEAUIPhysicalEntity@@XZ 0000000035084300 f   physicalworld.obj
 0001:000833c0       ?This@CPhysicalEntityIt@CPhysicalWorld@@UEAAPEAUIPhysicalEntity@@XZ 00000000350843c0 f   physicalworld.obj
 0001:000833f0       ?MoveFirst@CPhysicalEntityIt@CPhysicalWorld@@UEAAXXZ 00000000350843f0 f   physicalworld.obj
 0001:00083440       ?GetEntityProfileType@@YAHPEAVCPhysicalEntity@@@Z 0000000035084440 f   physicalworld.obj
 0001:00083520       ?Cleanup@CPhysicalWorld@@UEAAXXZ 0000000035084520 f   physicalworld.obj
 0001:00083550       ?DeactivateOnDemandGrid@CPhysicalWorld@@UEAAXXZ 0000000035084550 f   physicalworld.obj
 0001:00083640       ?SetSurfaceParameters@CPhysicalWorld@@UEAAHHMMI@Z 0000000035084640 f   physicalworld.obj
 0001:000836c0       ?GetSurfaceParameters@CPhysicalWorld@@UEAAHHAEAM0AEAI@Z 00000000350846c0 f   physicalworld.obj
 0001:00083700       ?SetSurfaceParameters@CPhysicalWorld@@UEAAHHMMMMMMI@Z 0000000035084700 f   physicalworld.obj
 0001:00083790       ?GetSurfaceParameters@CPhysicalWorld@@UEAAHHAEAM00000AEAI@Z 0000000035084790 f   physicalworld.obj
 0001:00083820       ?CleanseEventsQueue@CPhysicalWorld@@QEAAXXZ 0000000035084820 f   physicalworld.obj
 0001:000838d0       ?PatchEventsQueue@CPhysicalWorld@@QEAAXPEAUIPhysicalEntity@@PEAXH@Z 00000000350848d0 f   physicalworld.obj
 0001:00083980       ?GetFreeEntId@CPhysicalWorld@@QEAAHXZ 0000000035084980 f   physicalworld.obj
 0001:00083a70       ?GetPhysicalEntityId@CPhysicalWorld@@UEAAHPEAUIPhysicalEntity@@@Z 0000000035084a70 f   physicalworld.obj
 0001:00083a90       ?GetPhysicalEntityById@CPhysicalWorld@@UEAAPEAUIPhysicalEntity@@H@Z 0000000035084a90 f   physicalworld.obj
 0001:00083f50       ?GroupByOuterEntity@@YAXPEAPEAVCPhysicalEntity@@HH@Z 0000000035084f50 f   physicalworld.obj
 0001:00084040       ?ScheduleForStep@CPhysicalWorld@@QEAAXPEAVCPhysicalEntity@@M@Z 0000000035085040 f   physicalworld.obj
 0001:000840c0       ?Stop@SPhysTask@@UEAAXXZ   00000000350850c0 f   physicalworld.obj
 0001:000840e0       ?ProcessNextEngagedIndependentEntity@CPhysicalWorld@@QEAAXH@Z 00000000350850e0 f   physicalworld.obj
 0001:00084250       ?ProcessNextIndependentEntity@CPhysicalWorld@@QEAAXMHH@Z 0000000035085250 f   physicalworld.obj
 0001:00084400       ?ChangeEntitySimClass@CPhysicalWorld@@QEAAHPEAVCPhysicalEntity@@@Z 0000000035085400 f   physicalworld.obj
 0001:000846d0       ?UnmarkEntityAsDeforming@CPhysicalWorld@@QEAAXPEAVCPhysicalEntity@@@Z 00000000350856d0 f   physicalworld.obj
 0001:00084760       ?PurgeDeletedEntities@CPhysicalWorld@@UEAAXXZ 0000000035085760 f   physicalworld.obj
 0001:00084980       ?DrawEntityHelperInformation@CPhysicalWorld@@UEAAXPEAUIPhysRenderer@@HH@Z 0000000035085980 f   physicalworld.obj
 0001:000849c0       ??_EIGeomManager@@UEAAPEAXI@Z 00000000350859c0 f i physicalworld.obj
 0001:000849c0       ??_GIGeomManager@@UEAAPEAXI@Z 00000000350859c0 f i physicalworld.obj
 0001:000849f0       ??_GICryUnknown@@MEAAPEAXI@Z 00000000350859f0 f i CryPhysics.obj
 0001:000849f0       ??_GIPhysUtils@@UEAAPEAXI@Z 00000000350859f0 f i physicalworld.obj
 0001:000849f0       ??_GCEngineModule_CryPhysics@@MEAAPEAXI@Z 00000000350859f0 f i CryPhysics.obj
 0001:000849f0       ??_EICryUnknown@@MEAAPEAXI@Z 00000000350859f0 f i CryPhysics.obj
 0001:000849f0       ??_ECEngineModule_CryPhysics@@MEAAPEAXI@Z 00000000350859f0 f i CryPhysics.obj
 0001:000849f0       ??_EIPhysUtils@@UEAAPEAXI@Z 00000000350859f0 f i physicalworld.obj
 0001:00084a20       ??_GIPhysicalWorld@@UEAAPEAXI@Z 0000000035085a20 f i physicalworld.obj
 0001:00084a20       ??_EIPhysicalWorld@@UEAAPEAXI@Z 0000000035085a20 f i physicalworld.obj
 0001:00084a50       ?AddEntityProfileInfo@CPhysicalWorld@@QEAAXPEAVCPhysicalEntity@@H@Z 0000000035085a50 f   physicalworld.obj
 0001:00084cc0       ?AddEventClient@CPhysicalWorld@@UEAAXHP6AHPEBUEventPhys@@@ZHM@Z 0000000035085cc0 f   physicalworld.obj
 0001:00084db0       ?RemoveEventClient@CPhysicalWorld@@UEAAHHP6AHPEBUEventPhys@@@ZH@Z 0000000035085db0 f   physicalworld.obj
 0001:00084e50       ?AllocEvent@CPhysicalWorld@@QEAAPEAUEventPhys@@HH@Z 0000000035085e50 f   physicalworld.obj
 0001:00084f30       ?GetPumpLoggedEventsTicks@CPhysicalWorld@@UEAAIXZ 0000000035085f30 f   physicalworld.obj
 0001:00084f50       ?ClearLoggedEvents@CPhysicalWorld@@UEAAXXZ 0000000035085f50 f   physicalworld.obj
 0001:00085010       ?RemoveExplosionShape@CPhysicalWorld@@UEAAXH@Z 0000000035086010 f   physicalworld.obj
 0001:00085130       ?GetExplosionShape@CPhysicalWorld@@QEAAPEAUIGeometry@@MHAEAMAEAH@Z 0000000035086130 f   physicalworld.obj
 0001:000853b0       ?GetWaterManagerParams@CPhysicalWorld@@UEAAHPEAUpe_params@@@Z 00000000350863b0 f   physicalworld.obj
 0001:000853d0       ?GetWatermanStatus@CPhysicalWorld@@UEAAHPEAUpe_status@@@Z 00000000350863d0 f   physicalworld.obj
 0001:000853f0       ??$ReallocateList@H@@YAPEAHAEAPEAHHH_N1@Z 00000000350863f0 f i physicalworld.obj
 0001:000854d0       ??$SignalEvent@UEventPhysEntityDeleted@@@CPhysicalWorld@@QEAAHPEAUEventPhysEntityDeleted@@H@Z 00000000350864d0 f i physicalworld.obj
 0001:00085560       ?UnregisterAllCracks@CGeomManager@@UEAAXP6AXPEAUIGeometry@@@Z@Z 0000000035086560 f i physicalworld.obj
 0001:000855e0       ?ReleaseGeomsImmediately@CGeomManager@@UEAAX_N@Z 00000000350865e0 f i physicalworld.obj
 0001:000855f0       ?CreateMesh@CGeomManager@@UEAAPEAUIGeometry@@V?$strided_pointer@$$CBU?$Vec3_tpl@M@@@@V?$strided_pointer@G@@PEADPEAHHHMHHM@Z 00000000350865f0 f i physicalworld.obj
 0001:00085690       ??_ECGeomManager@@UEAAPEAXI@Z 0000000035086690 f i physicalworld.obj
 0001:00085690       ??_GCGeomManager@@UEAAPEAXI@Z 0000000035086690 f i physicalworld.obj
 0001:000856e0       ?AllocateGrid@@YAXAEAUpe_entgrid@@AEBU?$Vec2_tpl@H@@@Z 00000000350866e0 f i physicalworld.obj
 0001:000857c0       ?GetTaskInfo@SPhysTask@@UEAAPEAUSThreadTaskInfo@@XZ 00000000350867c0 f i physicalworld.obj
 0001:000857d0       ?getPODcell@CPhysicalWorld@@QEAAPEAUpe_PODcell@@HH@Z 00000000350867d0 f i physicalworld.obj
 0001:000858d0       ?AddRef@CPhysicalEntityIt@CPhysicalWorld@@UEAAXXZ 00000000350868d0 f i physicalworld.obj
 0001:000858e0       ?Release@CPhysicalEntityIt@CPhysicalWorld@@UEAAXXZ 00000000350868e0 f i physicalworld.obj
 0001:00085900       ?Init@CPhysicalWorld@@UEAAXXZ 0000000035086900 f   physicalworld.obj
 0001:00085fc0       ?GetHeightfieldData@CPhysicalWorld@@UEAAPEAUIPhysicalEntity@@PEAUheightfield@primitives@@@Z 0000000035086fc0 f   physicalworld.obj
 0001:00086080       ?AddRefEntInPODGrid@CPhysicalWorld@@UEAAHPEAUIPhysicalEntity@@PEBU?$Vec3_tpl@M@@@Z 0000000035087080 f   physicalworld.obj
 0001:000862e0       ?GetPODGridCellBBox@CPhysicalWorld@@QEAAXHHAEAU?$Vec3_tpl@M@@0@Z 00000000350872e0 f   physicalworld.obj
 0001:00086400       ?CreatePhysicalPlaceholder@CPhysicalWorld@@UEAAPEAUIPhysicalEntity@@W4pe_type@@PEAUpe_params@@PEAXHH@Z 0000000035087400 f   physicalworld.obj
 0001:00086830       ??_ECPhysicalPlaceholder@@UEAAPEAXI@Z 0000000035087830 f i physicalworld.obj
 0001:000868b0       ?ReserveEntityCount@CPhysicalWorld@@UEAAHH@Z 00000000350878b0 f   physicalworld.obj
 0001:00086c50       ?SetPhysicalEntityId@CPhysicalWorld@@UEAAHPEAUIPhysicalEntity@@HHH@Z 0000000035087c50 f   physicalworld.obj
 0001:00086ef0       ?ReallocTmpEntList@CPhysicalWorld@@QEAAHAEAPEAPEAVCPhysicalEntity@@HH@Z 0000000035087ef0 f   physicalworld.obj
 0001:00087000       ?UpdateDeformingEntities@CPhysicalWorld@@UEAAXM@Z 0000000035088000 f   physicalworld.obj
 0001:000871b0       ?ProcessIslandSolverResults@CPhysicalWorld@@QEAAXHHMMHMAEAHPEAPEAUentity_contact@@HHH_J@Z 00000000350881b0 f   physicalworld.obj
 0001:00087790       ?ProcessNextEntityIsland@CPhysicalWorld@@QEAAXMHHAEAHH@Z 0000000035088790 f   physicalworld.obj
 0001:00087f80       ?ProcessNextLivingEntity@CPhysicalWorld@@QEAAXMHH@Z 0000000035088f80 f   physicalworld.obj
 0001:00088720       ?ProcessBreakingEntities@CPhysicalWorld@@QEAAXM@Z 0000000035089720 f   physicalworld.obj
 0001:00088890       ?ThreadProc@CPhysicalWorld@@QEAAXHPEAUSPhysTask@@@Z 0000000035089890 f   physicalworld.obj
 0001:00088ab0       ?DetachEntityGridThunks@CPhysicalWorld@@QEAAXPEAVCPhysicalPlaceholder@@@Z 0000000035089ab0 f   physicalworld.obj
 0001:00088d20       ?SortThunks@CPhysicalWorld@@QEAAXXZ 0000000035089d20 f   physicalworld.obj
 0001:00089470       ?IsAffectedByExplosion@CPhysicalWorld@@UEAAMPEAUIPhysicalEntity@@PEAU?$Vec3_tpl@M@@@Z 000000003508a470 f   physicalworld.obj
 0001:00089520       ?MarkEntityAsDeforming@CPhysicalWorld@@QEAAXPEAVCPhysicalEntity@@@Z 000000003508a520 f   physicalworld.obj
 0001:00089630       ?ResetDynamicEntities@CPhysicalWorld@@UEAAXXZ 000000003508a630 f   physicalworld.obj
 0001:000896d0       ?DestroyDynamicEntities@CPhysicalWorld@@UEAAXXZ 000000003508a6d0 f   physicalworld.obj
 0001:00089b50       ?DrawPhysicsHelperInformation@CPhysicalWorld@@UEAAXPEAUIPhysRenderer@@H@Z 000000003508ab50 f   physicalworld.obj
 0001:0008abc0       ?GetMemoryStatistics@CPhysicalWorld@@UEAAXPEAVICrySizer@@@Z 000000003508bbc0 f   physicalworld.obj
 0001:0008b320       ?AddFuncProfileInfo@CPhysicalWorld@@QEAAXPEBDH@Z 000000003508c320 f   physicalworld.obj
 0001:0008b520       ?PumpLoggedEvents@CPhysicalWorld@@UEAAXXZ 000000003508c520 f   physicalworld.obj
 0001:0008bbe0       ?AddExplosionShape@CPhysicalWorld@@UEAAHPEAUIGeometry@@MHM@Z 000000003508cbe0 f   physicalworld.obj
 0001:0008bee0       ?SetWaterManagerParams@CPhysicalWorld@@UEAAHPEAUpe_params@@@Z 000000003508cee0 f   physicalworld.obj
 0001:0008bf90       ?DestroyWaterManager@CPhysicalWorld@@UEAAXXZ 000000003508cf90 f   physicalworld.obj
 0001:0008bfd0       ?GetEntityMassAndCom@CPhysicalWorld@@UEAAXPEAUIPhysicalEntity@@AEAMAEAU?$Vec3_tpl@M@@@Z 000000003508cfd0 f   physicalworld.obj
 0001:0008c0c0       ?SerializeGarbageTypedSnapshot@CPhysicalWorld@@UEAAXV?$CSerializeWrapper@UISerialize@@@@HH@Z 000000003508d0c0 f   physicalworld.obj
 0001:0008c280       ?GetEntitiesIterator@CPhysicalWorld@@UEAAPEAUIPhysicalEntityIt@@XZ 000000003508d280 f   physicalworld.obj
 0001:0008c310       ?CryModuleCRTMalloc@@YAPEAX_K@Z 000000003508d310 f i physicalworld.obj
 0001:0008c380       ??_GCMultiThreadRefCount@@UEAAPEAXI@Z 000000003508d380 f i physicalworld.obj
 0001:0008c380       ??_GSThreadTaskInfo@@UEAAPEAXI@Z 000000003508d380 f i physicalworld.obj
 0001:0008c380       ??_ESThreadTaskInfo@@UEAAPEAXI@Z 000000003508d380 f i physicalworld.obj
 0001:0008c380       ??_ECMultiThreadRefCount@@UEAAPEAXI@Z 000000003508d380 f i physicalworld.obj
 0001:0008c3b0       ??_GSPhysTask@@UEAAPEAXI@Z 000000003508d3b0 f i physicalworld.obj
 0001:0008c3b0       ??_ESPhysTask@@UEAAPEAXI@Z 000000003508d3b0 f i physicalworld.obj
 0001:0008c3f0       ??_GITetrLattice@@UEAAPEAXI@Z 000000003508d3f0 f i tetrlattice.obj
 0001:0008c3f0       ??_GIPhysicalEntityIt@@UEAAPEAXI@Z 000000003508d3f0 f i physicalworld.obj
 0001:0008c3f0       ??_EIPhysicalEntityIt@@UEAAPEAXI@Z 000000003508d3f0 f i physicalworld.obj
 0001:0008c3f0       ??_GIBreakableGrid2d@@UEAAPEAXI@Z 000000003508d3f0 f i geoman.obj
 0001:0008c3f0       ??_EITetrLattice@@UEAAPEAXI@Z 000000003508d3f0 f i tetrlattice.obj
 0001:0008c3f0       ??_EIBreakableGrid2d@@UEAAPEAXI@Z 000000003508d3f0 f i geoman.obj
 0001:0008c3f0       ??_ECPhysicalEntityIt@CPhysicalWorld@@UEAAPEAXI@Z 000000003508d3f0 f i physicalworld.obj
 0001:0008c3f0       ??_GCPhysicalEntityIt@CPhysicalWorld@@UEAAPEAXI@Z 000000003508d3f0 f i physicalworld.obj
 0001:0008c420       ??0CPhysicalWorld@@QEAA@PEAUILog@@@Z 000000003508d420 f   physicalworld.obj
 0001:0008cb00       ?destroy@sp_counted_base@detail@boost@@UEAAXXZ 000000003508db00 f i CryPhysics.obj
 0001:0008cb00       ?Release@CTetrLattice@@UEAAXXZ 000000003508db00 f i tetrlattice.obj
 0001:0008cb00       ?Release@CBreakableGrid2d@@UEAAXXZ 000000003508db00 f i geoman.obj
 0001:0008cb00       ?Release@CPhysicalWorld@@UEAAXXZ 000000003508db00 f i physicalworld.obj
 0001:0008cb20       ?GetGeomManager@CPhysicalWorld@@UEAAPEAUIGeomManager@@XZ 000000003508db20 f i physicalworld.obj
 0001:0008cb30       ?GetPhysUtils@CPhysicalWorld@@UEAAPEAUIPhysUtils@@XZ 000000003508db30 f i physicalworld.obj
 0001:0008cb40       ?GetPhysVars@CPhysicalWorld@@UEAAPEAUPhysicsVars@@XZ 000000003508db40 f i physicalworld.obj
 0001:0008cb50       ?CreatePhysicalEntity@CPhysicalWorld@@UEAAPEAUIPhysicalEntity@@W4pe_type@@PEAUpe_params@@PEAXHH@Z 000000003508db50 f i physicalworld.obj
 0001:0008cb90       ?GetPhysicsTime@CPhysicalWorld@@UEAAMXZ 000000003508db90 f i physicalworld.obj
 0001:0008cba0       ?GetiPhysicsTime@CPhysicalWorld@@UEAAHXZ 000000003508dba0 f i physicalworld.obj
 0001:0008cbb0       ?SetPhysicsTime@CPhysicalWorld@@UEAAXM@Z 000000003508dbb0 f i physicalworld.obj
 0001:0008cbf0       ?SetiPhysicsTime@CPhysicalWorld@@UEAAXH@Z 000000003508dbf0 f i physicalworld.obj
 0001:0008cc10       ?SetSnapshotTime@CPhysicalWorld@@UEAAXMH@Z 000000003508dc10 f i physicalworld.obj
 0001:0008cc50       ?SetiSnapshotTime@CPhysicalWorld@@UEAAXHH@Z 000000003508dc50 f i physicalworld.obj
 0001:0008cc80       ?GetEntityCount@CPhysicalWorld@@UEAAHH@Z 000000003508dc80 f i physicalworld.obj
 0001:0008cc90       ?DeletePointer@CPhysicalWorld@@UEAAXPEAX@Z 000000003508dc90 f i physicalworld.obj
 0001:0008ccb0       ?SetPhysicsStreamer@CPhysicalWorld@@UEAAXPEAUIPhysicsStreamer@@@Z 000000003508dcb0 f i physicalworld.obj
 0001:0008ccc0       ?SetPhysicsEventClient@CPhysicalWorld@@UEAAXPEAUIPhysicsEventClient@@@Z 000000003508dcc0 f i physicalworld.obj
 0001:0008ccd0       ?GetLastEntityUpdateTime@CPhysicalWorld@@UEAAMPEAUIPhysicalEntity@@@Z 000000003508dcd0 f i physicalworld.obj
 0001:0008ccf0       ?GetInternalLock@CPhysicalWorld@@UEAAPECHH@Z 000000003508dcf0 f i physicalworld.obj
 0001:0008cd40       ?GetEntityProfileInfo@CPhysicalWorld@@UEAAHAEAPEAUphys_profile_info@@@Z 000000003508dd40 f i physicalworld.obj
 0001:0008cd60       ?GetFuncProfileInfo@CPhysicalWorld@@UEAAHAEAPEAUphys_profile_info@@@Z 000000003508dd60 f i physicalworld.obj
 0001:0008cd80       ?GetGroupProfileInfo@CPhysicalWorld@@UEAAHAEAPEAUphys_profile_info@@@Z 000000003508dd80 f i physicalworld.obj
 0001:0008cd90       ?GetJobProfileInfo@CPhysicalWorld@@UEAAHAEAPEAUphys_job_info@@@Z 000000003508dd90 f i physicalworld.obj
 0001:0008cda0       ?GetWaterMat@CPhysicalWorld@@UEAAHXZ 000000003508dda0 f i physicalworld.obj
 0001:0008cdb0       ?RemoveAllExplosionShapes@CPhysicalWorld@@UEAAXP6AXPEAUIGeometry@@@Z@Z 000000003508ddb0 f i physicalworld.obj
 0001:0008ce50       ?GetIWorld@CPhysicalWorld@@UEAAPEAUIPhysicalWorld@@XZ 000000003508de50 f i physicalworld.obj
 0001:0008ce60       ??$SignalEvent@UEventPhysEnvChange@@@CPhysicalWorld@@QEAAHPEAUEventPhysEnvChange@@H@Z 000000003508de60 f i physicalworld.obj
 0001:0008cef0       ??$SignalEvent@UEventPhysRWIResult@@@CPhysicalWorld@@QEAAHPEAUEventPhysRWIResult@@H@Z 000000003508def0 f i physicalworld.obj
 0001:0008cf80       ??$SignalEvent@UEventPhysPWIResult@@@CPhysicalWorld@@QEAAHPEAUEventPhysPWIResult@@H@Z 000000003508df80 f i physicalworld.obj
 0001:0008d010       ??_ECPhysicalWorld@@W7EAAPEAXI@Z 000000003508e010 f i physicalworld.obj
 0001:0008d020       ??_ECPhysicalWorld@@WBA@EAAPEAXI@Z 000000003508e020 f i physicalworld.obj
 0001:0008d030       ?CoverPolygonWithCircles@CPhysicalWorld@@UEAAHV?$strided_pointer@U?$Vec2_tpl@M@@@@H_NAEBU?$Vec2_tpl@M@@AEAPEAU3@AEAPEAMM@Z 000000003508e030 f i physicalworld.obj
 0001:0008d0a0       ?qhull@CPhysicalWorld@@UEAAHV?$strided_pointer@U?$Vec3_tpl@M@@@@HAEAPEAHP6APEAX_K@Z@Z 000000003508e0a0 f i physicalworld.obj
 0001:0008d0e0       ??$OnEvent@UEventPhysEnvChange@@@CPhysicalWorld@@QEAAHIPEAUEventPhysEnvChange@@PEAPEAU1@@Z 000000003508e0e0 f i physicalworld.obj
 0001:0008d1f0       ??$OnEvent@UEventPhysRWIResult@@@CPhysicalWorld@@QEAAHIPEAUEventPhysRWIResult@@PEAPEAU1@@Z 000000003508e1f0 f i physicalworld.obj
 0001:0008d2e0       ??$OnEvent@UEventPhysPWIResult@@@CPhysicalWorld@@QEAAHIPEAUEventPhysPWIResult@@PEAPEAU1@@Z 000000003508e2e0 f i physicalworld.obj
 0001:0008d3b0       ??$OnEvent@UEventPhysArea@@@CPhysicalWorld@@QEAAHIPEAUEventPhysArea@@PEAPEAU1@@Z 000000003508e3b0 f i physicalworld.obj
 0001:0008d480       ??$OnEvent@UEventPhysAreaChange@@@CPhysicalWorld@@QEAAHIPEAUEventPhysAreaChange@@PEAPEAU1@@Z 000000003508e480 f i physicalworld.obj
 0001:0008d560       ??$OnEvent@UEventPhysEntityDeleted@@@CPhysicalWorld@@QEAAHIPEAUEventPhysEntityDeleted@@PEAPEAU1@@Z 000000003508e560 f i physicalworld.obj
 0001:0008d630       ?RayWorldIntersection@CPhysicalWorld@@UEAAHAEBU?$Vec3_tpl@M@@0HIPEAUray_hit@@HPEAPEAUIPhysicalEntity@@HPEAXHPEBDPEAUray_hit_cached@@H@Z 000000003508e630 f i physicalworld.obj
 0001:0008d730       ?AddDeferredEvent@CPhysicalWorld@@UEAAPEAUEventPhys@@HPEAU2@@Z 000000003508e730 f i physicalworld.obj
 0001:0008da90       ?DeallocGThunksPool@CPhysicalWorld@@QEAAXXZ 000000003508ea90 f   physicalworld.obj
 0001:0008db10       ?SetHeightfieldData@CPhysicalWorld@@UEAAPEAUIPhysicalEntity@@PEBUheightfield@primitives@@PEAHH@Z 000000003508eb10 f   physicalworld.obj
 0001:0008e0c0       ?RegisterBBoxInPODGrid@CPhysicalWorld@@UEAAXPEBU?$Vec3_tpl@M@@@Z 000000003508f0c0 f   physicalworld.obj
 0001:0008e7d0       ?GetEntitiesAround@CPhysicalWorld@@QEAAHAEBU?$Vec3_tpl@M@@0AEAPEAPEAVCPhysicalEntity@@HPEAV3@HH@Z 000000003508f7d0 f   physicalworld.obj
 0001:000904d0       ?OnUpdate@SPhysTask@@UEAAXXZ 00000000350914d0 f   physicalworld.obj
 0001:000904e0       ??4SBreakRequest@@QEAAAEAU0@AEBU0@@Z 00000000350914e0 f i physicalworld.obj
 0001:00090750       ?ClonePhysGeomInEntity@CPhysicalWorld@@QEAAXPEAVCPhysicalEntity@@HPEAUIGeometry@@@Z 0000000035091750 f   physicalworld.obj
 0001:00090990       ?DeformEntityPart@CPhysicalWorld@@QEAAHPEAVCPhysicalEntity@@HPEAUpe_explosion@@PEAUgeom_world_data@@2H@Z 0000000035091990 f   physicalworld.obj
 0001:00091110       ?CalculateExplosionExposure@CPhysicalWorld@@UEAAMPEAUpe_explosion@@PEAUIPhysicalEntity@@@Z 0000000035092110 f   physicalworld.obj
 0001:00091760       ?CollideEntityWithBeam@CPhysicalWorld@@UEAAHPEAUIPhysicalEntity@@U?$Vec3_tpl@M@@1MPEAUray_hit@@@Z 0000000035092760 f   physicalworld.obj
 0001:00092130       ?CollideEntityWithPrimitive@CPhysicalWorld@@UEAAHPEAUIPhysicalEntity@@HPEAUprimitive@primitives@@U?$Vec3_tpl@M@@PEAUray_hit@@PEAUintersection_params@@@Z 0000000035093130 f   physicalworld.obj
 0001:00093310       ?RayTraceEntity@CPhysicalWorld@@UEAAHPEAUIPhysicalEntity@@U?$Vec3_tpl@M@@1PEAUray_hit@@PEAUpe_params_pos@@I@Z 0000000035094310 f   physicalworld.obj
 0001:000940b0       ?SavePhysicalEntityPtr@CPhysicalWorld@@UEAAXV?$CSerializeWrapper@UISerialize@@@@PEAUIPhysicalEntity@@@Z 00000000350950b0 f   physicalworld.obj
 0001:000941a0       ?LoadPhysicalEntityPtr@CPhysicalWorld@@UEAAPEAUIPhysicalEntity@@V?$CSerializeWrapper@UISerialize@@@@@Z 00000000350951a0 f   physicalworld.obj
 0001:000944b0       ?SetStateFromTypedSnapshot@CPhysicalEntity@@UEAAHV?$CSerializeWrapper@UISerialize@@@@HH@Z 00000000350954b0 f   physicalworld.obj
 0001:000946a0       ??$ReallocQueue@USBreakRequest@@@CPhysicalWorld@@QEAAXAEAPEAUSBreakRequest@@HAEAH11H@Z 00000000350956a0 f i physicalworld.obj
 0001:00094830       ??$ReallocQueue@USPwiRequest@@@CPhysicalWorld@@QEAAXAEAPEAUSPwiRequest@@HAEAH11H@Z 0000000035095830 f i physicalworld.obj
 0001:000949e0       ?GetEntitiesInBox@CPhysicalWorld@@UEAAHU?$Vec3_tpl@M@@0AEAPEAPEAUIPhysicalEntity@@HH@Z 00000000350959e0 f i physicalworld.obj
 0001:00094a40       ?AllocGThunksPool@CPhysicalWorld@@QEAAXH@Z 0000000035095a40 f   physicalworld.obj
 0001:00094d40       ?Shutdown@CPhysicalWorld@@UEAAXH@Z 0000000035095d40 f   physicalworld.obj
 0001:00095780       ?RepositionEntity@CPhysicalWorld@@QEAAHPEAVCPhysicalPlaceholder@@HPEAU?$Vec3_tpl@M@@H@Z 0000000035096780 f   physicalworld.obj
 0001:00096720       ?DeformPhysicalEntity@CPhysicalWorld@@UEAAHPEAUIPhysicalEntity@@AEBU?$Vec3_tpl@M@@1MH@Z 0000000035097720 f   physicalworld.obj
 0001:00097450       ?SimulateExplosion@CPhysicalWorld@@UEAAXPEAUpe_explosion@@PEAPEAUIPhysicalEntity@@HHH@Z 0000000035098450 f   physicalworld.obj
 0001:0009ba60       ?PrimitiveWorldIntersection@CPhysicalWorld@@UEAAMAEBUSPWIParams@IPhysicalWorld@@AEAUWriteLockCond@@PEBD@Z 000000003509ca60 f   physicalworld.obj
 0001:0009da90       ??1CPhysicalWorld@@UEAA@XZ 000000003509ea90 f   physicalworld.obj
 0001:0009dc60       ?SetupEntityGrid@CPhysicalWorld@@UEAAXHU?$Vec3_tpl@M@@HHMMH@Z 000000003509ec60 f   physicalworld.obj
 0001:0009e010       ?CreatePhysicalEntity@CPhysicalWorld@@UEAAPEAUIPhysicalEntity@@W4pe_type@@MPEAUpe_params@@PEAXHHPEAU2@@Z 000000003509f010 f   physicalworld.obj
 0001:0009e990       ?DestroyPhysicalEntity@CPhysicalWorld@@UEAAHPEAUIPhysicalEntity@@HH@Z 000000003509f990 f   physicalworld.obj
 0001:0009f950       ?TimeStep@CPhysicalWorld@@UEAAXMH@Z 00000000350a0950 f   physicalworld.obj
 0001:000a20c0       ??_GCPhysicalWorld@@UEAAPEAXI@Z 00000000350a30c0 f i physicalworld.obj
 0001:000a20c0       ??_ECPhysicalWorld@@UEAAPEAXI@Z 00000000350a30c0 f i physicalworld.obj
 0001:000a20f0       ?update_followers@@YAXHHH@Z 00000000350a30f0 f   rigidbody.obj
 0001:000a21c0       ?add_route_follower@@YAXHHH@Z 00000000350a31c0 f   rigidbody.obj
 0001:000a2280       ?CleanupContactSolvers@@YAXXZ 00000000350a3280 f   rigidbody.obj
 0001:000a22d0       ??0RigidBody@@QEAA@XZ      00000000350a32d0 f   rigidbody.obj
 0001:000a2380       ?zero@RigidBody@@QEAAXXZ   00000000350a3380 f   rigidbody.obj
 0001:000a23b0       ?GetRBMemStats@@YAXPEAVICrySizer@@@Z 00000000350a33b0 f   rigidbody.obj
 0001:000a2420       ?should_swap@@YA_NPEAPEAUentity_contact_unproj@@HHAEAHH@Z 00000000350a3420 f   rigidbody.obj
 0001:000a2570       ?trace_unproj_route@@YAXHHH@Z 00000000350a3570 f   rigidbody.obj
 0001:000a26b0       ?RegisterContact@@YAXPEAUentity_contact@@@Z 00000000350a36b0 f   rigidbody.obj
 0001:000a2770       ?DisablePreCG@@YAXXZ       00000000350a3770 f   rigidbody.obj
 0001:000a27c0       ??$ReallocateList@D@@YAPEADAEAPEADHH_N1@Z 00000000350a37c0 f i rigidbody.obj
 0001:000a2c20       ?GetContactMatrix@RigidBody@@QEAAXAEBU?$Vec3_tpl@M@@AEAU?$Matrix33_tpl@M@@@Z 00000000350a3c20 f   rigidbody.obj
 0001:000a30d0       ?ComputeRc@@YANPEAVRigidBody@@PEAPEAUentity_contact@@HHH@Z 00000000350a40d0 f   rigidbody.obj
 0001:000a4120       ?AllocSolverTmpBuf@@YAPEADH@Z 00000000350a5120 f   rigidbody.obj
 0001:000a42b0       ?InvokeContactSolverMC@@YAHPEAUcontact_helper@@PEAUcontact_helper_constraint@@PEAUbody_helper@@HHMHMM@Z 00000000350a52b0 f   rigidbody.obj
 0001:000a6aa0       ?UpdateState@RigidBody@@QEAAXXZ 00000000350a7aa0 f   rigidbody.obj
 0001:000a6f40       ?InitContactSolver@@YAXM@Z 00000000350a7f40 f   rigidbody.obj
 0001:000a7020       ?Create@RigidBody@@QEAAXAEBU?$Vec3_tpl@M@@0AEBU?$Quat_tpl@M@@MM10@Z 00000000350a8020 f   rigidbody.obj
 0001:000a7390       ?Add@RigidBody@@QEAAXAEBU?$Vec3_tpl@M@@U2@AEBU?$Quat_tpl@M@@MM@Z 00000000350a8390 f   rigidbody.obj
 0001:000a84d0       ?Step@RigidBody@@QEAAXM@Z  00000000350a94d0 f   rigidbody.obj
 0001:000a8c90       ?InvokeContactSolver@@YAHMPEAUSolverSettings@@MAEAPEAPEAUentity_contact@@AEAHAEAPEAPEAVRigidBody@@@Z 00000000350a9c90 f   rigidbody.obj
 0001:000b63f0       ?CryFatalError@@YAXPEBDZZ  00000000350b73f0 f i rigidentity.obj
 0001:000b6490       ?AttachContact@CRigidEntity@@QEAAXPEAUentity_contact@@HPEAVCPhysicalEntity@@@Z 00000000350b7490 f   rigidentity.obj
 0001:000b65b0       ?DetachContact@CRigidEntity@@QEAAXPEAUentity_contact@@HH@Z 00000000350b75b0 f   rigidentity.obj
 0001:000b6730       ?GetParams@CRigidEntity@@UEBAHPEAUpe_params@@@Z 00000000350b7730 f   rigidentity.obj
 0001:000b68b0       ?HasContactsWith@CRigidEntity@@UEAAHPEAVCPhysicalEntity@@@Z 00000000350b78b0 f   rigidentity.obj
 0001:000b6910       ?HasCollisionContactsWith@CRigidEntity@@UEAAHPEAVCPhysicalEntity@@@Z 00000000350b7910 f   rigidentity.obj
 0001:000b6960       ?HasConstraintContactsWith@CRigidEntity@@UEBAHPEBVCPhysicalEntity@@H@Z 00000000350b7960 f   rigidentity.obj
 0001:000b6a40       ?HasPartContactsWith@CRigidEntity@@UEAAHPEAVCPhysicalEntity@@HH@Z 00000000350b7a40 f   rigidentity.obj
 0001:000b6c40       ?Awake@CRigidEntity@@UEAAHHH@Z 00000000350b7c40 f   rigidentity.obj
 0001:000b6ea0       ?AlertNeighbourhoodND@CRigidEntity@@UEAAXH@Z 00000000350b7ea0 f   rigidentity.obj
 0001:000b6fa0       ?MaskIgnoredColliders@CRigidEntity@@QEAA_KH@Z 00000000350b7fa0 f   rigidentity.obj
 0001:000b70d0       ?UnmaskIgnoredColliders@CRigidEntity@@QEAAX_KH@Z 00000000350b80d0 f   rigidentity.obj
 0001:000b71c0       ?IgnoreCollisionsWith@CRigidEntity@@UEBA_NPEBVCPhysicalEntity@@H@Z 00000000350b81c0 f   rigidentity.obj
 0001:000b7360       ?wait_for_ent@@YAHPECVCPhysicalEntity@@@Z 00000000350b8360 f i rigidentity.obj
 0001:000b7390       ?CleanupAfterContactsCheck@CRigidEntity@@QEAAXH@Z 00000000350b8390 f   rigidentity.obj
 0001:000b7410       ?RemoveConstraint@CRigidEntity@@QEAAHH@Z 00000000350b8410 f   rigidentity.obj
 0001:000b74f0       ?BreakableConstraintsUpdated@CRigidEntity@@UEAAXXZ 00000000350b84f0 f   rigidentity.obj
 0001:000b7700       ?ComputeBBoxRE@CRigidEntity@@QEAAXPEAUcoord_block_BBox@@@Z 00000000350b8700 f   rigidentity.obj
 0001:000b7850       ?UpdatePosition@CRigidEntity@@QEAAXH@Z 00000000350b8850 f   rigidentity.obj
 0001:000b7ba0       ?StartStep@CRigidEntity@@UEAAXM@Z 00000000350b8ba0 f   rigidentity.obj
 0001:000b7bc0       ?GetContactCount@CRigidEntity@@UEAAHH@Z 00000000350b8bc0 f   rigidentity.obj
 0001:000b7c60       ?GetDamping@CRigidEntity@@UEAAMM@Z 00000000350b8c60 f   rigidentity.obj
 0001:000b7cd0       ?UpdateSequenceDeltaAverage@SRigidEntityNetStateHistory@@AEAAXEH@Z 00000000350b8cd0 f   rigidentity.obj
 0001:000b7d50       ?WriteContacts@CRigidEntity@@QEAAHAEAVCStream@@H@Z 00000000350b8d50 f   rigidentity.obj
 0001:000b7eb0       ?GetLocalSequenceNumber@CRigidEntity@@QEAAEXZ 00000000350b8eb0 f   rigidentity.obj
 0001:000b7f30       ?GetInterpSequenceNumber@CRigidEntity@@QEAAMXZ 00000000350b8f30 f   rigidentity.obj
 0001:000b7fe0       ?GetStateChecksum@CRigidEntity@@UEAAIXZ 00000000350b8fe0 f   rigidentity.obj
 0001:000b8360       ?ReportConstraintBreak@CRigidEntity@@QEAAAEAUEventPhysJointBroken@@AEAU2@H@Z 00000000350b9360 f   rigidentity.obj
 0001:000b84c0       ?GetMemoryStatistics@CRigidEntity@@UEBAXPEAVICrySizer@@@Z 00000000350b94c0 f   rigidentity.obj
 0001:000b85c0       ??0?$AngleAxis_tpl@M@@QEAA@AEBU?$Quat_tpl@M@@@Z 00000000350b95c0 f i rigidentity.obj
 0001:000b86e0       ??$?0M@?$Ang3_tpl@M@@QEAA@AEBU?$Quat_tpl@M@@@Z 00000000350b96e0 f i rigidentity.obj
 0001:000b88b0       ?FreeContact@CPhysicalWorld@@QEAAXPEAUentity_contact@@@Z 00000000350b98b0 f i rigidentity.obj
 0001:000b8910       ?Glob2Loc@@YA?AU?$Vec3_tpl@M@@AEBUentity_contact@@H@Z 00000000350b9910 f i rigidentity.obj
 0001:000b8c10       ??0pe_params_rope@@QEAA@XZ 00000000350b9c10 f i rigidentity.obj
 0001:000b8ea0       ??0CRigidEntity@@QEAA@PEAVCPhysicalWorld@@@Z 00000000350b9ea0 f   rigidentity.obj
 0001:000b91d0       ?IsAwake@CRigidEntity@@UEBAHH@Z 00000000350ba1d0 f i rigidentity.obj
 0001:000b91e0       ?GetRigidBody@CRigidEntity@@UEAAPEAVRigidBody@@HH@Z 00000000350ba1e0 f i rigidentity.obj
 0001:000b91f0       ?GetSleepSpeedChange@CRigidEntity@@UEAAXHAEAU?$Vec3_tpl@M@@0@Z 00000000350ba1f0 f i rigidentity.obj
 0001:000b9230       ?GetContactMatrix@CRigidEntity@@UEAAXAEBU?$Vec3_tpl@M@@HAEAU?$Matrix33_tpl@M@@@Z 00000000350ba230 f i rigidentity.obj
 0001:000b9280       ??1CRigidEntity@@UEAA@XZ   00000000350ba280 f   rigidentity.obj
 0001:000b9390       ?DetachAllContacts@CRigidEntity@@QEAAXXZ 00000000350ba390 f   rigidentity.obj
 0001:000b94c0       ?DetachPartContacts@CRigidEntity@@UEAAXHHPEAVCPhysicalEntity@@HH@Z 00000000350ba4c0 f   rigidentity.obj
 0001:000b95c0       ?_AllocData@?$CryStackStringT@D$0CAA@@@QEAAX_K@Z 00000000350ba5c0 f i rigidentity.obj
 0001:000b9640       ?RemoveCollider@CRigidEntity@@UEAAHPEAVCPhysicalEntity@@_N@Z 00000000350ba640 f   rigidentity.obj
 0001:000b9800       ?AddCollider@CRigidEntity@@UEAAHPEAVCPhysicalEntity@@@Z 00000000350ba800 f   rigidentity.obj
 0001:000b9940       ?RemoveContactPoint@CRigidEntity@@UEAAHPEAVCPhysicalEntity@@AEBU?$Vec3_tpl@M@@M@Z 00000000350ba940 f   rigidentity.obj
 0001:000b9a80       ?RegisterConstraint@CRigidEntity@@QEAAHAEBU?$Vec3_tpl@M@@0HPEAVCPhysicalEntity@@HHH@Z 00000000350baa80 f   rigidentity.obj
 0001:000b9e20       ?VerifyExistingContacts@CRigidEntity@@QEAAXM@Z 00000000350bae20 f   rigidentity.obj
 0001:000b9fe0       ?CalcEnergy@CRigidEntity@@UEAAMM@Z 00000000350bafe0 f   rigidentity.obj
 0001:000ba640       ?PushReceivedState@SRigidEntityNetStateHistory@@QEAAXAEBUSRigidEntityNetSerialize@@@Z 00000000350bb640 f   rigidentity.obj
 0001:000ba760       ?PushReceivedSequenceDelta@SRigidEntityNetStateHistory@@QEAAXE@Z 00000000350bb760 f   rigidentity.obj
 0001:000ba8e0       ?GetStateSnapshot@CRigidEntity@@UEAAHAEAVCStream@@MH@Z 00000000350bb8e0 f   rigidentity.obj
 0001:000ba9e0       ?Serialize@SRigidEntityNetSerialize@@QEAAXV?$CSerializeWrapper@UISerialize@@@@@Z 00000000350bb9e0 f   rigidentity.obj
 0001:000baac0       ?PostSetStateFromSnapshot@CRigidEntity@@UEAAHXZ 00000000350bbac0 f   rigidentity.obj
 0001:000baff0       ?CompactContactBlock@CRigidEntity@@QEBAHPEAUentity_contact@@HMHAEAHAEAPEAU2@AEAU?$Vec3_tpl@M@@AEAMAEBU3@5@Z 00000000350bbff0 f   rigidentity.obj
 0001:000bc010       ??$AllocPooledObj@Uentity_contact@@@CPhysicalWorld@@QEAAPEAUentity_contact@@AEAPEAU1@AEAH1AECH@Z 00000000350bd010 f i rigidentity.obj
 0001:000bc180       ?MoveConstrainedObjects@CRigidEntity@@QEAAXAEBU?$Vec3_tpl@M@@AEBU?$Quat_tpl@M@@@Z 00000000350bd180 f   rigidentity.obj
 0001:000bc5a0       ?RemoveGeometry@CRigidEntity@@UEAAXHH@Z 00000000350bd5a0 f   rigidentity.obj
 0001:000bc750       ?SaveConstraintFrames@CRigidEntity@@QEAAXH@Z 00000000350bd750 f   rigidentity.obj
 0001:000bca50       ?RecomputeMassDistribution@CRigidEntity@@UEAAXHH@Z 00000000350bda50 f   rigidentity.obj
 0001:000bd5a0       ?GetStatus@CRigidEntity@@UEBAHPEAUpe_status@@@Z 00000000350be5a0 f   rigidentity.obj
 0001:000bded0       ?FakeRayCollision@CRigidEntity@@QEAAXPEAVCPhysicalEntity@@M@Z 00000000350beed0 f   rigidentity.obj
 0001:000bec20       ?GetPotentialColliders@CRigidEntity@@UEAAHAEAPEAPEAVCPhysicalEntity@@M@Z 00000000350bfc20 f   rigidentity.obj
 0001:000bf5a0       ?ProcessContactEvents@CRigidEntity@@QEAAXPEAUgeom_contact@@HH@Z 00000000350c05a0 f   rigidentity.obj
 0001:000bff70       ?CheckForNewContacts@CRigidEntity@@QEAAHPEAUgeom_world_data@@PEAUintersection_params@@AEAHU?$Vec3_tpl@M@@HH@Z 00000000350c0f70 f   rigidentity.obj
 0001:000c2540       ?OnContactResolved@CRigidEntity@@UEAAXPEAUentity_contact@@HH@Z 00000000350c3540 f   rigidentity.obj
 0001:000c28a0       ?UpdateConstraints@CRigidEntity@@QEAAXM@Z 00000000350c38a0 f   rigidentity.obj
 0001:000c5170       ?CapBodyVel@CRigidEntity@@QEAAXXZ 00000000350c6170 f   rigidentity.obj
 0001:000c59b0       ?CheckContactConflicts@CRigidEntity@@QEAAXPEAUgeom_contact@@HH@Z 00000000350c69b0 f   rigidentity.obj
 0001:000c6690       ?PostStepNotify@CRigidEntity@@QEAAHMPEAUpe_params_buoyancy@@H@Z 00000000350c7690 f   rigidentity.obj
 0001:000c6a10       ?GetMaxTimeStep@CRigidEntity@@UEAAMM@Z 00000000350c7a10 f   rigidentity.obj
 0001:000c7d10       ?ArchiveContact@CRigidEntity@@QEAAXPEAUentity_contact@@MHM@Z 00000000350c8d10 f   rigidentity.obj
 0001:000c8430       ?RegisterContacts@CRigidEntity@@UEAAHMH@Z 00000000350c9430 f   rigidentity.obj
 0001:000c8df0       ?StepBack@CRigidEntity@@UEAAXM@Z 00000000350c9df0 f   rigidentity.obj
 0001:000c9800       ?Update@CRigidEntity@@UEAAHMM@Z 00000000350ca800 f   rigidentity.obj
 0001:000cae90       ?SetNetworkAuthority@CRigidEntity@@UEAAXHH@Z 00000000350cbe90 f   rigidentity.obj
 0001:000caf90       ?SetStateFromSnapshot@CRigidEntity@@UEAAHV?$CSerializeWrapper@UISerialize@@@@H@Z 00000000350cbf90 f   rigidentity.obj
 0001:000cbae0       ?ReadContacts@CRigidEntity@@QEAAHAEAVCStream@@H@Z 00000000350ccae0 f   rigidentity.obj
 0001:000cc080       ?ApplyBuoyancy@CRigidEntity@@QEAAXMAEBU?$Vec3_tpl@M@@PEAUpe_params_buoyancy@@H@Z 00000000350cd080 f   rigidentity.obj
 0001:000cde00       ?ExtractConstraintInfo@CRigidEntity@@QEAAHH_KAEAUpe_action_add_constraint@@@Z 00000000350cee00 f   rigidentity.obj
 0001:000ce2e0       ?OnNeighbourSplit@CRigidEntity@@UEAAXPEAVCPhysicalEntity@@0@Z 00000000350cf2e0 f   rigidentity.obj
 0001:000cf540       ?AddGeometry@CRigidEntity@@UEAAHPEAUphys_geometry@@PEAUpe_geomparams@@HH@Z 00000000350d0540 f   rigidentity.obj
 0001:000cfe90       ?SetParams@CRigidEntity@@UEAAHPEAUpe_params@@H@Z 00000000350d0e90 f   rigidentity.obj
 0001:000d1290       ?Action@CRigidEntity@@UEAAHPEAUpe_action@@H@Z 00000000350d2290 f   rigidentity.obj
 0001:000d4340       ?RegisterContactPoint@CRigidEntity@@QEAAPEAUentity_contact@@HAEBU?$Vec3_tpl@M@@PEBUgeom_contact@@HHHHHMH0@Z 00000000350d5340 f   rigidentity.obj
 0001:000d5800       ?ProcessCanopyContact@CRigidEntity@@QEAAXPEAUgeom_contact@@HMH@Z 00000000350d6800 f   rigidentity.obj
 0001:000d64a0       ?DelayedIntersect@CRigidEntity@@UEAAXPEAUgeom_contact@@HPEAPEAVCPhysicalEntity@@PEAY01H@Z 00000000350d74a0 f   rigidentity.obj
 0001:000d7370       ?GetStateSnapshot@CRigidEntity@@UEAAHV?$CSerializeWrapper@UISerialize@@@@MH@Z 00000000350d8370 f   rigidentity.obj
 0001:000d7b10       ?SetStateFromSnapshot@CRigidEntity@@UEAAHAEAVCStream@@H@Z 00000000350d8b10 f   rigidentity.obj
 0001:000d8810       ?GetInterpolatedState@CRigidEntity@@QEAA_NMAEAUSRigidEntityNetSerialize@@@Z 00000000350d9810 f   rigidentity.obj
 0001:000d9060       ?Format@?$CryStackStringT@D$0CAA@@@QEAAAEAV1@PEBDZZ 00000000350da060 f i rigidentity.obj
 0001:000d9150       ?UpdateStateFromNetwork@CRigidEntity@@QEAAXXZ 00000000350da150 f   rigidentity.obj
 0001:000d9260       ?DrawHelperInformation@CRigidEntity@@UEAAXPEAUIPhysRenderer@@H@Z 00000000350da260 f   rigidentity.obj
 0001:000da390       ?Step@CRigidEntity@@UEAAHM@Z 00000000350db390 f   rigidentity.obj
 0001:000dcd80       ??1CRopeEntity@@UEAA@XZ    00000000350ddd80 f   ropeentity.obj
 0001:000dce50       ?GetType@CRopeEntity@@UEBA?AW4pe_type@@XZ 00000000350dde50 f i ropeentity.obj
 0001:000dce50       ?GetType@CVoxelGeom@@UEAAHXZ 00000000350dde50 f i geoman.obj
 0001:000dce60       ?IsAwake@CRopeEntity@@UEBAHH@Z 00000000350dde60 f i ropeentity.obj
 0001:000dce60       ?IsAwake@CSoftEntity@@UEBAHH@Z 00000000350dde60 f i softentity.obj
 0001:000dce70       ?GetMass@CRopeEntity@@UEAAMH@Z 00000000350dde70 f i ropeentity.obj
 0001:000dce90       ?GetMassInv@CRopeEntity@@UEAAMXZ 00000000350dde90 f i ropeentity.obj
 0001:000dcea0       ?CalcEnergy@CRopeEntity@@UEAAMM@Z 00000000350ddea0 f i ropeentity.obj
 0001:000dcec0       ?GetLastTimeStep@CRopeEntity@@UEAAMM@Z 00000000350ddec0 f i ropeentity.obj
 0001:000dced0       ?GetMemoryStatistics@CRopeEntity@@UEBAXPEAVICrySizer@@@Z 00000000350dded0 f   ropeentity.obj
 0001:000dcf40       ?GetCheckPart@CPhysicalEntity@@QEAAHH@Z 00000000350ddf40 f i ropeentity.obj
 0001:000dd0e0       ?GetDamping@CRopeEntity@@UEAAMM@Z 00000000350de0e0 f i ropeentity.obj
 0001:000dd120       ??_ECRopeEntity@@UEAAPEAXI@Z 00000000350de120 f i ropeentity.obj
 0001:000dd120       ??_GCRopeEntity@@UEAAPEAXI@Z 00000000350de120 f i ropeentity.obj
 0001:000dd150       ?Awake@CRopeEntity@@UEAAHHH@Z 00000000350de150 f   ropeentity.obj
 0001:000dd390       ?GetStatus@CRopeEntity@@UEBAHPEAUpe_status@@@Z 00000000350de390 f   ropeentity.obj
 0001:000dd6f0       ?StartStep@CRopeEntity@@UEAAXM@Z 00000000350de6f0 f   ropeentity.obj
 0001:000dd7b0       ?GetMaxTimeStep@CRopeEntity@@UEAAMM@Z 00000000350de7b0 f   ropeentity.obj
 0001:000dd820       ?ZeroLengthStraighten@CRopeEntity@@QEAAXM@Z 00000000350de820 f   ropeentity.obj
 0001:000de3d0       ?Solver@CRopeEntity@@QEAAMMM@Z 00000000350df3d0 f   ropeentity.obj
 0001:000e0e20       ?OnDelayedStep@CRopeEntity@@UEAAXAEAVCMemStreamA@@@Z 00000000350e1e20 f   ropeentity.obj
 0001:000e0fb0       ?GetStateSnapshot@CRopeEntity@@UEAAHAEAVCStream@@MH@Z 00000000350e1fb0 f   ropeentity.obj
 0001:000e1000       ?ComputeExtent@CRopeEntity@@UEBAMAEAUGeomQuery@@W4EGeomForm@@@Z 00000000350e2000 f   ropeentity.obj
 0001:000e1260       ??$ReallocateList@USPrecompPartBV@@@@YAPEAUSPrecompPartBV@@AEAPEAU0@HH_N1@Z 00000000350e2260 f i ropeentity.obj
 0001:000e1260       ??$ReallocateList@USStructuralJoint@@@@YAPEAUSStructuralJoint@@AEAPEAU0@HH_N1@Z 00000000350e2260 f i physicalentity.obj
 0001:000e1350       ??0CRopeEntity@@QEAA@PEAVCPhysicalWorld@@@Z 00000000350e2350 f   ropeentity.obj
 0001:000e17d0       ?AlertNeighbourhoodND@CRopeEntity@@UEAAXH@Z 00000000350e27d0 f   ropeentity.obj
 0001:000e18c0       ?RecalcBBox@CRopeEntity@@QEAAXXZ 00000000350e28c0 f   ropeentity.obj
 0001:000e1b70       ?GetParams@CRopeEntity@@UEBAHPEAUpe_params@@@Z 00000000350e2b70 f   ropeentity.obj
 0001:000e20d0       ?AllocSubVtx@CRopeEntity@@QEAAXXZ 00000000350e30d0 f   ropeentity.obj
 0001:000e2250       ?FillVtxContactData@CRopeEntity@@QEAAXPEAUrope_vtx@@HAEAUSRopeCheckPart@@PEAUgeom_contact@@@Z 00000000350e3250 f   ropeentity.obj
 0001:000e25c0       ?CheckCollisions@CRopeEntity@@QEAAXHPEAUSRopeCheckPart@@HMM@Z 00000000350e35c0 f   ropeentity.obj
 0001:000e4010       ?RegisterContacts@CRopeEntity@@UEAAHMH@Z 00000000350e5010 f   ropeentity.obj
 0001:000e5d30       ?Update@CRopeEntity@@UEAAHMM@Z 00000000350e6d30 f   ropeentity.obj
 0001:000e6cc0       ?RayTrace@CRopeEntity@@UEAAHAEAUSRayTraceRes@@@Z 00000000350e7cc0 f   ropeentity.obj
 0001:000e73e0       ?ApplyVolumetricPressure@CRopeEntity@@UEAAXAEBU?$Vec3_tpl@M@@MM@Z 00000000350e83e0 f   ropeentity.obj
 0001:000e7d40       ?OnNeighbourSplit@CRopeEntity@@UEAAXPEAVCPhysicalEntity@@0@Z 00000000350e8d40 f   ropeentity.obj
 0001:000e7fc0       ?SetStateFromSnapshot@CRopeEntity@@UEAAHV?$CSerializeWrapper@UISerialize@@@@H@Z 00000000350e8fc0 f   ropeentity.obj
 0001:000e8cb0       ?DrawHelperInformation@CRopeEntity@@UEAAXPEAUIPhysRenderer@@H@Z 00000000350e9cb0 f   ropeentity.obj
 0001:000e9390       ?GetRandomPos@CRopeEntity@@UEBAXAEAURandomPos@@AEAUGeomQuery@@W4EGeomForm@@@Z 00000000350ea390 f   ropeentity.obj
 0001:000e9720       ?SetParams@CRopeEntity@@UEAAHPEAUpe_params@@H@Z 00000000350ea720 f   ropeentity.obj
 0001:000eb510       ?EnforceConstraints@CRopeEntity@@QEAAXMAEBU?$Quat_tpl@M@@AEBU?$Vec3_tpl@M@@MH@Z 00000000350ec510 f   ropeentity.obj
 0001:000ec8e0       ?Action@CRopeEntity@@UEAAHPEAUpe_action@@H@Z 00000000350ed8e0 f   ropeentity.obj
 0001:000edbe0       ?StepSubdivided@CRopeEntity@@QEAAXMPEAUSRopeCheckPart@@HM@Z 00000000350eebe0 f   ropeentity.obj
 0001:000f2590       ?ApplyStiffness@CRopeEntity@@QEAAXMHAEBU?$Quat_tpl@M@@AEBU?$Vec3_tpl@M@@M@Z 00000000350f3590 f   ropeentity.obj
 0001:000f3a70       ?Step@CRopeEntity@@UEAAHM@Z 00000000350f4a70 f   ropeentity.obj
 0001:000f94d0       ?GetStateSnapshot@CRopeEntity@@UEAAHV?$CSerializeWrapper@UISerialize@@@@MH@Z 00000000350fa4d0 f   ropeentity.obj
 0001:000f9b00       ?GetRigidBodyData@CRopeEntity@@UEAAPEAVRigidBody@@PEAV2@H@Z 00000000350fab00 f   ropeentity.obj
 0001:000f9f80       ?GetLocTransform@CRopeEntity@@UEAAXHAEAU?$Vec3_tpl@M@@AEAU?$Quat_tpl@M@@AEAM@Z 00000000350faf80 f   ropeentity.obj
 0001:000fa240       ?RemoveCore@CSoftEntity@@QEAAXXZ 00000000350fb240 f   softentity.obj
 0001:000fa2b0       ?AlertNeighbourhoodND@CSoftEntity@@UEAAXH@Z 00000000350fb2b0 f   softentity.obj
 0001:000fa3a0       ?Awake@CSoftEntity@@UEAAHHH@Z 00000000350fb3a0 f   softentity.obj
 0001:000fa3f0       ?GetParams@CSoftEntity@@UEBAHPEAUpe_params@@@Z 00000000350fb3f0 f   softentity.obj
 0001:000fa590       ?StartStep@CSoftEntity@@UEAAXM@Z 00000000350fb590 f   softentity.obj
 0001:000fa5b0       ?GetMemoryStatistics@CSoftEntity@@UEBAXPEAVICrySizer@@@Z 00000000350fb5b0 f   softentity.obj
 0001:000fa670       ??0CSoftEntity@@QEAA@PEAVCPhysicalWorld@@@Z 00000000350fb670 f   softentity.obj
 0001:000fa860       ?GetType@CSoftEntity@@UEBA?AW4pe_type@@XZ 00000000350fb860 f i softentity.obj
 0001:000fa870       ?GetMass@CSoftEntity@@UEAAMH@Z 00000000350fb870 f i softentity.obj
 0001:000fa890       ?GetStatus@CSoftEntity@@UEBAHPEAUpe_status@@@Z 00000000350fb890 f   softentity.obj
 0001:000fad80       ?GetMaxTimeStep@CSoftEntity@@UEAAMM@Z 00000000350fbd80 f   softentity.obj
 0001:000fadf0       ?OnDelayedStep@CSoftEntity@@UEAAXAEAVCMemStreamA@@@Z 00000000350fbdf0 f   softentity.obj
 0001:000fb3d0       ?RecalcTriNormal@CTriMesh@@QEAAXH@Z 00000000350fc3d0 f i softentity.obj
 0001:000fb540       ??1CSoftEntity@@UEAA@XZ    00000000350fc540 f   softentity.obj
 0001:000fb6e0       ?BakeCurrentPose@CSoftEntity@@QEAAXXZ 00000000350fc6e0 f   softentity.obj
 0001:000fbdc0       ?RemoveGeometry@CSoftEntity@@UEAAXHH@Z 00000000350fcdc0 f   softentity.obj
 0001:000fbf50       ?AttachPoints@CSoftEntity@@QEAAXPEAUpe_action_attach_points@@PEAVCPhysicalEntity@@HMMHAEBU?$Vec3_tpl@M@@AEBU?$Quat_tpl@M@@@Z 00000000350fcf50 f   softentity.obj
 0001:000fc330       ?Action@CSoftEntity@@UEAAHPEAUpe_action@@H@Z 00000000350fd330 f   softentity.obj
 0001:000fef90       ?ApplyVolumetricPressure@CSoftEntity@@UEAAXAEBU?$Vec3_tpl@M@@MM@Z 00000000350fff90 f   softentity.obj
 0001:000ff610       ?RayTrace@CSoftEntity@@UEAAHAEAUSRayTraceRes@@@Z 0000000035100610 f   softentity.obj
 0001:000ffaf0       ?GetStateSnapshot@CSoftEntity@@UEAAHV?$CSerializeWrapper@UISerialize@@@@MH@Z 0000000035100af0 f   softentity.obj
 0001:000ffc10       ?SetStateFromSnapshot@CSoftEntity@@UEAAHV?$CSerializeWrapper@UISerialize@@@@H@Z 0000000035100c10 f   softentity.obj
 0001:000fffb0       ?DrawHelperInformation@CSoftEntity@@UEAAXPEAUIPhysRenderer@@H@Z 0000000035100fb0 f   softentity.obj
 0001:00100480       ??_GCSoftEntity@@UEAAPEAXI@Z 0000000035101480 f i softentity.obj
 0001:00100480       ??_ECSoftEntity@@UEAAPEAXI@Z 0000000035101480 f i softentity.obj
 0001:001004b0       ?AddGeometry@CSoftEntity@@UEAAHPEAUphys_geometry@@PEAUpe_geomparams@@HH@Z 00000000351014b0 f   softentity.obj
 0001:00102ae0       ?SetParams@CSoftEntity@@UEAAHPEAUpe_params@@H@Z 0000000035103ae0 f   softentity.obj
 0001:00103c70       ?StepInner@CSoftEntity@@QEAAXMHPEAUcheck_part@@HAEBUplane@primitives@@AEBU?$Vec3_tpl@M@@M2AEBU?$Quat_tpl@M@@PEAUse_vertex@@@Z 0000000035104c70 f   softentity.obj
 0001:0010a4a0       ?Step@CSoftEntity@@UEAAHM@Z 000000003510b4a0 f   softentity.obj
 0001:0010e420       ?MaxPrimsInNode@CHeightfieldBV@@UEAAHXZ 000000003510f420 f i waterman.obj
 0001:0010e430       ??_ECHeightfieldBV@@UEAAPEAXI@Z 000000003510f430 f i waterman.obj
 0001:0010e430       ??_GCHeightfieldBV@@UEAAPEAXI@Z 000000003510f430 f i waterman.obj
 0001:0010e480       ?GetPrimitiveId@CTriMesh@@UEAAHHH@Z 000000003510f480 f i waterman.obj
 0001:0010e4a0       ?GetForeignIdx@CTriMesh@@UEAAHH@Z 000000003510f4a0 f i waterman.obj
 0001:0010e4c0       ?GetNormal@CTriMesh@@UEAA?AU?$Vec3_tpl@M@@HAEBU2@@Z 000000003510f4c0 f i waterman.obj
 0001:0010e4f0       ?GetPrimitiveCount@CTriMesh@@UEAAHXZ 000000003510f4f0 f i waterman.obj
 0001:0010e500       ?GetSubtractionsCount@CTriMesh@@UEAAHXZ 000000003510f500 f i waterman.obj
 0001:0010e510       ?GetTriMesh@CTriMesh@@UEAAPEAUIGeometry@@H@Z 000000003510f510 f i waterman.obj
 0001:0010e570       ?GetErrorCount@CTriMesh@@UEAAHXZ 000000003510f570 f i waterman.obj
 0001:0010e580       ?GetForeignData@CTriMesh@@UEAAPEAXH@Z 000000003510f580 f i waterman.obj
 0001:0010e5a0       ?SetForeignData@CTriMesh@@UEAAXPEAXH@Z 000000003510f5a0 f i waterman.obj
 0001:0010e5d0       ?DestroyAuxilaryMeshData@CTriMesh@@UEAAXH@Z 000000003510f5d0 f i waterman.obj
 0001:0010e650       ?GetType@CSingleBoxTree@@UEAAHXZ 000000003510f650 f i livingentity.obj
 0001:0010e650       ?GetType@CRigidEntity@@UEBA?AW4pe_type@@XZ 000000003510f650 f i rigidentity.obj
 0001:0010e650       ?GetType@CHeightfield@@UEAAHXZ 000000003510f650 f i waterman.obj
 0001:0010e660       ?GetBVTree@CHeightfield@@UEAAPEAVCBVTree@@XZ 000000003510f660 f i waterman.obj
 0001:0010e670       ?GetData@CHeightfield@@UEAAPEBUprimitive@primitives@@XZ 000000003510f670 f i waterman.obj
 0001:0010e680       ??_ECHeightfield@@UEAAPEAXI@Z 000000003510f680 f i waterman.obj
 0001:0010e680       ??_GCHeightfield@@UEAAPEAXI@Z 000000003510f680 f i waterman.obj
 0001:0010e700       ?GetParams@CWaterMan@@QEAAHPEAUpe_params@@@Z 000000003510f700 f   waterman.obj
 0001:0010e760       ?GetBBox@CTriMesh@@UEAAXPEAUbox@primitives@@@Z 000000003510f760 f i waterman.obj
 0001:0010e7b0       ?GetBBox@CTriMesh@@UEAAXPEAUbox@primitives@@H@Z 000000003510f7b0 f i waterman.obj
 0001:0010e800       ?Load@CTriMesh@@UEAAXAEAVCMemStream@@@Z 000000003510f800 f i waterman.obj
 0001:0010e840       ?GetCenter@CHeightfield@@UEAA?AU?$Vec3_tpl@M@@XZ 000000003510f840 f i waterman.obj
 0001:0010e920       ??0CWaterMan@@QEAA@PEAVCPhysicalWorld@@@Z 000000003510f920 f   waterman.obj
 0001:0010ea20       ??1CWaterMan@@QEAA@XZ      000000003510fa20 f   waterman.obj
 0001:0010eb00       ?GetStatus@CWaterMan@@QEAAHPEAUpe_status@@@Z 000000003510fb00 f   waterman.obj
 0001:0010ec60       ?TimeStep@CWaterMan@@QEAAXM@Z 000000003510fc60 f   waterman.obj
 0001:0010f520       ?check_cell@jgrid_checker@@QEAAHAEBU?$Vec2_tpl@H@@AEAH@Z 0000000035110520 f i waterman.obj
 0001:0010fc00       ?MarkCellInteriorQueue@jgrid_checker@@QEAAXH@Z 0000000035110c00 f i waterman.obj
 0001:0010fdc0       ?GetPrimitive@CHeightfield@@UEAAHHPEAUprimitive@primitives@@@Z 0000000035110dc0 f i waterman.obj
 0001:0010fe70       ?OnWaterHit@CWaterMan@@QEAAXAEBU?$Vec3_tpl@M@@0@Z 0000000035110e70 f   waterman.obj
 0001:001100f0       ??$DrawRayOnGrid@Ujgrid_checker@@@@YAHPEAUgrid@primitives@@AEAU?$Vec3_tpl@M@@1AEAUjgrid_checker@@@Z 00000000351110f0 f i waterman.obj
 0001:00110840       ??0CHeightfield@@QEAA@XZ   0000000035111840 f i waterman.obj
 0001:00110880       ?OnWaterInteraction@CWaterMan@@QEAAXPEAVCPhysicalEntity@@@Z 0000000035111880 f   waterman.obj
 0001:00113850       ?SetViewerPos@CWaterMan@@QEAAXAEBU?$Vec3_tpl@M@@H@Z 0000000035114850 f   waterman.obj
 0001:00114430       ?DrawHelpers@CWaterMan@@QEAAXPEAUIPhysRenderer@@@Z 0000000035115430 f   waterman.obj
 0001:00114930       ?SetParams@CWaterMan@@QEAAHPEAUpe_params@@@Z 0000000035115930 f   waterman.obj
 0001:00114d70       ?AlertNeighbourhoodND@CWheeledVehicleEntity@@UEAAXH@Z 0000000035115d70 f   wheeledvehicleentity.obj
 0001:00114dd0       ?OnContactResolved@CWheeledVehicleEntity@@UEAAXPEAUentity_contact@@HH@Z 0000000035115dd0 f   wheeledvehicleentity.obj
 0001:00114df0       ?GetMaxTimeStep@CWheeledVehicleEntity@@UEAAMM@Z 0000000035115df0 f   wheeledvehicleentity.obj
 0001:00114e50       ?GetDamping@CWheeledVehicleEntity@@UEAAMM@Z 0000000035115e50 f   wheeledvehicleentity.obj
 0001:00114ea0       ?HasContactsWith@CWheeledVehicleEntity@@UEAAHPEAVCPhysicalEntity@@@Z 0000000035115ea0 f   wheeledvehicleentity.obj
 0001:00114ef0       ?HasPartContactsWith@CWheeledVehicleEntity@@UEAAHPEAVCPhysicalEntity@@HH@Z 0000000035115ef0 f   wheeledvehicleentity.obj
 0001:00114fa0       ?RemoveCollider@CWheeledVehicleEntity@@UEAAHPEAVCPhysicalEntity@@_N@Z 0000000035115fa0 f   wheeledvehicleentity.obj
 0001:00115020       ?Update@CWheeledVehicleEntity@@UEAAHMM@Z 0000000035116020 f   wheeledvehicleentity.obj
 0001:001151e0       ?GetMemoryStatistics@CWheeledVehicleEntity@@UEBAXPEAVICrySizer@@@Z 00000000351161e0 f   wheeledvehicleentity.obj
 0001:00115230       ?GetParams@CWheeledVehicleEntity@@UEBAHPEAUpe_params@@@Z 0000000035116230 f   wheeledvehicleentity.obj
 0001:001155f0       ?ComputeBBox@CWheeledVehicleEntity@@UEAAXPEAU?$Vec3_tpl@M@@H@Z 00000000351165f0 f   wheeledvehicleentity.obj
 0001:001156b0       ?ComputeDrivingTorque@CWheeledVehicleEntity@@QEAAMM@Z 00000000351166b0 f   wheeledvehicleentity.obj
 0001:00115c60       ?GetStateSnapshot@CWheeledVehicleEntity@@UEAAHAEAVCStream@@MH@Z 0000000035116c60 f   wheeledvehicleentity.obj
 0001:00115d60       ?SetStateFromSnapshot@CWheeledVehicleEntity@@UEAAHAEAVCStream@@H@Z 0000000035116d60 f   wheeledvehicleentity.obj
 0001:00115f70       ?Serialize@SWheeledVehicleEntityNetSerialize@@QEAAXV?$CSerializeWrapper@UISerialize@@@@H@Z 0000000035116f70 f   wheeledvehicleentity.obj
 0001:00116020       ?GetStateSnapshot@CWheeledVehicleEntity@@UEAAHV?$CSerializeWrapper@UISerialize@@@@MH@Z 0000000035117020 f   wheeledvehicleentity.obj
 0001:001160e0       ?DrawHelperInformation@CWheeledVehicleEntity@@UEAAXPEAUIPhysRenderer@@H@Z 00000000351170e0 f   wheeledvehicleentity.obj
 0001:00116230       ??0pe_cargeomparams@@QEAA@AEAUpe_geomparams@@@Z 0000000035117230 f i wheeledvehicleentity.obj
 0001:00116370       ?SetParams@CWheeledVehicleEntity@@UEAAHPEAUpe_params@@H@Z 0000000035117370 f   wheeledvehicleentity.obj
 0001:00116f70       ?RemoveGeometry@CWheeledVehicleEntity@@UEAAXHH@Z 0000000035117f70 f   wheeledvehicleentity.obj
 0001:00117120       ?AddAdditionalImpulses@CWheeledVehicleEntity@@UEAAXM@Z 0000000035118120 f   wheeledvehicleentity.obj
 0001:00118df0       ?RegisterContacts@CWheeledVehicleEntity@@UEAAHMH@Z 0000000035119df0 f   wheeledvehicleentity.obj
 0001:001192f0       ?SetStateFromSnapshot@CWheeledVehicleEntity@@UEAAHV?$CSerializeWrapper@UISerialize@@@@H@Z 000000003511a2f0 f   wheeledvehicleentity.obj
 0001:00119420       ??0CWheeledVehicleEntity@@QEAA@PEAVCPhysicalWorld@@@Z 000000003511a420 f   wheeledvehicleentity.obj
 0001:001195b0       ?IsConvex@CGeometry@@UEAAHM@Z 000000003511a5b0 f i livingentity.obj
 0001:001195b0       ?GetStateSnapshot@CSoftEntity@@UEAAHAEAVCStream@@MH@Z 000000003511a5b0 f i softentity.obj
 0001:001195b0       ?Step@CPhysicalEntity@@UEAAHM@Z 000000003511a5b0 f i physicalentity.obj
 0001:001195b0       ?MaxPrimsInNode@CBVTree@@UEAAHXZ 000000003511a5b0 f i livingentity.obj
 0001:001195b0       ?SanityCheck@CGeometry@@UEAAHXZ 000000003511a5b0 f i livingentity.obj
 0001:001195b0       ?IsAPrimitive@CPrimitive@@UEAAHXZ 000000003511a5b0 f i livingentity.obj
 0001:001195b0       ?FlushDynPool@CPhysicalWorld@@UEAAHXZ 000000003511a5b0 f i physicalworld.obj
 0001:001195b0       ?PostSetStateFromSnapshot@CPhysicalEntity@@UEAAHXZ 000000003511a5b0 f i livingentity.obj
 0001:001195b0       ?GetType@CTriMesh@@UEAAHXZ 000000003511a5b0 f i trimesh.obj
 0001:001195b0       ?GetType@CPhysicalStub@@UEBA?AW4pe_type@@XZ 000000003511a5b0 f i physarea.obj
 0001:001195b0       ?PrepareForIntersectionTest@CGeometry@@UEAAHPEAUgeometry_under_test@@PEAV1@0_N@Z 000000003511a5b0 f i livingentity.obj
 0001:001195b0       ?SanityCheck@CBVTree@@UEAAHXZ 000000003511a5b0 f i livingentity.obj
 0001:001195b0       ?DoStep@CPhysicalEntity@@UEAAHMH@Z 000000003511a5b0 f i articulatedentity.obj
 0001:001195b0       ?GetType@CAABBTree@@UEAAHXZ 000000003511a5b0 f i trimesh.obj
 0001:001195b0       ?GetSnapshotVersion@CWheeledVehicleEntity@@UEAAHXZ 000000003511a5b0 f i wheeledvehicleentity.obj
 0001:001195b0       ?GetPrimitiveCount@CGeometry@@UEAAHXZ 000000003511a5b0 f i livingentity.obj
 0001:001195b0       ?default_overlap_check@@YAHPEBUprimitive@primitives@@0PEAVCOverlapChecker@@@Z 000000003511a5b0 f i overlapchecks.obj
 0001:001195b0       ?IsAPrimitive@CRayGeom@@UEAAHXZ 000000003511a5b0 f i livingentity.obj
 0001:001195b0       ?GetType@CPhysicalEntity@@UEBA?AW4pe_type@@XZ 000000003511a5b0 f i physicalentity.obj
 0001:001195b0       ?HasPartContactsWith@CPhysicalEntity@@UEAAHPEAV1@HH@Z 000000003511a5b0 f i livingentity.obj
 0001:001195b0       ?Update@CPhysicalEntity@@UEAAHMM@Z 000000003511a5b0 f i particleentity.obj
 0001:001195b0       ?DoStep@CPhysicalPlaceholder@@UEAAHMH@Z 000000003511a5b0 f i physarea.obj
 0001:001195c0       ??_GCRigidEntity@@UEAAPEAXI@Z 000000003511a5c0 f i rigidentity.obj
 0001:001195c0       ??_ECRigidEntity@@UEAAPEAXI@Z 000000003511a5c0 f i rigidentity.obj
 0001:001195c0       ??_GCWheeledVehicleEntity@@UEAAPEAXI@Z 000000003511a5c0 f i wheeledvehicleentity.obj
 0001:001195c0       ??_ECWheeledVehicleEntity@@UEAAPEAXI@Z 000000003511a5c0 f i wheeledvehicleentity.obj
 0001:001195f0       ?RecalcSuspStiffness@CWheeledVehicleEntity@@QEAAXXZ 000000003511a5f0 f   wheeledvehicleentity.obj
 0001:00119f70       ?AddGeometry@CWheeledVehicleEntity@@UEAAHPEAUphys_geometry@@PEAUpe_geomparams@@HH@Z 000000003511af70 f   wheeledvehicleentity.obj
 0001:0011ae80       ?Action@CWheeledVehicleEntity@@UEAAHPEAUpe_action@@H@Z 000000003511be80 f   wheeledvehicleentity.obj
 0001:0011baa0       ?GetStatus@CWheeledVehicleEntity@@UEBAHPEAUpe_status@@@Z 000000003511caa0 f   wheeledvehicleentity.obj
 0001:0011ce90       ?CheckAdditionalGeometry@CWheeledVehicleEntity@@UEAAXM@Z 000000003511de90 f   wheeledvehicleentity.obj
 0001:001218b0       ?line_seg_inters@@YAHPEBU?$Vec2_tpl@M@@0PEAU1@@Z 00000000351228b0 f i boolean2d.obj
 0001:00121c30       ?check_if_inside@@YAHHAEAU?$Vec2_tpl@H@@AEBU1@PEBU?$Vec2_tpl@M@@AEBU2@@Z 0000000035122c30 f i boolean2d.obj
 0001:00121e90       ?boolean2d@@YAHW4booltype@@PEAU?$Vec2_tpl@M@@H1HHAEAPEAU2@AEAPEAH@Z 0000000035122e90 f   boolean2d.obj
 0001:001238b0       ??_Gbop_meshupdate_thunk@@UEAAPEAXI@Z 00000000351248b0 f i boolean3d.obj
 0001:001238b0       ??_Ebop_meshupdate_thunk@@UEAAPEAXI@Z 00000000351248b0 f i boolean3d.obj
 0001:00123900       ??1bop_meshupdate@@UEAA@XZ 0000000035124900 f   boolean3d.obj
 0001:00123a00       ?TriangulatePolyBruteforce@@YAHPEAU?$Vec2_tpl@M@@HPEAHH@Z 0000000035124a00 f   boolean3d.obj
 0001:00124200       ?TriangulatePoly@@YAHPEAU?$Vec2_tpl@M@@HPEAHH@Z 0000000035125200 f   boolean3d.obj
 0001:001257e0       ??$ReallocateList@U?$Vec3_tpl@M@@@@YAPEAU?$Vec3_tpl@M@@AEAPEAU0@HH_N1@Z 00000000351267e0 f i boolean3d.obj
 0001:001258d0       ??$ReallocateList@Ubop_newvtx@@@@YAPEAUbop_newvtx@@AEAPEAU0@HH_N1@Z 00000000351268d0 f i boolean3d.obj
 0001:001259b0       ??$ReallocateList@Utrinfo@@@@YAPEAUtrinfo@@AEAPEAU0@HH_N1@Z 00000000351269b0 f i boolean3d.obj
 0001:00125a90       ??_Gbop_meshupdate@@UEAAPEAXI@Z 0000000035126a90 f i boolean3d.obj
 0001:00125a90       ??_Ebop_meshupdate@@UEAAPEAXI@Z 0000000035126a90 f i boolean3d.obj
 0001:00125ac0       ?insertBorderVtx@@YAXPEAUtessvtx@@HHAEBU?$Vec3_tpl@M@@H@Z 0000000035126ac0 f   boolean3d.obj
 0001:00126050       ?Subtract@CTriMesh@@UEAAHPEAUIGeometry@@PEAUgeom_world_data@@1H@Z 0000000035127050 f   boolean3d.obj
 0001:0012d880       ?zero@?$matrix_tpl@N@@QEAAAEAV1@XZ 000000003512e880 f i matrixnm.obj
 0001:0012d8f0       ?LUdecomposition@?$matrix_tpl@M@@QEBAHAEAPEAMAEAPEAH@Z 000000003512e8f0 f i matrixnm.obj
 0001:0012de60       ?solveAx_b@?$matrix_tpl@M@@QEBAHPEAM00PEAH@Z 000000003512ee60 f i matrixnm.obj
 0001:0012e250       ?identity@?$matrix_tpl@N@@QEAAAEAV1@XZ 000000003512f250 f i matrixnm.obj
 0001:0012e330       ?T@?$matrix_tpl@M@@QEBA?AV1@XZ 000000003512f330 f i matrixnm.obj
 0001:0012e600       ?jacobi_transformation@?$matrix_tpl@M@@QEBAHAEAV1@PEAMM@Z 000000003512f600 f i matrixnm.obj
 0001:0012f2e0       ?jacobi_transformation@?$matrix_tpl@N@@QEBAHAEAV1@PEANN@Z 00000000351302e0 f i matrixnm.obj
 0001:00130040       ?transpose@?$matrix_tpl@M@@QEAAAEAV1@XZ 0000000035131040 f i matrixnm.obj
 0001:00130250       ?invert@?$matrix_tpl@M@@QEAAAEAV1@XZ 0000000035131250 f i matrixnm.obj
 0001:001308f0       ?qhull2d@@YAHPEAUptitem2d@@HPEAUedgeitem@@@Z 00000000351318f0 f   qhull.obj
 0001:001315f0       ?e_cansee@@YA_NAEBU?$Vec3_tpl@M@@0M@Z 00000000351325f0 f i qhull.obj
 0001:001316f0       ?associate_ptlist_with_trilist@@YAXPEAUptitem@@PEAUqhtritem@@0V?$strided_pointer@UVec3mem@@@@@Z 00000000351326f0 f   qhull.obj
 0001:00131860       ?qhull@@YAHV?$strided_pointer@U?$Vec3_tpl@M@@@@HAEAPEAHP6APEAX_K@Z@Z 0000000035132860 f   qhull.obj
 0001:001341e0       ?float2int@@YAHM@Z         00000000351351e0 f   utils.obj
 0001:00134200       ?compute_projection_integrals@@YAXPEAU?$Vec3_tpl@N@@QEAN@Z 0000000035135200 f   utils.obj
 0001:001346b0       ??0SOcclusionCubeMap@@QEAA@XZ 00000000351356b0 f   utils.obj
 0001:001346f0       ?get_cubemap_cell_buddy@@YAHHHH@Z 00000000351356f0 f i utils.obj
 0001:001347f0       ?GrowAndCompareCubemaps@@YAXPEAUSOcclusionCubeMap@@0HAEAH1@Z 00000000351357f0 f   utils.obj
 0001:00134b40       ?crop_polygon_with_plane@@YAHPEBU?$Vec3_tpl@M@@HPEAU1@AEBU1@M@Z 0000000035135b40 f   utils.obj
 0001:00134fa0       ?bin2ascii@@YAHPEBEHPEAE@Z 0000000035135fa0 f   utils.obj
 0001:00135110       ?ascii2bin@@YAHPEBEHPEAE@Z 0000000035136110 f   utils.obj
 0001:00135340       ?WritePacked@@YAXAEAVCStream@@H@Z 0000000035136340 f   utils.obj
 0001:00135360       ?ReadPacked@@YAXAEAVCStream@@AEAH@Z 0000000035136360 f   utils.obj
 0001:00135390       ?Free@SOcclusionCubeMap@@QEAAXXZ 0000000035136390 f   utils.obj
 0001:00135400       ?Allocate@SOcclusionCubeMap@@QEAAXH@Z 0000000035136400 f   utils.obj
 0001:001354d0       ?Reset@SOcclusionCubeMap@@QEAAXXZ 00000000351364d0 f   utils.obj
 0001:00135530       ?ProcessRmin@SOcclusionCubeMap@@QEAAXXZ 0000000035136530 f   utils.obj
 0001:00135680       ?GetMemoryStatistics@SOcclusionCubeMap@@QEAAXPEAVICrySizer@@@Z 0000000035136680 f   utils.obj
 0001:001356e0       ?DebugDrawToScreen@SOcclusionCubeMap@@QEAAXMMM@Z 00000000351366e0 f   utils.obj
 0001:00135e30       ?Raster@?$Rasteriser@$02@@SAXPEBU?$Vec3_tpl@M@@HPEAUSOcclusionCubeMap@@@Z 0000000035136e30 f i utils.obj
 0001:001370b0       ?Raster@?$Rasteriser@$03@@SAXPEBU?$Vec3_tpl@M@@HPEAUSOcclusionCubeMap@@@Z 00000000351380b0 f i utils.obj
 0001:00138460       ?Raster@?$Rasteriser@$07@@SAXPEBU?$Vec3_tpl@M@@HPEAUSOcclusionCubeMap@@@Z 0000000035139460 f i utils.obj
 0001:00139c20       ?compute_face_integrals@@YAXPEAU?$Vec3_tpl@N@@U1@QEAN@Z 000000003513ac20 f   utils.obj
 0001:0013a010       ?ComputeMassProperties@@YANV?$strided_pointer@$$CBU?$Vec3_tpl@M@@@@PEBHHAEAU?$Vec3_tpl@N@@AEAU?$Matrix33_tpl@N@@@Z 000000003513b010 f   utils.obj
 0001:0013a850       ?ChoosePrimitiveForMesh@@YAHV?$strided_pointer@$$CBU?$Vec3_tpl@M@@@@V?$strided_pointer@$$CBG@@HPEBU?$Vec3_tpl@N@@AEBU3@HMAEAPEAUprimitive@primitives@@@Z 000000003513b850 f   utils.obj
 0001:0013f4c0       ?get_xqs_from_matrices@@YAXPEAU?$Matrix34_tpl@M@@PEAU?$Matrix33_tpl@M@@AEAU?$Vec3_tpl@M@@AEAU?$Quat_tpl@M@@AEAM@Z 00000000351404c0 f   utils.obj
 0001:0013f980       ?CalcMediumResistance@@YAXPEBU?$Vec3_tpl@M@@HAEBU1@AEBUplane@primitives@@111AEAU1@3@Z 0000000035140980 f   utils.obj
 0001:00140a50       ?CoverPolygonWithCircles@@YAHV?$strided_pointer@U?$Vec2_tpl@M@@@@H_NAEBU?$Vec2_tpl@M@@AEAPEAU2@AEAPEAMM@Z 0000000035141a50 f   utils.obj
 0001:001416d0       ?RasterizePolygonIntoCubemap@@YAXPEBU?$Vec3_tpl@M@@HHPEAUSOcclusionCubeMap@@@Z 00000000351426d0 f   utils.obj
 0001:00141710       ??1SOcclusionCubeMap@@QEAA@XZ 0000000035142710 f   utils.obj
 0001:00141720       ?Init@SOcclusionCubeMap@@QEAAXHMM@Z 0000000035142720 f   utils.obj
 0001:001417c0       ?ExtrudeBox@@YAXPEBUbox@primitives@@AEBU?$Vec3_tpl@M@@MPEAU12@@Z 00000000351427c0 f   utils.obj
 0001:00141e50       ?ReadCompressedQuat@@YAXAEAVCStream@@AEAU?$Quat_tpl@M@@@Z 0000000035142e50 f   utils.obj
 0001:00142130       ?SetGeomConvex@CAABBTree@@UEAAXXZ 0000000035143130 f   aabbtree.obj
 0001:00142160       ?ReleaseLastSweptBVs@CAABBTree@@UEAAXH@Z 0000000035143160 f   aabbtree.obj
 0001:00142180       ?GetNodeContents@CAABBTree@@UEAAHHPEAUBV@@HHPEAUgeometry_under_test@@1@Z 0000000035143180 f   aabbtree.obj
 0001:00142220       ?GetRootNodeDim@CAABBTree@@QEAAXAEAU?$Vec3_tpl@M@@0@Z 0000000035143220 f i aabbtree.obj
 0001:00142440       ?GetBBox@CAABBTree@@UEAAXPEAUbox@primitives@@@Z 0000000035143440 f   aabbtree.obj
 0001:001424b0       ?GetNodeBV@CAABBTree@@UEAAXAEAPEAUBV@@HH@Z 00000000351434b0 f   aabbtree.obj
 0001:00142570       ?GetNodeBV@CAABBTree@@UEAAXAEAPEAUBV@@AEBU?$Vec3_tpl@M@@MHH@Z 0000000035143570 f   aabbtree.obj
 0001:00142640       ?SplitPriority@CAABBTree@@UEAAMPEBUBV@@@Z 0000000035143640 f   aabbtree.obj
 0001:00142680       ?GetNodeChildrenBVs@CAABBTree@@UEAAXAEBU?$Matrix33_tpl@M@@AEBU?$Vec3_tpl@M@@MPEBUBV@@AEAPEAU4@3H@Z 0000000035143680 f   aabbtree.obj
 0001:00142bc0       ?GetNodeChildrenBVs@CAABBTree@@UEAAXPEBUBV@@AEAPEAU2@1H@Z 0000000035143bc0 f   aabbtree.obj
 0001:00143210       ?GetNodeChildrenBVs@CAABBTree@@UEAAXPEBUBV@@AEBU?$Vec3_tpl@M@@MAEAPEAU2@2H@Z 0000000035144210 f   aabbtree.obj
 0001:001438e0       ?MarkUsedTriangle@CAABBTree@@UEAAXHPEAUgeometry_under_test@@@Z 00000000351448e0 f   aabbtree.obj
 0001:001439c0       ?PrepareForIntersectionTest@CAABBTree@@UEAAHPEAUgeometry_under_test@@PEAVCGeometry@@0@Z 00000000351449c0 f   aabbtree.obj
 0001:00143af0       ?GetMemoryStatistics@CAABBTree@@UEAAXPEAVICrySizer@@@Z 0000000035144af0 f   aabbtree.obj
 0001:00143ba0       ?SanityCheck@CAABBTree@@UEAAHXZ 0000000035144ba0 f   aabbtree.obj
 0001:00143bb0       ?SetParams@CAABBTree@@QEAAXHHMAEBU?$Matrix33_tpl@M@@H@Z 0000000035144bb0 f   aabbtree.obj
 0001:00143cb0       ?BuildNode@CAABBTree@@QEAAMHHHU?$Vec3_tpl@M@@0PEAY02U2@H@Z 0000000035144cb0 f   aabbtree.obj
 0001:00144d90       ?Save@CAABBTree@@UEAAXAEAVCMemStream@@@Z 0000000035145d90 f   aabbtree.obj
 0001:00144fe0       ?Load@CAABBTree@@UEAAXAEAVCMemStream@@PEAVCGeometry@@@Z 0000000035145fe0 f   aabbtree.obj
 0001:001453d0       ?Build@CAABBTree@@UEAAMPEAVCGeometry@@@Z 00000000351463d0 f   aabbtree.obj
 0001:00145e30       ?GetNodeBV@CAABBTree@@UEAAXAEBU?$Matrix33_tpl@M@@AEBU?$Vec3_tpl@M@@MAEAPEAUBV@@HH@Z 0000000035146e30 f   aabbtree.obj
 0001:001461b0       ?PrepareForIntersectionTest@CBoxGeom@@UEAAHPEAUgeometry_under_test@@PEAVCGeometry@@0_N@Z 00000000351471b0 f   boxgeom.obj
 0001:00146280       ?GetMemoryStatistics@CBoxGeom@@UEAAXPEAVICrySizer@@@Z 0000000035147280 f   boxgeom.obj
 0001:001462a0       ?PointInsideStatus@CBoxGeom@@UEAAHAEBU?$Vec3_tpl@M@@@Z 00000000351472a0 f   boxgeom.obj
 0001:001463d0       ?GetFeature@CBoxGeom@@UEAAHHHPEAU?$Vec3_tpl@M@@@Z 00000000351473d0 f   boxgeom.obj
 0001:001468a0       ?BuildTriMesh@CBoxGeom@@QEAAXAEAVCTriMesh@@H@Z 00000000351478a0 f   boxgeom.obj
 0001:00147020       ?GetErrorCount@CGeometry@@UEAAHXZ 0000000035148020 f   livingentity.obj
 0001:00147020       ?default_unprojection@@YAHPEAUunprojection_mode@@PEBUprimitive@primitives@@H1HPEAUcontact@@PEAUgeom_contact_area@@@Z 0000000035148020 f   linunprojectionchecks.obj
 0001:00147020       ?AddRef@CPhysicalStub@@UEAAHXZ 0000000035148020 f   physarea.obj
 0001:00147020       ?GetStateSnapshotTxt@CPhysicalStub@@UEAAHPEADHM@Z 0000000035148020 f   physarea.obj
 0001:00147020       ?RegisterContacts@CPhysicalEntity@@UEAAHMH@Z 0000000035148020 f   particleentity.obj
 0001:00147020       ?HasConstraintContactsWith@CPhysicalEntity@@UEBAHPEBV1@H@Z 0000000035148020 f   livingentity.obj
 0001:00147020       ?Step@CPhysicalStub@@UEAAHM@Z 0000000035148020 f   physarea.obj
 0001:00147020       ?GetStatus@CPhysicalStub@@UEBAHPEAUpe_status@@@Z 0000000035148020 f   physarea.obj
 0001:00147020       ?GetType@COBBTree@@UEAAHXZ 0000000035148020 f   trimesh.obj
 0001:00147020       ?GetStateChecksum@CPhysicalStub@@UEAAIXZ 0000000035148020 f   physarea.obj
 0001:00147020       ?UnprojectSphere@CGeometry@@UEAAHU?$Vec3_tpl@M@@MMPEAUcontact@@@Z 0000000035148020 f   livingentity.obj
 0001:00147020       ?SetStateFromTypedSnapshot@CPhysicalStub@@UEAAHV?$CSerializeWrapper@UISerialize@@@@HH@Z 0000000035148020 f   physarea.obj
 0001:00147020       ?Awake@CPhysicalEntity@@UEAAHHH@Z 0000000035148020 f   physicalentity.obj
 0001:00147020       ?SetStateFromSnapshot@CPhysicalEntity@@UEAAHAEAVCStream@@H@Z 0000000035148020 f   physicalentity.obj
 0001:00147020       ?SetStateFromSnapshot@CPhysicalStub@@UEAAHV?$CSerializeWrapper@UISerialize@@@@H@Z 0000000035148020 f   physarea.obj
 0001:00147020       ?SetParams@CPhysicalStub@@UEAAHPEAUpe_params@@H@Z 0000000035148020 f   physarea.obj
 0001:00147020       ?FindClosestPoint@CGeometry@@UEAAHPEAUgeom_world_data@@AEAH1AEBU?$Vec3_tpl@M@@2PEAU3@H@Z 0000000035148020 f   livingentity.obj
 0001:00147020       ?HasCollisionContactsWith@CPhysicalEntity@@UEAAHPEAV1@@Z 0000000035148020 f   livingentity.obj
 0001:00147020       ?DoStep@CPhysicalStub@@UEAAHMH@Z 0000000035148020 f   physarea.obj
 0001:00147020       ?Boxify@CGeometry@@UEAAHPEAUbox@primitives@@HAEBUSBoxificationParams@IGeometry@@@Z 0000000035148020 f   livingentity.obj
 0001:00147020       ?PreparePolygon@CGeometry@@UEAAHPEAUcoord_plane@primitives@@HHPEAUgeometry_under_test@@AEAPEAU?$Vec2_tpl@M@@AEAPEAH3@Z 0000000035148020 f   livingentity.obj
 0001:00147020       ?SetStateFromSnapshot@CParticleEntity@@UEAAHAEAVCStream@@H@Z 0000000035148020 f   particleentity.obj
 0001:00147020       ?GetIWorld@CGeomManager@@UEAAPEAUIPhysicalWorld@@XZ 0000000035148020 f   physicalworld.obj
 0001:00147020       ?RayTrace@CPhysicalEntity@@UEAAHAEAUSRayTraceRes@@@Z 0000000035148020 f   rwi.obj
 0001:00147020       ?SetStateFromSnapshot@CSoftEntity@@UEAAHAEAVCStream@@H@Z 0000000035148020 f   softentity.obj
 0001:00147020       ?GetPrimitiveList@CGeometry@@UEAAHHHHPEAUprimitive@primitives@@HPEAUgeometry_under_test@@10PEAD@Z 0000000035148020 f   livingentity.obj
 0001:00147020       ?GetStateChecksum@CPhysicalEntity@@UEAAIXZ 0000000035148020 f   livingentity.obj
 0001:00147020       ?GetBVTree@CGeometry@@UEAAPEAVCBVTree@@XZ 0000000035148020 f   livingentity.obj
 0001:00147020       ?Subtract@CGeometry@@UEAAHPEAUIGeometry@@PEAUgeom_world_data@@1H@Z 0000000035148020 f   livingentity.obj
 0001:00147020       ?PreparePolyline@CGeometry@@UEAAHPEAUcoord_plane@primitives@@HHPEAUgeometry_under_test@@AEAPEAU?$Vec2_tpl@M@@AEAPEAH3@Z 0000000035148020 f   livingentity.obj
 0001:00147020       ?GetWorld@CPhysicalStub@@UEBAPEAUIPhysicalWorld@@XZ 0000000035148020 f   physarea.obj
 0001:00147020       ?GetFeature@CGeometry@@UEAAHHHPEAU?$Vec3_tpl@M@@@Z 0000000035148020 f   livingentity.obj
 0001:00147020       ?SerializeWorld@CPhysicalWorld@@UEAAHPEBDH@Z 0000000035148020 f   physicalworld.obj
 0001:00147020       ?GetParams@CPhysicalStub@@UEBAHPEAUpe_params@@@Z 0000000035148020 f   physarea.obj
 0001:00147020       ?CalcPhysicalProperties@CGeometry@@UEAAHPEAUphys_geometry@@@Z 0000000035148020 f   livingentity.obj
 0001:00147020       ?Release@CPhysicalStub@@UEAAHXZ 0000000035148020 f   physarea.obj
 0001:00147020       ?GetiForeignData@CPhysicalStub@@UEBAHXZ 0000000035148020 f   physarea.obj
 0001:00147020       ?IsAwake@CPhysicalEntity@@UEBAHH@Z 0000000035148020 f   livingentity.obj
 0001:00147020       ?GetStateSnapshot@CPhysicalEntity@@UEAAHAEAVCStream@@MH@Z 0000000035148020 f   physicalentity.obj
 0001:00147020       ?get_deleter@?$sp_counted_impl_p@VCEngineModule_CryPhysics@@@detail@boost@@UEAAPEAXAEBVsp_typeinfo@23@@Z 0000000035148020 f   CryPhysics.obj
 0001:00147020       ?Action@CPhysicalStub@@UEAAHPEAUpe_action@@H@Z 0000000035148020 f   physarea.obj
 0001:00147020       ?GetTriMesh@CBoxGeom@@UEAAPEAUIGeometry@@H@Z 0000000035148020 f   boxgeom.obj
 0001:00147020       ?GetTriMesh@CGeometry@@UEAAPEAUIGeometry@@H@Z 0000000035148020 f   livingentity.obj
 0001:00147020       ?GetType@CBoxGeom@@UEAAHXZ 0000000035148020 f   physicalentity.obj
 0001:00147020       ?IsConvex@CVoxelGeom@@UEAAHM@Z 0000000035148020 f   geoman.obj
 0001:00147020       ?GetForeignData@CPhysicalStub@@UEBAPEAXH@Z 0000000035148020 f   physarea.obj
 0001:00147020       ?GetSubtractionsCount@CGeometry@@UEAAHXZ 0000000035148020 f   livingentity.obj
 0001:00147020       ?SerializeGeometries@CPhysicalWorld@@UEAAHPEBDH@Z 0000000035148020 f   physicalworld.obj
 0001:00147020       ?PostSetStateFromSnapshot@CPhysicalStub@@UEAAHXZ 0000000035148020 f   physarea.obj
 0001:00147020       ?IsConvex@CHeightfield@@UEAAHM@Z 0000000035148020 f   waterman.obj
 0001:00147020       ?SetStateFromSnapshot@CLivingEntity@@UEAAHAEAVCStream@@H@Z 0000000035148020 f   livingentity.obj
 0001:00147020       ?default_intersection@@YAHPEBUprimitive@primitives@@0PEAUprim_inters@@@Z 0000000035148020 f   intersectionchecks.obj
 0001:00147020       ?SetStateFromSnapshot@CArticulatedEntity@@UEAAHAEAVCStream@@H@Z 0000000035148020 f   articulatedentity.obj
 0001:00147020       ?CheckSelfCollision@CRigidEntity@@UEAAHHH@Z 0000000035148020 f   rigidentity.obj
 0001:00147020       ?QueryComposite@CEngineModule_CryPhysics@@MEBAPEAXPEBD@Z 0000000035148020 f   CryPhysics.obj
 0001:00147020       ?SetStateFromSnapshot@CRopeEntity@@UEAAHAEAVCStream@@H@Z 0000000035148020 f   ropeentity.obj
 0001:00147020       ?SetStateFromSnapshot@CPhysicalStub@@UEAAHAEAVCStream@@H@Z 0000000035148020 f   physarea.obj
 0001:00147020       ?GetSizeFast@CGeometry@@UEAAHXZ 0000000035148020 f   livingentity.obj
 0001:00147020       ?DrawToOcclusionCubemap@CGeometry@@UEAAHPEBUgeom_world_data@@HHHPEAUSOcclusionCubeMap@@@Z 0000000035148020 f   livingentity.obj
 0001:00147020       ?GetContactCount@CPhysicalEntity@@UEAAHH@Z 0000000035148020 f   livingentity.obj
 0001:00147020       ?AddRef@CPhysicalPlaceholder@@UEAAHXZ 0000000035148020 f   physarea.obj
 0001:00147020       ?GetStateSnapshot@CPhysicalStub@@UEAAHV?$CSerializeWrapper@UISerialize@@@@MH@Z 0000000035148020 f   physarea.obj
 0001:00147020       ?Release@CPhysicalPlaceholder@@UEAAHXZ 0000000035148020 f   physarea.obj
 0001:00147020       ?HasContactsWith@CPhysicalEntity@@UEAAHPEAV1@@Z 0000000035148020 f   livingentity.obj
 0001:00147020       ?IsAPrimitive@CGeometry@@UEAAHXZ 0000000035148020 f   livingentity.obj
 0001:00147020       ?GetStateSnapshot@CPhysicalStub@@UEAAHAEAVCStream@@MH@Z 0000000035148020 f   physarea.obj
 0001:00147030       ?CalcVolumetricPressure@CBoxGeom@@UEAAXPEAUgeom_world_data@@AEBU?$Vec3_tpl@M@@MM1AEAU3@2@Z 0000000035148030 f   boxgeom.obj
 0001:001470e0       ?CalculateBuoyancy@CBoxGeom@@UEAAMPEBUplane@primitives@@PEBUgeom_world_data@@AEAU?$Vec3_tpl@M@@@Z 00000000351480e0 f   boxgeom.obj
 0001:00147170       ?DrawWireframe@CBoxGeom@@UEAAXPEAUIPhysRenderer@@PEAUgeom_world_data@@HH@Z 0000000035148170 f   boxgeom.obj
 0001:001472c0       ?CreateBox@CBoxGeom@@QEAAPEAV1@PEAUbox@primitives@@@Z 00000000351482c0 f   boxgeom.obj
 0001:00147410       ?FindClosestPoint@CBoxGeom@@UEAAHPEAUgeom_world_data@@AEAH1AEBU?$Vec3_tpl@M@@2PEAU3@H@Z 0000000035148410 f   boxgeom.obj
 0001:00148bd0       ?UnprojectSphere@CBoxGeom@@UEAAHU?$Vec3_tpl@M@@MMPEAUcontact@@@Z 0000000035149bd0 f   boxgeom.obj
 0001:00148d00       ?Save@CBoxGeom@@UEAAXAEAVCMemStream@@@Z 0000000035149d00 f   boxgeom.obj
 0001:00148da0       ?Load@CBoxGeom@@UEAAXAEAVCMemStream@@@Z 0000000035149da0 f   boxgeom.obj
 0001:00148e20       ?CalcPhysicalProperties@CBoxGeom@@UEAAHPEAUphys_geometry@@@Z 0000000035149e20 f   boxgeom.obj
 0001:001490f0       ?PrepareBox@CBoxGeom@@QEAAXPEAUbox@primitives@@PEAUgeometry_under_test@@@Z 000000003514a0f0 f   boxgeom.obj
 0001:00149470       ?PreparePrimitive@CBoxGeom@@UEAAHPEAUgeom_world_data@@AEAPEAUprimitive@primitives@@H@Z 000000003514a470 f   boxgeom.obj
 0001:00149810       ?GetPrimitiveList@CBoxGeom@@UEAAHHHHPEAUprimitive@primitives@@HPEAUgeometry_under_test@@10PEAD@Z 000000003514a810 f   boxgeom.obj
 0001:00149ad0       ?GetUnprojectionCandidates@CBoxGeom@@UEAAHHPEBUcontact@@AEAPEAUprimitive@primitives@@AEAPEAHPEAUgeometry_under_test@@@Z 000000003514aad0 f   boxgeom.obj
 0001:0014a200       ?PreparePolygon@CBoxGeom@@UEAAHPEAUcoord_plane@primitives@@HHPEAUgeometry_under_test@@AEAPEAU?$Vec2_tpl@M@@AEAPEAH3@Z 000000003514b200 f   boxgeom.obj
 0001:0014ac30       ?PreparePolyline@CBoxGeom@@UEAAHPEAUcoord_plane@primitives@@HHPEAUgeometry_under_test@@AEAPEAU?$Vec2_tpl@M@@AEAPEAH3@Z 000000003514bc30 f   boxgeom.obj
 0001:0014b3d0       ?CalculateMediumResistance@CBoxGeom@@UEAAXPEBUplane@primitives@@PEBUgeom_world_data@@AEAU?$Vec3_tpl@M@@2@Z 000000003514c3d0 f   boxgeom.obj
 0001:0014bca0       ?DrawToOcclusionCubemap@CBoxGeom@@UEAAHPEBUgeom_world_data@@HHHPEAUSOcclusionCubeMap@@@Z 000000003514cca0 f   boxgeom.obj
 0001:0014c560       ?PrepareForIntersectionTest@CCapsuleGeom@@UEAAHPEAUgeometry_under_test@@PEAVCGeometry@@0_N@Z 000000003514d560 f   capsulegeom.obj
 0001:0014c5a0       ?PointInsideStatus@CCapsuleGeom@@UEAAHAEBU?$Vec3_tpl@M@@@Z 000000003514d5a0 f   capsulegeom.obj
 0001:0014c780       ?CalculateBuoyancy@CCapsuleGeom@@UEAAMPEBUplane@primitives@@PEBUgeom_world_data@@AEAU?$Vec3_tpl@M@@@Z 000000003514d780 f   capsulegeom.obj
 0001:0014c790       ?CreateCapsule@CCapsuleGeom@@QEAAPEAV1@PEAUcapsule@primitives@@@Z 000000003514d790 f   capsulegeom.obj
 0001:0014c9c0       ?GetUnprojectionCandidates@CCapsuleGeom@@UEAAHHPEBUcontact@@AEAPEAUprimitive@primitives@@AEAPEAHPEAUgeometry_under_test@@@Z 000000003514d9c0 f   capsulegeom.obj
 0001:0014cc80       ?FindClosestPoint@CCapsuleGeom@@UEAAHPEAUgeom_world_data@@AEAH1AEBU?$Vec3_tpl@M@@2PEAU3@H@Z 000000003514dc80 f   capsulegeom.obj
 0001:0014db60       ?UnprojectSphere@CCapsuleGeom@@UEAAHU?$Vec3_tpl@M@@MMPEAUcontact@@@Z 000000003514eb60 f   capsulegeom.obj
 0001:0014dfd0       ?CalculateMediumResistance@CCapsuleGeom@@UEAAXPEBUplane@primitives@@PEBUgeom_world_data@@AEAU?$Vec3_tpl@M@@2@Z 000000003514efd0 f   capsulegeom.obj
 0001:0014eb00       ?DrawToOcclusionCubemap@CCapsuleGeom@@UEAAHPEBUgeom_world_data@@HHHPEAUSOcclusionCubeMap@@@Z 000000003514fb00 f   capsulegeom.obj
 0001:0014ecc0       ?CalcPhysicalProperties@CCapsuleGeom@@UEAAHPEAUphys_geometry@@@Z 000000003514fcc0 f   capsulegeom.obj
 0001:0014ef70       ?PrepareForIntersectionTest@CCylinderGeom@@UEAAHPEAUgeometry_under_test@@PEAVCGeometry@@0_N@Z 000000003514ff70 f   cylindergeom.obj
 0001:0014f080       ?ComputeExtent@CCylinderGeom@@UEAAMAEAUGeomQuery@@W4EGeomForm@@@Z 0000000035150080 f   cylindergeom.obj
 0001:0014f100       ?GetMemoryStatistics@CCylinderGeom@@UEAAXPEAVICrySizer@@@Z 0000000035150100 f   cylindergeom.obj
 0001:0014f120       ?PointInsideStatus@CCylinderGeom@@UEAAHAEBU?$Vec3_tpl@M@@@Z 0000000035150120 f   cylindergeom.obj
 0001:0014f210       ?PrepareCylinder@CCylinderGeom@@QEAAXPEAUcylinder@primitives@@PEAUgeometry_under_test@@@Z 0000000035150210 f   cylindergeom.obj
 0001:0014f3a0       ?PreparePrimitive@CCylinderGeom@@UEAAHPEAUgeom_world_data@@AEAPEAUprimitive@primitives@@H@Z 00000000351503a0 f   cylindergeom.obj
 0001:0014f550       ?GetPrimitiveList@CCylinderGeom@@UEAAHHHHPEAUprimitive@primitives@@HPEAUgeometry_under_test@@10PEAD@Z 0000000035150550 f   cylindergeom.obj
 0001:0014f580       ?PreparePolyline@CCylinderGeom@@UEAAHPEAUcoord_plane@primitives@@HHPEAUgeometry_under_test@@AEAPEAU?$Vec2_tpl@M@@AEAPEAH3@Z 0000000035150580 f   cylindergeom.obj
 0001:0014f9a0       ?DrawWireframe@CCylinderGeom@@UEAAXPEAUIPhysRenderer@@PEAUgeom_world_data@@HH@Z 00000000351509a0 f   cylindergeom.obj
 0001:0014faf0       ?CreateCylinder@CCylinderGeom@@QEAAPEAV1@PEAUcylinder@primitives@@@Z 0000000035150af0 f   cylindergeom.obj
 0001:0014fd20       ?GetRandomPos@CCylinderGeom@@UEAAXAEAURandomPos@@AEAUGeomQuery@@W4EGeomForm@@@Z 0000000035150d20 f   cylindergeom.obj
 0001:001502e0       ?GetUnprojectionCandidates@CCylinderGeom@@UEAAHHPEBUcontact@@AEAPEAUprimitive@primitives@@AEAPEAHPEAUgeometry_under_test@@@Z 00000000351512e0 f   cylindergeom.obj
 0001:00150670       ?PreparePolygon@CCylinderGeom@@UEAAHPEAUcoord_plane@primitives@@HHPEAUgeometry_under_test@@AEAPEAU?$Vec2_tpl@M@@AEAPEAH3@Z 0000000035151670 f   cylindergeom.obj
 0001:00150e30       ?UnprojectSphere@CCylinderGeom@@UEAAHU?$Vec3_tpl@M@@MMPEAUcontact@@@Z 0000000035151e30 f   cylindergeom.obj
 0001:001510d0       ?CalcVolumetricPressure@CCylinderGeom@@UEAAXPEAUgeom_world_data@@AEBU?$Vec3_tpl@M@@MM1AEAU3@2@Z 00000000351520d0 f   cylindergeom.obj
 0001:00151450       ?CalculateBuoyancy@CCylinderGeom@@UEAAMPEBUplane@primitives@@PEBUgeom_world_data@@AEAU?$Vec3_tpl@M@@@Z 0000000035152450 f   cylindergeom.obj
 0001:001524a0       ?crop_polyarc2d_with_line@@YAHPEBU?$Vec2_tpl@M@@PEBHHMPEAU1@PEAHAEBU1@4@Z 00000000351534a0 f   cylindergeom.obj
 0001:00152e60       ?CalculateMediumResistance@CCylinderGeom@@UEAAXPEBUplane@primitives@@PEBUgeom_world_data@@AEAU?$Vec3_tpl@M@@2@Z 0000000035153e60 f   cylindergeom.obj
 0001:00154a40       ?DrawToOcclusionCubemap@CCylinderGeom@@UEAAHPEBUgeom_world_data@@HHHPEAUSOcclusionCubeMap@@@Z 0000000035155a40 f   cylindergeom.obj
 0001:00154be0       ?Save@CCylinderGeom@@UEAAXAEAVCMemStream@@@Z 0000000035155be0 f   cylindergeom.obj
 0001:00154c90       ?Load@CCylinderGeom@@UEAAXAEAVCMemStream@@@Z 0000000035155c90 f   cylindergeom.obj
 0001:00154d00       ?findroots@?$polynomial_tpl@N$03@@QEBAHNNPEANHH_N@Z 0000000035155d00 f i cylindergeom.obj
 0001:00155ec0       ?CalcPhysicalProperties@CCylinderGeom@@UEAAHPEAUphys_geometry@@@Z 0000000035156ec0 f   cylindergeom.obj
 0001:00156150       ?FindClosestPoint@CCylinderGeom@@UEAAHPEAUgeom_world_data@@AEAH1AEBU?$Vec3_tpl@M@@2PEAU3@H@Z 0000000035157150 f   cylindergeom.obj
 0001:00158500       ?InitGeoman@CGeomManager@@UEAAXXZ 0000000035159500 f   geoman.obj
 0001:00158540       ?ShutDownGeoman@CGeomManager@@UEAAXXZ 0000000035159540 f   geoman.obj
 0001:00158660       ?DestroyGeometry@CGeomManager@@UEAAXPEAUIGeometry@@@Z 0000000035159660 f   geoman.obj
 0001:00158670       ?AddRefGeometry@CGeomManager@@UEAAHPEAUphys_geometry@@@Z 0000000035159670 f   geoman.obj
 0001:00158680       ?UnregisterGeometry@CGeomManager@@UEAAHPEAUphys_geometry@@@Z 0000000035159680 f   geoman.obj
 0001:00158760       ?Release@CGeometry@@UEAAXXZ 0000000035159760 f   geoman.obj
 0001:001587c0       ?FlushOldGeoms@CGeomManager@@QEAAXXZ 00000000351597c0 f   geoman.obj
 0001:00158820       ?SetGeomMatMapping@CGeomManager@@UEAAXPEAUphys_geometry@@PEAHH@Z 0000000035159820 f   geoman.obj
 0001:001588c0       ?CreateTetrLattice@CGeomManager@@UEAAPEAUITetrLattice@@PEBU?$Vec3_tpl@M@@HPEBHH@Z 00000000351598c0 f   geoman.obj
 0001:00158950       ?Build@CRayBV@@UEAAMPEAVCGeometry@@@Z 0000000035159950 f i livingentity.obj
 0001:00158950       ?Build@CVoxelBV@@UEAAMPEAVCGeometry@@@Z 0000000035159950 f i geoman.obj
 0001:00158960       ?MaxPrimsInNode@CVoxelBV@@UEAAHXZ 0000000035159960 f i geoman.obj
 0001:00158970       ?GetNodeBV@CVoxelBV@@UEAAXAEAPEAUBV@@AEBU?$Vec3_tpl@M@@MHH@Z 0000000035159970 f i geoman.obj
 0001:00158980       ?GetNodeBV@CVoxelBV@@UEAAXAEBU?$Matrix33_tpl@M@@AEBU?$Vec3_tpl@M@@MAEAPEAUBV@@1MHH@Z 0000000035159980 f i geoman.obj
 0001:001589b0       ?ResetCollisionArea@CVoxelBV@@UEAAXXZ 00000000351599b0 f i geoman.obj
 0001:001589d0       ??0CBreakableGrid2d@@QEAA@XZ 00000000351599d0 f i geoman.obj
 0001:00158a40       ?GetGridData@CBreakableGrid2d@@UEAAPEAUgrid@primitives@@XZ 0000000035159a40 f i geoman.obj
 0001:00158a50       ?IsEmpty@CBreakableGrid2d@@UEAA_NXZ 0000000035159a50 f i geoman.obj
 0001:00158a60       ?GetFracture@CBreakableGrid2d@@UEAAMXZ 0000000035159a60 f i geoman.obj
 0001:00158a80       ?GetMemoryStatistics@CBreakableGrid2d@@UEBAXPEAVICrySizer@@@Z 0000000035159a80 f i geoman.obj
 0001:00158b00       ??_GCBreakableGrid2d@@UEAAPEAXI@Z 0000000035159b00 f i geoman.obj
 0001:00158b00       ??_ECBreakableGrid2d@@UEAAPEAXI@Z 0000000035159b00 f i geoman.obj
 0001:00158b80       ?GenerateBreakableGrid@CGeomManager@@UEAAPEAUIBreakableGrid2d@@PEAU?$Vec2_tpl@M@@HAEBU?$Vec2_tpl@H@@HH@Z 0000000035159b80 f   geoman.obj
 0001:00158c00       ??0CRayGeom@@QEAA@PEBUray@primitives@@@Z 0000000035159c00 f i geoman.obj
 0001:00158d30       ?GetFreeGeomSlot@CGeomManager@@QEAAPEAUphys_geometry@@XZ 0000000035159d30 f   geoman.obj
 0001:00158e50       ?RegisterGeometry@CGeomManager@@UEAAPEAUphys_geometry@@PEAUIGeometry@@HPEAHH@Z 0000000035159e50 f   geoman.obj
 0001:00159000       ?SaveGeometry@CGeomManager@@UEAAXAEAVCMemStream@@PEAUIGeometry@@@Z 000000003515a000 f   geoman.obj
 0001:00159070       ?LoadGeometry@CGeomManager@@UEAAPEAUIGeometry@@AEAVCMemStream@@V?$strided_pointer@$$CBU?$Vec3_tpl@M@@@@V?$strided_pointer@G@@PEAD@Z 000000003515a070 f   geoman.obj
 0001:00159320       ?SavePhysGeometry@CGeomManager@@UEAAXAEAVCMemStream@@PEAUphys_geometry@@@Z 000000003515a320 f   geoman.obj
 0001:001594b0       ?LoadPhysGeometry@CGeomManager@@UEAAPEAUphys_geometry@@AEAVCMemStream@@V?$strided_pointer@$$CBU?$Vec3_tpl@M@@@@V?$strided_pointer@G@@PEAD@Z 000000003515a4b0 f   geoman.obj
 0001:00159710       ??$ComputeMeshEigenBasis@G@@YAXV?$strided_pointer@$$CBU?$Vec3_tpl@M@@@@V?$strided_pointer@G@@HPEAU?$Vec3_tpl@N@@AEAU2@@Z 000000003515a710 f i geoman.obj
 0001:0015a260       ??1CMemStream@@UEAA@XZ     000000003515b260 f i geoman.obj
 0001:0015a2d0       ?Prealloc@CMemStream@@UEAAXXZ 000000003515b2d0 f i geoman.obj
 0001:0015a360       ?GrowBuf@CMemStream@@UEAAXH@Z 000000003515b360 f i geoman.obj
 0001:0015a400       ??_ECMemStream@@UEAAPEAXI@Z 000000003515b400 f i geoman.obj
 0001:0015a400       ??_GCMemStream@@UEAAPEAXI@Z 000000003515b400 f i geoman.obj
 0001:0015a430       ??0CVoxelGeom@@QEAA@XZ     000000003515b430 f i geoman.obj
 0001:0015a490       ?GetData@CTriMesh@@UEAAPEBUprimitive@primitives@@XZ 000000003515b490 f i geoman.obj
 0001:0015a4a0       ?GetBVTree@CVoxelGeom@@UEAAPEAVCBVTree@@XZ 000000003515b4a0 f i geoman.obj
 0001:0015a4b0       ??_GCVoxelGeom@@UEAAPEAXI@Z 000000003515b4b0 f i geoman.obj
 0001:0015a4b0       ??_ECVoxelGeom@@UEAAPEAXI@Z 000000003515b4b0 f i geoman.obj
 0001:0015a530       ?GetPrimitive@CTriMesh@@UEAAHHPEAUprimitive@primitives@@@Z 000000003515b530 f i geoman.obj
 0001:0015a5f0       ?CreateMesh@CGeomManager@@UEAAPEAUIGeometry@@V?$strided_pointer@$$CBU?$Vec3_tpl@M@@@@V?$strided_pointer@G@@PEADPEAHHHMPEAUSMeshBVParams@@@Z 000000003515b5f0 f   geoman.obj
 0001:0015a920       ?CreatePrimitive@CGeomManager@@UEAAPEAUIGeometry@@HPEBUprimitive@primitives@@@Z 000000003515b920 f   geoman.obj
 0001:0015ac40       ?RegisterCrack@CGeomManager@@UEAAHPEAUIGeometry@@PEAU?$Vec3_tpl@M@@H@Z 000000003515bc40 f   geoman.obj
 0001:0015b800       ?UnregisterCrack@CGeomManager@@UEAAXH@Z 000000003515c800 f   geoman.obj
 0001:0015b8f0       ?GetCrackGeom@CGeomManager@@UEAAPEAUIGeometry@@PEBU?$Vec3_tpl@M@@HPEAUgeom_world_data@@@Z 000000003515c8f0 f   geoman.obj
 0001:0015cd60       ?CloneGeometry@CGeomManager@@UEAAPEAUIGeometry@@PEAU2@@Z 000000003515dd60 f   geoman.obj
 0001:0015cf10       ??0InitGeometryGlobals@@QEAA@XZ 000000003515df10 f   geometry.obj
 0001:0015cfe0       ?RadiusCheckBVs@@YAHPEAUradius_check_data@@PEAUBV@@@Z 000000003515dfe0 f   geometry.obj
 0001:0015d0f0       ?SphereCheckBVs@@YAHPEAVCBVTree@@PEAUsphere@primitives@@PEAUBV@@H@Z 000000003515e0f0 f   geometry.obj
 0001:0015d1e0       ?IntersectLocked@CGeometry@@UEAAHPEAUIGeometry@@PEAUgeom_world_data@@1PEAUintersection_params@@AEAPEAUgeom_contact@@AEAUWriteLockCond@@H@Z 000000003515e1e0 f   geometry.obj
 0001:0015d2b0       ?TestBV@@YAXPEAVCBVTree@@PEAUBV@@HHAEA_NH@Z 000000003515e2b0 f   geometry.obj
 0001:0015d380       ?ComputeExtent@CGeometry@@UEAAMAEAUGeomQuery@@W4EGeomForm@@@Z 000000003515e380 f   geometry.obj
 0001:0015d420       ?SanityCheckTree@@YAHPEAVCBVTree@@H@Z 000000003515e420 f   geometry.obj
 0001:0015d4f0       ?BoxRandomPos@@YAXAEAURandomPos@@W4EGeomForm@@AEBU?$Vec3_tpl@M@@@Z 000000003515e4f0 f i geometry.obj
 0001:0015d7e0       ?IntersectBVs@@YAHPEAUgeometry_under_test@@PEAUBV@@1@Z 000000003515e7e0 f   geometry.obj
 0001:0015dd80       ?SweepTestBVs@@YAHPEAUgeometry_under_test@@PEAUBV@@1@Z 000000003515ed80 f   geometry.obj
 0001:0015e420       ?BuildOcclusionCubemap@CGeometry@@UEAAMPEAUgeom_world_data@@HPEAUSOcclusionCubeMap@@1H@Z 000000003515f420 f   geometry.obj
 0001:0015e710       ?RegisterIntersection@CGeometry@@UEAAHPEAUprimitive@primitives@@0PEAUgeometry_under_test@@1PEAUprim_inters@@@Z 000000003515f710 f   geometry.obj
 0001:0015ef20       ?GetRandomPos@CGeometry@@UEAAXAEAURandomPos@@AEAUGeomQuery@@W4EGeomForm@@@Z 000000003515ff20 f   geometry.obj
 0001:0015f0d0       ?SphereCheck@CGeometry@@QEAAHAEBU?$Vec3_tpl@M@@MH@Z 00000000351600d0 f   geometry.obj
 0001:0015f260       ?GTestPrepPartDeux@@YAXPEAUgeometry_under_test@@AEAU?$Vec3_tpl@N@@@Z 0000000035160260 f   geometry.obj
 0001:0015f720       ?Intersect@CGeometry@@UEAAHPEAUIGeometry@@PEAUgeom_world_data@@1PEAUintersection_params@@AEAPEAUgeom_contact@@@Z 0000000035160720 f   geometry.obj
 0001:001617c0       ?DrawBBox@@YAXPEAUIPhysRenderer@@HPEAUgeom_world_data@@PEAVCBVTree@@PEAUBBox@@HHH@Z 00000000351627c0 f   geometry.obj
 0001:00161b70       ?Intersect@CPrimitive@@UEAAHPEAUIGeometry@@PEAUgeom_world_data@@1PEAUintersection_params@@AEAPEAUgeom_contact@@@Z 0000000035162b70 f   geometry.obj
 0001:00163a60       ?Build@CHeightfieldBV@@UEAAMPEAVCGeometry@@@Z 0000000035164a60 f   heightfieldbv.obj
 0001:00163aa0       ?MarkUsedTriangle@CHeightfieldBV@@UEAAXHPEAUgeometry_under_test@@@Z 0000000035164aa0 f   heightfieldbv.obj
 0001:00163ac0       ?GetBBox@CHeightfieldBV@@UEAAXPEAUbox@primitives@@@Z 0000000035164ac0 f   heightfieldbv.obj
 0001:00163b70       ?GetNodeBV@CHeightfieldBV@@UEAAXAEAPEAUBV@@HH@Z 0000000035164b70 f   heightfieldbv.obj
 0001:00163cc0       ?project_box_on_grid@@YAXPEAUbox@primitives@@PEAUgrid@2@PEAUgeometry_under_test@@AEAH333AEAM@Z 0000000035164cc0 f   heightfieldbv.obj
 0001:00164300       ?GetNodeContents@CHeightfieldBV@@UEAAHHPEAUBV@@HHPEAUgeometry_under_test@@1@Z 0000000035165300 f   heightfieldbv.obj
 0001:001645c0       ?GetNodeBV@CHeightfieldBV@@UEAAXAEBU?$Matrix33_tpl@M@@AEBU?$Vec3_tpl@M@@MAEAPEAUBV@@HH@Z 00000000351655c0 f   heightfieldbv.obj
 0001:001648f0       ?GetMemoryStatistics@CHeightfield@@UEAAXPEAVICrySizer@@@Z 00000000351658f0 f   heightfieldgeom.obj
 0001:00164930       ?PointInsideStatus@CHeightfield@@UEAAHAEBU?$Vec3_tpl@M@@@Z 0000000035165930 f   heightfieldgeom.obj
 0001:00164b40       ?CreateHeightfield@CHeightfield@@QEAAPEAV1@PEAUheightfield@primitives@@@Z 0000000035165b40 f   heightfieldgeom.obj
 0001:00164d70       ?check_cell@hf_cell_checker@@QEAAHAEBU?$Vec2_tpl@H@@AEAH@Z 0000000035165d70 f i heightfieldgeom.obj
 0001:001651f0       ?PrepareForIntersectionTest@CHeightfield@@UEAAHPEAUgeometry_under_test@@PEAVCGeometry@@0_N@Z 00000000351661f0 f   heightfieldgeom.obj
 0001:00165d80       ?CheckPtEdgeDist@@YAXPEBU?$Vec3_tpl@M@@AEBU1@AEAU1@AEAH@Z 0000000035166d80 f i heightfieldgeom.obj
 0001:00165fc0       ?CheckPtTriDist@@YAXAEBUtriangle@primitives@@AEBU?$Vec3_tpl@M@@AEAU3@AEAH@Z 0000000035166fc0 f i heightfieldgeom.obj
 0001:001663d0       ?FindClosestPoint@CHeightfield@@UEAAHPEAUgeom_world_data@@AEAH1AEBU?$Vec3_tpl@M@@2PEAU3@H@Z 00000000351673d0 f   heightfieldgeom.obj
 0001:00166b90       ?DrawToOcclusionCubemap@CHeightfield@@UEAAHPEBUgeom_world_data@@HHHPEAUSOcclusionCubeMap@@@Z 0000000035167b90 f   heightfieldgeom.obj
 0001:001674f0       ??$DrawRayOnGrid@Uhf_cell_checker@@@@YAHPEAUgrid@primitives@@AEAU?$Vec3_tpl@M@@1AEAUhf_cell_checker@@@Z 00000000351684f0 f i heightfieldgeom.obj
 0001:00167c50       ?Intersect@CHeightfield@@UEAAHPEAUIGeometry@@PEAUgeom_world_data@@1PEAUintersection_params@@AEAPEAUgeom_contact@@@Z 0000000035168c50 f   heightfieldgeom.obj
 0001:00169060       ?box_sphere_intersection@@YAHPEBUbox@primitives@@PEBUsphere@2@PEAUprim_inters@@@Z 000000003516a060 f   intersectionchecks.obj
 0001:00169400       ?sphere_box_intersection@@YAHPEBUsphere@primitives@@PEBUbox@2@PEAUprim_inters@@@Z 000000003516a400 f   intersectionchecks.obj
 0001:00169470       ?sphere_sphere_intersection@@YAHPEBUsphere@primitives@@0PEAUprim_inters@@@Z 000000003516a470 f   intersectionchecks.obj
 0001:00169660       ?tri_tri_intersection@@YAHPEBUtriangle@primitives@@0PEAUprim_inters@@@Z 000000003516a660 f   intersectionchecks.obj
 0001:0016a080       ?tri_sphere_intersection@@YAHPEBUtriangle@primitives@@PEBUsphere@2@PEAUprim_inters@@@Z 000000003516b080 f   intersectionchecks.obj
 0001:0016abf0       ?sphere_tri_intersection@@YAHPEBUsphere@primitives@@PEBUtriangle@2@PEAUprim_inters@@@Z 000000003516bbf0 f   intersectionchecks.obj
 0001:0016ac60       ?ray_tri_intersection@@YAHPEBUray@primitives@@PEBUtriangle@2@PEAUprim_inters@@@Z 000000003516bc60 f   intersectionchecks.obj
 0001:0016b300       ?tri_ray_intersection@@YAHPEBUtriangle@primitives@@PEBUray@2@PEAUprim_inters@@@Z 000000003516c300 f   intersectionchecks.obj
 0001:0016b370       ?box_cylinder_intersection@@YAHPEBUbox@primitives@@PEBUcylinder@2@PEAUprim_inters@@@Z 000000003516c370 f   intersectionchecks.obj
 0001:0016cd90       ?cylinder_box_intersection@@YAHPEBUcylinder@primitives@@PEBUbox@2@PEAUprim_inters@@@Z 000000003516dd90 f   intersectionchecks.obj
 0001:0016ce00       ?box_capsule_intersection@@YAHPEBUbox@primitives@@PEBUcapsule@2@PEAUprim_inters@@@Z 000000003516de00 f   intersectionchecks.obj
 0001:0016e6e0       ?capsule_box_intersection@@YAHPEBUcapsule@primitives@@PEBUbox@2@PEAUprim_inters@@@Z 000000003516f6e0 f   intersectionchecks.obj
 0001:0016e750       ?box_ray_intersection@@YAHPEBUbox@primitives@@PEBUray@2@PEAUprim_inters@@@Z 000000003516f750 f   intersectionchecks.obj
 0001:0016ecb0       ?ray_box_intersection@@YAHPEBUray@primitives@@PEBUbox@2@PEAUprim_inters@@@Z 000000003516fcb0 f   intersectionchecks.obj
 0001:0016ecf0       ?cylinder_cylinder_intersection@@YAHPEBUcylinder@primitives@@0PEAUprim_inters@@@Z 000000003516fcf0 f   intersectionchecks.obj
 0001:001708c0       ?cylinder_sphere_intersection@@YAHPEBUcylinder@primitives@@PEBUsphere@2@PEAUprim_inters@@@Z 00000000351718c0 f   intersectionchecks.obj
 0001:00170cc0       ?sphere_cylinder_intersection@@YAHPEBUsphere@primitives@@PEBUcylinder@2@PEAUprim_inters@@@Z 0000000035171cc0 f   intersectionchecks.obj
 0001:00170d00       ?cylinder_capsule_intersection@@YAHPEBUcylinder@primitives@@PEBUcapsule@2@PEAUprim_inters@@@Z 0000000035171d00 f   intersectionchecks.obj
 0001:00171e40       ?capsule_cylinder_intersection@@YAHPEBUcapsule@primitives@@PEBUcylinder@2@PEAUprim_inters@@@Z 0000000035172e40 f   intersectionchecks.obj
 0001:00171e80       ?cylinder_ray_intersection@@YAHPEBUcylinder@primitives@@PEBUray@2@PEAUprim_inters@@@Z 0000000035172e80 f   intersectionchecks.obj
 0001:00172a10       ?ray_cylinder_intersection@@YAHPEBUray@primitives@@PEBUcylinder@2@PEAUprim_inters@@@Z 0000000035173a10 f   intersectionchecks.obj
 0001:00172a50       ?sphere_ray_intersection@@YAHPEBUsphere@primitives@@PEBUray@2@PEAUprim_inters@@@Z 0000000035173a50 f   intersectionchecks.obj
 0001:00172d10       ?ray_sphere_intersection@@YAHPEBUray@primitives@@PEBUsphere@2@PEAUprim_inters@@@Z 0000000035173d10 f   intersectionchecks.obj
 0001:00172d50       ?capsule_capsule_intersection@@YAHPEBUcapsule@primitives@@0PEAUprim_inters@@@Z 0000000035173d50 f   intersectionchecks.obj
 0001:00173590       ?capsule_sphere_intersection@@YAHPEBUcylinder@primitives@@PEBUsphere@2@PEAUprim_inters@@@Z 0000000035174590 f   intersectionchecks.obj
 0001:00173810       ?sphere_capsule_intersection@@YAHPEBUsphere@primitives@@PEBUcapsule@2@PEAUprim_inters@@@Z 0000000035174810 f   intersectionchecks.obj
 0001:00173850       ?capsule_ray_intersection@@YAHPEBUcapsule@primitives@@PEBUray@2@PEAUprim_inters@@@Z 0000000035174850 f   intersectionchecks.obj
 0001:001743a0       ?ray_capsule_intersection@@YAHPEBUray@primitives@@PEBUcapsule@2@PEAUprim_inters@@@Z 00000000351753a0 f   intersectionchecks.obj
 0001:001743e0       ?tri_box_intersection@@YAHPEBUtriangle@primitives@@PEBUbox@2@PEAUprim_inters@@@Z 00000000351753e0 f   intersectionchecks.obj
 0001:00176060       ?box_tri_intersection@@YAHPEBUbox@primitives@@PEBUtriangle@2@PEAUprim_inters@@@Z 0000000035177060 f   intersectionchecks.obj
 0001:00176100       ?tri_cylinder_intersection@@YAHPEBUtriangle@primitives@@PEBUcylinder@2@PEAUprim_inters@@@Z 0000000035177100 f   intersectionchecks.obj
 0001:001799c0       ?cylinder_tri_intersection@@YAHPEBUcylinder@primitives@@PEBUtriangle@2@PEAUprim_inters@@@Z 000000003517a9c0 f   intersectionchecks.obj
 0001:00179a30       ?tri_capsule_intersection@@YAHPEBUtriangle@primitives@@PEBUcapsule@2@PEAUprim_inters@@@Z 000000003517aa30 f   intersectionchecks.obj
 0001:0017c2e0       ?capsule_tri_intersection@@YAHPEBUcapsule@primitives@@PEBUtriangle@2@PEAUprim_inters@@@Z 000000003517d2e0 f   intersectionchecks.obj
 0001:0017c350       ?box_box_intersection@@YAHPEBUbox@primitives@@0PEAUprim_inters@@@Z 000000003517d350 f   intersectionchecks.obj
 0001:0017ce90       ?crop_polygon_with_bound@@YAHPEBU?$Vec2_tpl@M@@PEBHHAEBU1@HHPEAU1@PEAH@Z 000000003517de90 f   linunprojectionchecks.obj
 0001:0017d150       ?crop_segment_with_bound@@YAXPEAU?$Vec2_tpl@M@@MHPEAH1HH@Z 000000003517e150 f   linunprojectionchecks.obj
 0001:0017d2e0       ?flip_contact@@YAXPEBUunprojection_mode@@PEAUcontact@@PEAUgeom_contact_area@@@Z 000000003517e2e0 f   linunprojectionchecks.obj
 0001:0017d5a0       ?tri_tri_lin_unprojection@@YAHPEAUunprojection_mode@@PEBUtriangle@primitives@@H1HPEAUcontact@@PEAUgeom_contact_area@@@Z 000000003517e5a0 f   linunprojectionchecks.obj
 0001:0017e860       ?tri_box_lin_unprojection@@YAHPEAUunprojection_mode@@PEBUtriangle@primitives@@HPEBUbox@3@HPEAUcontact@@PEAUgeom_contact_area@@@Z 000000003517f860 f   linunprojectionchecks.obj
 0001:00180020       ?box_tri_lin_unprojection@@YAHPEAUunprojection_mode@@PEBUbox@primitives@@HPEBUtriangle@3@HPEAUcontact@@PEAUgeom_contact_area@@@Z 0000000035181020 f   linunprojectionchecks.obj
 0001:00180190       ?tri_cylinder_lin_unprojection@@YAHPEAUunprojection_mode@@PEBUtriangle@primitives@@HPEBUcylinder@3@HPEAUcontact@@PEAUgeom_contact_area@@@Z 0000000035181190 f   linunprojectionchecks.obj
 0001:00183d80       ?cylinder_tri_lin_unprojection@@YAHPEAUunprojection_mode@@PEBUcylinder@primitives@@HPEBUtriangle@3@HPEAUcontact@@PEAUgeom_contact_area@@@Z 0000000035184d80 f   linunprojectionchecks.obj
 0001:00183ef0       ?tri_sphere_lin_unprojection@@YAHPEAUunprojection_mode@@PEBUtriangle@primitives@@HPEBUsphere@3@HPEAUcontact@@PEAUgeom_contact_area@@@Z 0000000035184ef0 f   linunprojectionchecks.obj
 0001:00185010       ?sphere_tri_lin_unprojection@@YAHPEAUunprojection_mode@@PEBUsphere@primitives@@HPEBUtriangle@3@HPEAUcontact@@PEAUgeom_contact_area@@@Z 0000000035186010 f   linunprojectionchecks.obj
 0001:00185180       ?tri_capsule_lin_unprojection@@YAHPEAUunprojection_mode@@PEBUtriangle@primitives@@HPEBUcapsule@3@HPEAUcontact@@PEAUgeom_contact_area@@@Z 0000000035186180 f   linunprojectionchecks.obj
 0001:001853b0       ?capsule_tri_lin_unprojection@@YAHPEAUunprojection_mode@@PEBUcapsule@primitives@@HPEBUtriangle@3@HPEAUcontact@@PEAUgeom_contact_area@@@Z 00000000351863b0 f   linunprojectionchecks.obj
 0001:00185520       ?tri_ray_lin_unprojection@@YAHPEAUunprojection_mode@@PEBUtriangle@primitives@@HPEBUray@3@HPEAUcontact@@PEAUgeom_contact_area@@@Z 0000000035186520 f   linunprojectionchecks.obj
 0001:001864d0       ?ray_tri_lin_unprojection@@YAHPEAUunprojection_mode@@PEBUray@primitives@@HPEBUtriangle@3@HPEAUcontact@@PEAUgeom_contact_area@@@Z 00000000351874d0 f   linunprojectionchecks.obj
 0001:00186640       ?box_cylinder_lin_unprojection@@YAHPEAUunprojection_mode@@PEBUbox@primitives@@HPEBUcylinder@3@HPEAUcontact@@PEAUgeom_contact_area@@@Z 0000000035187640 f   linunprojectionchecks.obj
 0001:0018c3f0       ?cylinder_box_lin_unprojection@@YAHPEAUunprojection_mode@@PEBUcylinder@primitives@@HPEBUbox@3@HPEAUcontact@@PEAUgeom_contact_area@@@Z 000000003518d3f0 f   linunprojectionchecks.obj
 0001:0018c4d0       ?box_sphere_lin_unprojection@@YAHPEAUunprojection_mode@@PEBUbox@primitives@@HPEBUsphere@3@HPEAUcontact@@PEAUgeom_contact_area@@@Z 000000003518d4d0 f   linunprojectionchecks.obj
 0001:0018d970       ?sphere_box_lin_unprojection@@YAHPEAUunprojection_mode@@PEBUsphere@primitives@@HPEBUbox@3@HPEAUcontact@@PEAUgeom_contact_area@@@Z 000000003518e970 f   linunprojectionchecks.obj
 0001:0018dae0       ?box_capsule_lin_unprojection@@YAHPEAUunprojection_mode@@PEBUbox@primitives@@HPEBUcapsule@3@HPEAUcontact@@PEAUgeom_contact_area@@@Z 000000003518eae0 f   linunprojectionchecks.obj
 0001:0018e050       ?capsule_box_lin_unprojection@@YAHPEAUunprojection_mode@@PEBUcapsule@primitives@@HPEBUbox@3@HPEAUcontact@@PEAUgeom_contact_area@@@Z 000000003518f050 f   linunprojectionchecks.obj
 0001:0018e130       ?sphere_sphere_lin_unprojection@@YAHPEAUunprojection_mode@@PEBUsphere@primitives@@H1HPEAUcontact@@PEAUgeom_contact_area@@@Z 000000003518f130 f   linunprojectionchecks.obj
 0001:0018e560       ?ray_box_lin_unprojection@@YAHPEAUunprojection_mode@@PEBUray@primitives@@HPEBUbox@3@HPEAUcontact@@PEAUgeom_contact_area@@@Z 000000003518f560 f   linunprojectionchecks.obj
 0001:0018f5b0       ?box_ray_lin_unprojection@@YAHPEAUunprojection_mode@@PEBUbox@primitives@@HPEBUray@3@HPEAUcontact@@PEAUgeom_contact_area@@@Z 00000000351905b0 f   linunprojectionchecks.obj
 0001:0018f720       ?ray_cylinder_lin_unprojection@@YAHPEAUunprojection_mode@@PEBUray@primitives@@HPEBUcylinder@3@HPEAUcontact@@PEAUgeom_contact_area@@@Z 0000000035190720 f   linunprojectionchecks.obj
 0001:00191e10       ?cylinder_ray_lin_unprojection@@YAHPEAUunprojection_mode@@PEBUcylinder@primitives@@HPEBUray@3@HPEAUcontact@@PEAUgeom_contact_area@@@Z 0000000035192e10 f   linunprojectionchecks.obj
 0001:00191f80       ?ray_sphere_lin_unprojection@@YAHPEAUunprojection_mode@@PEBUray@primitives@@HPEBUsphere@3@HPEAUcontact@@PEAUgeom_contact_area@@@Z 0000000035192f80 f   linunprojectionchecks.obj
 0001:00192a10       ?sphere_ray_lin_unprojection@@YAHPEAUunprojection_mode@@PEBUsphere@primitives@@HPEBUray@3@HPEAUcontact@@PEAUgeom_contact_area@@@Z 0000000035193a10 f   linunprojectionchecks.obj
 0001:00192b80       ?ray_capsule_lin_unprojection@@YAHPEAUunprojection_mode@@PEBUray@primitives@@HPEBUcapsule@3@HPEAUcontact@@PEAUgeom_contact_area@@@Z 0000000035193b80 f   linunprojectionchecks.obj
 0001:00192db0       ?capsule_ray_lin_unprojection@@YAHPEAUunprojection_mode@@PEBUcapsule@primitives@@HPEBUray@3@HPEAUcontact@@PEAUgeom_contact_area@@@Z 0000000035193db0 f   linunprojectionchecks.obj
 0001:00192f20       ?box_box_lin_unprojection@@YAHPEAUunprojection_mode@@PEBUbox@primitives@@H1HPEAUcontact@@PEAUgeom_contact_area@@@Z 0000000035193f20 f   linunprojectionchecks.obj
 0001:001965f0       ?cylinder_sphere_lin_unprojection@@YAHPEAUunprojection_mode@@PEBUcylinder@primitives@@HPEBUsphere@3@HPEAUcontact@@PEAUgeom_contact_area@@@Z 00000000351975f0 f   linunprojectionchecks.obj
 0001:001981c0       ?sphere_cylinder_lin_unprojection@@YAHPEAUunprojection_mode@@PEBUsphere@primitives@@HPEBUcylinder@3@HPEAUcontact@@PEAUgeom_contact_area@@@Z 00000000351991c0 f   linunprojectionchecks.obj
 0001:00198330       ?cyl_cyl_lin_unprojection@@YAHPEAUunprojection_mode@@PEBUcylinder@primitives@@H1HPEAUcontact@@PEAUgeom_contact_area@@@Z 0000000035199330 f   linunprojectionchecks.obj
 0001:001a06a0       ?cylinder_capsule_lin_unprojection@@YAHPEAUunprojection_mode@@PEBUcylinder@primitives@@HPEBUcapsule@3@HPEAUcontact@@PEAUgeom_contact_area@@@Z 00000000351a16a0 f   linunprojectionchecks.obj
 0001:001a0c10       ?capsule_cylinder_lin_unprojection@@YAHPEAUunprojection_mode@@PEBUcapsule@primitives@@HPEBUcylinder@3@HPEAUcontact@@PEAUgeom_contact_area@@@Z 00000000351a1c10 f   linunprojectionchecks.obj
 0001:001a0cf0       ?capsule_capsule_lin_unprojection@@YAHPEAUunprojection_mode@@PEBUcapsule@primitives@@H1HPEAUcontact@@PEAUgeom_contact_area@@@Z 00000000351a1cf0 f   linunprojectionchecks.obj
 0001:001a1800       ?sphere_capsule_lin_unprojection@@YAHPEAUunprojection_mode@@PEBUsphere@primitives@@HPEBUcapsule@3@HPEAUcontact@@PEAUgeom_contact_area@@@Z 00000000351a2800 f   linunprojectionchecks.obj
 0001:001a1d60       ?capsule_sphere_lin_unprojection@@YAHPEAUunprojection_mode@@PEBUcapsule@primitives@@HPEBUsphere@3@HPEAUcontact@@PEAUgeom_contact_area@@@Z 00000000351a2d60 f   linunprojectionchecks.obj
 0001:001a1f50       ?SetParams@COBBTree@@QEAAXHHM@Z 00000000351a2f50 f   obbtree.obj
 0001:001a1f60       ?SetGeomConvex@COBBTree@@UEAAXXZ 00000000351a2f60 f   obbtree.obj
 0001:001a1f90       ?ReleaseLastSweptBVs@COBBTree@@UEAAXH@Z 00000000351a2f90 f   obbtree.obj
 0001:001a1f90       ?ReleaseLastBVs@COBBTree@@UEAAXH@Z 00000000351a2f90 f   obbtree.obj
 0001:001a1f90       ?ReleaseLastBVs@CAABBTree@@UEAAXH@Z 00000000351a2f90 f   aabbtree.obj
 0001:001a1fb0       ?GetNodeContents@COBBTree@@UEAAHHPEAUBV@@HHPEAUgeometry_under_test@@1@Z 00000000351a2fb0 f   obbtree.obj
 0001:001a2040       ?CleanupAfterIntersectionTest@CAABBTree@@UEAAXPEAUgeometry_under_test@@@Z 00000000351a3040 f   aabbtree.obj
 0001:001a2040       ?CleanupAfterIntersectionTest@COBBTree@@UEAAXPEAUgeometry_under_test@@@Z 00000000351a3040 f   obbtree.obj
 0001:001a2110       ?SanityCheck@COBBTree@@UEAAHXZ 00000000351a3110 f   obbtree.obj
 0001:001a2120       ?SplitPriority@COBBTree@@UEAAMPEBUBV@@@Z 00000000351a3120 f   obbtree.obj
 0001:001a2160       ?MarkUsedTriangle@COBBTree@@UEAAXHPEAUgeometry_under_test@@@Z 00000000351a3160 f   obbtree.obj
 0001:001a2280       ?PrepareForIntersectionTest@COBBTree@@UEAAHPEAUgeometry_under_test@@PEAVCGeometry@@0@Z 00000000351a3280 f   obbtree.obj
 0001:001a23b0       ?GetMemoryStatistics@COBBTree@@UEAAXPEAVICrySizer@@@Z 00000000351a33b0 f   obbtree.obj
 0001:001a2440       ?GetBBox@COBBTree@@UEAAXPEAUbox@primitives@@@Z 00000000351a3440 f   obbtree.obj
 0001:001a2500       ?GetNodeBV@COBBTree@@UEAAXAEAPEAUBV@@HH@Z 00000000351a3500 f   obbtree.obj
 0001:001a2660       ?GetNodeBV@COBBTree@@UEAAXAEAPEAUBV@@AEBU?$Vec3_tpl@M@@MHH@Z 00000000351a3660 f   obbtree.obj
 0001:001a27f0       ?GetNodeChildrenBVs@COBBTree@@UEAAXPEBUBV@@AEAPEAU2@1H@Z 00000000351a37f0 f   obbtree.obj
 0001:001a2a20       ?GetNodeChildrenBVs@COBBTree@@UEAAXPEBUBV@@AEBU?$Vec3_tpl@M@@MAEAPEAU2@2H@Z 00000000351a3a20 f   obbtree.obj
 0001:001a2ca0       ?Save@COBBTree@@UEAAXAEAVCMemStream@@@Z 00000000351a3ca0 f   obbtree.obj
 0001:001a2e00       ?Load@COBBTree@@UEAAXAEAVCMemStream@@PEAVCGeometry@@@Z 00000000351a3e00 f   obbtree.obj
 0001:001a2f50       ??$ComputeMeshEigenBasis@H@@YAXV?$strided_pointer@$$CBU?$Vec3_tpl@M@@@@V?$strided_pointer@H@@HPEAU?$Vec3_tpl@N@@AEAU2@@Z 00000000351a3f50 f i obbtree.obj
 0001:001a3aa0       ?BuildNode@COBBTree@@QEAAMHHHH@Z 00000000351a4aa0 f   obbtree.obj
 0001:001a5520       ?GetNodeBV@COBBTree@@UEAAXAEBU?$Matrix33_tpl@M@@AEBU?$Vec3_tpl@M@@MAEAPEAUBV@@HH@Z 00000000351a6520 f   obbtree.obj
 0001:001a5950       ?GetNodeChildrenBVs@COBBTree@@UEAAXAEBU?$Matrix33_tpl@M@@AEBU?$Vec3_tpl@M@@MPEBUBV@@AEAPEAU4@3H@Z 00000000351a6950 f   obbtree.obj
 0001:001a6080       ?Build@COBBTree@@UEAAMPEAVCGeometry@@@Z 00000000351a7080 f   obbtree.obj
 0001:001a6270       ?box_ray_overlap_check@@YAHPEBUbox@primitives@@PEBUray@2@PEAVCOverlapChecker@@@Z 00000000351a7270 f   overlapchecks.obj
 0001:001a6610       ?ray_box_overlap_check@@YAHPEBUray@primitives@@PEBUbox@2@PEAVCOverlapChecker@@@Z 00000000351a7610 f   overlapchecks.obj
 0001:001a6620       ?box_sphere_overlap_check@@YAHPEBUbox@primitives@@PEBUsphere@2@PEAVCOverlapChecker@@@Z 00000000351a7620 f   overlapchecks.obj
 0001:001a67b0       ?sphere_box_overlap_check@@YAHPEBUsphere@primitives@@PEBUbox@2@PEAVCOverlapChecker@@@Z 00000000351a77b0 f   overlapchecks.obj
 0001:001a67c0       ?sphere_sphere_overlap_check@@YAHPEBUsphere@primitives@@0PEAVCOverlapChecker@@@Z 00000000351a77c0 f   overlapchecks.obj
 0001:001a6810       ?heightfield_sphere_overlap_check@@YAHPEBUheightfield@primitives@@PEBUsphere@2@PEAVCOverlapChecker@@@Z 00000000351a7810 f   overlapchecks.obj
 0001:001a6a30       ?sphere_heightfield_overlap_check@@YAHPEBUsphere@primitives@@PEBUheightfield@2@PEAVCOverlapChecker@@@Z 00000000351a7a30 f   overlapchecks.obj
 0001:001a6a40       ?box_tri_overlap_check@@YAHPEBUbox@primitives@@PEBUtriangle@2@PEAVCOverlapChecker@@@Z 00000000351a7a40 f   overlapchecks.obj
 0001:001a7240       ?tri_box_overlap_check@@YAHPEBUtriangle@primitives@@PEBUbox@2@PEAVCOverlapChecker@@@Z 00000000351a8240 f   overlapchecks.obj
 0001:001a7250       ?tri_sphere_dist2@@YA?AV?$quotient_tpl@M@@PEBUtriangle@primitives@@PEBUsphere@3@AEAH@Z 00000000351a8250 f   overlapchecks.obj
 0001:001a7860       ?tri_sphere_overlap_check@@YAHPEBUtriangle@primitives@@PEBUsphere@2@PEAVCOverlapChecker@@@Z 00000000351a8860 f   overlapchecks.obj
 0001:001a78b0       ?sphere_tri_overlap_check@@YAHPEBUsphere@primitives@@PEBUtriangle@2@PEAVCOverlapChecker@@@Z 00000000351a88b0 f   overlapchecks.obj
 0001:001a7900       ?box_box_overlap_check@@YAHPEBUbox@primitives@@0PEAVCOverlapChecker@@@Z 00000000351a8900 f   overlapchecks.obj
 0001:001a8350       ?box_heightfield_overlap_check@@YAHPEBUbox@primitives@@PEBUheightfield@2@PEAVCOverlapChecker@@@Z 00000000351a9350 f   overlapchecks.obj
 0001:001a8df0       ?heightfield_box_overlap_check@@YAHPEBUheightfield@primitives@@PEBUbox@2@PEAVCOverlapChecker@@@Z 00000000351a9df0 f   overlapchecks.obj
 0001:001a8e00       ?box_voxgrid_overlap_check@@YAHPEBUbox@primitives@@PEBUvoxelgrid@2@PEAVCOverlapChecker@@@Z 00000000351a9e00 f   overlapchecks.obj
 0001:001a99a0       ?voxgrid_box_overlap_check@@YAHPEBUvoxelgrid@primitives@@PEBUbox@2@PEAVCOverlapChecker@@@Z 00000000351aa9a0 f   overlapchecks.obj
 0001:001a99b0       ?GetNodeContents@CRayBV@@UEAAHHPEAUBV@@HHPEAUgeometry_under_test@@1@Z 00000000351aa9b0 f   raybv.obj
 0001:001a9a20       ?GetNodeBV@CRayBV@@UEAAXAEAPEAUBV@@HH@Z 00000000351aaa20 f   raybv.obj
 0001:001a9aa0       ?GetNodeBV@CRayBV@@UEAAXAEBU?$Matrix33_tpl@M@@AEBU?$Vec3_tpl@M@@MAEAPEAUBV@@HH@Z 00000000351aaaa0 f   raybv.obj
 0001:001a9c60       ?PreparePrimitive@CRayGeom@@UEAAHPEAUgeom_world_data@@AEAPEAUprimitive@primitives@@H@Z 00000000351aac60 f   raygeom.obj
 0001:001a9e10       ?PrepareRay@CRayGeom@@QEAAXPEAUray@primitives@@PEAUgeometry_under_test@@@Z 00000000351aae10 f   raygeom.obj
 0001:001a9f90       ?GetUnprojectionCandidates@CRayGeom@@UEAAHHPEBUcontact@@AEAPEAUprimitive@primitives@@AEAPEAHPEAUgeometry_under_test@@@Z 00000000351aaf90 f   raygeom.obj
 0001:001a9fd0       ?GetPrimitiveList@CRayGeom@@UEAAHHHHPEAUprimitive@primitives@@HPEAUgeometry_under_test@@10PEAD@Z 00000000351aafd0 f   raygeom.obj
 0001:001aa000       ?RegisterIntersection@CRayGeom@@UEAAHPEAUprimitive@primitives@@0PEAUgeometry_under_test@@1PEAUprim_inters@@@Z 00000000351ab000 f   raygeom.obj
 0001:001aa230       ?GetBBox@CRayGeom@@UEAAXPEAUbox@primitives@@@Z 00000000351ab230 f   raygeom.obj
 0001:001aa320       ?PrepareForIntersectionTest@CRayGeom@@UEAAHPEAUgeometry_under_test@@PEAVCGeometry@@0_N@Z 00000000351ab320 f   raygeom.obj
 0001:001aa3d0       ?tri_tri_rot_unprojection@@YAHPEAUunprojection_mode@@PEBUtriangle@primitives@@H1HPEAUcontact@@PEAUgeom_contact_area@@@Z 00000000351ab3d0 f   rotunprojectionchecks.obj
 0001:001acfe0       ?ray_tri_rot_unprojection@@YAHPEAUunprojection_mode@@PEBUray@primitives@@HPEBUtriangle@3@HPEAUcontact@@PEAUgeom_contact_area@@@Z 00000000351adfe0 f   rotunprojectionchecks.obj
 0001:001aea30       ?tri_ray_rot_unprojection@@YAHPEAUunprojection_mode@@PEBUtriangle@primitives@@HPEBUray@3@HPEAUcontact@@PEAUgeom_contact_area@@@Z 00000000351afa30 f   rotunprojectionchecks.obj
 0001:001aee40       ?ray_box_rot_unprojection@@YAHPEAUunprojection_mode@@PEBUray@primitives@@HPEBUbox@3@HPEAUcontact@@PEAUgeom_contact_area@@@Z 00000000351afe40 f   rotunprojectionchecks.obj
 0001:001b0ab0       ?box_ray_rot_unprojection@@YAHPEAUunprojection_mode@@PEBUbox@primitives@@HPEBUray@3@HPEAUcontact@@PEAUgeom_contact_area@@@Z 00000000351b1ab0 f   rotunprojectionchecks.obj
 0001:001b0ec0       ?ray_cyl_rot_unprojection@@YAHPEAUunprojection_mode@@PEBUray@primitives@@HPEBUcylinder@3@HPEAUcontact@@PEAUgeom_contact_area@@@Z 00000000351b1ec0 f   rotunprojectionchecks.obj
 0001:001b7990       ?cyl_ray_rot_unprojection@@YAHPEAUunprojection_mode@@PEBUcylinder@primitives@@HPEBUray@3@HPEAUcontact@@PEAUgeom_contact_area@@@Z 00000000351b8990 f   rotunprojectionchecks.obj
 0001:001b7da0       ?ray_capsule_rot_unprojection@@YAHPEAUunprojection_mode@@PEBUray@primitives@@HPEBUcapsule@3@HPEAUcontact@@PEAUgeom_contact_area@@@Z 00000000351b8da0 f   rotunprojectionchecks.obj
 0001:001be460       ?capsule_ray_rot_unprojection@@YAHPEAUunprojection_mode@@PEBUcapsule@primitives@@HPEBUray@3@HPEAUcontact@@PEAUgeom_contact_area@@@Z 00000000351bf460 f   rotunprojectionchecks.obj
 0001:001be870       ?ray_sphere_rot_unprojection@@YAHPEAUunprojection_mode@@PEBUray@primitives@@HPEBUsphere@3@HPEAUcontact@@PEAUgeom_contact_area@@@Z 00000000351bf870 f   rotunprojectionchecks.obj
 0001:001c0d80       ?sphere_ray_rot_unprojection@@YAHPEAUunprojection_mode@@PEBUsphere@primitives@@HPEBUray@3@HPEAUcontact@@PEAUgeom_contact_area@@@Z 00000000351c1d80 f   rotunprojectionchecks.obj
 0001:001c1190       ??0entity_grid_checker@@QEAA@XZ 00000000351c2190 f i rwi.obj
 0001:001c1310       ?RayWater@CPhysicalWorld@@QEAAXAEBU?$Vec3_tpl@M@@0AEAUentity_grid_checker@@HHPEAUray_hit@@@Z 00000000351c2310 f   rwi.obj
 0001:001c17d0       ??$ReallocQueue@USRwiRequest@@@CPhysicalWorld@@QEAAXAEAPEAUSRwiRequest@@HAEAH11H@Z 00000000351c27d0 f i rwi.obj
 0001:001c1920       ?check_cell@entity_grid_checker@@QEAAHAEBU?$Vec2_tpl@H@@AEAH@Z 00000000351c2920 f i rwi.obj
 0001:001c3100       ?RayHeightfield@CPhysicalWorld@@QEAAXAEBU?$Vec3_tpl@M@@AEAU2@PEAUray_hit@@HH@Z 00000000351c4100 f   rwi.obj
 0001:001c34e0       ?TracePendingRays@CPhysicalWorld@@UEAAHH@Z 00000000351c44e0 f   rwi.obj
 0001:001c3b40       ??$DrawRayOnGrid@Uentity_grid_checker@@@@YAHPEAUgrid@primitives@@AEAU?$Vec3_tpl@M@@1AEAUentity_grid_checker@@@Z 00000000351c4b40 f i rwi.obj
 0001:001c4290       ?RayWorldIntersection@CPhysicalWorld@@UEAAHAEBUSRWIParams@IPhysicalWorld@@PEBDH@Z 00000000351c5290 f   rwi.obj
 0001:001c56b0       ?GetNodeContents@CSingleBoxTree@@UEAAHHPEAUBV@@HHPEAUgeometry_under_test@@1@Z 00000000351c66b0 f   singleboxtree.obj
 0001:001c5720       ?PrepareForIntersectionTest@CSingleBoxTree@@UEAAHPEAUgeometry_under_test@@PEAVCGeometry@@0@Z 00000000351c6720 f   singleboxtree.obj
 0001:001c5740       ?Build@CSingleBoxTree@@UEAAMPEAVCGeometry@@@Z 00000000351c6740 f   singleboxtree.obj
 0001:001c5760       ?GetNodeBV@CSingleBoxTree@@UEAAXAEAPEAUBV@@HH@Z 00000000351c6760 f   singleboxtree.obj
 0001:001c5820       ?GetNodeBV@CSingleBoxTree@@UEAAXAEAPEAUBV@@AEBU?$Vec3_tpl@M@@MHH@Z 00000000351c6820 f   singleboxtree.obj
 0001:001c5930       ?MarkUsedTriangle@CSingleBoxTree@@UEAAXHPEAUgeometry_under_test@@@Z 00000000351c6930 f   singleboxtree.obj
 0001:001c5950       ?GetBBox@CSingleBoxTree@@UEAAXPEAUbox@primitives@@@Z 00000000351c6950 f   singleboxtree.obj
 0001:001c59b0       ?GetMemoryStatistics@CSingleBoxTree@@UEAAXPEAVICrySizer@@@Z 00000000351c69b0 f   singleboxtree.obj
 0001:001c5a00       ?SetBox@CSingleBoxTree@@QEAAXPEAUbox@primitives@@@Z 00000000351c6a00 f   singleboxtree.obj
 0001:001c5b00       ?Save@CSingleBoxTree@@UEAAXAEAVCMemStream@@@Z 00000000351c6b00 f   singleboxtree.obj
 0001:001c5bc0       ?Load@CSingleBoxTree@@UEAAXAEAVCMemStream@@PEAVCGeometry@@@Z 00000000351c6bc0 f   singleboxtree.obj
 0001:001c5c30       ?GetNodeBV@CSingleBoxTree@@UEAAXAEBU?$Matrix33_tpl@M@@AEBU?$Vec3_tpl@M@@MAEAPEAUBV@@HH@Z 00000000351c6c30 f   singleboxtree.obj
 0001:001c5f80       ?GetNodeBV@CSingleBoxTree@@UEAAXAEBU?$Matrix33_tpl@M@@AEBU?$Vec3_tpl@M@@MAEAPEAUBV@@1MHH@Z 00000000351c6f80 f   singleboxtree.obj
 0001:001c6330       ?PrepareForIntersectionTest@CSphereGeom@@UEAAHPEAUgeometry_under_test@@PEAVCGeometry@@0_N@Z 00000000351c7330 f   spheregeom.obj
 0001:001c63e0       ?GetMemoryStatistics@CSphereGeom@@UEAAXPEAVICrySizer@@@Z 00000000351c73e0 f   spheregeom.obj
 0001:001c6400       ?CreateSphere@CSphereGeom@@QEAAPEAV1@PEAUsphere@primitives@@@Z 00000000351c7400 f   spheregeom.obj
 0001:001c64d0       ?CalcPhysicalProperties@CSphereGeom@@UEAAHPEAUphys_geometry@@@Z 00000000351c74d0 f   spheregeom.obj
 0001:001c6550       ?PointInsideStatus@CSphereGeom@@UEAAHAEBU?$Vec3_tpl@M@@@Z 00000000351c7550 f   spheregeom.obj
 0001:001c65a0       ?ComputeExtent@CSphereGeom@@UEAAMAEAUGeomQuery@@W4EGeomForm@@@Z 00000000351c75a0 f   spheregeom.obj
 0001:001c65f0       ?PreparePrimitive@CSphereGeom@@UEAAHPEAUgeom_world_data@@AEAPEAUprimitive@primitives@@H@Z 00000000351c75f0 f   spheregeom.obj
 0001:001c6700       ?GetPrimitiveList@CSphereGeom@@UEAAHHHHPEAUprimitive@primitives@@HPEAUgeometry_under_test@@10PEAD@Z 00000000351c7700 f   spheregeom.obj
 0001:001c6810       ?GetUnprojectionCandidates@CSphereGeom@@UEAAHHPEBUcontact@@AEAPEAUprimitive@primitives@@AEAPEAHPEAUgeometry_under_test@@@Z 00000000351c7810 f   spheregeom.obj
 0001:001c6930       ?CalculateBuoyancy@CSphereGeom@@UEAAMPEBUplane@primitives@@PEBUgeom_world_data@@AEAU?$Vec3_tpl@M@@@Z 00000000351c7930 f   spheregeom.obj
 0001:001c6ba0       ?DrawWireframe@CSphereGeom@@UEAAXPEAUIPhysRenderer@@PEAUgeom_world_data@@HH@Z 00000000351c7ba0 f   spheregeom.obj
 0001:001c6cf0       ?FindClosestPoint@CSphereGeom@@UEAAHPEAUgeom_world_data@@AEAH1AEBU?$Vec3_tpl@M@@2PEAU3@H@Z 00000000351c7cf0 f   spheregeom.obj
 0001:001c70c0       ?UnprojectSphere@CSphereGeom@@UEAAHU?$Vec3_tpl@M@@MMPEAUcontact@@@Z 00000000351c80c0 f   spheregeom.obj
 0001:001c7240       ?CalculateMediumResistance@CSphereGeom@@UEAAXPEBUplane@primitives@@PEBUgeom_world_data@@AEAU?$Vec3_tpl@M@@2@Z 00000000351c8240 f   spheregeom.obj
 0001:001c7c70       ?CalcVolumetricPressure@CSphereGeom@@UEAAXPEAUgeom_world_data@@AEBU?$Vec3_tpl@M@@MM1AEAU3@2@Z 00000000351c8c70 f   spheregeom.obj
 0001:001c7de0       ?DrawToOcclusionCubemap@CSphereGeom@@UEAAHPEBUgeom_world_data@@HHHPEAUSOcclusionCubeMap@@@Z 00000000351c8de0 f   spheregeom.obj
 0001:001c8250       ?Save@CSphereGeom@@UEAAXAEAVCMemStream@@@Z 00000000351c9250 f   spheregeom.obj
 0001:001c82c0       ?Load@CSphereGeom@@UEAAXAEAVCMemStream@@@Z 00000000351c92c0 f   spheregeom.obj
 0001:001c8310       ?GetRandomPos@CSphereGeom@@UEAAXAEAURandomPos@@AEAUGeomQuery@@W4EGeomForm@@@Z 00000000351c9310 f   spheregeom.obj
 0001:001c8540       ?GetParams@CTetrLattice@@UEAAHPEAUpe_params@@@Z 00000000351c9540 f   tetrlattice.obj
 0001:001c8580       ??0CTetrLattice@@QEAA@PEAUIPhysicalWorld@@@Z 00000000351c9580 f   tetrlattice.obj
 0001:001c8610       ??1CTetrLattice@@UEAA@XZ   00000000351c9610 f   tetrlattice.obj
 0001:001c8690       ?SetParams@CTetrLattice@@UEAAHPEAUpe_params@@@Z 00000000351c9690 f   tetrlattice.obj
 0001:001c8900       ??4STetrahedron@@QEAAAEAU0@AEBU0@@Z 00000000351c9900 f i tetrlattice.obj
 0001:001c8a00       ?DrawWireframe@CTetrLattice@@UEAAXPEAUIPhysRenderer@@PEAUgeom_world_data@@H@Z 00000000351c9a00 f   tetrlattice.obj
 0001:001c90a0       ?CreateSkinMesh@CTetrLattice@@UEAAPEAUIGeometry@@H@Z 00000000351ca0a0 f   tetrlattice.obj
 0001:001c92a0       ?CropSpikes@CBreakableGrid2d@@QEAAHHHPEAHHHHM@Z 00000000351ca2a0 f i tetrlattice.obj
 0001:001c9850       ?BreakIntoChunks@CBreakableGrid2d@@UEAAPEAHAEBU?$Vec2_tpl@M@@MAEAPEAU2@HMHMM@Z 00000000351ca850 f   tetrlattice.obj
 0001:001caf10       ??_GCTetrLattice@@UEAAPEAXI@Z 00000000351cbf10 f i tetrlattice.obj
 0001:001caf10       ??_ECTetrLattice@@UEAAPEAXI@Z 00000000351cbf10 f i tetrlattice.obj
 0001:001caf40       ??0CTetrLattice@@QEAA@PEAV0@H@Z 00000000351cbf40 f   tetrlattice.obj
 0001:001cb2b0       ?CreateLattice@CTetrLattice@@QEAAPEAV1@PEBU?$Vec3_tpl@M@@HPEBHH@Z 00000000351cc2b0 f   tetrlattice.obj
 0001:001cc410       ?AddImpulse@CTetrLattice@@QEAAHAEBU?$Vec3_tpl@M@@000M@Z 00000000351cd410 f   tetrlattice.obj
 0001:001cca00       ?Defragment@CTetrLattice@@QEAAHXZ 00000000351cda00 f   tetrlattice.obj
 0001:001cccf0       ?SetGrid@CTetrLattice@@QEAAXAEBUbox@primitives@@@Z 00000000351cdcf0 f   tetrlattice.obj
 0001:001cde30       ?Subtract@CTetrLattice@@QEAAXPEAUIGeometry@@PEBUgeom_world_data@@1@Z 00000000351cee30 f   tetrlattice.obj
 0001:001cf8b0       ?CheckStructure@CTetrLattice@@QEAAHMAEBU?$Vec3_tpl@M@@PEBUplane@primitives@@HPEAUpe_explosion@@HH@Z 00000000351d08b0 f   tetrlattice.obj
 0001:001d3ca0       ?Split@CTetrLattice@@QEAAXPEAPEAVCTriMesh@@HPEAPEAV1@@Z 00000000351d4ca0 f   tetrlattice.obj
 0001:001d51f0       ?CheckPoint@CTetrLattice@@UEAAHAEBU?$Vec3_tpl@M@@PEAHPEAM@Z 00000000351d61f0 f   tetrlattice.obj
 0001:001d5ce0       ?SetMesh@CTetrLattice@@QEAAXPEAVCTriMesh@@@Z 00000000351d6ce0 f   tetrlattice.obj
 0001:001d5d20       ?Generate@CBreakableGrid2d@@QEAAXPEAU?$Vec2_tpl@M@@HAEBU?$Vec2_tpl@H@@HH@Z 00000000351d6d20 f   tetrlattice.obj
 0001:001d6d60       ?MaxPrimsInNode@COBBTree@@UEAAHXZ 00000000351d7d60 f i trimesh.obj
 0001:001d6d60       ?GetiForeignData@CGeometry@@UEAAHXZ 00000000351d7d60 f i livingentity.obj
 0001:001d6d70       ?GetNodeContentsIdx@COBBTree@@UEAAHHAEAH@Z 00000000351d7d70 f i trimesh.obj
 0001:001d6d90       ??_GCOBBTree@@UEAAPEAXI@Z  00000000351d7d90 f i trimesh.obj
 0001:001d6d90       ??_ECOBBTree@@UEAAPEAXI@Z  00000000351d7d90 f i trimesh.obj
 0001:001d6e00       ??0InitTriMeshGlobals@@QEAA@XZ 00000000351d7e00 f   trimesh.obj
 0001:001d6ea0       ?qsort@@YAXPEAHHH@Z        00000000351d7ea0 f   trimesh.obj
 0001:001d6f80       ?CleanupAfterIntersectionTest@CTriMesh@@UEAAXPEAUgeometry_under_test@@@Z 00000000351d7f80 f   trimesh.obj
 0001:001d7130       ?GetNeighbouringEdgeId@CTriMesh@@QEAAHHH@Z 00000000351d8130 f   trimesh.obj
 0001:001d7250       ?CleanupGlobalLoadState@CTriMesh@@SAXXZ 00000000351d8250 f   trimesh.obj
 0001:001d72a0       ?GetMemoryUsage@TriMeshStaticData@@YAXPEAVICrySizer@@@Z 00000000351d82a0 f   trimesh.obj
 0001:001d7300       ?SanityCheck@CTriMesh@@UEAAHXZ 00000000351d8300 f   trimesh.obj
 0001:001d7310       ??1?$vector2_w_enforcer@M@@QEAA@XZ 00000000351d8310 f i trimesh.obj
 0001:001d7390       ?MaxPrimsInNode@CAABBTree@@UEAAHXZ 00000000351d8390 f i trimesh.obj
 0001:001d73a0       ?GetNodeContentsIdx@CAABBTree@@UEAAHHAEAH@Z 00000000351d83a0 f i trimesh.obj
 0001:001d73c0       ??_ECAABBTree@@UEAAPEAXI@Z 00000000351d83c0 f i trimesh.obj
 0001:001d73c0       ??_GCAABBTree@@UEAAPEAXI@Z 00000000351d83c0 f i trimesh.obj
 0001:001d7430       ?GetMaxSkipDim@CAABBTree@@UEAAMXZ 00000000351d8430 f i trimesh.obj
 0001:001d7490       ?GetMaxSkipDim@COBBTree@@UEAAMXZ 00000000351d8490 f i trimesh.obj
 0001:001d74f0       ?TriRandomPoint@@YAXQEAMW4EGeomForm@@@Z 00000000351d84f0 f i trimesh.obj
 0001:001d7640       ??1CTriMesh@@UEAA@XZ       00000000351d8640 f   trimesh.obj
 0001:001d7800       ?PointInsideStatus@CTriMesh@@UEAAHAEBU?$Vec3_tpl@M@@@Z 00000000351d8800 f i trimesh.obj
 0001:001d7810       ?GetBVTree@CTriMesh@@UEAAPEAVCBVTree@@XZ 00000000351d8810 f i trimesh.obj
 0001:001d7820       ?GetRandomPos@CTriMesh@@UEAAXAEAURandomPos@@AEAUGeomQuery@@W4EGeomForm@@@Z 00000000351d8820 f   trimesh.obj
 0001:001d79f0       ?GetCenter@CTriMesh@@UEAA?AU?$Vec3_tpl@M@@XZ 00000000351d89f0 f   trimesh.obj
 0001:001d7c00       ?GetFeature@CTriMesh@@UEAAHHHPEAU?$Vec3_tpl@M@@@Z 00000000351d8c00 f   trimesh.obj
 0001:001d7d30       ?PrepareTriangle@CTriMesh@@QEAAXHPEAUtriangle@primitives@@PEBUgeometry_under_test@@@Z 00000000351d8d30 f   trimesh.obj
 0001:001d8060       ?PreparePrimitive@CTriMesh@@UEAAHPEAUgeom_world_data@@AEAPEAUprimitive@primitives@@H@Z 00000000351d9060 f   trimesh.obj
 0001:001d8350       ?GetPrimitiveList@CTriMesh@@UEAAHHHHPEAUprimitive@primitives@@HPEAUgeometry_under_test@@10PEAD@Z 00000000351d9350 f   trimesh.obj
 0001:001d8aa0       ?HashTrianglesToPlane@CTriMesh@@QEAAXAEBUcoord_plane@primitives@@AEBU?$Vec2_tpl@M@@AEAUgrid@3@AEAPEAH3M@Z 00000000351d9aa0 f   trimesh.obj
 0001:001d98b0       ?CalculateMediumResistance@CTriMesh@@UEAAXPEBUplane@primitives@@PEBUgeom_world_data@@AEAU?$Vec3_tpl@M@@2@Z 00000000351da8b0 f   trimesh.obj
 0001:001d9a40       ?DrawToOcclusionCubemap@CTriMesh@@UEAAHPEBUgeom_world_data@@HHHPEAUSOcclusionCubeMap@@@Z 00000000351daa40 f   trimesh.obj
 0001:001d9e30       ?DrawWireframe@CTriMesh@@UEAAXPEAUIPhysRenderer@@PEAUgeom_world_data@@HH@Z 00000000351dae30 f   trimesh.obj
 0001:001da310       ?GetMemoryStatistics@CTriMesh@@UEAAXPEAVICrySizer@@@Z 00000000351db310 f   trimesh.obj
 0001:001da720       ?Save@CTriMesh@@UEAAXAEAVCMemStream@@@Z 00000000351db720 f   trimesh.obj
 0001:001dacf0       ?CompactMemory@CTriMesh@@UEAAXXZ 00000000351dbcf0 f   trimesh.obj
 0001:001dae70       ?ExpandVtxList@CTriMesh@@QEAAHXZ 00000000351dbe70 f   trimesh.obj
 0001:001dafd0       ?CroppedRectArea@@YAMAEBU?$Vec2_tpl@M@@000@Z 00000000351dbfd0 f   trimesh.obj
 0001:001db220       ??$qsort@M@@YAXPEAHV?$strided_pointer@M@@HH@Z 00000000351dc220 f i trimesh.obj
 0001:001db370       ??0CTriMesh@@QEAA@XZ       00000000351dc370 f   trimesh.obj
 0001:001db4c0       ??_ECTriMesh@@UEAAPEAXI@Z  00000000351dc4c0 f i trimesh.obj
 0001:001db4c0       ??_GCTriMesh@@UEAAPEAXI@Z  00000000351dc4c0 f i trimesh.obj
 0001:001db4f0       ?CalculateTopology@CTriMesh@@QEAAHPEAHH@Z 00000000351dc4f0 f   trimesh.obj
 0001:001dbde0       ?RebuildBVTree@CTriMesh@@QEAAXPEAVCBVTree@@@Z 00000000351dcde0 f   trimesh.obj
 0001:001dc970       ?BuildIslandMap@CTriMesh@@QEAAHXZ 00000000351dd970 f   trimesh.obj
 0001:001dd1b0       ?CompactTriangleList@CTriMesh@@QEAAXPEAH_N@Z 00000000351de1b0 f   trimesh.obj
 0001:001dd570       ?ComputeExtent@CTriMesh@@UEAAMAEAUGeomQuery@@W4EGeomForm@@@Z 00000000351de570 f   trimesh.obj
 0001:001dda70       ?IsConvex@CTriMesh@@UEAAHM@Z 00000000351dea70 f   trimesh.obj
 0001:001ddd50       ?TraceTriangleInters@CTriMesh@@QEAAHHQEAPEAUprimitive@primitives@@HHPEAUprim_inters@@PEAUgeometry_under_test@@PEAUborder_trace@@@Z 00000000351ded50 f   trimesh.obj
 0001:001de330       ?GetUnprojectionCandidates@CTriMesh@@UEAAHHPEBUcontact@@AEAPEAUprimitive@primitives@@AEAPEAHPEAUgeometry_under_test@@@Z 00000000351df330 f   trimesh.obj
 0001:001decd0       ?update_unprojection@@YAXNPEAUunprojection_mode@@PEAUgeometry_under_test@@@Z 00000000351dfcd0 f   trimesh.obj
 0001:001df210       ?PreparePolygon@CTriMesh@@UEAAHPEAUcoord_plane@primitives@@HHPEAUgeometry_under_test@@AEAPEAU?$Vec2_tpl@M@@AEAPEAH3@Z 00000000351e0210 f   trimesh.obj
 0001:001e07d0       ?PreparePolyline@CTriMesh@@UEAAHPEAUcoord_plane@primitives@@HHPEAUgeometry_under_test@@AEAPEAU?$Vec2_tpl@M@@AEAPEAH3@Z 00000000351e17d0 f   trimesh.obj
 0001:001e1320       ?FindClosestPoint@CTriMesh@@UEAAHPEAUgeom_world_data@@AEAH1AEBU?$Vec3_tpl@M@@2PEAU3@H@Z 00000000351e2320 f   trimesh.obj
 0001:001e33e0       ?PointInsideStatusMesh@CTriMesh@@UEAAHAEBU?$Vec3_tpl@M@@PEAUindexed_triangle@primitives@@@Z 00000000351e43e0 f   trimesh.obj
 0001:001e3860       ?PrepareForRayTest@CTriMesh@@UEAAXM@Z 00000000351e4860 f   trimesh.obj
 0001:001e3f90       ?Intersect@CTriMesh@@UEAAHPEAUIGeometry@@PEAUgeom_world_data@@1PEAUintersection_params@@AEAPEAUgeom_contact@@@Z 00000000351e4f90 f   trimesh.obj
 0001:001e64e0       ?CalcVolumetricPressure@CTriMesh@@UEAAXPEAUgeom_world_data@@AEBU?$Vec3_tpl@M@@MM1AEAU3@2@Z 00000000351e74e0 f   trimesh.obj
 0001:001e7750       ?CalcPyramidVolume@@YAMAEBU?$Vec3_tpl@M@@000AEAU1@@Z 00000000351e8750 f   trimesh.obj
 0001:001e78d0       ?RemapForeignIdx@CTriMesh@@UEAAXPEAH0H@Z 00000000351e88d0 f   trimesh.obj
 0001:001e7fa0       ?AppendVertices@CTriMesh@@UEAAXPEAU?$Vec3_tpl@M@@PEAHH@Z 00000000351e8fa0 f   trimesh.obj
 0001:001e8190       ?GetIslandDisk@CTriMesh@@QEAAMHAEBU?$Vec3_tpl@M@@AEAU2@1AEAM@Z 00000000351e9190 f   trimesh.obj
 0001:001e8e70       ?Load@CTriMesh@@UEAAXAEAVCMemStream@@V?$strided_pointer@$$CBU?$Vec3_tpl@M@@@@V?$strided_pointer@G@@PEAD@Z 00000000351e9e70 f   trimesh.obj
 0001:001e9920       ?UnprojectSphere@CTriMesh@@UEAAHU?$Vec3_tpl@M@@MMPEAUcontact@@@Z 00000000351ea920 f   trimesh.obj
 0001:001eac30       ?SVD3x3@@YA?AU?$Vec3_tpl@M@@AEBU?$Matrix33_tpl@M@@@Z 00000000351ebc30 f   trimesh.obj
 0001:001eaeb0       ?CreateTriMesh@CTriMesh@@QEAAPEAV1@V?$strided_pointer@$$CBU?$Vec3_tpl@M@@@@V?$strided_pointer@G@@PEADPEAHHHHHM@Z 00000000351ebeb0 f   trimesh.obj
 0001:001ec6f0       ?SplitIntoIslands@CTriMesh@@QEAAPEAV1@PEAUplane@primitives@@HH@Z 00000000351ed6f0 f   trimesh.obj
 0001:001edfd0       ?FilterMesh@CTriMesh@@QEAAHMM@Z 00000000351eefd0 f   trimesh.obj
 0001:001ef2b0       ?CalcPhysicalProperties@CTriMesh@@UEAAHPEAUphys_geometry@@@Z 00000000351f02b0 f   trimesh.obj
 0001:001ef780       ?PrepareForIntersectionTest@CTriMesh@@UEAAHPEAUgeometry_under_test@@PEAVCGeometry@@0_N@Z 00000000351f0780 f   trimesh.obj
 0001:001efaa0       ?RegisterIntersection@CTriMesh@@UEAAHPEAUprimitive@primitives@@0PEAUgeometry_under_test@@1PEAUprim_inters@@@Z 00000000351f0aa0 f   trimesh.obj
 0001:001f3d10       ?Voxelize@CTriMesh@@QEAA?AUvoxgrid@1@U?$Quat_tpl@M@@M@Z 00000000351f4d10 f   trimesh.obj
 0001:001f4be0       ?Boxify@CTriMesh@@UEAAHPEAUbox@primitives@@HAEBUSBoxificationParams@IGeometry@@@Z 00000000351f5be0 f   trimesh.obj
 0001:001f9c60       ?Clone@CTriMesh@@QEAAPEAV1@PEAV1@H@Z 00000000351fac60 f   trimesh.obj
 0001:001fa310       ?CalculateBuoyancy@CTriMesh@@UEAAMPEBUplane@primitives@@PEBUgeom_world_data@@AEAU?$Vec3_tpl@M@@@Z 00000000351fb310 f   trimesh.obj
 0001:001fb2b0       ?GetVolume@CTriMesh@@UEAAMXZ 00000000351fc2b0 f   trimesh.obj
 0001:001fb370       ?CleanupAfterIntersectionTest@CVoxelBV@@UEAAXPEAUgeometry_under_test@@@Z 00000000351fc370 f   voxelbv.obj
 0001:001fb440       ?GetBBox@CVoxelBV@@UEAAXPEAUbox@primitives@@@Z 00000000351fc440 f   voxelbv.obj
 0001:001fb500       ?MarkUsedTriangle@CVoxelBV@@UEAAXHPEAUgeometry_under_test@@@Z 00000000351fc500 f   voxelbv.obj
 0001:001fb550       ?GetNodeBV@CVoxelBV@@UEAAXAEAPEAUBV@@HH@Z 00000000351fc550 f   voxelbv.obj
 0001:001fb7c0       ?project_box_on_3dgrid@@YAXPEAUbox@primitives@@PEAUgrid3d@2@PEAUgeometry_under_test@@PEAU?$Vec3_tpl@H@@@Z 00000000351fc7c0 f   voxelbv.obj
 0001:001fbe10       ?GetNodeContents@CVoxelBV@@UEAAHHPEAUBV@@HHPEAUgeometry_under_test@@1@Z 00000000351fce10 f   voxelbv.obj
 0001:001fc250       ?PrepareForIntersectionTest@CVoxelBV@@UEAAHPEAUgeometry_under_test@@PEAVCGeometry@@0@Z 00000000351fd250 f   voxelbv.obj
 0001:001fc4c0       ?GetNodeBV@CVoxelBV@@UEAAXAEBU?$Matrix33_tpl@M@@AEBU?$Vec3_tpl@M@@MAEAPEAUBV@@HH@Z 00000000351fd4c0 f   voxelbv.obj
 0001:001fc990       ?GetMemoryStatistics@CVoxelGeom@@UEAAXPEAVICrySizer@@@Z 00000000351fd990 f   voxelgeom.obj
 0001:001fca60       ?CreateVoxelGrid@CVoxelGeom@@QEAAPEAV1@PEAUgrid3d@primitives@@@Z 00000000351fda60 f   voxelgeom.obj
 0001:001fd1f0       ?DrawToOcclusionCubemap@CVoxelGeom@@UEAAHPEBUgeom_world_data@@HHHPEAUSOcclusionCubeMap@@@Z 00000000351fe1f0 f   voxelgeom.obj
 0001:001fd990       ?Intersect@CVoxelGeom@@UEAAHPEAUIGeometry@@PEAUgeom_world_data@@1PEAUintersection_params@@AEAPEAUgeom_contact@@@Z 00000000351fe990 f   voxelgeom.obj
 0001:001ff360       ??0CryEvent@@QEAA@XZ       0000000035200360 f   CryPhysics.obj
 0001:001ff390       ??1CryEvent@@QEAA@XZ       0000000035200390 f   CryPhysics.obj
 0001:001ff3a0       ?Set@CryEvent@@QEAAXXZ     00000000352003a0 f   CryPhysics.obj
 0001:001ff3b0       ?Wait@CryEvent@@QEBAXXZ    00000000352003b0 f   CryPhysics.obj
 0001:001ff3c0       ?CryPureCallHandler@@YAXXZ 00000000352003c0 f   CryPhysics.obj
 0001:001ff3d0       ?CryInvalidParameterHandler@@YAXPEB_W00I_K@Z 00000000352003d0 f   CryPhysics.obj
 0001:001ff3e0       ModuleInitISystem          00000000352003e0 f   CryPhysics.obj
 0001:001ff4b0       ?cry_rand32@@YAIXZ         00000000352004b0 f   CryPhysics.obj
 0001:001ff4d0       ?cry_frand@@YAMXZ          00000000352004d0 f   CryPhysics.obj
 0001:001ff510       ?Init@_CryMemoryManagerPoolHelper@@SAXXZ 0000000035200510 f i CryPhysics.obj
 0001:001ff710       ?CryGetIMemoryManager@@YAPEAUIMemoryManager@@XZ 0000000035200710 f   CryPhysics.obj
 0001:001ff760       ?CryInterlockedIncrement@@YAJPECH@Z 0000000035200760 f   CryPhysics.obj
 0001:001ff770       ?CryInterlockedDecrement@@YAJPECH@Z 0000000035200770 f   CryPhysics.obj
 0001:001ff780       ?CryInterlockedCompareExchange@@YAJPECJJJ@Z 0000000035200780 f   CryPhysics.obj
 0001:001ff790       ?CryCreateCriticalSectionInplace@@YAXPEAX@Z 0000000035200790 f   CryPhysics.obj
 0001:001ff7a0       ?CryDeleteCriticalSectionInplace@@YAXPEAX@Z 00000000352007a0 f   CryPhysics.obj
 0001:001ff7d0       ?CryGetCurrentThreadId@@YAIXZ 00000000352007d0 f   CryPhysics.obj
 0001:001ff7e0       ?CryQueryPerformanceCounter@@YA_JXZ 00000000352007e0 f   CryPhysics.obj
 0001:001ff7f0       CryModuleGetMemoryInfo     00000000352007f0 f   CryPhysics.obj
 0001:001ff7f0       CryGetMemoryInfoForModule  00000000352007f0 f   CryPhysics.obj
 0001:001ff830       ?OnSystemEvent@CSystemEventListner_Physics@@UEAAXW4ESystemEvent@@_K1@Z 0000000035200830 f i CryPhysics.obj
 0001:001ff890       CryModuleMalloc            0000000035200890 f   CryPhysics.obj
 0001:001ff930       CryModuleFree              0000000035200930 f   CryPhysics.obj
 0001:001ff9a0       CryModuleMemalign          00000000352009a0 f   CryPhysics.obj
 0001:001ffa50       ??2@YAPEAX_K@Z             0000000035200a50 f   CryPhysics.obj
 0001:001ffac0       ??_U@YAPEAX_K@Z            0000000035200ac0 f   CryPhysics.obj
 0001:001ffb30       ??3@YAXPEAX@Z              0000000035200b30 f   CryPhysics.obj
 0001:001ffbd0       ??_V@YAXPEAX@Z             0000000035200bd0 f   CryPhysics.obj
 0001:001ffc70       ??_EICryFactory@@MEAAPEAXI@Z 0000000035200c70 f i CryPhysics.obj
 0001:001ffc70       ??_GICryFactory@@MEAAPEAXI@Z 0000000035200c70 f i CryPhysics.obj
 0001:001ffca0       ??0InitPhysicsGlobals@@QEAA@XZ 0000000035200ca0 f i CryPhysics.obj
 0001:002002b0       CreatePhysicalWorld        00000000352012b0 f   CryPhysics.obj
 0001:00200380       ?GetFactory@CEngineModule_CryPhysics@@UEBAPEAUICryFactory@@XZ 0000000035201380 f i CryPhysics.obj
 0001:00200390       ?GetName@CEngineModule_CryPhysics@@MEAAPEBDXZ 0000000035201390 f i CryPhysics.obj
 0001:002003a0       ?GetCategory@CEngineModule_CryPhysics@@MEAAPEBDXZ 00000000352013a0 f i CryPhysics.obj
 0001:002003b0       ?Initialize@CEngineModule_CryPhysics@@MEAA_NAEAUSSystemGlobalEnvironment@@AEBUSSystemInitParams@@@Z 00000000352013b0 f i CryPhysics.obj
 0001:002004b0       ??_GISystemEventListener@@UEAAPEAXI@Z 00000000352014b0 f i CryPhysics.obj
 0001:002004b0       ??_EISystemEventListener@@UEAAPEAXI@Z 00000000352014b0 f i CryPhysics.obj
 0001:002004b0       ??_ECSystemEventListner_Physics@@UEAAPEAXI@Z 00000000352014b0 f i CryPhysics.obj
 0001:002004b0       ??_GCSystemEventListner_Physics@@UEAAPEAXI@Z 00000000352014b0 f i CryPhysics.obj
 0001:002004e0       ??0CFactory@CEngineModule_CryPhysics@@AEAA@XZ 00000000352014e0 f i CryPhysics.obj
 0001:00200580       ?sp_enable_shared_from_this@detail@boost@@YAXZZ 0000000035201580 f i CryPhysics.obj
 0001:002005a0       ?GetClassNameA@CFactory@CEngineModule_CryPhysics@@UEBAPEBDXZ 00000000352015a0 f i CryPhysics.obj
 0001:002005b0       ?GetClassID@CFactory@CEngineModule_CryPhysics@@UEBAAEBUCryGUID@@XZ 00000000352015b0 f i CryPhysics.obj
 0001:002005c0       ?ClassSupports@CFactory@CEngineModule_CryPhysics@@UEBA_NAEBUCryGUID@@@Z 00000000352015c0 f i CryPhysics.obj
 0001:00200600       ?ClassSupports@CFactory@CEngineModule_CryPhysics@@UEBAXAEAPEBUCryGUID@@AEA_K@Z 0000000035201600 f i CryPhysics.obj
 0001:00200610       ?dispose@?$sp_counted_impl_p@VCEngineModule_CryPhysics@@@detail@boost@@UEAAXXZ 0000000035201610 f i CryPhysics.obj
 0001:00200630       ??_GCFactory@CEngineModule_CryPhysics@@UEAAPEAXI@Z 0000000035201630 f i CryPhysics.obj
 0001:00200630       ??_ECFactory@CEngineModule_CryPhysics@@UEAAPEAXI@Z 0000000035201630 f i CryPhysics.obj
 0001:00200670       ??$?0VCEngineModule_CryPhysics@@@shared_count@detail@boost@@QEAA@PEAVCEngineModule_CryPhysics@@@Z 0000000035201670 f i CryPhysics.obj
 0001:00200780       ??_G?$sp_counted_impl_p@VCEngineModule_CryPhysics@@@detail@boost@@UEAAPEAXI@Z 0000000035201780 f i CryPhysics.obj
 0001:00200780       ??_Esp_counted_base@detail@boost@@UEAAPEAXI@Z 0000000035201780 f i CryPhysics.obj
 0001:00200780       ??_Gsp_counted_base@detail@boost@@UEAAPEAXI@Z 0000000035201780 f i CryPhysics.obj
 0001:00200780       ??_E?$sp_counted_impl_p@VCEngineModule_CryPhysics@@@detail@boost@@UEAAPEAXI@Z 0000000035201780 f i CryPhysics.obj
 0001:002007b0       ??_Gbad_alloc@std@@UEAAPEAXI@Z 00000000352017b0 f i CryPhysics.obj
 0001:002007b0       ??_Ebad_alloc@std@@UEAAPEAXI@Z 00000000352017b0 f i CryPhysics.obj
 0001:002007f0       ?QueryInterface@CEngineModule_CryPhysics@@MEBAPEAXAEBUCryGUID@@@Z 00000000352017f0 f i CryPhysics.obj
 0001:00200840       ?CreateClassInstance@CFactory@CEngineModule_CryPhysics@@UEBA?AV?$shared_ptr@UICryUnknown@@@boost@@XZ 0000000035201840 f i CryPhysics.obj
 0001:00200910       ?DeInitialize@?$Node_Alloc_Lock@$00$00@@SAXXZ 0000000035201910 f i StdAfx.obj
 0001:00200978       cosf                       0000000035201978 f   MSVCRT:MSVCR100.dll
 0001:0020097e       sinf                       000000003520197e f   MSVCRT:MSVCR100.dll
 0001:00200984       _purecall                  0000000035201984 f   MSVCRT:MSVCR100.dll
 0001:0020098a       asinf                      000000003520198a f   MSVCRT:MSVCR100.dll
 0001:00200990       atan2f                     0000000035201990 f   MSVCRT:MSVCR100.dll
 0001:00200996       memcpy                     0000000035201996 f   MSVCRT:MSVCR100.dll
 0001:0020099c       memset                     000000003520199c f   MSVCRT:MSVCR100.dll
 0001:002009a4       _onexit                    00000000352019a4 f   MSVCRT:atonexit.obj
 0001:00200a54       atexit                     0000000035201a54 f   MSVCRT:atonexit.obj
 0001:00200a6c       acosf                      0000000035201a6c f   MSVCRT:MSVCR100.dll
 0001:00200a72       cos                        0000000035201a72 f   MSVCRT:MSVCR100.dll
 0001:00200a78       sin                        0000000035201a78 f   MSVCRT:MSVCR100.dll
 0001:00200a7e       atan2                      0000000035201a7e f   MSVCRT:MSVCR100.dll
 0001:00200a84       exp                        0000000035201a84 f   MSVCRT:MSVCR100.dll
 0001:00200a8a       log                        0000000035201a8a f   MSVCRT:MSVCR100.dll
 0001:00200aa0       __chkstk                   0000000035201aa0 f   MSVCRT:chkstk.obj
 0001:00200aa0       _alloca_probe              0000000035201aa0     MSVCRT:chkstk.obj
 0001:00200aee       tanf                       0000000035201aee f   MSVCRT:MSVCR100.dll
 0001:00200af4       atanf                      0000000035201af4 f   MSVCRT:MSVCR100.dll
 0001:00200afa       expf                       0000000035201afa f   MSVCRT:MSVCR100.dll
 0001:00200b00       logf                       0000000035201b00 f   MSVCRT:MSVCR100.dll
 0001:00200b06       ?what@exception@std@@UEBAPEBDXZ 0000000035201b06 f   MSVCRT:MSVCR100.dll
 0001:00200b6c       _CRT_INIT                  0000000035201b6c f   MSVCRT:crtdll.obj
 0001:00200f04       _DllMainCRTStartup         0000000035201f04 f   MSVCRT:crtdll.obj
 0001:00200f42       __C_specific_handler       0000000035201f42 f   MSVCRT:MSVCR100.dll
 0001:00200f48       _unlock                    0000000035201f48 f   MSVCRT:MSVCR100.dll
 0001:00200f4e       __dllonexit                0000000035201f4e f   MSVCRT:MSVCR100.dll
 0001:00200f54       _lock                      0000000035201f54 f   MSVCRT:MSVCR100.dll
 0001:00200f5c       __clean_type_info_names    0000000035201f5c f   MSVCRT:tncleanup.obj
 0001:00200f68       _RTC_Initialize            0000000035201f68 f   MSVCRT:_initsect_.obj
 0001:00200fa0       _RTC_Terminate             0000000035201fa0 f   MSVCRT:_initsect_.obj
 0001:00200fe0       _ValidateImageBase         0000000035201fe0 f   MSVCRT:pesect.obj
 0001:00201010       _FindPESection             0000000035202010 f   MSVCRT:pesect.obj
 0001:00201060       _IsNonwritableInCurrentImage 0000000035202060 f   MSVCRT:pesect.obj
 0001:002010a2       _initterm                  00000000352020a2 f   MSVCRT:MSVCR100.dll
 0001:002010a8       _initterm_e                00000000352020a8 f   MSVCRT:MSVCR100.dll
 0001:002010ae       _amsg_exit                 00000000352020ae f   MSVCRT:MSVCR100.dll
 0001:002010b4       __CppXcptFilter            00000000352020b4 f   MSVCRT:MSVCR100.dll
 0001:002010bc       DllMain                    00000000352020bc f   MSVCRT:dllmain.obj
 0001:002010e0       __security_init_cookie     00000000352020e0 f   MSVCRT:gs_support.obj
 0001:00201194       __clean_type_info_names_internal 0000000035202194 f   MSVCRT:MSVCR100.dll
 0001:002016e0       ??__Fs_dummyMemReplay@?1??CryGetIMemReplay@@YAPEAUIMemReplay@@XZ@YAXXZ 00000000352026e0 f i articulatedentity.obj
 0001:00201710       ??__FserializeString@?1??SetSharedSerializeString@?$CSerializeWrapper@UISerialize@@@@QEAAAEAUSSerializeString@@AEBV?$CryStringT@D@@@Z@YAXXZ 0000000035202710 f i physicalentity.obj
 0001:00201930       ??__Fp@?1??CreateClassInstance@CFactory@CEngineModule_CryPhysics@@UEBA?AV?$shared_ptr@UICryUnknown@@@boost@@XZ@YAXXZ 0000000035202930 f i CryPhysics.obj
 0002:00000000       __imp_TlsGetValue          0000000035203000     kernel32:KERNEL32.dll
 0002:00000008       __imp_TlsAlloc             0000000035203008     kernel32:KERNEL32.dll
 0002:00000010       __imp_TlsSetValue          0000000035203010     kernel32:KERNEL32.dll
 0002:00000018       __imp_QueryPerformanceCounter 0000000035203018     kernel32:KERNEL32.dll
 0002:00000020       __imp_Sleep                0000000035203020     kernel32:KERNEL32.dll
 0002:00000028       __imp_CreateEventA         0000000035203028     kernel32:KERNEL32.dll
 0002:00000030       __imp_CloseHandle          0000000035203030     kernel32:KERNEL32.dll
 0002:00000038       __imp_SetEvent             0000000035203038     kernel32:KERNEL32.dll
 0002:00000040       __imp_WaitForSingleObject  0000000035203040     kernel32:KERNEL32.dll
 0002:00000048       __imp_InitializeCriticalSection 0000000035203048     kernel32:KERNEL32.dll
 0002:00000050       __imp_DeleteCriticalSection 0000000035203050     kernel32:KERNEL32.dll
 0002:00000058       __imp_EnterCriticalSection 0000000035203058     kernel32:KERNEL32.dll
 0002:00000060       __imp_LeaveCriticalSection 0000000035203060     kernel32:KERNEL32.dll
 0002:00000068       __imp_GetCurrentThreadId   0000000035203068     kernel32:KERNEL32.dll
 0002:00000070       __imp_LoadLibraryA         0000000035203070     kernel32:KERNEL32.dll
 0002:00000078       __imp_GetProcAddress       0000000035203078     kernel32:KERNEL32.dll
 0002:00000080       __imp_GetModuleHandleA     0000000035203080     kernel32:KERNEL32.dll
 0002:00000088       __imp_GetCurrentProcessId  0000000035203088     kernel32:KERNEL32.dll
 0002:00000090       __imp_GetTickCount         0000000035203090     kernel32:KERNEL32.dll
 0002:00000098       __imp_DisableThreadLibraryCalls 0000000035203098     kernel32:KERNEL32.dll
 0002:000000a0       __imp_DecodePointer        00000000352030a0     kernel32:KERNEL32.dll
 0002:000000a8       __imp_EncodePointer        00000000352030a8     kernel32:KERNEL32.dll
 0002:000000b0       __imp_GetSystemTimeAsFileTime 00000000352030b0     kernel32:KERNEL32.dll
 0002:000000b8       \177KERNEL32_NULL_THUNK_DATA 00000000352030b8     kernel32:KERNEL32.dll
 0002:000000c0       __imp_asinf                00000000352030c0     MSVCRT:MSVCR100.dll
 0002:000000c8       __imp_atan2f               00000000352030c8     MSVCRT:MSVCR100.dll
 0002:000000d0       __imp_memcpy               00000000352030d0     MSVCRT:MSVCR100.dll
 0002:000000d8       __imp_memset               00000000352030d8     MSVCRT:MSVCR100.dll
 0002:000000e0       __imp__snprintf            00000000352030e0     MSVCRT:MSVCR100.dll
 0002:000000e8       __imp_memmove              00000000352030e8     MSVCRT:MSVCR100.dll
 0002:000000f0       __imp_acosf                00000000352030f0     MSVCRT:MSVCR100.dll
 0002:000000f8       __imp_cos                  00000000352030f8     MSVCRT:MSVCR100.dll
 0002:00000100       __imp__purecall            0000000035203100     MSVCRT:MSVCR100.dll
 0002:00000108       __imp_sin                  0000000035203108     MSVCRT:MSVCR100.dll
 0002:00000110       __imp_atan2                0000000035203110     MSVCRT:MSVCR100.dll
 0002:00000118       __imp_exp                  0000000035203118     MSVCRT:MSVCR100.dll
 0002:00000120       __imp_log                  0000000035203120     MSVCRT:MSVCR100.dll
 0002:00000128       __imp_sprintf              0000000035203128     MSVCRT:MSVCR100.dll
 0002:00000130       __imp_strtoul              0000000035203130     MSVCRT:MSVCR100.dll
 0002:00000138       __imp_tanf                 0000000035203138     MSVCRT:MSVCR100.dll
 0002:00000140       __imp_atanf                0000000035203140     MSVCRT:MSVCR100.dll
 0002:00000148       __imp_expf                 0000000035203148     MSVCRT:MSVCR100.dll
 0002:00000150       __imp_logf                 0000000035203150     MSVCRT:MSVCR100.dll
 0002:00000158       __imp__set_invalid_parameter_handler 0000000035203158     MSVCRT:MSVCR100.dll
 0002:00000160       __imp__set_purecall_handler 0000000035203160     MSVCRT:MSVCR100.dll
 0002:00000168       __imp_exit                 0000000035203168     MSVCRT:MSVCR100.dll
 0002:00000170       __imp_??0exception@std@@QEAA@AEBQEBDH@Z 0000000035203170     MSVCRT:MSVCR100.dll
 0002:00000178       __imp_?what@exception@std@@UEBAPEBDXZ 0000000035203178     MSVCRT:MSVCR100.dll
 0002:00000180       __imp_??1exception@std@@UEAA@XZ 0000000035203180     MSVCRT:MSVCR100.dll
 0002:00000188       __imp___C_specific_handler 0000000035203188     MSVCRT:MSVCR100.dll
 0002:00000190       __imp__unlock              0000000035203190     MSVCRT:MSVCR100.dll
 0002:00000198       __imp___dllonexit          0000000035203198     MSVCRT:MSVCR100.dll
 0002:000001a0       __imp__lock                00000000352031a0     MSVCRT:MSVCR100.dll
 0002:000001a8       __imp__onexit              00000000352031a8     MSVCRT:MSVCR100.dll
 0002:000001b0       __imp_vsnprintf_s          00000000352031b0     MSVCRT:MSVCR100.dll
 0002:000001b0       __imp__vsnprintf_s         00000000352031b0     MSVCRT:MSVCR100.dll
 0002:000001b8       __imp__vsnprintf           00000000352031b8     MSVCRT:MSVCR100.dll
 0002:000001b8       __imp_vsnprintf            00000000352031b8     MSVCRT:MSVCR100.dll
 0002:000001c0       __imp__malloc_crt          00000000352031c0     MSVCRT:MSVCR100.dll
 0002:000001c8       __imp__initterm            00000000352031c8     MSVCRT:MSVCR100.dll
 0002:000001d0       __imp__initterm_e          00000000352031d0     MSVCRT:MSVCR100.dll
 0002:000001d8       __imp_free                 00000000352031d8     MSVCRT:MSVCR100.dll
 0002:000001e0       __imp__encoded_null        00000000352031e0     MSVCRT:MSVCR100.dll
 0002:000001e8       __imp__amsg_exit           00000000352031e8     MSVCRT:MSVCR100.dll
 0002:000001f0       __imp___CppXcptFilter      00000000352031f0     MSVCRT:MSVCR100.dll
 0002:000001f8       __imp___clean_type_info_names_internal 00000000352031f8     MSVCRT:MSVCR100.dll
 0002:00000200       __imp_sinf                 0000000035203200     MSVCRT:MSVCR100.dll
 0002:00000208       __imp_cosf                 0000000035203208     MSVCRT:MSVCR100.dll
 0002:00000210       __imp__ltoa                0000000035203210     MSVCRT:MSVCR100.dll
 0002:00000210       __imp_ltoa                 0000000035203210     MSVCRT:MSVCR100.dll
 0002:00000218       __imp__isnan               0000000035203218     MSVCRT:MSVCR100.dll
 0002:00000220       \177MSVCR100_NULL_THUNK_DATA 0000000035203220     MSVCRT:MSVCR100.dll
 0002:00000228       __imp_MessageBoxA          0000000035203228     user32:USER32.dll
 0002:00000230       \177USER32_NULL_THUNK_DATA 0000000035203230     user32:USER32.dll
 0002:00000238       __xc_a                     0000000035203238     MSVCRT:cinitexe.obj
 0002:000002c0       __xc_z                     00000000352032c0     MSVCRT:cinitexe.obj
 0002:000002c8       __xi_a                     00000000352032c8     MSVCRT:cinitexe.obj
 0002:000002d8       __xi_z                     00000000352032d8     MSVCRT:cinitexe.obj
 0002:00000310       __mask@@AbsFloat@          0000000035203310     articulatedentity.obj
 0002:00000320       ??_7IMemReplay@@6B@        0000000035203320     articulatedentity.obj
 0002:00000450       __real@3f800000            0000000035203450     articulatedentity.obj
 0002:00000454       __real@3f000000            0000000035203454     articulatedentity.obj
 0002:00000458       __real@bf800000            0000000035203458     articulatedentity.obj
 0002:0000045c       __real@7149f2ca            000000003520345c     articulatedentity.obj
 0002:00000460       __real@00000000            0000000035203460     articulatedentity.obj
 0002:00000470       __mask@@NegFloat@          0000000035203470     articulatedentity.obj
 0002:00000480       __real@3c23d70a            0000000035203480     articulatedentity.obj
 0002:00000484       __real@3fc90fdb            0000000035203484     articulatedentity.obj
 0002:00000490       ??_7CDummyMemReplay@@6B@   0000000035203490     articulatedentity.obj
 0002:000005c0       ??_7CArticulatedEntity@@6B@ 00000000352035c0     articulatedentity.obj
 0002:00000828       __real@42c80000            0000000035203828     articulatedentity.obj
 0002:0000082c       __real@40000000            000000003520382c     articulatedentity.obj
 0002:00000830       ??_C@_04OACGEDLG@qext?$AA@ 0000000035203830     articulatedentity.obj
 0002:00000838       ??_C@_01IIACKFLH@q?$AA@    0000000035203838     articulatedentity.obj
 0002:00000840       ??_C@_0EN@FCJJGCPA@?$CFs?3?5?$CI?$CF?450s?5?$EA?5?$CF?41f?0?$CF?41f?0?$CF?41f?$CJ?5Val@ 0000000035203840     articulatedentity.obj
 0002:00000890       ??_C@_02IKMLBCHJ@q0?$AA@   0000000035203890     articulatedentity.obj
 0002:00000898       ??_C@_0DN@ECLMILFI@?$CFs?3?5?$CI?$CF?450s?5?$EA?5?$CF?41f?0?$CF?41f?0?$CF?41f?$CJ?5Val@ 0000000035203898     articulatedentity.obj
 0002:000008d8       ??_C@_05JHLBIJAO@pivot?$AA@ 00000000352038d8     articulatedentity.obj
 0002:000008de       ??_C@_00CNPNBAHC@?$AA@     00000000352038de     articulatedentity.obj
 0002:000008e0       ??_C@_05HKIHAKL@ipart?$AA@ 00000000352038e0     articulatedentity.obj
 0002:000008e8       ??_C@_05BBEJFBFA@point?$AA@ 00000000352038e8     articulatedentity.obj
 0002:000008f0       __real@5368d4a5            00000000352038f0     articulatedentity.obj
 0002:000008f8       ??_C@_0L@CLGAEIII@angImpulse?$AA@ 00000000352038f8     articulatedentity.obj
 0002:00000904       __real@5a0e1bca            0000000035203904     articulatedentity.obj
 0002:00000910       ??_C@_0EN@KMHCOBOM@?$CFs?3?5?$CI?$CF?450s?5?$EA?5?$CF?41f?0?$CF?41f?0?$CF?41f?$CJ?5Val@ 0000000035203910     articulatedentity.obj
 0002:00000960       ??_C@_07LKMFNFAN@impulse?$AA@ 0000000035203960     articulatedentity.obj
 0002:00000968       __real@6753c21c            0000000035203968     articulatedentity.obj
 0002:0000096c       __real@1e3ce508            000000003520396c     articulatedentity.obj
 0002:00000970       __real@3e45798ee2308c3a    0000000035203970     articulatedentity.obj
 0002:00000978       __real@3f7d70a4            0000000035203978     articulatedentity.obj
 0002:0000097c       __real@3e860a92            000000003520397c     articulatedentity.obj
 0002:00000980       __real@41200000            0000000035203980     articulatedentity.obj
 0002:00000984       __real@3f7f7cff            0000000035203984     articulatedentity.obj
 0002:00000988       __real@401921fb54442d18    0000000035203988     articulatedentity.obj
 0002:00000990       __real@c00921fb54442d18    0000000035203990     articulatedentity.obj
 0002:00000998       __real@41700000            0000000035203998     articulatedentity.obj
 0002:000009a0       __real@3eb0c6f7a0b5ed8d    00000000352039a0     articulatedentity.obj
 0002:000009a8       __real@3dcccccd            00000000352039a8     articulatedentity.obj
 0002:000009b0       ??_C@_09GMEIBLE@offsPivot?$AA@ 00000000352039b0     articulatedentity.obj
 0002:000009c0       ??_C@_09OMNEEBCL@numjoints?$AA@ 00000000352039c0     articulatedentity.obj
 0002:000009cc       ??_C@_05LAFFIJJO@quat0?$AA@ 00000000352039cc     articulatedentity.obj
 0002:000009d8       ??_C@_09MBCEGBCG@q0changed?$AA@ 00000000352039d8     articulatedentity.obj
 0002:000009e4       ??_C@_02HJEEANKG@dq?$AA@   00000000352039e4     articulatedentity.obj
 0002:000009e8       ??_C@_05LDAEHAKN@joint?$AA@ 00000000352039e8     articulatedentity.obj
 0002:000009f0       ??_C@_03BHLLPCMD@vel?$AA@  00000000352039f0     articulatedentity.obj
 0002:000009f4       ??_C@_03PCBNCGFH@pos?$AA@  00000000352039f4     articulatedentity.obj
 0002:000009f8       ??_C@_05BJPFJFDJ@awake?$AA@ 00000000352039f8     articulatedentity.obj
 0002:00000a00       __real@40800000            0000000035203a00     articulatedentity.obj
 0002:00000a04       __real@41c80000            0000000035203a04     articulatedentity.obj
 0002:00000a08       __real@40c00000            0000000035203a08     articulatedentity.obj
 0002:00000a0c       __real@40a00000            0000000035203a0c     articulatedentity.obj
 0002:00000a10       __real@3716feb5            0000000035203a10     articulatedentity.obj
 0002:00000a20       ??_C@_0FD@NAFJCAP@CArticulatedEntity?3?3AddGeometry?3@ 0000000035203a20     articulatedentity.obj
 0002:00000a74       __real@447a0000            0000000035203a74     articulatedentity.obj
 0002:00000a78       __real@49742400            0000000035203a78     articulatedentity.obj
 0002:00000a7c       __real@40400000            0000000035203a7c     articulatedentity.obj
 0002:00000a80       ??_C@_0CK@MJPDAFHG@CArticulatedEntity?3Action?$CIaction@ 0000000035203a80     articulatedentity.obj
 0002:00000aac       __real@3d23d70a            0000000035203aac     articulatedentity.obj
 0002:00000ab0       __real@be800000            0000000035203ab0     articulatedentity.obj
 0002:00000ab4       __real@3e800000            0000000035203ab4     articulatedentity.obj
 0002:00000ab8       __real@3e4ccccd            0000000035203ab8     articulatedentity.obj
 0002:00000abc       __real@bf000000            0000000035203abc     articulatedentity.obj
 0002:00000ac0       __real@3d8efa35            0000000035203ac0     articulatedentity.obj
 0002:00000ac4       __real@3fcccccd            0000000035203ac4     articulatedentity.obj
 0002:00000ac8       __real@3f99999a            0000000035203ac8     articulatedentity.obj
 0002:00000acc       __real@3727c5ac            0000000035203acc     articulatedentity.obj
 0002:00000ad0       __real@51ba43b7            0000000035203ad0     articulatedentity.obj
 0002:00000ad4       __real@501502f9            0000000035203ad4     articulatedentity.obj
 0002:00000ad8       __real@3c8efa35            0000000035203ad8     articulatedentity.obj
 0002:00000adc       __real@358637bd            0000000035203adc     articulatedentity.obj
 0002:00000ae0       __real@3a83126f            0000000035203ae0     articulatedentity.obj
 0002:00000ae4       __real@38d1b717            0000000035203ae4     articulatedentity.obj
 0002:00000ae8       __real@322bcc77            0000000035203ae8     articulatedentity.obj
 0002:00000aec       __real@3f666666            0000000035203aec     articulatedentity.obj
 0002:00000af0       __real@3d8f5c29            0000000035203af0     articulatedentity.obj
 0002:00000af4       __real@40200000            0000000035203af4     articulatedentity.obj
 0002:00000af8       __real@3fc45f306dc9c883    0000000035203af8     articulatedentity.obj
 0002:00000b00       __real@3f4f5c28            0000000035203b00     articulatedentity.obj
 0002:00000b04       __real@3e99999a            0000000035203b04     articulatedentity.obj
 0002:00000b08       ??_C@_0BJ@NDOEJGHE@CArticulatedEntity?3?3Step?$AA@ 0000000035203b08     articulatedentity.obj
 0002:00000b28       ??_C@_0CL@ECFNLKDN@CArticulatedEntity?3SetParams?$CIpar@ 0000000035203b28     articulatedentity.obj
 0002:00000b54       __real@c0c90fdb            0000000035203b54     articulatedentity.obj
 0002:00000b58       __real@40c90fdb            0000000035203b58     articulatedentity.obj
 0002:00000b5c       __real@40490fdb            0000000035203b5c     articulatedentity.obj
 0002:00000b60       __real@2edbe6ff            0000000035203b60     articulatedentity.obj
 0002:00000b70       ??_7CBVTree@@6B@           0000000035203b70     livingentity.obj
 0002:00000c50       ??_7IGeometry@@6B@         0000000035203c50     livingentity.obj
 0002:00000dd0       ??_7CRayBV@@6B@            0000000035203dd0     livingentity.obj
 0002:00000eb0       ??_7CLivingEntity@@6B@     0000000035203eb0     livingentity.obj
 0002:000010e8       __real@404ca5dc1a63c1f8    00000000352040e8     livingentity.obj
 0002:000010f0       ??_7CGeometry@@6B@         00000000352040f0     livingentity.obj
 0002:000012e0       __real@43a3d5c3            00000000352042e0     livingentity.obj
 0002:000012e4       __real@c2c80000            00000000352042e4     livingentity.obj
 0002:000012e8       __real@3b480190            00000000352042e8     livingentity.obj
 0002:000012ec       __real@414c0000            00000000352042ec     livingentity.obj
 0002:000012f0       __real@41a00000            00000000352042f0     livingentity.obj
 0002:000012f8       __real@404436720cee34f2    00000000352042f8     livingentity.obj
 0002:00001300       __real@40c45f07af68ecef    0000000035204300     livingentity.obj
 0002:00001308       __real@36800000            0000000035204308     livingentity.obj
 0002:0000130c       __real@3da0a0a1            000000003520430c     livingentity.obj
 0002:00001310       __real@3f9954a49d7f2b6f    0000000035204310     livingentity.obj
 0002:00001318       __real@3f19222d989f5e57    0000000035204318     livingentity.obj
 0002:00001320       ??_C@_0N@DIIBGNIK@velRequested?$AA@ 0000000035204320     livingentity.obj
 0002:00001330       __real@c0800000            0000000035204330     livingentity.obj
 0002:00001338       ??_C@_0N@MHIKDJFP@sizeCollider?$AA@ 0000000035204338     livingentity.obj
 0002:00001348       __real@461c4000            0000000035204348     livingentity.obj
 0002:00001350       ??_C@_09EOJBHBBH@heightEye?$AA@ 0000000035204350     livingentity.obj
 0002:00001360       ??_C@_0M@FLAOEHJJ@heightPivot?$AA@ 0000000035204360     livingentity.obj
 0002:0000136c       ??_C@_02EDDPJOD@dt?$AA@    000000003520436c     livingentity.obj
 0002:00001370       ??_C@_03DAPAKLGM@dir?$AA@  0000000035204370     livingentity.obj
 0002:00001380       ??_7CSingleBoxTree@@6B@    0000000035204380     livingentity.obj
 0002:00001460       ??_7CCylinderGeom@@6B@     0000000035204460     livingentity.obj
 0002:00001650       ??_7CCapsuleGeom@@6B@      0000000035204650     livingentity.obj
 0002:00001840       __real@4010c152382d7365    0000000035204840     livingentity.obj
 0002:00001850       ??_7CRayGeom@@6B@          0000000035204850     livingentity.obj
 0002:00001a40       __real@3fb999999999999a    0000000035204a40     livingentity.obj
 0002:00001a48       __real@3b83126f            0000000035204a48     livingentity.obj
 0002:00001a50       __real@3ff39a816dfbe7fa    0000000035204a50     livingentity.obj
 0002:00001a58       __real@3fee28c7460698c7    0000000035204a58     livingentity.obj
 0002:00001a60       __real@3fe41b2f7ba3bcbe    0000000035204a60     livingentity.obj
 0002:00001a68       __real@3f91df46a2529d39    0000000035204a68     livingentity.obj
 0002:00001a70       ??_C@_0CL@HEHKAFBI@CLivingEntity?3SetParams?$CIplayer_d@ 0000000035204a70     livingentity.obj
 0002:00001aa0       __real@3f847ae147ae147b    0000000035204aa0     livingentity.obj
 0002:00001aa8       __real@3f8147ae            0000000035204aa8     livingentity.obj
 0002:00001aac       __real@3b23d70b            0000000035204aac     livingentity.obj
 0002:00001ab0       __real@40555555            0000000035204ab0     livingentity.obj
 0002:00001ab8       ??_C@_0CF@GMDAKOKI@CLivingEntity?3Action?$CIaction_impu@ 0000000035204ab8     livingentity.obj
 0002:00001ae0       ??_C@_0CC@ELHODBNL@CLivingEntity?3Action?$CIaction_move@ 0000000035204ae0     livingentity.obj
 0002:00001b04       __real@45cccccd            0000000035204b04     livingentity.obj
 0002:00001b08       __real@42480000            0000000035204b08     livingentity.obj
 0002:00001b0c       __real@3f866666            0000000035204b0c     livingentity.obj
 0002:00001b10       __real@41000000            0000000035204b10     livingentity.obj
 0002:00001b14       __real@3f333333            0000000035204b14     livingentity.obj
 0002:00001b18       __real@3ff0000000000000    0000000035204b18     livingentity.obj
 0002:00001b20       __real@4000000000000000    0000000035204b20     livingentity.obj
 0002:00001b28       __real@3f7746ea            0000000035204b28     livingentity.obj
 0002:00001b2c       __real@3e8483ee            0000000035204b2c     livingentity.obj
 0002:00001b30       __real@3fb33333            0000000035204b30     livingentity.obj
 0002:00001b38       __real@3fd0000000000000    0000000035204b38     livingentity.obj
 0002:00001b40       __real@bfc00000            0000000035204b40     livingentity.obj
 0002:00001b44       __real@d01502f9            0000000035204b44     livingentity.obj
 0002:00001b48       __real@3db22d0e            0000000035204b48     livingentity.obj
 0002:00001b4c       __real@3f19999a            0000000035204b4c     livingentity.obj
 0002:00001b50       __real@3e23d70b            0000000035204b50     livingentity.obj
 0002:00001b54       __real@3f7ff2e5            0000000035204b54     livingentity.obj
 0002:00001b58       __real@3ca3d70a            0000000035204b58     livingentity.obj
 0002:00001b5c       __real@bf8147ae            0000000035204b5c     livingentity.obj
 0002:00001b60       __real@c0000000            0000000035204b60     livingentity.obj
 0002:00001b64       __real@3f733333            0000000035204b64     livingentity.obj
 0002:00001b68       __real@3f400000            0000000035204b68     livingentity.obj
 0002:00001b6c       __real@3f733334            0000000035204b6c     livingentity.obj
 0002:00001b70       __real@358637be            0000000035204b70     livingentity.obj
 0002:00001b74       __real@3ecccccd            0000000035204b74     livingentity.obj
 0002:00001b78       __real@3fc00000            0000000035204b78     livingentity.obj
 0002:00001b80       ??_C@_0BE@PGDCIADM@CLivingEntity?3?3Step?$AA@ 0000000035204b80     livingentity.obj
 0002:00001b94       __real@00800000            0000000035204b94     particleentity.obj
 0002:00001ba0       ??_7CParticleEntity@@6B@   0000000035204ba0     particleentity.obj
 0002:00001dd8       __real@3f4ccccd            0000000035204dd8     particleentity.obj
 0002:00001ddc       __real@c11cf5c3            0000000035204ddc     particleentity.obj
 0002:00001de0       __real@c47a0000            0000000035204de0     particleentity.obj
 0002:00001de4       ??_C@_06IKLLLDHL@normal?$AA@ 0000000035204de4     particleentity.obj
 0002:00001df0       ??_C@_07MBJMFGGL@heading?$AA@ 0000000035204df0     particleentity.obj
 0002:00001df8       ??_C@_09GLPKLBIH@thickness?$AA@ 0000000035204df8     particleentity.obj
 0002:00001e04       ??_C@_04IAGNFIBA@size?$AA@ 0000000035204e04     particleentity.obj
 0002:00001e0c       ??_C@_04IJEANHEE@mass?$AA@ 0000000035204e0c     particleentity.obj
 0002:00001e18       ??_C@_0P@LKCCAGNB@ParticleEntity?$AA@ 0000000035204e18     particleentity.obj
 0002:00001e28       ??_C@_07OKNHCJLM@ifawake?$AA@ 0000000035204e28     particleentity.obj
 0002:00001e30       ??_C@_0CO@DMIGAK@CParticleEntity?3SetParams?$CIpe_par@ 0000000035204e30     particleentity.obj
 0002:00001e60       __real@43c80000            0000000035204e60     particleentity.obj
 0002:00001e64       __real@3d888889            0000000035204e64     particleentity.obj
 0002:00001e68       __real@3f7851ec            0000000035204e68     particleentity.obj
 0002:00001e6c       __real@3c23d70b            0000000035204e6c     particleentity.obj
 0002:00001e70       __real@42200000            0000000035204e70     particleentity.obj
 0002:00001e78       __real@3f1a36e2eb1c432d    0000000035204e78     particleentity.obj
 0002:00001e80       ??_C@_0CE@EPNDKOAE@RayWorldIntersection?$CIPhysParticl@ 0000000035204e80     particleentity.obj
 0002:00001ea4       __real@bf8ccccd            0000000035204ea4     particleentity.obj
 0002:00001ea8       ??_C@_0BI@KOOFBDI@CParticleEntity?3?3DoStep?$AA@ 0000000035204ea8     particleentity.obj
 0002:00001ed0       ??_7IPhysicalEntity@@6B@   0000000035204ed0     physarea.obj
 0002:00001fb0       __mask@@AbsDouble@         0000000035204fb0     physarea.obj
 0002:00001fc0       __real@2f800000            0000000035204fc0     physarea.obj
 0002:00001fc8       __real@3fe0000000000000    0000000035204fc8     physarea.obj
 0002:00001fd0       __real@3fd5555555555555    0000000035204fd0     physarea.obj
 0002:00001fd8       __real@3bc79ca10c924223    0000000035204fd8     physarea.obj
 0002:00001fe0       __real@3ddb7cdfd9d7bdbb    0000000035204fe0     physarea.obj
 0002:00001ff0       ??_7CPhysicalPlaceholder@@6B@ 0000000035204ff0     physarea.obj
 0002:000020e0       ??_7CPhysicalStub@@6B@     00000000352050e0     physarea.obj
 0002:000021d0       ??_7CPhysArea@@6B@         00000000352051d0     physarea.obj
 0002:000022d8       __real@be4ccccd            00000000352052d8     physarea.obj
 0002:000022e0       __real@4008000000000000    00000000352052e0     physarea.obj
 0002:000022e8       __real@bfd0000000000000    00000000352052e8     physarea.obj
 0002:000022f0       __real@4020000000000000    00000000352052f0     physarea.obj
 0002:000022f8       __real@3fe8000000000000    00000000352052f8     physarea.obj
 0002:00002300       __real@3e112e0be826d695    0000000035205300     physarea.obj
 0002:00002308       __real@be112e0be826d695    0000000035205308     physarea.obj
 0002:00002310       __real@4415af1d78b58c40    0000000035205310     physarea.obj
 0002:00002318       __real@c415af1d78b58c40    0000000035205318     physarea.obj
 0002:00002320       __real@3fc5555555555555    0000000035205320     physarea.obj
 0002:00002328       __real@0000000000000000    0000000035205328     physarea.obj
 0002:00002330       __mask@@NegDouble@         0000000035205330     physarea.obj
 0002:00002340       __real@4010000000000000    0000000035205340     physarea.obj
 0002:00002348       __real@3d4ccccd            0000000035205348     physarea.obj
 0002:0000234c       __real@ff7843b0            000000003520534c     physarea.obj
 0002:00002350       __real@7f7843b0            0000000035205350     physarea.obj
 0002:00002354       __real@3ffeb852            0000000035205354     physarea.obj
 0002:00002360       __real@e0ad78ec            0000000035205360     physicalentity.obj
 0002:00002364       __real@60ad78ec            0000000035205364     physicalentity.obj
 0002:00002370       ??_7CPhysicalEntity@@6B@   0000000035205370     physicalentity.obj
 0002:000025a8       ??_C@_05MHMEBBGO@scale?$AA@ 00000000352055a8     physicalentity.obj
 0002:000025b0       ??_C@_0BF@LALMAGNL@?5pos?3?5?$CF?41f?0?$CF?41f?0?$CF?41f?$AA@ 00000000352055b0     physicalentity.obj
 0002:000025d0       ??_C@_0FA@PBHKFAEH@?$CFs?3?5?$CI?$CF?450s?5?$EA?5?$CF?41f?0?$CF?41f?0?$CF?41f?$CJ?5Val@ 00000000352055d0     physicalentity.obj
 0002:00002620       ??_C@_0CI@IOBNLHFK@?$CIperhaps?5non?9uniform?5scaling?5was@ 0000000035205620     physicalentity.obj
 0002:00002648       ??_C@_07CEEBLDMK@BBox?$FL1?$FN?$AA@ 0000000035205648     physicalentity.obj
 0002:00002650       ??_C@_07CFIDNJPN@BBox?$FL0?$FN?$AA@ 0000000035205650     physicalentity.obj
 0002:00002658       ??_C@_0BE@NGINBJG@?5pt?3?5?$CF?41f?0?$CF?41f?0?$CF?41f?$AA@ 0000000035205658     physicalentity.obj
 0002:00002670       ??_C@_0DF@BCOOIFOK@?$CIperhaps?5non?9uniform?5scaling?5was@ 0000000035205670     physicalentity.obj
 0002:000026a8       ??_C@_07HAFFKDBK@density?$AA@ 00000000352056a8     physicalentity.obj
 0002:000026b0       __real@4cbebc20            00000000352056b0     physicalentity.obj
 0002:000026b4       __real@ccbebc20            00000000352056b4     physicalentity.obj
 0002:000026b8       __real@bf7ff972            00000000352056b8     physicalentity.obj
 0002:000026c0       ??_7CBoxGeom@@6B@          00000000352056c0     physicalentity.obj
 0002:000028b0       ??_7CSphereGeom@@6B@       00000000352058b0     physicalentity.obj
 0002:00002aa0       __real@3cf5c28f            0000000035205aa0     physicalentity.obj
 0002:00002aa8       ??_C@_0BM@NPMINFME@CPhysicalEntity?3AddGeometry?$AA@ 0000000035205aa8     physicalentity.obj
 0002:00002ac4       __real@41100000            0000000035205ac4     physicalentity.obj
 0002:00002ac8       __real@43480000            0000000035205ac8     physicalentity.obj
 0002:00002acc       __real@3ba3d70a            0000000035205acc     physicalentity.obj
 0002:00002ad0       __real@3b03126f            0000000035205ad0     physicalentity.obj
 0002:00002ad4       __real@d8635fa9            0000000035205ad4     physicalentity.obj
 0002:00002ad8       __real@58635fa9            0000000035205ad8     physicalentity.obj
 0002:00002adc       ??_C@_04GGBPDDBN@?$CF?41f?$AA@ 0000000035205adc     physicalentity.obj
 0002:00002ae8       ??_C@_09PHALKAAM@?$CF?41f?1?$CF?41f?$AA@ 0000000035205ae8     physicalentity.obj
 0002:00002af8       ??_C@_0BB@EIMABIKF@twist?3?5?$CF?41f?1?$CF?41f?$AA@ 0000000035205af8     physicalentity.obj
 0002:00002b10       ??_C@_0BA@MGOMOLHA@bend?3?5?$CF?41f?1?$CF?41f?$AA@ 0000000035205b10     physicalentity.obj
 0002:00002b20       ??_C@_0BA@KIPLJKAO@push?3?5?$CF?41f?1?$CF?41f?$AA@ 0000000035205b20     physicalentity.obj
 0002:00002b30       ??_C@_0BA@FIGEHIAC@pull?3?5?$CF?41f?1?$CF?41f?$AA@ 0000000035205b30     physicalentity.obj
 0002:00002b40       ??_C@_0BB@OCIOGPEL@shift?3?5?$CF?41f?1?$CF?41f?$AA@ 0000000035205b40     physicalentity.obj
 0002:00002b54       __real@beb15b57            0000000035205b54     physicalentity.obj
 0002:00002b58       __real@3df833fa            0000000035205b58     physicalentity.obj
 0002:00002b5c       __real@be99999a            0000000035205b5c     physicalentity.obj
 0002:00002b60       __real@bdd4d402            0000000035205b60     physicalentity.obj
 0002:00002b64       __real@3df836bf            0000000035205b64     physicalentity.obj
 0002:00002b68       __real@3c30efd3            0000000035205b68     physicalentity.obj
 0002:00002b6c       __real@bdcccccd            0000000035205b6c     physicalentity.obj
 0002:00002b70       __real@3d0de2ac            0000000035205b70     physicalentity.obj
 0002:00002b74       __real@3e315b57            0000000035205b74     physicalentity.obj
 0002:00002b78       __real@be315b57            0000000035205b78     physicalentity.obj
 0002:00002b7c       ??_C@_06GJCCMIGE@?$CF?42fkg?$AA@ 0000000035205b7c     physicalentity.obj
 0002:00002b84       __real@3f8ccccd            0000000035205b84     physicalentity.obj
 0002:00002b88       __real@be428f5f            0000000035205b88     physicalentity.obj
 0002:00002b90       ??_C@_0BJ@KINLGGMJ@Lattice?5tension?3?5?$CFf?5?$CI?$CFs?$CJ?$AA@ 0000000035205b90     physicalentity.obj
 0002:00002bac       ??_C@_04JFAPGDHH@bend?$AA@ 0000000035205bac     physicalentity.obj
 0002:00002bb4       ??_C@_05MOLGPPCG@twist?$AA@ 0000000035205bb4     physicalentity.obj
 0002:00002bbc       ??_C@_05CLOOKOFG@shift?$AA@ 0000000035205bbc     physicalentity.obj
 0002:00002bc4       ??_C@_04BEGLKOGM@pull?$AA@ 0000000035205bc4     physicalentity.obj
 0002:00002bcc       ??_C@_04GHHNIPCF@push?$AA@ 0000000035205bcc     physicalentity.obj
 0002:00002bd4       __real@48435000            0000000035205bd4     physicalentity.obj
 0002:00002bd8       __real@47c35000            0000000035205bd8     physicalentity.obj
 0002:00002bdc       __real@48c35000            0000000035205bdc     physicalentity.obj
 0002:00002be0       ??_C@_0CK@CECADMJN@CPhysicalEntity?3SetParams?$CIpe_par@ 0000000035205be0     physicalentity.obj
 0002:00002c10       ??_C@_0CL@MNMOENND@CPhysicalEntity?3?3SetParams?$CIpe_pa@ 0000000035205c10     physicalentity.obj
 0002:00002c40       ??_C@_0CJ@DICFJNIC@CPhysicalEntity?3SetParams?$CIpe_par@ 0000000035205c40     physicalentity.obj
 0002:00002c6c       ??_C@_06CPGPAJPB@hasDfm?$AA@ 0000000035205c6c     physicalentity.obj
 0002:00002c78       ??_C@_09BMMJDEMI@usedParts?$AA@ 0000000035205c78     physicalentity.obj
 0002:00002c88       ??_C@_0O@NOMKKJCH@dampingConstr?$AA@ 0000000035205c88     physicalentity.obj
 0002:00002c98       ??_C@_0M@ODBAFIDM@limitConstr?$AA@ 0000000035205c98     physicalentity.obj
 0002:00002ca4       ??_C@_05LDEILEND@axisx?$AA@ 0000000035205ca4     physicalentity.obj
 0002:00002cb0       ??_C@_08KGHNBEIB@szHelper?$AA@ 0000000035205cb0     physicalentity.obj
 0002:00002cc0       ??_C@_0L@GDBJIHOA@bBreakable?$AA@ 0000000035205cc0     physicalentity.obj
 0002:00002cd0       ??_C@_0P@DEBFNDAF@maxTorqueTwist?$AA@ 0000000035205cd0     physicalentity.obj
 0002:00002ce0       ??_C@_0O@DJBOCDGJ@maxTorqueBend?$AA@ 0000000035205ce0     physicalentity.obj
 0002:00002cf0       ??_C@_0O@MBJBNLLP@maxForceShift?$AA@ 0000000035205cf0     physicalentity.obj
 0002:00002d00       ??_C@_0N@LOFJHOOI@maxForcePull?$AA@ 0000000035205d00     physicalentity.obj
 0002:00002d10       ??_C@_0N@MNEPFPKB@maxForcePush?$AA@ 0000000035205d10     physicalentity.obj
 0002:00002d20       ??_C@_01EFFIKLCJ@n?$AA@    0000000035205d20     physicalentity.obj
 0002:00002d24       ??_C@_02BPBMPCEP@pt?$AA@   0000000035205d24     physicalentity.obj
 0002:00002d28       ??_C@_06IHFONFKC@ipart1?$AA@ 0000000035205d28     physicalentity.obj
 0002:00002d30       ??_C@_06JOEFOEOD@ipart0?$AA@ 0000000035205d30     physicalentity.obj
 0002:00002d38       ??_C@_02EGCJHIOB@id?$AA@   0000000035205d38     physicalentity.obj
 0002:00002d40       ??_C@_07FOFEHKBC@nJoints?$AA@ 0000000035205d40     physicalentity.obj
 0002:00002d48       ??_C@_09LGGKDIJE@hasJoints?$AA@ 0000000035205d48     physicalentity.obj
 0002:00002d60       ??_7IGeomManager@@6B@      0000000035205d60     physicalworld.obj
 0002:00002e18       ??_7IThreadTask@@6B@       0000000035205e18     physicalworld.obj
 0002:00002e38       ??_7SThreadTaskInfo@@6B@   0000000035205e38     physicalworld.obj
 0002:00002e38       ??_7CMultiThreadRefCount@@6B@ 0000000035205e38     physicalworld.obj
 0002:00002e40       ??_7IBreakableGrid2d@@6B@  0000000035205e40     geoman.obj
 0002:00002e40       ??_7ITetrLattice@@6B@      0000000035205e40     tetrlattice.obj
 0002:00002e40       ??_7IPhysicalEntityIt@@6B@ 0000000035205e40     physicalworld.obj
 0002:00002e80       ??_7IPhysicalWorld@@6B@    0000000035205e80     physicalworld.obj
 0002:00003150       ??_7IPhysUtils@@6B@        0000000035206150     physicalworld.obj
 0002:00003150       ??_7ICryUnknown@@6B@       0000000035206150     CryPhysics.obj
 0002:00003170       __real@3fe5555555555555    0000000035206170     physicalworld.obj
 0002:00003178       __real@3ef0001000100010    0000000035206178     physicalworld.obj
 0002:00003180       __real@477fff00            0000000035206180     physicalworld.obj
 0002:00003190       ??_C@_0EI@EOAKOGBE@Error?3?5?$CKmajor?$CK?5problem?5?9?5trying?5@ 0000000035206190     physicalworld.obj
 0002:000031d8       ??_C@_06LNKFDEGN@noname?$AA@ 00000000352061d8     physicalworld.obj
 0002:000031e0       __real@38000000            00000000352061e0     physicalworld.obj
 0002:000031f0       ??_7CGeomManager@@6B@      00000000352061f0     physicalworld.obj
 0002:000032b0       ??_7SPhysTask@@6B@         00000000352062b0     physicalworld.obj
 0002:000032d0       ??_7CPhysicalEntityIt@CPhysicalWorld@@6B@ 00000000352062d0     physicalworld.obj
 0002:00003308       __real@37d1b717            0000000035206308     physicalworld.obj
 0002:00003310       ??_C@_08KIKMFGJF@Physics0?$AA@ 0000000035206310     physicalworld.obj
 0002:00003320       ??_C@_08LBLHGHNE@Physics1?$AA@ 0000000035206320     physicalworld.obj
 0002:00003330       ??_C@_08JKJKDEBH@Physics2?$AA@ 0000000035206330     physicalworld.obj
 0002:00003340       ??_C@_08IDIBAFFG@Physics3?$AA@ 0000000035206340     physicalworld.obj
 0002:00003350       ??_C@_0BE@EHHKEKKG@?$CFd?5active?5object?$CIs?$CJ?$AA@ 0000000035206350     physicalworld.obj
 0002:00003370       ??_C@_0EF@JNHCCPCP@?$CFs?5?$EA?5?$CF7?42f?0?$CF7?42f?0?$CF7?42f?0?5mass?5?$CF?42@ 0000000035206370     physicalworld.obj
 0002:000033b8       __real@42700000            00000000352063b8     physicalworld.obj
 0002:000033bc       __real@42f00000            00000000352063bc     physicalworld.obj
 0002:000033c8       ??_C@_0BE@LFJFAKMB@Static?5TriMesh?5Data?$AA@ 00000000352063c8     physicalworld.obj
 0002:000033e0       ??_C@_0BE@OKHLKODM@external?5geometries?$AA@ 00000000352063e0     physicalworld.obj
 0002:000033f8       ??_C@_0L@NEGCPNMO@geometries?$AA@ 00000000352063f8     physicalworld.obj
 0002:00003404       ??_C@_05EPHILNBP@areas?$AA@ 0000000035206404     physicalworld.obj
 0002:00003410       ??_C@_0BA@CPFEOAFC@hidden?5entities?$AA@ 0000000035206410     physicalworld.obj
 0002:00003420       ??_C@_08PNMNOKOB@entities?$AA@ 0000000035206420     physicalworld.obj
 0002:00003430       ??_C@_0N@OILCNOIE@placeholders?$AA@ 0000000035206430     physicalworld.obj
 0002:00003440       ??_C@_0N@KOGLEBGK@world?5queues?$AA@ 0000000035206440     physicalworld.obj
 0002:00003450       ??_C@_0BB@CJHEBAIA@world?5structures?$AA@ 0000000035206450     physicalworld.obj
 0002:00003468       ??_C@_0BE@KJDJFMJA@STL?5Allocator?5Waste?$AA@ 0000000035206468     physicalworld.obj
 0002:00003480       ??_C@_0BA@NFPONAAD@static?5entities?$AA@ 0000000035206480     physicalworld.obj
 0002:00003490       ??_C@_0BC@CKIFBHJ@physical?5entities?$AA@ 0000000035206490     physicalworld.obj
 0002:000034a8       ??_C@_0BA@DBEKKOOB@living?5entities?$AA@ 00000000352064a8     physicalworld.obj
 0002:000034b8       ??_C@_0BC@FMIIKKPA@detached?5entities?$AA@ 00000000352064b8     physicalworld.obj
 0002:000034d0       ??_C@_08CFJOODNG@triggers?$AA@ 00000000352064d0     physicalworld.obj
 0002:000034e0       ??_C@_0BB@PLIHMJIB@deleted?5entities?$AA@ 00000000352064e0     physicalworld.obj
 0002:000034f8       ??_C@_0CG@LGHEGFDG@Error?3?5queued?5RWI?5hits?5pool?5corr@ 00000000352064f8     physicalworld.obj
 0002:00003520       ??_C@_0BI@BBMELPMJ@PhysEventHandler?$CI?$CFd?0?$CFd?$CJ?$AA@ 0000000035206520     physicalworld.obj
 0002:00003538       ??_C@_0CB@IEBMEMCB@CPhysicalWorld?3?3PumpLoggedEvents@ 0000000035206538     physicalworld.obj
 0002:00003560       ??_C@_0BB@EBHBFJFK@rb_primintersect?$AA@ 0000000035206560     physicalworld.obj
 0002:00003578       ??_C@_0N@DMLBCAGA@featherstone?$AA@ 0000000035206578     physicalworld.obj
 0002:00003588       ??_C@_0N@MGKFCACL@rope?5?5?5?5?5?5?5?5?$AA@ 0000000035206588     physicalworld.obj
 0002:00003598       ??_C@_0N@EIICPGEA@cloth?5?5?5?5?5?5?5?$AA@ 0000000035206598     physicalworld.obj
 0002:000035a8       ??_C@_0N@PAEACHLK@solver?5?5?5?5?5?5?$AA@ 00000000352065a8     physicalworld.obj
 0002:000035b8       ??_C@_0BB@GEEHMKJE@rb_geomintersect?$AA@ 00000000352065b8     physicalworld.obj
 0002:000035d0       ??_C@_0BB@DHBNBKPP@World?5step?5total?$AA@ 00000000352065d0     physicalworld.obj
 0002:000035e8       ??_C@_0BA@NILGEFEO@Queued?5requests?$AA@ 00000000352065e8     physicalworld.obj
 0002:000035f8       ??_C@_0P@COOONLDP@Entities?5total?$AA@ 00000000352065f8     physicalworld.obj
 0002:00003608       ??_C@_0BC@GKAHDKOK@Kinematic?5objects?$AA@ 0000000035206608     physicalworld.obj
 0002:00003620       ??_C@_0BE@LMPPICDB@Character?5skeletons?$AA@ 0000000035206620     physicalworld.obj
 0002:00003638       ??_C@_0BC@DHLIMEHH@Ropes?5?$CIcharacter?$CJ?$AA@ 0000000035206638     physicalworld.obj
 0002:00003650       ??_C@_0BD@KBBCJMME@Ropes?5?$CIvegetation?$CJ?$AA@ 0000000035206650     physicalworld.obj
 0002:00003664       ??_C@_05GKKHKKE@Cloth?$AA@ 0000000035206664     physicalworld.obj
 0002:00003670       ??_C@_0BD@HBBFNCLM@Ropes?5?$CIstandalone?$CJ?$AA@ 0000000035206670     physicalworld.obj
 0002:00003688       ??_C@_08KLCKKNPF@Ragdolls?$AA@ 0000000035206688     physicalworld.obj
 0002:00003698       ??_C@_0BH@GBMNCFJC@Physicalized?5particles?$AA@ 0000000035206698     physicalworld.obj
 0002:000036b0       ??_C@_06DCPPBEOJ@Actors?$AA@ 00000000352066b0     physicalworld.obj
 0002:000036b8       ??_C@_0BB@INJEDGPL@Wheeled?5vehicles?$AA@ 00000000352066b8     physicalworld.obj
 0002:000036d0       ??_C@_0N@FFLNJJI@Rigid?5bodies?$AA@ 00000000352066d0     physicalworld.obj
 0002:000036e0       ??_7CPhysicalWorld@@6BCGeomManager@@@ 00000000352066e0     physicalworld.obj
 0002:000037a0       ??_7CPhysicalWorld@@6BIPhysicalWorld@@@ 00000000352067a0     physicalworld.obj
 0002:00003a80       ??_7CPhysicalWorld@@6BIPhysUtils@@@ 0000000035206a80     physicalworld.obj
 0002:00003aa0       __real@3b800000            0000000035206aa0     physicalworld.obj
 0002:00003ab0       ??_C@_0FJ@OGBDLIAD@GetEntitiesInBox?3?5too?5many?5cells@ 0000000035206ab0     physicalworld.obj
 0002:00003b0c       ??_C@_04IBBNLEM@Game?$AA@  0000000035206b0c     physicalworld.obj
 0002:00003b18       ??_C@_0BM@NPIOPJJB@GetEntitiesAround?$CIExternal?$CJ?$AA@ 0000000035206b18     physicalworld.obj
 0002:00003b38       ??_C@_0BL@PFOGMOID@GetEntitiesAround?$CIPhysics?$CJ?$AA@ 0000000035206b38     physicalworld.obj
 0002:00003b58       ??_C@_0CC@FMONOPEM@CPhysicalWorld?3?3GetEntitiesAroun@ 0000000035206b58     physicalworld.obj
 0002:00003b7c       __real@4e6e6b28            0000000035206b7c     physicalworld.obj
 0002:00003b80       ??_C@_0CG@DAIPOGMA@CPhysicalWorld?3?3CollideEntityWit@ 0000000035206b80     physicalworld.obj
 0002:00003ba8       ??_C@_0CL@DKEANCLN@CPhysicalWorld?3?3CollideEntityWit@ 0000000035206ba8     physicalworld.obj
 0002:00003bd4       ??_C@_03GEPAOBPJ@com?$AA@  0000000035206bd4     physicalworld.obj
 0002:00003bd8       ??_C@_08PGIAAJBG@simclass?$AA@ 0000000035206bd8     physicalworld.obj
 0002:00003be8       ??_C@_0L@LDLJOCKM@entity_ptr?$AA@ 0000000035206be8     physicalworld.obj
 0002:00003bf8       ??_C@_0BD@INDOKC@Physical?5Grid?5Pool?$AA@ 0000000035206bf8     physicalworld.obj
 0002:00003c10       ??_C@_0EI@FEBOPGDO@Error?3?5too?5many?5entity?5grid?5thun@ 0000000035206c10     physicalworld.obj
 0002:00003c58       ??_C@_0DD@GLNFKCFH@Error?3?5?$CFs?5?$EA?5?$CF?41f?0?$CF?41f?0?$CF?41f?5is?5to@ 0000000035206c58     physicalworld.obj
 0002:00003c8c       ??_C@_06GOJKNBFM@entity?$AA@ 0000000035206c8c     physicalworld.obj
 0002:00003c94       __real@43800000            0000000035206c94     physicalworld.obj
 0002:00003c98       __real@c3480000            0000000035206c98     physicalworld.obj
 0002:00003c9c       __real@bf4ccccd            0000000035206c9c     physicalworld.obj
 0002:00003ca0       __real@34000000            0000000035206ca0     physicalworld.obj
 0002:00003ca8       ??_C@_0CC@HNDNKDHE@CPhysicalWorld?3?3SimulateExplosio@ 0000000035206ca8     physicalworld.obj
 0002:00003cd0       __real@4202a05f20000000    0000000035206cd0     physicalworld.obj
 0002:00003cd8       ??_C@_0CL@EIIFGMOL@CPhysicalWorld?3?3PrimitiveWorldIn@ 0000000035206cd8     physicalworld.obj
 0002:00003d08       ??_C@_0BF@HMDKKHBB@CreatePhysicalEntity?$AA@ 0000000035206d08     physicalworld.obj
 0002:00003d20       ??_C@_0CF@MPBHKPK@CPhysicalWorld?3?3CreatePhysicalEn@ 0000000035206d20     physicalworld.obj
 0002:00003d48       ??_C@_0CG@NDJJNCNB@CPhysicalWorld?3?3DestroyPhysicalE@ 0000000035206d48     physicalworld.obj
 0002:00003d70       ??_C@_0BC@NNEDADDI@D?3?2worldgeoms?4txt?$AA@ 0000000035206d70     physicalworld.obj
 0002:00003d88       ??_C@_0BB@PHBCIJJB@D?3?2worldents?4txt?$AA@ 0000000035206d88     physicalworld.obj
 0002:00003da0       ??_C@_0BE@MNKPLEKN@PhysicsWorkerThread?$AA@ 0000000035206da0     physicalworld.obj
 0002:00003db8       ??_C@_0BJ@KLNIBABK@CPhysicalWorld?3?3TimeStep?$AA@ 0000000035206db8     physicalworld.obj
 0002:00003dd8       ??_C@_0P@JAKLJLMO@RB?5thread?5data?$AA@ 0000000035206dd8     rigidbody.obj
 0002:00003de8       __real@3f8020c5            0000000035206de8     rigidbody.obj
 0002:00003dec       ??_C@_05EBOPLLCF@LCPMC?$AA@ 0000000035206dec     rigidbody.obj
 0002:00003df8       ??_C@_0BH@JPFBLAOJ@Physics?5Contact?5Solver?$AA@ 0000000035206df8     rigidbody.obj
 0002:00003e10       __real@4034000000000000    0000000035206e10     rigidbody.obj
 0002:00003e18       ??_C@_0N@CNCBJKKN@LCPCG?9unproj?$AA@ 0000000035206e18     rigidbody.obj
 0002:00003e28       __real@3f50624dd2f1a9fc    0000000035206e28     rigidbody.obj
 0002:00003e30       __real@4049000000000000    0000000035206e30     rigidbody.obj
 0002:00003e38       ??_C@_05CPBNFDCL@LCPCG?$AA@ 0000000035206e38     rigidbody.obj
 0002:00003e40       __real@80000000            0000000035206e40     rigidbody.obj
 0002:00003e48       __real@bf8eb851e0000000    0000000035206e48     rigidbody.obj
 0002:00003e50       __real@bf70624de0000000    0000000035206e50     rigidbody.obj
 0002:00003e58       __real@bd4ccccd            0000000035206e58     rigidbody.obj
 0002:00003e60       __real@407f400000000000    0000000035206e60     rigidbody.obj
 0002:00003e68       __real@39b4484bfeebc2a0    0000000035206e68     rigidbody.obj
 0002:00003e70       ??_C@_05LNAIGO@PreCG?$AA@  0000000035206e70     rigidbody.obj
 0002:00003e78       ??_C@_0BE@OAMBIDAL@InvokeContactSolver?$AA@ 0000000035206e78     rigidbody.obj
 0002:00003e8c       ??_C@_06HPGEIPLA@?$DMnull?$DO?$AA@ 0000000035206e8c     rigidentity.obj
 0002:00003e98       ??_C@_07KAALEJHI@?$DMlocal?$DO?$AA@ 0000000035206e98     rigidentity.obj
 0002:00003ea8       ??_C@_02DKCKIIND@?$CFs?$AA@ 0000000035206ea8     rigidentity.obj
 0002:00003eac       __real@c3000000            0000000035206eac     rigidentity.obj
 0002:00003eb0       __real@c3800000            0000000035206eb0     rigidentity.obj
 0002:00003eb4       __real@43000000            0000000035206eb4     rigidentity.obj
 0002:00003eb8       __real@44800000            0000000035206eb8     rigidentity.obj
 0002:00003ec0       ??_C@_0CI@IOKCCNHB@Deleting?5Reference?5Counted?5Objec@ 0000000035206ec0     rigidentity.obj
 0002:00003ef0       ??_7CRigidEntity@@6B@      0000000035206ef0     rigidentity.obj
 0002:00004158       __real@44cccb33            0000000035207158     rigidentity.obj
 0002:0000415c       __real@4423d5c3            000000003520715c     rigidentity.obj
 0002:00004160       ??_C@_0P@BDPDOPPG@sequenceNumber?$AA@ 0000000035207160     rigidentity.obj
 0002:00004170       ??_C@_06JPLOHAIH@angvel?$AA@ 0000000035207170     rigidentity.obj
 0002:00004178       ??_C@_03BHFFHIBL@rot?$AA@  0000000035207178     rigidentity.obj
 0002:0000417c       __real@3cb851ec            000000003520717c     rigidentity.obj
 0002:00004180       __real@3f7ff972            0000000035207180     rigidentity.obj
 0002:00004184       __real@bf99999a            0000000035207184     rigidentity.obj
 0002:00004188       __real@41f00000            0000000035207188     rigidentity.obj
 0002:0000418c       __real@3eaaaaab            000000003520718c     rigidentity.obj
 0002:00004190       __real@c1200000            0000000035207190     rigidentity.obj
 0002:00004194       __real@3f80a3d7            0000000035207194     rigidentity.obj
 0002:00004198       __real@43960000            0000000035207198     rigidentity.obj
 0002:0000419c       __real@3f70a3d7            000000003520719c     rigidentity.obj
 0002:000041a0       __real@bf59999a            00000000352071a0     rigidentity.obj
 0002:000041a4       __real@3fd9999a            00000000352071a4     rigidentity.obj
 0002:000041a8       __real@3e19999a            00000000352071a8     rigidentity.obj
 0002:000041b0       ??_C@_0BP@EANKIJJH@CRigidEntity?3?3RegisterContacts?$AA@ 00000000352071b0     rigidentity.obj
 0002:000041d0       ??_C@_0O@KJLDCHNC@maxBendTorque?$AA@ 00000000352071d0     rigidentity.obj
 0002:000041e0       ??_C@_0N@PCBEGNKJ@breakableAng?$AA@ 00000000352071e0     rigidentity.obj
 0002:000041f0       ??_C@_0N@NHHOIIFK@maxPullForce?$AA@ 00000000352071f0     rigidentity.obj
 0002:00004200       ??_C@_0N@NEPDBILI@breakableLin?$AA@ 0000000035207200     rigidentity.obj
 0002:00004210       ??_C@_06KGHINEPG@radius?$AA@ 0000000035207210     rigidentity.obj
 0002:00004218       ??_C@_07IANOJGAO@damping?$AA@ 0000000035207218     rigidentity.obj
 0002:00004220       ??_C@_05GECEPKB@flags?$AA@ 0000000035207220     rigidentity.obj
 0002:00004228       ??_C@_06CNGEOGNK@yzlim1?$AA@ 0000000035207228     rigidentity.obj
 0002:00004230       ??_C@_06DEHPNHJL@yzlim0?$AA@ 0000000035207230     rigidentity.obj
 0002:00004238       ??_C@_05DHNHFHMF@yzlim?$AA@ 0000000035207238     rigidentity.obj
 0002:00004240       ??_C@_05DFPCKMPE@xlim1?$AA@ 0000000035207240     rigidentity.obj
 0002:00004248       ??_C@_05CMOJJNLF@xlim0?$AA@ 0000000035207248     rigidentity.obj
 0002:00004250       ??_C@_04BGNKAOBC@xlim?$AA@ 0000000035207250     rigidentity.obj
 0002:00004258       ??_C@_07LBPEBLNH@qframe1?$AA@ 0000000035207258     rigidentity.obj
 0002:00004260       ??_C@_07NKFCNLOK@qf1used?$AA@ 0000000035207260     rigidentity.obj
 0002:00004268       ??_C@_07KIOPCKJG@qframe0?$AA@ 0000000035207268     rigidentity.obj
 0002:00004270       ??_C@_07BBAOAIEP@qf0used?$AA@ 0000000035207270     rigidentity.obj
 0002:00004278       ??_C@_07JOFJMAFF@partid1?$AA@ 0000000035207278     rigidentity.obj
 0002:00004280       ??_C@_07IHECPBBE@partid0?$AA@ 0000000035207280     rigidentity.obj
 0002:00004288       ??_C@_03CACBEHEB@pt1?$AA@  0000000035207288     rigidentity.obj
 0002:0000428c       ??_C@_03DJDKHGAA@pt0?$AA@  000000003520728c     rigidentity.obj
 0002:00004290       ??_C@_0L@HOHHMJMM@constraint?$AA@ 0000000035207290     rigidentity.obj
 0002:0000429c       ??_C@_05IOMEMJEC@count?$AA@ 000000003520729c     rigidentity.obj
 0002:000042a8       ??_C@_0M@JGLONDGH@constraints?$AA@ 00000000352072a8     rigidentity.obj
 0002:000042c0       ??_C@_0EL@PLDAGNFJ@Error?3?5Rigid?5Body?5?$CI?$EA?$CF?41f?0?$CF?41f?0?$CF?4@ 00000000352072c0     rigidentity.obj
 0002:0000430c       __real@bf7f7cee            000000003520730c     rigidentity.obj
 0002:00004310       __real@3c4ccccd            0000000035207310     rigidentity.obj
 0002:00004320       ??_C@_0EN@EHOJENEE@CRigidEntity?3?3AddGeometry?3?5?$CI?$CFs?5a@ 0000000035207320     rigidentity.obj
 0002:00004370       ??_C@_0CE@MCBDAAIP@CRigidEntity?3Action?$CIaction_impul@ 0000000035207370     rigidentity.obj
 0002:00004394       __real@3d75c28f            0000000035207394     rigidentity.obj
 0002:00004398       ??_C@_0CD@BGBGOAEC@CRigidEntity?3?3RegisterContactPoi@ 0000000035207398     rigidentity.obj
 0002:000043bc       __real@40600000            00000000352073bc     rigidentity.obj
 0002:000043c0       ??_C@_0BP@ODPDJPC@CRigidEntity?3?3DelayedIntersect?$AA@ 00000000352073c0     rigidentity.obj
 0002:000043e0       __real@3a200140            00000000352073e0     rigidentity.obj
 0002:000043e4       __real@3ac80190            00000000352073e4     rigidentity.obj
 0002:000043e8       ??_C@_07OHHAEMPA@seq?3?5?$CFf?$AA@ 00000000352073e8     rigidentity.obj
 0002:000043f0       ??_C@_07NFEGCOHC@seq?3?5?$CFd?$AA@ 00000000352073f0     rigidentity.obj
 0002:000043f8       __real@ba83126f            00000000352073f8     rigidentity.obj
 0002:000043fc       __real@3f35c28f            00000000352073fc     rigidentity.obj
 0002:00004400       __real@3d7a35dd            0000000035207400     rigidentity.obj
 0002:00004404       __real@3e428f5c            0000000035207404     rigidentity.obj
 0002:00004408       ??_C@_0BD@GCCCEIEI@CRigidEntity?3?3Step?$AA@ 0000000035207408     rigidentity.obj
 0002:00004430       ??_7CRopeEntity@@6B@       0000000035207430     ropeentity.obj
 0002:00004668       __real@6aa56fa6            0000000035207668     ropeentity.obj
 0002:0000466c       ??_C@_03HCMCBFLP@_?$CFd?$AA@ 000000003520766c     ropeentity.obj
 0002:00004670       __real@26901d7d            0000000035207670     ropeentity.obj
 0002:00004674       __real@bba3d70a            0000000035207674     ropeentity.obj
 0002:00004678       ??_C@_0P@BGLENKAJ@Rope?5solver?5MC?$AA@ 0000000035207678     ropeentity.obj
 0002:00004688       ??_C@_0P@HIEGDCAH@Rope?5solver?5CG?$AA@ 0000000035207688     ropeentity.obj
 0002:00004698       __real@3f59999a            0000000035207698     ropeentity.obj
 0002:0000469c       __real@3f100000            000000003520769c     ropeentity.obj
 0002:000046a0       __real@bf7eb852            00000000352076a0     ropeentity.obj
 0002:000046a4       ??_C@_04DMCMFBAM@tied?$AA@ 00000000352076a4     ropeentity.obj
 0002:000046ac       ??_C@_04OHHBHOGB@link?$AA@ 00000000352076ac     ropeentity.obj
 0002:000046b8       ??_C@_08BLGKBCOE@saveties?$AA@ 00000000352076b8     ropeentity.obj
 0002:000046c8       ??_C@_08JFDIBHCE@pt_tied1?$AA@ 00000000352076c8     ropeentity.obj
 0002:000046d8       ??_C@_08IMCDCGGF@pt_tied0?$AA@ 00000000352076d8     ropeentity.obj
 0002:000046e4       ??_C@_05FDOEMPCF@Verts?$AA@ 00000000352076e4     ropeentity.obj
 0002:000046ec       ??_C@_04OFJFANPM@nvtx?$AA@ 00000000352076ec     ropeentity.obj
 0002:000046f4       ??_C@_04DBMENFI@Segs?$AA@  00000000352076f4     ropeentity.obj
 0002:00004700       ??_C@_07DDKGOFMH@pos_end?$AA@ 0000000035207700     ropeentity.obj
 0002:00004708       ??_C@_09IAPMPKID@pos_start?$AA@ 0000000035207708     ropeentity.obj
 0002:00004718       ??_C@_08EAMLKELC@strained?$AA@ 0000000035207718     ropeentity.obj
 0002:00004724       ??_C@_05IHMDFKMI@nsegs?$AA@ 0000000035207724     ropeentity.obj
 0002:0000472c       __real@322bcc76            000000003520772c     ropeentity.obj
 0002:00004730       __real@3ea00000            0000000035207730     ropeentity.obj
 0002:00004734       __real@3ec00000            0000000035207734     ropeentity.obj
 0002:00004738       __real@3f7ae148            0000000035207738     ropeentity.obj
 0002:0000473c       __real@3d23d70b            000000003520773c     ropeentity.obj
 0002:00004740       __real@3db851ec            0000000035207740     ropeentity.obj
 0002:00004748       __real@3f1cd5f99c38b04b    0000000035207748     ropeentity.obj
 0002:00004750       __real@3fa66666            0000000035207750     ropeentity.obj
 0002:00004754       __real@3f7860ab            0000000035207754     ropeentity.obj
 0002:00004758       ??_C@_0P@EFOJKOHM@Rope?5collision?$AA@ 0000000035207758     ropeentity.obj
 0002:00004768       __real@3da3d70a            0000000035207768     ropeentity.obj
 0002:00004770       ??_C@_0BC@KAOKIHJG@CRopeEntity?3?3Step?$AA@ 0000000035207770     ropeentity.obj
 0002:00004790       ??_7CSoftEntity@@6B@       0000000035207790     softentity.obj
 0002:000049c8       ??_C@_0CD@HHJJGFJC@CSoftEntity?3Action?$CIaction_impuls@ 00000000352079c8     softentity.obj
 0002:000049ec       ??_C@_03CEPBOMNB@vtx?$AA@  00000000352079ec     softentity.obj
 0002:000049f0       ??_C@_07OOCOMFL@updated?$AA@ 00000000352079f0     softentity.obj
 0002:000049f8       ??_C@_0BC@LKGJNKHC@CSoftEntity?3?3Step?$AA@ 00000000352079f8     softentity.obj
 0002:00004a20       ??_7CHeightfieldBV@@6B@    0000000035207a20     waterman.obj
 0002:00004b00       ??_7CHeightfield@@6B@      0000000035207b00     waterman.obj
 0002:00004d00       __real@bf8020c5            0000000035207d00     waterman.obj
 0002:00004d04       __real@3fc147ae            0000000035207d04     waterman.obj
 0002:00004d08       __real@bf028f5c            0000000035207d08     waterman.obj
 0002:00004d18       __real@4023193d66ed2bfb    0000000035207d18     wheeledvehicleentity.obj
 0002:00004d20       __real@44ffe000            0000000035207d20     wheeledvehicleentity.obj
 0002:00004d24       __real@4223d1ec            0000000035207d24     wheeledvehicleentity.obj
 0002:00004d28       __real@3a001002            0000000035207d28     wheeledvehicleentity.obj
 0002:00004d2c       __real@3cc80640            0000000035207d2c     wheeledvehicleentity.obj
 0002:00004d30       ??_C@_07IODEONID@curGear?$AA@ 0000000035207d30     wheeledvehicleentity.obj
 0002:00004d38       ??_C@_09DGHJKKCO@handbrake?$AA@ 0000000035207d38     wheeledvehicleentity.obj
 0002:00004d48       ??_C@_07OAMHNPGL@wengine?$AA@ 0000000035207d48     wheeledvehicleentity.obj
 0002:00004d50       ??_C@_05JADEHCLC@steer?$AA@ 0000000035207d50     wheeledvehicleentity.obj
 0002:00004d58       ??_C@_05CANEEOEI@pedal?$AA@ 0000000035207d58     wheeledvehicleentity.obj
 0002:00004d60       __real@3fbacee9f37bebd5    0000000035207d60     wheeledvehicleentity.obj
 0002:00004d68       __real@c01921fb54442d18    0000000035207d68     wheeledvehicleentity.obj
 0002:00004d70       ??_7CWheeledVehicleEntity@@6B@ 0000000035207d70     wheeledvehicleentity.obj
 0002:00004fe0       ??_C@_0EF@EDDEFNIG@CWheeledVehicleEntity?3?3AddGeomet@ 0000000035207fe0     wheeledvehicleentity.obj
 0002:00005028       __real@40e00000            0000000035208028     wheeledvehicleentity.obj
 0002:0000502c       __real@bc23d70a            000000003520802c     wheeledvehicleentity.obj
 0002:00005030       ??_C@_0CP@CDDJNAEK@CWheeledVehicleEntity?3?3CheckAddi@ 0000000035208030     wheeledvehicleentity.obj
 0002:00005060       __real@33d6bf95            0000000035208060     boolean2d.obj
 0002:00005064       __real@36a7c5ac            0000000035208064     boolean2d.obj
 0002:00005070       ??_7bop_meshupdate_thunk@@6B@ 0000000035208070     boolean3d.obj
 0002:00005078       ??_7bop_meshupdate@@6B@    0000000035208078     boolean3d.obj
 0002:00005080       __real@3b449ba6            0000000035208080     boolean3d.obj
 0002:00005084       __real@3a03126f            0000000035208084     boolean3d.obj
 0002:00005088       __real@3f7fbe77            0000000035208088     boolean3d.obj
 0002:00005090       ??_C@_0BD@IANNIDHM@CTriMesh?3?3Subtract?$AA@ 0000000035208090     boolean3d.obj
 0002:000050a8       __real@bff0000000000000    00000000352080a8     matrixnm.obj
 0002:000050b0       __real@bb03126f            00000000352080b0     qhull.obj
 0002:000050b4       __real@fcf0bdc2            00000000352080b4     qhull.obj
 0002:000050c8       __real@bfa999999999999a    00000000352080c8     utils.obj
 0002:000050d0       __real@bfb5555555555555    00000000352080d0     utils.obj
 0002:000050d8       __real@bfc5555555555555    00000000352080d8     utils.obj
 0002:000050e0       __real@bf91111111111111    00000000352080e0     utils.obj
 0002:000050e8       __real@3fa999999999999a    00000000352080e8     utils.obj
 0002:000050f0       __real@3fb5555555555555    00000000352080f0     utils.obj
 0002:000050f8       __real@3fa5555555555555    00000000352080f8     utils.obj
 0002:00005100       __real@3f91111111111111    0000000035208100     utils.obj
 0002:00005108       ??_C@_0BB@KMIBLBAG@ReadPacked?5i?$DN?$DN?$CFi?$AA@ 0000000035208108     utils.obj
 0002:0000511c       __real@3b000000            000000003520811c     utils.obj
 0002:00005120       __real@45000000            0000000035208120     utils.obj
 0002:00005128       __real@3bc79ca100000000    0000000035208128     utils.obj
 0002:00005130       __real@37800080            0000000035208130     utils.obj
 0002:00005138       __real@3fee666660000000    0000000035208138     utils.obj
 0002:00005140       __real@41800000            0000000035208140     utils.obj
 0002:00005148       __real@3fb45f306dc9c883    0000000035208148     utils.obj
 0002:00005150       __real@3fd3333333333333    0000000035208150     utils.obj
 0002:00005158       __real@3fe6666666666666    0000000035208158     utils.obj
 0002:00005160       __real@3ee4f8b588e368f1    0000000035208160     utils.obj
 0002:00005168       ??_C@_0DC@MJBDGDCG@Unsupported?5polygon?5size?5for?5Occ@ 0000000035208168     utils.obj
 0002:0000519c       __real@be860a92            000000003520819c     utils.obj
 0002:000051a0       __real@3f09222d989f5e57    00000000352081a0     utils.obj
 0002:000051a8       __real@3c800000            00000000352081a8     aabbtree.obj
 0002:000051b0       ??_C@_0L@PDPAOLJI@AABB?5trees?$AA@ 00000000352081b0     aabbtree.obj
 0002:000051bc       __real@42fe0000            00000000352081bc     aabbtree.obj
 0002:000051c0       __real@42800000            00000000352081c0     aabbtree.obj
 0002:000051c4       __real@c9742400            00000000352081c4     aabbtree.obj
 0002:000051d8       __real@3eb0c6f7a0000000    00000000352081d8     capsulegeom.obj
 0002:000051e0       __real@be960418            00000000352081e0     capsulegeom.obj
 0002:000051e4       __real@3f34fdf4            00000000352081e4     capsulegeom.obj
 0002:000051e8       __real@3f2aaaab            00000000352081e8     capsulegeom.obj
 0002:000051ec       __real@40860a92            00000000352081ec     capsulegeom.obj
 0002:00005200       __real@3ff921fb54442d18    0000000035208200     cylindergeom.obj
 0002:00005208       __real@3faaaaab            0000000035208208     cylindergeom.obj
 0002:0000520c       __real@3e000000            000000003520820c     cylindergeom.obj
 0002:00005210       __real@beaaaaab            0000000035208210     cylindergeom.obj
 0002:00005230       ??_7CVoxelBV@@6B@          0000000035208230     geoman.obj
 0002:00005308       ??_7CBreakableGrid2d@@6B@  0000000035208308     geoman.obj
 0002:00005340       ??_C@_0BA@JHFFHIMH@brekable2d?5grid?$AA@ 0000000035208340     geoman.obj
 0002:00005350       ??_7CMemStream@@6B@        0000000035208350     geoman.obj
 0002:00005370       ??_7CVoxelGeom@@6B@        0000000035208370     geoman.obj
 0002:00005588       __real@3f60624dd2f1a9fc    0000000035208588     heightfieldgeom.obj
 0002:00005590       __real@3f1a36e2e0000000    0000000035208590     heightfieldgeom.obj
 0002:00005598       __real@3fe6a09e667f3bcd    0000000035208598     heightfieldgeom.obj
 0002:000055a8       __real@2f52f8ac174d6123    00000000352085a8     intersectionchecks.obj
 0002:000055b0       __real@3feff7ced916872b    00000000352085b0     intersectionchecks.obj
 0002:000055b8       __real@3e2aaaab            00000000352085b8     intersectionchecks.obj
 0002:000055bc       __real@3d17b426            00000000352085bc     intersectionchecks.obj
 0002:000055c0       __real@3fef5c2900000000    00000000352085c0     intersectionchecks.obj
 0002:000055c8       __real@c000000000000000    00000000352085c8     intersectionchecks.obj
 0002:000055d0       __real@bf3504f3            00000000352085d0     intersectionchecks.obj
 0002:000055d4       __real@3f3504f3            00000000352085d4     intersectionchecks.obj
 0002:000055d8       ??_C@_0BB@PKNEGLNF@RB_PrimIntersect?$AA@ 00000000352085d8     jobq.obj
 0002:000055f0       ??_C@_0N@IPMPGLJF@Featherstone?$AA@ 00000000352085f0     jobq.obj
 0002:00005600       ??_C@_04FEDAIEKO@Rope?$AA@ 0000000035208600     jobq.obj
 0002:00005608       ??_C@_09HHOKDCAB@RB_Solver?$AA@ 0000000035208608     jobq.obj
 0002:00005618       ??_C@_0BB@NPOCPIBL@RB_GeomIntersect?$AA@ 0000000035208618     jobq.obj
 0002:00005640       __real@bfffd70a40000000    0000000035208640     linunprojectionchecks.obj
 0002:00005648       __real@c007eb8520000000    0000000035208648     linunprojectionchecks.obj
 0002:00005650       __real@3fa99999a0000000    0000000035208650     linunprojectionchecks.obj
 0002:00005658       __real@3fefef9db22d0e56    0000000035208658     linunprojectionchecks.obj
 0002:00005660       __real@3f847ae140000000    0000000035208660     linunprojectionchecks.obj
 0002:00005668       __real@3f40624dd2f1a9fc    0000000035208668     linunprojectionchecks.obj
 0002:00005670       __real@3fefae147ae147ae    0000000035208670     linunprojectionchecks.obj
 0002:00005678       __real@3ff028f5c28f5c29    0000000035208678     linunprojectionchecks.obj
 0002:00005680       __real@3f804189            0000000035208680     linunprojectionchecks.obj
 0002:00005688       __real@3ff00418a0000000    0000000035208688     linunprojectionchecks.obj
 0002:00005690       __real@3feff7cee0000000    0000000035208690     linunprojectionchecks.obj
 0002:00005698       __real@3fa2f684bda12f68    0000000035208698     linunprojectionchecks.obj
 0002:000056a0       __real@3efa36e2d7731900    00000000352086a0     linunprojectionchecks.obj
 0002:000056a8       __real@3f689374c0000000    00000000352086a8     linunprojectionchecks.obj
 0002:000056b0       __real@3f747ae140000000    00000000352086b0     linunprojectionchecks.obj
 0002:000056b8       __real@3f50624de0000000    00000000352086b8     linunprojectionchecks.obj
 0002:000056c0       ??_C@_09HCPCMEJO@OBB?5trees?$AA@ 00000000352086c0     obbtree.obj
 0002:000056d0       __real@ffee42d130773b76    00000000352086d0     obbtree.obj
 0002:000056d8       __real@7fee42d130773b76    00000000352086d8     obbtree.obj
 0002:000056e8       __real@3feeb851eb851eb8    00000000352086e8     rotunprojectionchecks.obj
 0002:000056f0       __real@3ff0a3d70a3d70a4    00000000352086f0     rotunprojectionchecks.obj
 0002:000056f8       __real@3ff0525460aa64c3    00000000352086f8     rotunprojectionchecks.obj
 0002:00005700       __real@3fef5cfaacd9e83e    0000000035208700     rotunprojectionchecks.obj
 0002:00005718       ??_C@_0CD@LFICKIIJ@PrimitiveWorldIntersection?$CIQueue@ 0000000035208718     rwi.obj
 0002:00005740       ??_C@_0BN@NCMAGHFA@RayWorldIntersection?$CIQueued?$CJ?$AA@ 0000000035208740     rwi.obj
 0002:00005760       ??_C@_0CF@KIKHOLPD@CPhysicalWorld?3?3RayWorldIntersec@ 0000000035208760     rwi.obj
 0002:00005788       ??_C@_0BA@CEOHFAK@SingleBox?5trees?$AA@ 0000000035208788     singleboxtree.obj
 0002:000057a8       __real@41490fdb            00000000352087a8     spheregeom.obj
 0002:000057ac       __real@bf7fbe77            00000000352087ac     spheregeom.obj
 0002:000057b0       __real@3fe6a09e667f3bcc    00000000352087b0     spheregeom.obj
 0002:000057b8       __real@3f828f5c            00000000352087b8     spheregeom.obj
 0002:000057c0       ??_7CTetrLattice@@6B@      00000000352087c0     tetrlattice.obj
 0002:000057f8       ??_C@_0BN@LFEFBEHO@CTetrLattice?3?3CheckStructure?$AA@ 00000000352087f8     tetrlattice.obj
 0002:00005818       __real@3f004189            0000000035208818     tetrlattice.obj
 0002:0000581c       __real@bfc147ae            000000003520881c     tetrlattice.obj
 0002:00005830       ??_7COBBTree@@6B@          0000000035208830     trimesh.obj
 0002:00005910       ??_7CAABBTree@@6B@         0000000035208910     trimesh.obj
 0002:000059f0       ??_7CTriMesh@@6B@          00000000352089f0     trimesh.obj
 0002:00005bf0       ??_C@_0O@EBEONEPM@auxilary?5data?$AA@ 0000000035208bf0     trimesh.obj
 0002:00005c00       ??_C@_0BB@NABIJMGH@wasted?5mesh?5data?$AA@ 0000000035208c00     trimesh.obj
 0002:00005c18       ??_C@_09HDIEJGOE@mesh?5data?$AA@ 0000000035208c18     trimesh.obj
 0002:00005c28       ??_C@_0BI@PKAJMKLJ@CTriMesh?3?3RebuildBVTree?$AA@ 0000000035208c28     trimesh.obj
 0002:00005c40       __real@39d1b717            0000000035208c40     trimesh.obj
 0002:00005c44       __real@40029cbc            0000000035208c44     trimesh.obj
 0002:00005c48       __real@3efae147            0000000035208c48     trimesh.obj
 0002:00005c4c       __real@3951b717            0000000035208c4c     trimesh.obj
 0002:00005c50       __real@40001062            0000000035208c50     trimesh.obj
 0002:00005c60       ??_C@_0M@KMODIPJI@voxel?5grids?$AA@ 0000000035208c60     voxelgeom.obj
 0002:00005c70       ??_7ISystemEventListener@@6B@ 0000000035208c70     CryPhysics.obj
 0002:00005c80       ??_C@_0BD@PJOKHJBB@Pure?5function?5call?$AA@ 0000000035208c80     CryPhysics.obj
 0002:00005c98       ??_C@_0CL@LKHBOBAH@Invalid?5parameter?5detected?5in?5CR@ 0000000035208c98     CryPhysics.obj
 0002:00005cc8       ??_C@_0DJ@DLJMMMP@Could?5not?5access?5CrySystem?4dll?5?$CI@ 0000000035208cc8     CryPhysics.obj
 0002:00005d08       ??_C@_0P@NHEMOHAI@Memory?5Manager?$AA@ 0000000035208d08     CryPhysics.obj
 0002:00005d18       ??_C@_0O@FFDHMLKN@CrySystem?4dll?$AA@ 0000000035208d18     CryPhysics.obj
 0002:00005d28       ??_C@_0BO@JDKBDPNB@CryGetIMemoryManagerInterface?$AA@ 0000000035208d28     CryPhysics.obj
 0002:00005d48       ??_C@_0BB@PNKHDABP@CrySystemCrtFree?$AA@ 0000000035208d48     CryPhysics.obj
 0002:00005d60       ??_C@_0BB@MFMFBMDO@CrySystemCrtSize?$AA@ 0000000035208d60     CryPhysics.obj
 0002:00005d78       ??_C@_0BD@BBIFHONI@CrySystemCrtMalloc?$AA@ 0000000035208d78     CryPhysics.obj
 0002:00005d90       ??_C@_0O@LCCIKADF@CryGetMemSize?$AA@ 0000000035208d90     CryPhysics.obj
 0002:00005da0       ??_C@_07CKAGCLEE@CryFree?$AA@ 0000000035208da0     CryPhysics.obj
 0002:00005da8       ??_C@_0L@FICCDMFO@CryRealloc?$AA@ 0000000035208da8     CryPhysics.obj
 0002:00005db8       ??_C@_09MCKPOEAK@CryMalloc?$AA@ 0000000035208db8     CryPhysics.obj
 0002:00005dc8       ??_C@_0BO@HAMEIFMK@Critical?5Section?5hanging?5lock?$AA@ 0000000035208dc8     CryPhysics.obj
 0002:00005de8       ?iid@?1??IID@ICryUnknown@@CAAEBUCryGUID@@XZ@4U3@B 0000000035208de8     CryPhysics.obj
 0002:00005df8       ?iid@?1??IID@IEngineModule@@CAAEBUCryGUID@@XZ@4U3@B 0000000035208df8     CryPhysics.obj
 0002:00005e08       ??_7ICryFactory@@6B@       0000000035208e08     CryPhysics.obj
 0002:00005e38       ??_7CSystemEventListner_Physics@@6B@ 0000000035208e38     CryPhysics.obj
 0002:00005e60       __real@3ac90fdb            0000000035208e60     CryPhysics.obj
 0002:00005e68       ??_C@_0L@CODMBEB@CryPhysics?$AA@ 0000000035208e68     CryPhysics.obj
 0002:00005e78       ??_7CEngineModule_CryPhysics@@6B@ 0000000035208e78     CryPhysics.obj
 0002:00005eb0       ??_C@_09BHIABECK@CryEngine?$AA@ 0000000035208eb0     CryPhysics.obj
 0002:00005ec0       ??_7CFactory@CEngineModule_CryPhysics@@6B@ 0000000035208ec0     CryPhysics.obj
 0002:00005ef0       ??_7bad_alloc@std@@6B@     0000000035208ef0     CryPhysics.obj
 0002:00005f00       ??_C@_0P@GHFPNOJB@bad?5allocation?$AA@ 0000000035208f00     CryPhysics.obj
 0002:00005f10       ??_7sp_counted_base@detail@boost@@6B@ 0000000035208f10     CryPhysics.obj
 0002:00005f30       ??_C@_0BI@KMAEJCIO@EngineModule_CryPhysics?$AA@ 0000000035208f30     CryPhysics.obj
 0002:00005f48       ?cid@?1??GetClassID@CFactory@CEngineModule_CryPhysics@@UEBAAEBUCryGUID@@XZ@4U4@B 0000000035208f48     CryPhysics.obj
 0002:00005f58       ??_7?$sp_counted_impl_p@VCEngineModule_CryPhysics@@@detail@boost@@6B@ 0000000035208f58     CryPhysics.obj
 0002:00005f78       ??_C@_0BN@FOKPCDPC@Boost?5threw?5an?5exception?3?5?$CFs?$AA@ 0000000035208f78     CryPhysics.obj
 0002:00005fa0       _pRawDllMain               0000000035208fa0     MSVCRT:crtdll.obj
 0002:00005fa0       _pDefaultRawDllMain        0000000035208fa0     MSVCRT:crtdll.obj
 0002:00006000       __rtc_iaa                  0000000035209000     MSVCRT:_initsect_.obj
 0002:00006008       __rtc_izz                  0000000035209008     MSVCRT:_initsect_.obj
 0002:00006010       __rtc_taa                  0000000035209010     MSVCRT:_initsect_.obj
 0002:00006018       __rtc_tzz                  0000000035209018     MSVCRT:_initsect_.obj
 0002:00013aac       __IMPORT_DESCRIPTOR_KERNEL32 0000000035216aac     kernel32:KERNEL32.dll
 0002:00013ac0       __IMPORT_DESCRIPTOR_USER32 0000000035216ac0     user32:USER32.dll
 0002:00013ad4       __IMPORT_DESCRIPTOR_MSVCR100 0000000035216ad4     MSVCRT:MSVCR100.dll
 0002:00013ae8       __NULL_IMPORT_DESCRIPTOR   0000000035216ae8     kernel32:KERNEL32.dll
 0003:00000000       ?fVec3_One@?$Vec3Constants@M@@2U?$Vec3_tpl@M@@B 0000000035218000     articulatedentity.obj
 0003:00000050       ?g_stub@@3VCPhysicalStub@@A 0000000035218050     physarea.obj
 0003:00000078       ?sEmptyStringBuffer@?1??_emptyHeader@?$CryStringT@D@@KAPEAUStrHeader@2@XZ@4PAU32@A 0000000035218078     physicalentity.obj
 0003:000000a8       ?__cursubstep@@3HA         00000000352180a8     physicalworld.obj
 0003:00000230       ?fVec3_Zero@?$Vec3Constants@M@@2U?$Vec3_tpl@M@@B 0000000035218230     rigidentity.obj
 0003:00000240       ?fVec2_Zero@?$Vec2Constants@M@@2U?$Vec2_tpl@M@@A 0000000035218240     rigidentity.obj
 0003:00000248       ?fVec2_OneX@?$Vec2Constants@M@@2U?$Vec2_tpl@M@@A 0000000035218248     rigidentity.obj
 0003:00000250       ?fVec2_OneY@?$Vec2Constants@M@@2U?$Vec2_tpl@M@@A 0000000035218250     rigidentity.obj
 0003:00000258       ?fVec2_One@?$Vec2Constants@M@@2U?$Vec2_tpl@M@@A 0000000035218258     rigidentity.obj
 0003:000002c0       ?g_bSaferBooleans@@3HA     00000000352182c0     boolean3d.obj
 0003:000002e4       ?mtx_pool_size@?$matrix_tpl@M@@2HA 00000000352182e4     matrixnm.obj
 0003:000002e8       ?vecn_pool_size@?$vectorn_tpl@M@@2HA 00000000352182e8     matrixnm.obj
 0003:000002ec       ?mtx_pool_size@?$matrix_tpl@N@@2HA 00000000352182ec     matrixnm.obj
 0003:000004d0       ?defgwd@@3Ugeom_world_data@@A 00000000352184d0     geometry.obj
 0003:00000530       ?defip@@3Uintersection_params@@A 0000000035218530     geometry.obj
 0003:000005e0       ?table@CIntersectionChecker@@2PAY07P6AHPEBUprimitive@primitives@@0PEAUprim_inters@@@ZA 00000000352185e0     intersectionchecks.obj
 0003:000007e0       ?default_function@CIntersectionChecker@@2P6AHPEBUprimitive@primitives@@0PEAUprim_inters@@@ZEA 00000000352187e0     intersectionchecks.obj
 0003:00000808       ?g_jobName@@3PAPEADA       0000000035218808     jobq.obj
 0003:00000840       ?table@CUnprojectionChecker@@2PAY177P6AHPEAUunprojection_mode@@PEBUprimitive@primitives@@H1HPEAUcontact@@PEAUgeom_contact_area@@@ZA 0000000035218840     linunprojectionchecks.obj
 0003:00000c80       ?table@COverlapChecker@@2PAY07P6AHPEBUprimitive@primitives@@0PEAV1@@ZA 0000000035218c80     overlapchecks.obj
 0003:00000e80       ?default_function@COverlapChecker@@2P6AHPEBUprimitive@primitives@@0PEAV1@@ZEA 0000000035218e80     overlapchecks.obj
 0003:00000ff0       ?g_Overlapper@@3VCOverlapChecker@@A 0000000035218ff0     trimesh.obj
 0003:00001060       ?m_seed@CLCGRndGen@@0_KA   0000000035219060     CryPhysics.obj
 0003:000010ac       _fltused                   00000000352190ac     MSVCRT:dllsupp.obj
 0003:000010b0       __native_dllmain_reason    00000000352190b0     MSVCRT:natstart.obj
 0003:000010b4       __native_vcclrit_reason    00000000352190b4     MSVCRT:natstart.obj
 0003:000010b8       __security_cookie          00000000352190b8     MSVCRT:gs_cookie.obj
 0003:000010c0       __security_cookie_complement 00000000352190c0     MSVCRT:gs_cookie.obj
 0003:000010d0       ?__ae_step@@3HA            00000000352190d0     articulatedentity.obj
 0003:000010d4       ?__maxdiff@@3MA            00000000352190d4     articulatedentity.obj
 0003:000010d8       ?s_pMemReplay@?1??CryGetIMemReplay@@YAPEAUIMemReplay@@XZ@4PEAU2@EA 00000000352190d8     articulatedentity.obj
 0003:000010e0       ?s_dummyMemReplay@?1??CryGetIMemReplay@@YAPEAUIMemReplay@@XZ@4UCDummyMemReplay@@A 00000000352190e0     articulatedentity.obj
 0003:000010e8       ??_B?1??CryGetIMemReplay@@YAPEAUIMemReplay@@XZ@51 00000000352190e8     articulatedentity.obj
 0003:00001840       ?g_pCurParticle@CParticleEntity@@2PAPEAV1@A 0000000035219840     particleentity.obj
 0003:00002b48       ?s_EmptyElems@?1??set_null@?$SmallDynStorage@MHUStandardAlloc@NAlloc@@@NArray@@IEAAXXZ@4PEAMEA 000000003521ab48     physarea.obj
 0003:00002b50       ?s_EmptyHeader@?1??set_null@?$SmallDynStorage@MHUStandardAlloc@NAlloc@@@NArray@@IEAAXXZ@4UEmptyHeader@23@A 000000003521ab50     physarea.obj
 0003:00002b58       ??_B?1??set_null@?$SmallDynStorage@MHUStandardAlloc@NAlloc@@@NArray@@IEAAXXZ@51 000000003521ab58     physarea.obj
 0003:00002b60       ?s_EmptyElems@?1??set_null@?$SmallDynStorage@UGeomQuery@@HUStandardAlloc@NAlloc@@@NArray@@IEAAXXZ@4PEAUGeomQuery@@EA 000000003521ab60     physarea.obj
 0003:00002b68       ?s_EmptyHeader@?1??set_null@?$SmallDynStorage@UGeomQuery@@HUStandardAlloc@NAlloc@@@NArray@@IEAAXXZ@4UEmptyHeader@23@A 000000003521ab68     physarea.obj
 0003:00002b74       ??_B?1??set_null@?$SmallDynStorage@UGeomQuery@@HUStandardAlloc@NAlloc@@@NArray@@IEAAXXZ@51 000000003521ab74     physarea.obj
 0003:00002b80       ?g_parts@CPhysicalEntity@@2PEAUSPartHelper@@EA 000000003521ab80     physicalentity.obj
 0003:00002b88       ?g_joints@CPhysicalEntity@@2PEAUSStructuralJointHelper@@EA 000000003521ab88     physicalentity.obj
 0003:00002b90       ?g_jointsDbg@CPhysicalEntity@@2PEAUSStructuralJointDebugHelper@@EA 000000003521ab90     physicalentity.obj
 0003:00002b98       ?g_jointidx@CPhysicalEntity@@2PEAHEA 000000003521ab98     physicalentity.obj
 0003:00002ba0       ?g_nPartsAlloc@CPhysicalEntity@@2HA 000000003521aba0     physicalentity.obj
 0003:00002ba4       ?g_nJointsAlloc@CPhysicalEntity@@2HA 000000003521aba4     physicalentity.obj
 0003:00002ba8       ?g_pSliceMesh@@3PEAVCTriMesh@@EA 000000003521aba8     physicalentity.obj
 0003:00002bb0       ?g_StaticRigidBodies@@3PAVRigidBody@@A 000000003521abb0     physicalentity.obj
 0003:00002f00       ?g_StaticPhysicalEntity@@3VCPhysicalEntity@@A 000000003521af00     physicalentity.obj
 0003:00003060       ?m_defpart@CPhysicalEntity@@2Ugeom@@A 000000003521b060     physicalentity.obj
 0003:000030e8       ?s_used_memory@?1??_usedMemory@?$CryStringT@D@@SA_K_J@Z@4_KA 000000003521b0e8     physicalentity.obj
 0003:00005b48       ?serializeString@?1??SetSharedSerializeString@?$CSerializeWrapper@UISerialize@@@@QEAAAEAUSSerializeString@@AEBV?$CryStringT@D@@@Z@4U3@A 000000003521db48     physicalentity.obj
 0003:00005b50       ??_B?1??SetSharedSerializeString@?$CSerializeWrapper@UISerialize@@@@QEAAAEAUSSerializeString@@AEBV?$CryStringT@D@@@Z@51 000000003521db50     physicalentity.obj
 0003:00005b60       ?g_nPhysWorlds@@3HA        000000003521db60     physicalworld.obj
 0003:00005b64       ?g_pidxPhysThreadidx@@3HA  000000003521db64     physicalworld.obj
 0003:00005b70       ?g_pPhysWorlds@@3PAPEAVCPhysicalWorld@@A 000000003521db70     physicalworld.obj
 0003:00005d70       ?g_dummyBuf@@3PAHA         000000003521dd70     physicalworld.obj
 0003:00005db0       ?g_timeFiber@@3_JC         000000003521ddb0     physicalworld.obj
 0003:00005db8       ?__curstep@@3HA            000000003521ddb8     physicalworld.obj
 0003:00005dbc       ?g_initg_pidxPhysThread@@3UInitg_pidxPhysThread@@A 000000003521ddbc     physicalworld.obj
 0003:0000fc20       ?g_RBdata@@3PAPEAURBdata@@A 0000000035227c20     rigidbody.obj
 0003:0000fc40       ?__solver_step@@3HA        0000000035227c40     rigidbody.obj
 0003:00010e70       ?g_REdata@@3PAUREdata@@A   0000000035228e70     rigidentity.obj
 0003:00013698       ?__bstop@@3HA              000000003522b698     rigidentity.obj
 0003:000136c0       ?s_used_memory@?1??_usedMemory@?$CryStackStringT@D$0CAA@@@SA_K_K@Z@4_KA 000000003522b6c0     rigidentity.obj
 0003:000148a0       ?str@?1??numbered_tag@@YAPEBDPEBDI@Z@4PADA 000000003522c8a0     ropeentity.obj
 0003:00015a10       ?g_lockProcessedAux@CPhysicalEntity@@2HC 000000003522da10     softentity.obj
 0003:00018620       ?g_BoolHash@@3PAIA         0000000035230620     boolean2d.obj
 0003:00020620       ?g_BoolGrid@@3PAHA         0000000035238620     boolean2d.obj
 0003:00024620       ?g_BoolIdBuf@@3PAHA        000000003523c620     boolean2d.obj
 0003:00028630       ?g_BoolPtBuf@@3PAU?$Vec2_tpl@M@@A 0000000035240630     boolean2d.obj
 0003:00030630       ?g_BoolInters@@3PAUinters2d@@A 0000000035248630     boolean2d.obj
 0003:00031630       ?g_nTriangulationErrors@@3HA 0000000035249630     boolean3d.obj
 0003:000319e0       ?mtx_pool@?$matrix_tpl@M@@2PAMA 00000000352499e0     matrixnm.obj
 0003:000321e0       ?vecn_pool@?$vectorn_tpl@M@@2PAMA 000000003524a1e0     matrixnm.obj
 0003:000325e0       ?mtx_pool@?$matrix_tpl@N@@2PANA 000000003524a5e0     matrixnm.obj
 0003:000335e0       ?g_bHasSSE@@3HA            000000003524b5e0     matrixnm.obj
 0003:000335e4       ?mtx_pool_pos@?$matrix_tpl@M@@2HA 000000003524b5e4     matrixnm.obj
 0003:000335e8       ?vecn_pool_pos@?$vectorn_tpl@M@@2HA 000000003524b5e8     matrixnm.obj
 0003:000335ec       ?mtx_pool_pos@?$matrix_tpl@N@@2HA 000000003524b5ec     matrixnm.obj
 0003:000335f0       ?__qhullcalled@@3HA        000000003524b5f0     qhull.obj
 0003:000514e0       ?g_pLockIntersect@@3PECHEC 00000000352694e0     geometry.obj
 0003:000514f0       ?g_idata@@3PAUintersData@@A 00000000352694f0     geometry.obj
 0003:00141889       ?g_Intersector@@3VCIntersectionChecker@@A 0000000035359889     intersectionchecks.obj
 0003:00141890       ?g_pHFbuf@@3PAPEAVCHeightfield@@A 0000000035359890     jobq.obj
 0003:00141900       ?g_Unprojector@@3VCUnprojectionChecker@@A 0000000035359900     linunprojectionchecks.obj
 0003:00141960       ?dummyAreaPt@@3PAU?$Vec3_tpl@M@@A 0000000035359960     linunprojectionchecks.obj
 0003:00141a30       ?gSpuQuery3DengineForHeights@@3IA 0000000035359a30     rwi.obj
 0003:00141a50       ?g_RWIContacts@@3PAUgeom_contact@@A 0000000035359a50     rwi.obj
 0003:00143ff0       ?g_Faces@CTetrLattice@@2PEAUSCGFace@@EA 000000003535bff0     tetrlattice.obj
 0003:00143ff8       ?g_Tets@CTetrLattice@@2PEAUSCGTetr@@EA 000000003535bff8     tetrlattice.obj
 0003:00144000       ?g_nFacesAlloc@CTetrLattice@@2HA 000000003535c000     tetrlattice.obj
 0003:00144004       ?g_nTetsAlloc@CTetrLattice@@2HA 000000003535c004     tetrlattice.obj
 0003:001443ac       ?__gtrimesh@@3HA           000000003535c3ac     trimesh.obj
 0003:00144780       ?g_subrefBuf@@3PAUsubref@@A 000000003535c780     CryPhysics.obj
 0003:00144930       ?g_sintab@@3PAMA           000000003535c930     CryPhysics.obj
 0003:00145934       ?numAllocations@_CryMemoryManagerPoolHelper@@2HC 000000003535d934     CryPhysics.obj
 0003:00145938       ?requestedMemory@_CryMemoryManagerPoolHelper@@2JC 000000003535d938     CryPhysics.obj
 0003:0014593c       ?freedMemory@_CryMemoryManagerPoolHelper@@2JC 000000003535d93c     CryPhysics.obj
 0003:00145940       ?allocatedMemory@_CryMemoryManagerPoolHelper@@2JC 000000003535d940     CryPhysics.obj
 0003:00145948       ?g_subrefGeomParams@@3PAPEAUsubref@@A 000000003535d948     CryPhysics.obj
 0003:00145960       ?g_subrefAction@@3PAPEAUsubref@@A 000000003535d960     CryPhysics.obj
 0003:001459f0       ?g_subrefParams@@3PAPEAUsubref@@A 000000003535d9f0     CryPhysics.obj
 0003:00145ac8       ?g_szGeomParams@@3PAHA     000000003535dac8     CryPhysics.obj
 0003:00145ae0       ?g_szAction@@3PAHA         000000003535dae0     CryPhysics.obj
 0003:00145b30       ?g_szParams@@3PAHA         000000003535db30     CryPhysics.obj
 0003:00145b9c       ?g_bProfilerEnabled@@3_NA  000000003535db9c     CryPhysics.obj
 0003:00145ba0       ?gEnv@@3PEAUSSystemGlobalEnvironment@@EA 000000003535dba0     CryPhysics.obj
 0003:00145ba8       ?m_pFirst@Test@CryUnitTest@@2PEAU12@EA 000000003535dba8     CryPhysics.obj
 0003:00145bb0       ?m_pLast@Test@CryUnitTest@@2PEAU12@EA 000000003535dbb0     CryPhysics.obj
 0003:00145bb8       ?g_pHeadToRegFactories@@3PEAUSRegFactoryNode@@EA 000000003535dbb8     CryPhysics.obj
 0003:00145bc0       ?g_iTraceAllocations@@3HA  000000003535dbc0     CryPhysics.obj
 0003:00145bc4       ?m_bInitialized@_CryMemoryManagerPoolHelper@@2HA 000000003535dbc4     CryPhysics.obj
 0003:00145bc8       ?_CryMalloc@_CryMemoryManagerPoolHelper@@2P6APEAX_KAEA_K0@ZEA 000000003535dbc8     CryPhysics.obj
 0003:00145bd0       ?_CryGetMemSize@_CryMemoryManagerPoolHelper@@2P6A_KPEAX_K@ZEA 000000003535dbd0     CryPhysics.obj
 0003:00145bd8       ?_CryRealloc@_CryMemoryManagerPoolHelper@@2P6APEAXPEAX_KAEA_K21@ZEA 000000003535dbd8     CryPhysics.obj
 0003:00145be0       ?_CryFree@_CryMemoryManagerPoolHelper@@2P6A_KPEAX_K@ZEA 000000003535dbe0     CryPhysics.obj
 0003:00145be8       ?_CryCrtMalloc@_CryMemoryManagerPoolHelper@@2P6APEAX_K@ZEA 000000003535dbe8     CryPhysics.obj
 0003:00145bf0       ?_CryCrtRealloc@_CryMemoryManagerPoolHelper@@2P6APEAXPEAX_K@ZEA 000000003535dbf0     CryPhysics.obj
 0003:00145bf8       ?_CryCrtFree@_CryMemoryManagerPoolHelper@@2P6A_KPEAX@ZEA 000000003535dbf8     CryPhysics.obj
 0003:00145c00       ?_CryCrtSize@_CryMemoryManagerPoolHelper@@2P6A_KPEAX@ZEA 000000003535dc00     CryPhysics.obj
 0003:00145c08       ?_CryGetIMemoryManagerInterface@_CryMemoryManagerPoolHelper@@2P6AXPEAPEAX@ZEA 000000003535dc08     CryPhysics.obj
 0003:00145c10       ?g_random_generator@@3VCLCGRndGen@@A 000000003535dc10     CryPhysics.obj
 0003:00145c11       ?Now@@3VInitPhysicsGlobals@@A 000000003535dc11     CryPhysics.obj
 0003:00145c20       ?s_factory@CFactory@CEngineModule_CryPhysics@@0V12@A 000000003535dc20     CryPhysics.obj
 0003:00145c78       ?s_used_memory@?1??_usedMemory@?$CryStringT@_W@@SA_K_J@Z@4_KA 000000003535dc78     CryPhysics.obj
 0003:00145c80       ?supportedIIDs@?1???0CFactory@CEngineModule_CryPhysics@@AEAA@XZ@4PAUCryGUID@@A 000000003535dc80     CryPhysics.obj
 0003:00145ca0       ?p@?1??CreateClassInstance@CFactory@CEngineModule_CryPhysics@@UEBA?AV?$shared_ptr@UICryUnknown@@@boost@@XZ@4V?$shared_ptr@VCEngineModule_CryPhysics@@@5@A 000000003535dca0     CryPhysics.obj
 0003:00145cb0       ??_B?1??CreateClassInstance@CFactory@CEngineModule_CryPhysics@@UEBA?AV?$shared_ptr@UICryUnknown@@@boost@@XZ@51 000000003535dcb0     CryPhysics.obj
 0003:00145cc0       ?g_globalSections@?$Node_Alloc_Lock@$00$00@@2PAUInternalCriticalSectionDummy@@A 000000003535dcc0     StdAfx.obj
 0003:00146d40       ?m_bInitialized@?$Node_Alloc_Lock@$00$00@@2_NA 000000003535ed40     StdAfx.obj
 0003:00146d48       ?__type_info_root_node@@3U__type_info_node@@A 000000003535ed48     MSVCRT:tncleanup.obj
 0003:00146d58       __native_startup_state     000000003535ed58     <common>
 0003:00146d60       __native_startup_lock      000000003535ed60     <common>
 0003:00146d68       __dyn_tls_init_callback    000000003535ed68     <common>
 0003:00146d70       __onexitend                000000003535ed70     <common>
 0003:00146d78       __onexitbegin              000000003535ed78     <common>
 0005:00000000       ?m_Self@CrySimpleThreadSelf@@1PEAV1@EA 0000000035367000     CryPhysics.obj

 entry point at        0001:00200f04

 Static symbols

 0001:00047ea0       ?qsort@@YAXPEAMPEAHHH@Z    0000000035048ea0 f   physarea.obj
 0001:00048940       ?SignalEventAreaChange@@YAXPEAVCPhysicalWorld@@PEAVCPhysArea@@@Z 0000000035049940 f   physarea.obj
 0001:00083b70       ?qsort@@YAXPEAPEAVCPhysicalEntity@@PEAMPEAHHH@Z 0000000035084b70 f   physicalworld.obj
 0001:0008a500       ?qsort@@YAXPEAPEAVCPhysicalEntity@@AEBU?$Vec3_tpl@M@@1HH@Z 000000003508b500 f   physicalworld.obj
 0001:000a2880       ??$qsort@PEAUentity_contact@@@@YAXPEAPEAUentity_contact@@HHH@Z 00000000350a3880 f   rigidbody.obj
 0001:000a2990       ??$qsort@PEAVRigidBody@@@@YAXPEAPEAVRigidBody@@HHH@Z 00000000350a3990 f   rigidbody.obj
 0001:000a2b00       ??$qsort@PEAUentity_contact_unproj@@@@YAXPEAPEAUentity_contact_unproj@@HHH@Z 00000000350a3b00 f   rigidbody.obj
 0001:000b8110       ?qsort@@YAXPEAUedgeitem@@HH@Z 00000000350b9110 f   rigidentity.obj
 0001:001307e0       ?qsort@@YAXPEAHPEAPEAXHH@Z 00000000351317e0 f   qhull.obj
 0001:001dac30       ?ExpandGlobalLoadState@@YAXH@Z 00000000351dbc30 f   trimesh.obj
 0001:00200b0c       pre_c_init                 0000000035201b0c f   MSVCRT:crtdll.obj
 0001:00200dc8       __DllMainCRTStartup        0000000035201dc8 f   MSVCRT:crtdll.obj
 0001:002011a0       _onexit$fin$0              00000000352021a0 f   MSVCRT:atonexit.obj
 0001:002011bb       __DllMainCRTStartup$filt$0 00000000352021bb f   MSVCRT:crtdll.obj
 0001:002011eb       __DllMainCRTStartup$fin$1  00000000352021eb f   MSVCRT:crtdll.obj
 0001:00201210       _IsNonwritableInCurrentImage$filt$0 0000000035202210 f   MSVCRT:pesect.obj
 0001:00201240       ??__Eg_stub@@YAXXZ         0000000035202240 f   physarea.obj
 0001:00201250       ??__Eg_StaticRigidBodies@@YAXXZ 0000000035202250 f   physicalentity.obj
 0001:00201290       ??__Eg_StaticPhysicalEntity@@YAXXZ 0000000035202290 f   physicalentity.obj
 0001:002012c0       ??__Eg_initg_pidxPhysThread@@YAXXZ 00000000352022c0 f   physicalworld.obj
 0001:002012e0       ??__ECryUserInvalidID@@YAXXZ 00000000352022e0 f   rigidentity.obj
 0001:002012f0       ??__ECrySessionInvalidID@@YAXXZ 00000000352022f0 f   rigidentity.obj
 0001:00201300       ??__Eg_idata@@YAXXZ        0000000035202300 f   geometry.obj
 0001:00201590       ??__Enow@@YAXXZ            0000000035202590 f   geometry.obj
 0001:002015a0       ??__EinitHeightfieldGlobals@@YAXXZ 00000000352025a0 f   heightfieldbv.obj
 0001:002015e0       ??__EinitTriMeshGlobals@@YAXXZ 00000000352025e0 f   trimesh.obj
 0001:002015f0       ??__EinitVoxgridGlobals@@YAXXZ 00000000352025f0 f   voxelbv.obj
 0001:00201630       ??__Eg_random_generator@@YAXXZ 0000000035202630 f   CryPhysics.obj
 0001:00201640       ??__Eg_system_event_listener_physics@@YAXXZ 0000000035202640 f   CryPhysics.obj
 0001:00201650       ??__ENow@@YAXXZ            0000000035202650 f   CryPhysics.obj
 0001:00201660       ??__E?s_factory@CFactory@CEngineModule_CryPhysics@@0V12@A@@YAXXZ 0000000035202660 f   CryPhysics.obj
 0001:00201680       ??__EautoInitializer@@YAXXZ 0000000035202680 f   StdAfx.obj
 0001:002016f0       ??__Fg_stub@@YAXXZ         00000000352026f0 f   physarea.obj
 0001:00201700       ??__Fg_StaticPhysicalEntity@@YAXXZ 0000000035202700 f   physicalentity.obj
 0001:00201750       ??__Fg_entSoft@?1??SetStateFromTypedSnapshot@CPhysicalEntity@@UEAAHV?$CSerializeWrapper@UISerialize@@@@HH@Z@YAXXZ 0000000035202750 f   physicalworld.obj
 0001:00201760       ??__Fg_entRope@?1??SetStateFromTypedSnapshot@CPhysicalEntity@@UEAAHV?$CSerializeWrapper@UISerialize@@@@HH@Z@YAXXZ 0000000035202760 f   physicalworld.obj
 0001:00201770       ??__Fg_entArticulated@?1??SetStateFromTypedSnapshot@CPhysicalEntity@@UEAAHV?$CSerializeWrapper@UISerialize@@@@HH@Z@YAXXZ 0000000035202770 f   physicalworld.obj
 0001:00201780       ??__Fg_entParticle@?1??SetStateFromTypedSnapshot@CPhysicalEntity@@UEAAHV?$CSerializeWrapper@UISerialize@@@@HH@Z@YAXXZ 0000000035202780 f   physicalworld.obj
 0001:00201790       ??__Fg_entLiving@?1??SetStateFromTypedSnapshot@CPhysicalEntity@@UEAAHV?$CSerializeWrapper@UISerialize@@@@HH@Z@YAXXZ 0000000035202790 f   physicalworld.obj
 0001:002017a0       ??__Fg_entRigid@?1??SetStateFromTypedSnapshot@CPhysicalEntity@@UEAAHV?$CSerializeWrapper@UISerialize@@@@HH@Z@YAXXZ 00000000352027a0 f   physicalworld.obj
 0001:002017b0       ??__Fg_entStatic@?1??SetStateFromTypedSnapshot@CPhysicalEntity@@UEAAHV?$CSerializeWrapper@UISerialize@@@@HH@Z@YAXXZ 00000000352027b0 f   physicalworld.obj
 0001:002017c0       ??__Fg_entSoft@?1??SerializeGarbageTypedSnapshot@CPhysicalWorld@@UEAAXV?$CSerializeWrapper@UISerialize@@@@HH@Z@YAXXZ 00000000352027c0 f   physicalworld.obj
 0001:002017d0       ??__Fg_entRope@?1??SerializeGarbageTypedSnapshot@CPhysicalWorld@@UEAAXV?$CSerializeWrapper@UISerialize@@@@HH@Z@YAXXZ 00000000352027d0 f   physicalworld.obj
 0001:002017e0       ??__Fg_entArticulated@?1??SerializeGarbageTypedSnapshot@CPhysicalWorld@@UEAAXV?$CSerializeWrapper@UISerialize@@@@HH@Z@YAXXZ 00000000352027e0 f   physicalworld.obj
 0001:002017f0       ??__Fg_entParticle@?1??SerializeGarbageTypedSnapshot@CPhysicalWorld@@UEAAXV?$CSerializeWrapper@UISerialize@@@@HH@Z@YAXXZ 00000000352027f0 f   physicalworld.obj
 0001:00201800       ??__Fg_entLiving@?1??SerializeGarbageTypedSnapshot@CPhysicalWorld@@UEAAXV?$CSerializeWrapper@UISerialize@@@@HH@Z@YAXXZ 0000000035202800 f   physicalworld.obj
 0001:00201810       ??__Fg_entWheeled@?1??SerializeGarbageTypedSnapshot@CPhysicalWorld@@UEAAXV?$CSerializeWrapper@UISerialize@@@@HH@Z@YAXXZ 0000000035202810 f   physicalworld.obj
 0001:00201820       ??__Fg_entRigid@?1??SerializeGarbageTypedSnapshot@CPhysicalWorld@@UEAAXV?$CSerializeWrapper@UISerialize@@@@HH@Z@YAXXZ 0000000035202820 f   physicalworld.obj
 0001:00201830       ??__Fg_entStatic@?1??SerializeGarbageTypedSnapshot@CPhysicalWorld@@UEAAXV?$CSerializeWrapper@UISerialize@@@@HH@Z@YAXXZ 0000000035202830 f   physicalworld.obj
 0001:00201840       ??__Fg_entWheeled@?1??SetStateFromTypedSnapshot@CPhysicalEntity@@UEAAHV?$CSerializeWrapper@UISerialize@@@@HH@Z@YAXXZ 0000000035202840 f   physicalworld.obj
 0001:00201850       ??__FCrySessionInvalidID@@YAXXZ 0000000035202850 f   rigidentity.obj
 0001:002018a0       ??__FCryUserInvalidID@@YAXXZ 00000000352028a0 f   rigidentity.obj
 0001:002018f0       ??__Fg_system_event_listener_physics@@YAXXZ 00000000352028f0 f   CryPhysics.obj
 0001:00201900       ??__F?s_factory@CFactory@CEngineModule_CryPhysics@@0V12@A@@YAXXZ 0000000035202900 f   CryPhysics.obj
 0001:00201970       ??__FautoInitializer@@YAXXZ 0000000035202970 f   StdAfx.obj
